
 OS2KRNL

 Start         Length     Name                   Class
 0001:00000000 000000000H MPDATA                 MPDATA 32-bit
 0001:00000000 000000770H START                  LOWDATA 16-bit
 0001:00000770 000000B78H CONSTANTS              LOWDATA 16-bit
 0001:000012F0 000000400H IDTDATA                LOWDATA 16-bit
 0001:000016F0 0000057B8H DATA                   LOWDATA 16-bit
 0001:00006EA8 000000000H DWORDDATA              LOWDATA 16-bit
 0001:00006EA8 0000003DEH TABLE                  LOWDATA 16-bit
 0001:00007286 000000584H INTERRMSG              LOWDATA 16-bit
 0001:0000780A 00000005FH ABIOSDATA              LOWDATA 16-bit
 0001:00007869 000000008H LASTDATA               LOWDATA 16-bit
 0001:00007871 000000000H EENDDATA               LOWDATA 16-bit
 0002:00000000 000000238H FIRSTCODE              LOWCODE 16-bit
 0002:00000238 000004324H CODE                   LOWCODE 16-bit
 0002:0000455C 000000450H ABIOSCODE              LOWCODE 16-bit
 0002:000049AC 0000029ECH INITCODE               LOWCODE 16-bit
 0003:00000000 00000D23BH DCODE                  DCODE 16-bit
 0004:00000000 00000008AH DFIRST                 DDATA 16-bit
 0004:0000008A 00000A9ADH DDATA                  DDATA 16-bit
 0004:0000AA38 000000000H DCONST                 DDATA 16-bit
 0004:0000AA38 0000009B0H DBSS                   DDATA 16-bit
 0005:00000000 00000F994H TASKDUMMY              PTDADATA 16-bit
 0005:0000F994 00000066CH TASKDATA               PTDADATA 16-bit
 0006:00000000 000001510H GDTSTART               GDTDATA 16-bit
 0006:00001510 000000810H GDTCGSEG               GDTDATA 16-bit
 0006:00001D20 0000001A0H GDTPUBSEG              GDTDATA 16-bit
 0006:00001EC0 000000000H GDTEND                 GDTDATA 16-bit
 0007:00000000 00000158CH INITDATA               INITDATA 16-bit
 0007:0000158C 00000047AH INITTABLE              INITDATA 16-bit
 0007:00001A06 00000031EH INITSTRING             INITDATA 16-bit
 0007:00001D24 00000372AH INITBSS                INITDATA 16-bit
 0008:00000000 000002940H INITR3CODE             INITR3CODE 16-bit
 0009:00000000 0000001ACH MVDMINSTDATA           MIDATA 32-bit
 000A:00000000 0000019A4H SWAPINSTDATA           SIDATA 32-bit
 000B:00000000 000000304H CINIT_DATA             CINITDATA 32-bit
 000B:00000304 000001470H THUNKINIT_DATA         CINITDATA 32-bit
 000B:00001774 000001B6CH CSWAP_DATA             CSWAPDATA 32-bit
 000B:000032E0 00001CC50H _DATA                  DATA 32-bit
 000B:0001FF30 000000242H DOSMTE                 DATA 32-bit
 000B:00020172 000000000H DOSMTENAME             DATA 32-bit
 000B:00020172 000000003H DOSMTEMID              DATA 32-bit
 000B:00020175 000000CE7H DOSMTEENTRY            DATA 32-bit
 000B:00020E5C 000000018H DOSMTEAUX              DATA 32-bit
 000B:00020E74 0000000C2H FSHMTE                 DATA 32-bit
 000B:00020F36 000000000H FSHMTENAME             DATA 32-bit
 000B:00020F36 000000001H FSHMTEMID              DATA 32-bit
 000B:00020F37 0000000DCH FSHMTEENTRY            DATA 32-bit
 000B:00021013 0000000BAH VDDMTE                 DATA 32-bit
 000B:000210CD 000000000H VDDMTENAME             DATA 32-bit
 000B:000210CD 000000003H VDDMTEMID              DATA 32-bit
 000B:000210D0 000000298H VDDMTEENTRY            DATA 32-bit
 000B:00021368 000005690H PANICMSG               CONST 32-bit
 000B:000269F8 000000000H CONST                  CONST 32-bit
 000B:000269F8 000000138H _BSS                   BSS 32-bit
 000B:00026B30 000004CF2H c_common               BSS 32-bit
 000C:00000000 00000EF64H HIGH2CODE              HIGH2CODE 16-bit
 000D:00000000 00000B514H HIGH3CODE              HIGH3CODE 16-bit
 000E:00000000 0000046D4H HIGH4CODE              HIGH4CODE 16-bit
 000E:000046D4 000000000H HIGH4SWAPCODE          HIGH4CODE 16-bit
 000E:000046D4 000003BD0H FSSWAPCODE             HIGH4CODE 16-bit
 000E:000082A4 0000022ECH FATEASWAPCODE          HIGH4CODE 16-bit
 000E:0000A590 000000000H MONLOCKCODE            HIGH4CODE 16-bit
 000E:0000A590 000000000H MONSWAPCODE            HIGH4CODE 16-bit
 000E:0000A590 0000039A8H NMPIPESWAPCODE         HIGH4CODE 16-bit
 000E:0000DF38 000000000H ENDHIGH4CODE           HIGH4CODE 16-bit
 000F:00000000 000001124H HIGH5CODE              HIGH5CODE 16-bit
 000F:00001124 000000518H HIGH5SWAPCODE          HIGH5CODE 16-bit
 000F:0000163C 000000094H LOGSWAPCODE            HIGH5CODE 16-bit
 000F:000016D0 000000000H LOGLOCKCODE            HIGH5CODE 16-bit
 000F:000016D0 000001AD4H RASLOCKCODE            HIGH5CODE 16-bit
 000F:000031A4 000001218H RASSWAPCODE            HIGH5CODE 16-bit
 000F:000043BC 00000739CH HIGHINITCODE           HIGH5CODE 16-bit
 000F:0000B758 000000000H ENDHIGH5CODE           HIGH5CODE 16-bit
 0010:00000000 000001DDCH THUNK_TEXT             CODE 32-bit
 0010:00001DDC 00000DC20H HIGH32CODE             CODE 32-bit
 0010:0000F9FC 000030023H _TEXT                  CODE 32-bit
 0010:0003FA20 0000021F4H SMLOCK_TEXT            CODE 32-bit
 0010:00041C14 000002B28H HIGH32SWAP_TEXT        CODE 32-bit
 0010:0004473C 000000000H THUNKSWAP_TEXT         CODE 32-bit
 0010:0004473C 0000002BCH SWAP32_1               CODE 32-bit
 0010:000449F8 00000036CH SWAP32_2               CODE 32-bit
 0010:00044D64 000000B88H SWAP32_3               CODE 32-bit
 0010:000458EC 0000010FCH SWAP32_4               CODE 32-bit
 0010:000469E8 000000DB8H SWAP32_5               CODE 32-bit
 0010:000477A0 000000E64H SWAP32_6               CODE 32-bit
 0010:00048604 000000FF0H SWAP32_7               CODE 32-bit
 0010:000495F4 000001484H SWAP32_8               CODE 32-bit
 0010:0004AA78 0000008C4H SWAP32_9               CODE 32-bit
 0010:0004B33C 000000FA0H SWAP32_10              CODE 32-bit
 0010:0004C2DC 000000814H SWAP32_11              CODE 32-bit
 0010:0004CAF0 000000878H SWAP32_12              CODE 32-bit
 0010:0004D368 000003558H SWAP32_13              CODE 32-bit
 0010:000508C0 000002560H SWAP32_14              CODE 32-bit
 0010:00052E20 000002398H SWAP32_15              CODE 32-bit
 0010:000551B8 000000CBCH SWAP32_16              CODE 32-bit
 0010:00055E74 000000B88H SWAP32_17              CODE 32-bit
 0010:000569FC 000000A00H SWAP32_18              CODE 32-bit
 0010:000573FC 000000930H SWAP32_19              CODE 32-bit
 0010:00057D2C 000000A54H SWAP32_20              CODE 32-bit
 0010:00058780 0000003B4H SWAP32_21              CODE 32-bit
 0010:00058B34 000000C78H SWAP32_22              CODE 32-bit
 0010:000597AC 0000046A8H SWAP32_23              CODE 32-bit
 0010:0005DE54 000000FC4H SWAP32_24              CODE 32-bit
 0010:0005EE18 000000CC4H SWAP32_25              CODE 32-bit
 0010:0005FADC 000001518H SWAP32_26              CODE 32-bit
 0010:00060FF4 000002370H SWAP32_27              CODE 32-bit
 0010:00063364 0000008A4H SWAP32_28              CODE 32-bit
 0010:00063C08 000000000H LOAD_TUNE1_SWP         CODE 32-bit
 0010:00063C08 0000007D0H LOAD_TUNE4_SWP         CODE 32-bit
 0010:000643D8 000000000H LOAD_TUNE8_SWP         CODE 32-bit
 0010:000643D8 000000000H LOAD_TUNE9_SWP         CODE 32-bit
 0010:000643D8 000000000H LOAD_FTUNE2_SWP        CODE 32-bit
 0010:000643D8 0000018A0H LOAD_FTUNE1_SWP        CODE 32-bit
 0010:00065C78 000001748H LOAD_TUNEDIT1_SWP      CODE 32-bit
 0010:000673C0 000000000H LOAD_TUNEDOS5_SWP      CODE 32-bit
 0010:000673C0 00000004CH LOAD_TUNEDOS12_SWP     CODE 32-bit
 0010:0006740C 000000000H LOAD_TUNEDOS11_SWP     CODE 32-bit
 0010:0006740C 000000300H LOAD_TUNEDOS4_SWP      CODE 32-bit
 0010:0006770C 000000000H LOAD_EXITDOS1_SWP      CODE 32-bit
 0010:0006770C 000000154H LOAD_BEEP_SWP          CODE 32-bit
 0010:00067860 00000070CH EXMGSWAP_TEXT          CODE 32-bit
 0010:00067F6C 000009C1CH TKSWAP_TEXT            CODE 32-bit
 0010:00071B88 0000033E8H LDRSWAP_TEXT           CODE 32-bit
 0010:00074F70 000000F58H SELSWAP_TEXT           CODE 32-bit
 0010:00075EC8 00000195CH VMSWAP_TEXT            CODE 32-bit
 0010:00077824 000000768H PGSWAP_TEXT            CODE 32-bit
 0010:00077F8C 000006A24H MVDMSWAP_TEXT          CODE 32-bit
 0010:0007E9B0 000001274H QUERYSWAP_TEXT         CODE 32-bit
 0010:0007FC24 000002764H PERFSWAP_TEXT          CODE 32-bit
 0010:00082388 000002C50H DYNSWAP_TEXT           CODE 32-bit
 0010:00084FD8 000001AE4H DYNLOCK_TEXT           CODE 32-bit
 0010:00086ABC 000002F20H DEBUGLOCK_TEXT         CODE 32-bit
 0010:000899DC 000003FD8H DEBUGSWAP_TEXT         CODE 32-bit
 0010:0008D9B4 0000013CCH MON32SWAP_TEXT         CODE 32-bit
 0010:0008ED80 0000002E8H MON32LOCK_TEXT         CODE 32-bit
 0010:0008F068 000000140H PROFLOCK_TEXT          CODE 32-bit
 0010:0008F1A8 000002B2CH PROFSWAP_TEXT          CODE 32-bit
 0010:00091CD4 000009C08H CINIT_TEXT             CODE 32-bit
 0010:0009B8DC 000000148H THUNKINIT_TEXT         CODE 32-bit
 0010:0009BA24 000000000H ENDHIGH32CODE          CODE 32-bit

 Origin   Group
 000C:0   DOSHIGH2CODE
 000D:0   DOSHIGH3CODE
 000E:0   DOSHIGH4CODE
 000F:0   DOSHIGH5CODE
 0007:0   DOSINITDATA
 0010:0   DOSHIGH32CODE
 0008:0   DOSINITR3CODE
 0000:0   FLAT
 000B:0   DGROUP
 0009:0   DOSMVDMINSTDATA
 000A:0   DOSSWAPINSTDATA
 0003:0   DBGCODE
 0004:0   DBGDATA
 0002:0   DOSCODE
 0005:0   TASKAREA
 0001:0   DOSGROUP
 0006:0   DOSGDTDATA

  Address         Publics by Value

 0000:00000000  Imp  DOSIODELAYCNT        (DOSCALLS.427)
 0000:00000000  Abs  _EndOp
 0000:00000000  Abs  PVWMI_Ct_cpu_Int_0
 0000:00000001  Abs  _EndOpArg
 0000:00000001  Abs  PVWMI_Mt_cpu_ETInt_ETNotIdle_0
 0000:00000002  Abs  PVWMI_Mt_cpu_STInt_STNotIdle_0
 0000:00000002  Abs  _OutBlank
 0000:00000003  Abs  _OutBlanks
 0000:00000003  Abs  PVWMI_ET_cpu_NotIdle_0
 0000:00000004  Abs  RmSelLstNum
 0000:00000004  Abs  PVWMI_ST_cpu_NotIdle_0
 0000:00000004  Abs  _OutCrLf
 0000:00000005  Abs  PVWMI_Ct_cpu_Sched_0
 0000:00000005  Abs  _OutChar
 0000:00000006  Abs  PVWMI_Mt_mem_PageFault_0
 0000:00000006  Abs  PIPEDIRLEN
 0000:00000006  Abs  _OutStr
 0000:00000007  Abs  PVWMI_Mt_mem_PageFault_1
 0000:00000007  Abs  _OutStrlc
 0000:00000008  Abs  PVWMI_Ct_mem_DemandLd_0
 0000:00000008  Abs  _OutMsg
 0000:00000009  Abs  _OutMsglc
 0000:00000009  Abs  PVWMI_Ct_mem_Discard_0
 0000:0000000A  Abs  _OutMsgArg
 0000:0000000A  Abs  lblLen
 0000:0000000A  Abs  PVWMI_Ct_mem_SwapOut_0
 0000:0000000A  Abs  dhFrameIP
 0000:0000000B  Abs  _OutMsgArglc
 0000:0000000B  Abs  lbl2Len
 0000:0000000B  Abs  PVWMI_Ct_mem_SwapIn_0
 0000:0000000C  Abs  PVWMI_Ct_mem_Reassigned_0
 0000:0000000C  Abs  _OutStrPtr
 0000:0000000C  Abs  dhFrameCS
 0000:0000000D  Abs  PVWMI_Ct_mem_Reassigned_1
 0000:0000000D  Abs  _OutStrPtrlc
 0000:0000000E  Abs  _OutByteHexPtr
 0000:0000000E  Abs  PVWMI_LQ_mem_QUsed_0
 0000:0000000F  Abs  _OutByteHexAddr
 0000:0000000F  Abs  PVWMI_EQ_mem_QUsed_0
 0000:00000010  Abs  _OutWordHexPtr
 0000:00000010  Abs  PVWMI_LQ_mem_QCTResident_0
 0000:00000011  Abs  PVWMI_EQ_mem_QCTResident_0
 0000:00000011  Abs  _OutWordHexAddr
 0000:00000012  Abs  Bmp_SegSize
 0000:00000012  Abs  _OutWordHexArg
 0000:00000012  Abs  PVWMI_LQ_mem_QFree_0
 0000:00000013  Abs  PVWMI_EQ_mem_QFree_0
 0000:00000013  Abs  _Out24HexPtr
 0000:00000014  Abs  PVWMI_Ct_mem_Idled_0
 0000:00000014  Abs  _Out24HexArg
 0000:00000014  Abs  GPTTFCHECKSIZE
 0000:00000015  Abs  PVWMI_Ct_mem_Recovered_0
 0000:00000015  Abs  _OutGateOffstPtr
 0000:00000016  Abs  PVWMI_ET_cal_Masm_0
 0000:00000016  Abs  _OutDescLimitPtr
 0000:00000017  Abs  PVWMI_CtST_cal_Masm_0
 0000:00000017  Abs  _OutDescBasePtr
 0000:00000018  Abs  _OutDwordHexPtr
 0000:00000018  Abs  PVWMI_ET_cal_C_0
 0000:00000019  Abs  _OutDwordHexAddr
 0000:00000019  Abs  PVWMI_CtST_cal_C_0
 0000:0000001A  Abs  PVWMI_ET_thd_FileIOWait_0
 0000:0000001A  Abs  _OutDwordHexArg
 0000:0000001B  Abs  _OutByteDecPtr
 0000:0000001B  Abs  PVWMI_ET_thd_FileIOWait_1
 0000:0000001C  Abs  PVWMI_ET_thd_FileIOWait_2
 0000:0000001C  Abs  KMCHECKEVENTSIZE
 0000:0000001C  Abs  _OutWordDecPtr
 0000:0000001D  Abs  _OutBitFHexPtr
 0000:0000001D  Abs  PVWMI_ET_thd_FileIOWait_3
 0000:0000001E  Abs  _OutBitFHexArg
 0000:0000001E  Abs  PVWMI_ST_thd_FileIOWait_0
 0000:0000001F  Abs  PVWMI_ST_thd_FileIOWait_1
 0000:0000001F  Abs  _OutMsgIfBitSet
 0000:00000020  Abs  PVWMI_ST_thd_FileIOWait_2
 0000:00000020  Abs  _OutMsgIfBitClr
 0000:00000021  Abs  PVWMI_ST_thd_FileIOWait_3
 0000:00000021  Abs  _OutMsgIfBitSetArg
 0000:00000022  Abs  PVWMI_Ct_fbc_RdHit_0
 0000:00000022  Abs  _OutMsgIfBitClrArg
 0000:00000023  Abs  PVWMI_Ct_fbc_RdMiss_0
 0000:00000023  Abs  _OutMsgIfBitSetlc
 0000:00000024  Abs  _OutMsgIfBitSetAddrlc
 0000:00000024  Abs  PVWMI_Ct_fbc_WrtHit_0
 0000:00000025  Abs  _JumpIfEQ
 0000:00000025  Abs  PVWMI_Ct_fbc_WrtMiss_0
 0000:00000026  Abs  PVWMI_Ct_fbc_WrtActiv_0
 0000:00000026  Abs  _OutMsgIfBitClrlc
 0000:00000027  Abs  _OutMsgIfBitSetArglc
 0000:00000027  Abs  PVWMI_Ct_fbc_Bypass_0
 0000:00000028  Abs  PVWMI_ET_spr_Spare1_0
 0000:00000028  Abs  _OutMsgIfBitClrArglc
 0000:00000028  Abs  HeaderLen
 0000:00000029  Abs  _PushData
 0000:00000029  Abs  PVWMI_ST_spr_Spare1_0
 0000:0000002A  Abs  PVWMI_CtST_spr_Spare1_0
 0000:0000002A  Abs  _PushArg
 0000:0000002B  Abs  _LoadCache
 0000:0000002B  Abs  PVWMI_Ct_spr_Spare1_0
 0000:0000002C  Abs  PVWMI_ET_spr_Spare1_1
 0000:0000002C  Abs  _CallOp
 0000:0000002D  Abs  PVWMI_ST_spr_Spare1_1
 0000:0000002D  Abs  _JumpOp
 0000:0000002E  Abs  _OutMsgBitF
 0000:0000002E  Abs  PVWMI_CtST_spr_Spare1_1
 0000:0000002F  Abs  PVWMI_Ct_spr_Spare1_1
 0000:0000002F  Abs  _OutMsgBitFlc
 0000:00000030  Abs  PVWMI_ET_spr_Spare2_0
 0000:00000030  Abs  _JumpIfBitF
 0000:00000031  Abs  _JumpIfBitF_AE_DwordAddr
 0000:00000031  Abs  PVWMI_ST_spr_Spare2_0
 0000:00000032  Abs  _JumpIfBitSet
 0000:00000032  Abs  PVWMI_CtST_spr_Spare2_0
 0000:00000033  Abs  PVWMI_Ct_spr_Spare2_0
 0000:00000033  Abs  _JumpIfBitClr
 0000:00000034  Abs  PVWMI_ET_spr_Spare2_1
 0000:00000034  Abs  _JumpIfDwordNull
 0000:00000035  Abs  _JumpIfEnv286
 0000:00000035  Abs  PVWMI_ST_spr_Spare2_1
 0000:00000036  Abs  _JumpIfEnv386
 0000:00000036  Abs  PVWMI_CtST_spr_Spare2_1
 0000:00000037  Abs  _CaseJump
 0000:00000037  Abs  PVWMI_Ct_spr_Spare2_1
 0000:00000038  Abs  PVWMI_ET_spr_Spare3_0
 0000:00000038  Abs  _InSwitchStr
 0000:00000039  Abs  _InBytePtr
 0000:00000039  Abs  PVWMI_ST_spr_Spare3_0
 0000:0000003A  Abs  _InWordPtr
 0000:0000003A  Abs  PVWMI_CtST_spr_Spare3_0
 0000:0000003B  Abs  _InWordArg
 0000:0000003B  Abs  PVWMI_Ct_spr_Spare3_0
 0000:0000003C  Abs  PVWMI_ET_spr_Spare3_1
 0000:0000003C  Abs  _In24bitArg
 0000:0000003D  Abs  _InDwordArg
 0000:0000003D  Abs  PVWMI_ST_spr_Spare3_1
 0000:0000003E  Abs  _InBitFArg
 0000:0000003E  Abs  PVWMI_CtST_spr_Spare3_1
 0000:0000003F  Abs  _SetBitArg
 0000:0000003F  Abs  PVWMI_Ct_spr_Spare3_1
 0000:00000040  Abs  PVWMI_ET_spr_Spare4_0
 0000:00000040  Abs  _ClearBitArg
 0000:00000041  Abs  _ToggleBitArg
 0000:00000041  Abs  PVWMI_ST_spr_Spare4_0
 0000:00000042  Abs  _JumpIfInCharEQ
 0000:00000042  Abs  PVWMI_CtST_spr_Spare4_0
 0000:00000043  Abs  _JumpIfEOL
 0000:00000043  Abs  PVWMI_Ct_spr_Spare4_0
 0000:00000044  Abs  PVWMI_ET_spr_Spare4_1
 0000:00000044  Abs  _GetInBuf
 0000:00000045  Abs  PVWMI_ST_spr_Spare4_1
 0000:00000046  Abs  PVWMI_CtST_spr_Spare4_1
 0000:00000047  Abs  PVWMI_Ct_spr_Spare4_1
 0000:00000048  Abs  PVWMI_ET_spr_Spare5_0
 0000:00000049  Abs  PVWMI_ST_spr_Spare5_0
 0000:0000004A  Abs  PVWMI_CtST_spr_Spare5_0
 0000:0000004B  Abs  PVWMI_Ct_spr_Spare5_0
 0000:0000004C  Abs  PVWMI_ET_spr_Spare5_1
 0000:0000004D  Abs  PVWMI_ST_spr_Spare5_1
 0000:0000004E  Abs  PVWMI_CtST_spr_Spare5_1
 0000:0000004F  Abs  PVWMI_Ct_spr_Spare5_1
 0000:00000050  Abs  PVWMI_ET_spr_Spare6_0
 0000:00000051  Abs  PVWMI_ST_spr_Spare6_0
 0000:00000052  Abs  PVWMI_CtST_spr_Spare6_0
 0000:00000053  Abs  PVWMI_Ct_spr_Spare6_0
 0000:00000054  Abs  PVWMI_ET_spr_Spare6_1
 0000:00000055  Abs  PVWMI_ST_spr_Spare6_1
 0000:00000056  Abs  PVWMI_CtST_spr_Spare6_1
 0000:00000057  Abs  PVWMI_Ct_spr_Spare6_1
 0000:00000058  Abs  PVWMI_ET_spr_Spare7_0
 0000:00000059  Abs  PVWMI_ST_spr_Spare7_0
 0000:0000005A  Abs  PVWMI_CtST_spr_Spare7_0
 0000:0000005B  Abs  PVWMI_Ct_spr_Spare7_0
 0000:0000005C  Abs  PVWMI_ET_spr_Spare7_1
 0000:0000005D  Abs  PVWMI_ST_spr_Spare7_1
 0000:0000005E  Abs  PVWMI_CtST_spr_Spare7_1
 0000:0000005F  Abs  PVWMI_Ct_spr_Spare7_1
 0000:00000060  Abs  PVWMI_ET_spr_Spare8_0
 0000:00000061  Abs  PVWMI_ST_spr_Spare8_0
 0000:00000062  Abs  PVWMI_CtST_spr_Spare8_0
 0000:00000063  Abs  PVWMI_Ct_spr_Spare8_0
 0000:00000064  Abs  PVWMI_ET_spr_Spare8_1
 0000:00000065  Abs  PVWMI_ST_spr_Spare8_1
 0000:00000066  Abs  PVWMI_CtST_spr_Spare8_1
 0000:00000067  Abs  PVWMI_Ct_spr_Spare8_1
 0000:00000068  Abs  PVWMI_ET_spr_Spare9_0
 0000:00000069  Abs  PVWMI_ST_spr_Spare9_0
 0000:0000006A  Abs  PVWMI_CtST_spr_Spare9_0
 0000:0000006B  Abs  PVWMI_Ct_spr_Spare9_0
 0000:0000006C  Abs  PVWMI_ET_spr_Spare9_1
 0000:0000006D  Abs  PVWMI_ST_spr_Spare9_1
 0000:0000006E  Abs  PVWMI_CtST_spr_Spare9_1
 0000:0000006F  Abs  PVWMI_Ct_spr_Spare9_1
 0000:00000070  Abs  PVWMI_ET_spr_Spare10_0
 0000:00000071  Abs  PVWMI_ST_spr_Spare10_0
 0000:00000072  Abs  PVWMI_CtST_spr_Spare10_0
 0000:00000073  Abs  PVWMI_Ct_spr_Spare10_0
 0000:00000074  Abs  PVWMI_ET_spr_Spare10_1
 0000:00000075  Abs  PVWMI_ST_spr_Spare10_1
 0000:00000076  Abs  PVWMI_CtST_spr_Spare10_1
 0000:00000077  Abs  PVWMI_Ct_spr_Spare10_1
 0000:00000200  Abs  DFSTKLEN
 0000:00000400  Abs  NWDSTKLEN
 0000:00000400  Abs  MSSTACKSIZE
 0000:00000400  Abs  IDTLEN
 0000:00000800  Abs  MESSAGE_BUFFER_LENGTH
 0001:00000000       DosGroupBase
 0001:00000000       _StartSTART
 0001:00000000       SAS_base_area
 0001:00000020       SAS_dd_area
 0001:00000026       ABIOS_CDA_anchor_p
 0001:00000028       ABIOS_CDA_anchor_r
 0001:0000002C       SAS_vm_area
 0001:0000005C       SAS_task_area
 0001:0000006E       SAS_RAS_area
 0001:00000078       SAS_file_area
 0001:00000084       SysInfoSeg
 0001:00000084       _SysInfoSeg
 0001:00000086       LocInfoSeg
 0001:00000086       _LocInfoSeg
 0001:0000008A       LocInfoSegRM
 0001:0000008E       CDIB_selector
 0001:00000100       RAS_BIOS_data
 0001:00000280       SISData
 0001:00000280       _SISData
 0001:00000300       MSStack
 0001:00000707       TSS
 0001:00000707       _tssTK
 0001:00000770       _EndSTART
 0001:00000770       Country_Code
 0001:00000770       _StartCONSTANTS
 0001:00000772       LeadByteTable
 0001:0000077A       NullLeadByteTable
 0001:0000077C       CharType
 0001:0000087C       UNCfscList
 0001:000008A0       UNCfscLast
 0001:000008AC       ksemMFT
 0001:000008BC       ksemVPB
 0001:000008CE       dynam_API_table
 0001:000009CE       dynam_ret_table
 0001:000009F2       _flGlobalActions
 0001:000009F2       Resched
 0001:000009F2       _Resched
 0001:000009F7       InDos
 0001:000009F7       _cInDos
 0001:000009F8       sgspid
 0001:00000A18       state_nmi
 0001:00000A1A       NPX_Owner
 0001:00000A1C       UserNum
 0001:00000A1F       OEMNum
 0001:00000A20       RASDevHelpDS
 0001:00000A22       RASDevHelpDX
 0001:00000A24       DekkoPhysAddr
 0001:00000A28       ras_mec_table
 0001:00000A28       ras_mec_table_flat
 0001:00000A48       ras_systr_flags
 0001:00000A49       ras_systr_flags2
 0001:00000A4A       _ras_perf_mec_table
 0001:00000A4A       _ras_perf_mec_table_flat
 0001:00000A6A       ras_stda_addr
 0001:00000A6A       _RASselSTDA
 0001:00000A6C       ras_lost_events
 0001:00000A6E       ras_stda_oldest
 0001:00000A70       ras_stda_num
 0001:00000A72       ras_sync_Pid
 0001:00000A74       _ras_pname_head
 0001:00000A74       ras_pname_head
 0001:00000A78       ras_max_sysdata
 0001:00000A7A       TraceValue
 0001:00000A7B       ras_sysdata_flags
 0001:00000A7F       ras_lock_flags
 0001:00000A81       ras_lock_count
 0001:00000A9C       _ptcbTKEvap
 0001:00000AA0       TaskData
 0001:00000AA2       TaskNumber
 0001:00000AA2       _TaskNumber
 0001:00000AA6       _ThreadCount
 0001:00000AAA       COPROCFakeState
 0001:00000AAA       _COPROCFakeState
 0001:00000AAC       _MaxProcesses
 0001:00000AAC       MaxProcesses
 0001:00000AB0       MaxThreads
 0001:00000AB0       _MaxThreads
 0001:00000AB2       TCResched
 0001:00000AB2       _TCResched
 0001:00000AB3       DynTimeSlice
 0001:00000AB3       _DynTimeSlice
 0001:00000AB4       fAPMidle
 0001:00000AB4       _fAPMidle
 0001:00000AB5       papTCBPtrs
 0001:00000AB7       papTCBPtrs_seg
 0001:00000ABA       DevhlpFuncDisp
 0001:00000C46       SchedPtr
 0001:00000C4A       ScrnIoOk
 0001:00000C4B       CurProcSG
 0001:00000C4C       CurProcSW
 0001:00000C4E       CurProcPID
 0001:00000C54       VectorReboot
 0001:00000C58       VectorMSATS
 0001:00000C60       VectorSDF
 0001:00000C64       VectorDEKKO
 0001:00000C68       VectorRIPL
 0001:00000C90       DevClassTables
 0001:00000C94       LastDPB
 0001:00000C98       DHF
 0001:00000D6A       sysini_handle
 0001:00000D6C       SICG_SS_SP
 0001:00000D7C       _DOSCALL1
 0001:00000D84       LoadDevDrv
 0001:00000D86       Sctmask
 0001:00000D88       DBCS_Codepg
 0001:00000D8A       hVPBFirst
 0001:00000D8A       _hVPBFirst
 0001:00000D8C       pVPBBuf
 0001:00000D90       pVPBSem
 0001:00000D91       DriveLetter
 0001:00000DAB       DiffNam
 0001:00000DAC       MyName
 0001:00000DBC       MyNum
 0001:00000DBE       DPBHead
 0001:00000DC2       SFT_FreeHead
 0001:00000DC6       _MFT_hPTree
 0001:00000DC6       MFT_hPTree
 0001:00000DCA       Serial
 0001:00000DCC       RLRHead
 0001:00000DCE       BClock
 0001:00000DD4       EGAPresent
 0001:00000DD5       EGADevice
 0001:00000DD9       ConInpDev
 0001:00000DDF       ConOutDev
 0001:00000DE5       MaxSec
 0001:00000DE7       CDSAddr
 0001:00000DEB       NumIO
 0001:00000DEB       _NumIO
 0001:00000DEC       NumIORipl
 0001:00000DEC       _NumIORipl
 0001:00000DED       _NumIOReserveDriveLetter
 0001:00000DED       NumIOReserveDriveLetter
 0001:00000DEE       _ReserveDriveLetterStart
 0001:00000DEE       ReserveDriveLetterStart
 0001:00000DEF       uchLastDrive
 0001:00000DEF       _uchLastDrive
 0001:00000DF0       DevHlp
 0001:00000DF4       NULdev
 0001:00000DF4       DevHead
 0001:00000E0E       Splices
 0001:00000E10       CONdev
 0001:00000E2A       OEMdev
 0001:00000E44       CharDevRMPRec
 0001:00000E48       CharDevSem
 0001:00000E54       CNotifySem
 0001:00000E60       _UdelSem
 0001:00000E6C       SpoolDevRMPRec
 0001:00000E70       SpoolDevSem
 0001:00000E7C       MUF_Pid
 0001:00000E7E       HDE_Pid
 0001:00000E80       Day
 0001:00000E81       Month
 0001:00000E82       Year
 0001:00000E84       DayCnt
 0001:00000E86       WeekDay
 0001:00000E87       OEM_handler
 0001:00000E8B       ProtOnlySystem
 0001:00000E8C       DevConfigTbl
 0001:00000E8C       numPtr
 0001:00000E8D       numSerial
 0001:00000E8E       numDisk
 0001:00000E8F       mathCop
 0001:00000E8F       _mathcop
 0001:00000E90       devConReser
 0001:00000E91       pcType
 0001:00000E92       displAdap
 0001:00000E94       RSL_SelDS
 0001:00000E94       RmSelLst
 0001:00000E96       RSL_SelES
 0001:00000E98       RSL_SelDMAAdd
 0001:00000E9A       RSL_SelJFN1
 0001:00000E9C       GDTDesc
 0001:00000EA2       IDTDesc
 0001:00000EA8       _CpuType
 0001:00000EAC       _CpuStepping
 0001:00000EB0       _Pentium_Vendor_ID
 0001:00000EBC       _Pentium_Stepping
 0001:00000EC0       _Pentium_Feature_Flags
 0001:00000EC4       _SigFocus
 0001:00000EC4       SigFocus
 0001:00000F04       PendingSignals
 0001:00000F06       PendingSigArg
 0001:00000F16       _GDT_SAS
 0001:00000F18       _GDT_RLR
 0001:00000F1A       _GDT_VPB
 0001:00000F1C       _GDT_PTDA
 0001:00000F1E       _GDT_TSS
 0001:00000F20       _DOSGROUP
 0001:00000F22       _ABIOS_present
 0001:00000F22       ABIOS_present
 0001:00000F23       NoInt21Flag
 0001:00000F24       _CpuVendor
 0001:00000F28       _Sis2
 0001:00000F34       _Lis2
 0001:00000F40       rwSysInfoSeg
 0001:00000F42       SMHotKeyQ
 0001:00000F50       CtrlNumLkQ
 0001:00000F5E       SMDosSessionQ
 0001:00000F6C       HardErrPkt
 0001:00001280       CtrlPrtScQ
 0001:0000128E       JITLaunchPkt
 0001:000012A8       JITLaunchPkt2
 0001:000012E2       VideoPauseFlag
 0001:000012F0       _StartIDTDATA
 0001:000012F0       _EndCONSTANTS
 0001:000012F0       IDT
 0001:00001328       NPXNAVec
 0001:00001360       IDTTrap0E
 0001:000013F8       Int21Vec
 0001:000016F0       _StartDATA
 0001:000016F0       ReqPktSegs
 0001:000016F0       _EndIDTDATA
 0001:00001704       MaxReqPktsSegs
 0001:0000170A       FirstPacket
 0001:00003D9A       LastPacket
 0001:00003D9A       s2BmpSel
 0001:00003D9C       iDevCall
 0001:00003DC6       iRMNCall
 0001:00003DFE       LogDDCS
 0001:00003E00       LogDDIdc
 0001:00003E02       LogDDDS
 0001:00003E04       PhysDiskTablePtr
 0001:00003E10       CodePgBuff
 0001:00003E24       sSysPCB
 0001:00003E28       cProfCall
 0001:00003E2A       achMod
 0001:00003E38       _szTempBuf
 0001:00003F3C       _TempDelFileInfo
 0001:0000406C       DevPrefix
 0001:00004072       fFSSwapStarted
 0001:00004073       _CodeLockArray
 0001:0000426C       DOS_Abort_Close
 0001:0000427D       EADirName
 0001:000042B4       UNKNOWN_FSD_name
 0001:000042BC       FAT_FSD_name
 0001:000042C0       PRN_Device_Name
 0001:000042C4       LPT1_Device_Name
 0001:000042D0       MFSD_Stage
 0001:000042D1       szKBD
 0001:00004348       initfatchkdsk
 0001:0000434A       NmpBmpSel
 0001:0000434C       NmpRmpHand
 0001:0000435E       CNotifyGlobal_Count
 0001:00004376       NextCDSHandle
 0001:00004386       SFNAllocCtr
 0001:0000438A       SFT_GrowSem
 0001:0000438C       pbufWPT
 0001:00004390       semWPT
 0001:00004392       FSPrtyIO_Mode
 0001:00004394       FATCache
 0001:00004396       _GlobalPvwQSize
 0001:0000439A       _GlobalVME
 0001:0000439B       GlobalAutoFail
 0001:0000439C       _SuppressPopUps
 0001:0000439D       _PopUpLogDrive
 0001:0000439E       _UMB_ON
 0001:0000439F       _RASKData
 0001:000043A0       _DLLBasing
 0001:000043A6       PtoV_Selectors
 0001:0000442A       hDiscSegRmpStruc
 0001:00004432       _SMswapping
 0001:00004434       _SMCFGMinFree
 0001:00004438       _SMCFGSwapSize
 0001:0000443C       _SMCommit
 0001:0000443E       ShareRmpStruc
 0001:0000444A       ErrMap24
 0001:0000445F       ErrMap24End
 0001:0000445F       MsgMap24
 0001:00004474       MsgMap24End
 0001:00004478       MuxTable
 0001:00004EE2       DumpProc
 0001:00004EE6       _DUMP_ON
 0001:00004EE6       DUMP_ON
 0001:00004EE7       REIPL_ON
 0001:00004EE8       DumpDevice
 0001:00004EE8       _DumpDevice
 0001:00004EF0       ras_min_table
 0001:00004EF0       _ras_min_table
 0001:00004F22       _cTKNoBlock
 0001:00004F24       CurrentRamSemID
 0001:00004F26       SmlPostCt
 0001:00004F2A       Initialize_Flags
 0001:00004F32       SysSemDataTable
 0001:00005532       SysSemRmpHdl
 0001:0000573C       semaphore
 0001:0000573D       slot_present
 0001:0000573E       handler_list
 0001:0000595E       handler_max
 0001:00005960       semaphore_handle
 0001:00005D4C       XCPTXferBuffer
 0001:00005F2A       _InterruptLevel
 0001:00005F2A       InterruptLevel
 0001:00005F2E       CurrIntLevel
 0001:00005F32       CADCount
 0001:00005F34       CADHookHandle
 0001:00005F38       DiskDCTable
 0001:000061FC       MouseDCTable
 0001:00006250       fIBMSystem
 0001:00006252       ArenaInfo
 0001:00006256       RealInitDS
 0001:00006258       _ABIOS_Revision
 0001:00006258       ABIOS_Revision
 0001:00006259       ACHK_FLAG
 0001:0000625A       mFSD_FLAG
 0001:0000625B       pMiniFSD
 0001:0000625F       _ulPICMask
 0001:00006263       NPX_Type
 0001:00006263       _NPX_Type
 0001:00006264       twodiskboot
 0001:00006266       mifs_ptr
 0001:0000626A       _IsMiniIFS
 0001:0000626B       pLAZCur
 0001:0000626F       DMQS_Sel
 0001:00006271       APM_CodeSeg
 0001:00006273       APM_DataSeg
 0001:00006275       APM_Offset
 0001:00006277       APM_Flags
 0001:00006279       APM_Level
 0001:0000627B       APM_IdleHookRtn
 0001:00006281       APM_32CodeSeg
 0001:00006283       APM_32Offset
 0001:00006287       _DDInitTime
 0001:00006288       _InitCodeInvalid
 0001:00006289       syiGlobalFlags
 0001:0000628E       BytesPerSector
 0001:00006290       FatDirtyBit
 0001:000062BB       DirBufferSelector
 0001:000062C1       OS2DirBufferSelector
 0001:000062C3       OS2BOOTDirBufferSelector
 0001:000062D4       FileBufferAddress
 0001:000062D8       FileBufferLength
 0001:00006339       FileReadBuffer
 0001:00006340       BootBPB
 0001:00006360       _LDRDDOwner
 0001:00006362       _LDRFSDOwner
 0001:00006364       _pgPhysPageDir
 0001:000063DE       mutexCreateVDM
 0001:000063E2       eventCreateVDM
 0001:000063EA       NWDStackBase
 0001:000067EA       NWDTss
 0001:00006852       cMaxNMI
 0001:00006856       cMaxKNMI
 0001:0000685A       cNMI
 0001:00006862       fNWDEnabled
 0001:00006863       fNWD
 0001:000068F1       isa_error
 0001:000068F2       _ShutdownFlag
 0001:000068F6       fDebugOnly
 0001:000068F8       _tkPanicActive
 0001:000068F9       nPanic
 0001:000068FD       fPanicToScreen
 0001:0000695A       VPUserSelector
 0001:0000695C       _AssertAlignESP
 0001:00006960       _AssertAlignESPPanic
 0001:00006B48       DFStackBase
 0001:00006D48       DFTss
 0001:00006E20       ras_krnl_type
 0001:00006EA6       segDebugCS
 0001:00006EA8       _EndDWORDDATA
 0001:00006EA8       _StartDWORDDATA
 0001:00006EA8       lbl
 0001:00006EA8       _StartTABLE
 0001:00006EA8       _EndDATA
 0001:00006EB2       lbl2
 0001:00006EBD       minimumBPB
 0001:00006EDC       MSVERS
 0001:00006EDE       YRTAB
 0001:00006EE6       MONTAB
 0001:00006EF2       I21_MAP_E_TAB
 0001:0000705A       Err_Table_21
 0001:00007136       Err_Table_24
 0001:00007196       DOSTable
 0001:000071D7       RedirCallOut
 0001:00007224       pgMstable
 0001:00007259       Header
 0001:00007286       _StartINTERRMSG
 0001:00007286       _EndTABLE
 0001:0000780A       _StartABIOSDATA
 0001:0000780A       _EndINTERRMSG
 0001:00007810       ABIOS_DH_present
 0001:00007845       ABIOS_System_Parameter_Table
 0001:00007865       ProtSegSize
 0001:00007867       RealCDASel
 0001:00007869       _EndABIOSDATA
 0001:00007869       _StartLASTDATA
 0001:00007871       _StartEENDDATA
 0001:00007871       _EndLASTDATA
 0002:00000000       _StartFIRSTCODE
 0002:00000001       RETFDLabel
 0002:0000000C       BUGBITS
 0002:00000018       modesw$h_RealMode
 0002:0000001A       RealMode
 0002:00000168       modesw$h_RealModeNoInt
 0002:0000016A       RealModeNoInt
 0002:00000174       ProtModeSub
 0002:00000238       _StartCODE
 0002:00000238       _EndFIRSTCODE
 0002:00000238       h_w_Beep
 0002:0000023A       w_Beep
 0002:0000023A       DosBeep_PreTrace
 0002:00000255       DosBeep_PostTrace
 0002:00000258       h_DevDeInstall
 0002:0000025A       DevDeInstall
 0002:000002A8       h_DevIOCall
 0002:000002AC       h_DevIOCall2
 0002:000002B0       f_DevIOCall2
 0002:000002B2       DevIOCall2
 0002:000002B9       DevIOCall
 0002:0000041C       h_GetTCBReqPkt
 0002:00000420       f_GetTCBReqPkt
 0002:00000422       GetTCBReqPkt
 0002:00000488       h_w_CallPddIoctl
 0002:000004C4       h_S2AllocReqPkt
 0002:000004C8       f_AllocReqPacketWait
 0002:000004D0       h_AllocReqPacketWait
 0002:000004D2       AllocReqPacketWait
 0002:000004F1       S2AllocReqPkt
 0002:0000057C       dh_AllocReqPacket
 0002:000005FC       h_dh_FreeReqPacket
 0002:00000600       f_dh_FreeReqPacket
 0002:00000602       dh_FreeReqPacket
 0002:0000066C       h_FreeReqPacket
 0002:00000670       f_FreeReqPacket
 0002:00000672       FreeReqPacket
 0002:000006E4       h_SetRead
 0002:000006E6       SetRead
 0002:000006E8       SetRdNA
 0002:0000072D       h_SetWrite
 0002:0000072F       SetWrite
 0002:00000731       SetWrNA
 0002:00000740       h_SetReadNoAlloc
 0002:00000744       h_SetWriteNoAlloc
 0002:00000748       sNULdev
 0002:0000074E       iNULdev
 0002:00000750       sCONdev
 0002:00000756       iCONdev
 0002:00000758       dh_RealToProt
 0002:00000768       dh_ProtToReal
 0002:00000778       dh_RAS
 0002:00000790       dh_PerfSysTrace
 0002:000007C8       h_dh_AttachDD
 0002:000007CA       dh_AttachDD
 0002:0000085C       dh_InternalError
 0002:00000864       dh_LogEntry
 0002:00000950       Save_Message
 0002:0000095C       dh_VideoPause
 0002:000009A8       dh_Beep
 0002:000009DC       dh_RegisterBeep
 0002:000009F8       dh_RegisterFreq
 0002:00000A14       dh_MonWrite
 0002:00000A74       dh_MonFlush
 0002:00000A94       dh_MonitorCreate
 0002:00000AB0       dh_Register
 0002:00000ACC       dh_DeRegister
 0002:00000AE8       f_NotifyMonNotify
 0002:00000AF0       f_DoProfile
 0002:00000B20       CountTic
 0002:00000B64       use16Tick
 0002:00000BC8       flatTick
 0002:00000C54       dh_RegisterProfile
 0002:00000C6C       h_TestDBCSLOW
 0002:00000C70       f_TestDBCSLOW
 0002:00000C72       TestDBCSLOW
 0002:00000C84       h_FindChar
 0002:00000C88       f_FindChar
 0002:00000C8A       FindChar
 0002:00000CB4       GetRR
 0002:00000CC4       GetExtent
 0002:00000CD8       SetExtent
 0002:00000CF4       h_GetExtended
 0002:00000CF8       f_GetExtended
 0002:00000CFA       GetExtended
 0002:00000D08       GetRecSize
 0002:00000D18       f_FCBIO
 0002:00000EE0       FSH_INTERR
 0002:00000EF4       FSH_SEMREQUEST
 0002:00000F1C       FSH_SEMCLEAR
 0002:00000F3C       FSH_IOSEMCLEAR
 0002:00000F5C       FSH_YIELD
 0002:00000F64       misc$VerifyLog2
 0002:00000F78       h_SetVPB
 0002:00000F7A       SetVPB
 0002:00001094       h_RetryWait
 0002:00001098       f_RetryWait
 0002:0000109A       RetryWait
 0002:000010B4       misc$Far_SetBad
 0002:000010BC       misc$SetBad
 0002:000010D4       RedirDispAddr
 0002:000010D8       Redir_Dispatcher
 0002:000010E0       Far_RetCC
 0002:000010F4       h_VirtToPhysDM
 0002:000010F6       VirtToPhysDM
 0002:00001100       h_VirtToPhys
 0002:00001104       f_VirtToPhys
 0002:00001106       VirtToPhys
 0002:00001178       f_dh_PhysToUVirt
 0002:0000117A       dh_PhysToUVirt
 0002:00001210       AllocPhysDM
 0002:000012A8       FreePhysDM
 0002:000012EC       h_AllocateGDTSelector
 0002:00001314       dh_AllocateGDTSelector
 0002:00001330       h_FreeGDTSelector
 0002:00001332       FreeGDTSelector
 0002:00001332       dh_FreeGDTSelector
 0002:00001340       h_PhysToGDTSelector
 0002:00001342       dh_PhysToGDTSelector
 0002:00001342       PhysToGDTSelector
 0002:00001380       dh_PhysToGDTSel
 0002:00001390       dh_GetDescInfo
 0002:000013E0       f_PhysToVirtDM
 0002:000013E2       PhysToVirtDM
 0002:000013E2       dh_PhysToVirt
 0002:000013F4       h_PhysToVirt
 0002:000013F6       PhysToVirt
 0002:000014D0       UnPhysToVirtDM
 0002:000014D0       dh_UnPhysToVirt
 0002:000014E0       dh_VirtToLin
 0002:000014F0       dh_LinToGDTSelector
 0002:0000150C       dh_PageListToGDTSelector
 0002:00001608       SegLockDM
 0002:0000166C       SegUnlockDM
 0002:0000168C       dh_ReallocSeg
 0002:000016E4       dh_VMLock
 0002:00001734       dh_VMUnlock
 0002:00001768       dh_VMGlobalToProcess
 0002:000017B4       dh_VMProcessToGlobal
 0002:00001800       dh_VMAlloc
 0002:000018C8       dh_VMFree
 0002:00001918       dh_VMSetMem
 0002:0000194C       dh_VerifyAccess
 0002:00001978       dh_LinToPageList
 0002:000019A0       dh_PageListToLin
 0002:00001A3C       dh_DynamicAPI
 0002:00001A44       modesw$SelToPhys
 0002:00001AF0       h_SelToSeg
 0002:00001AF2       SelToSeg
 0002:00001B10       KFGotoReal
 0002:00001B40       KFGotoProt
 0002:00001B68       modesw$h_ProtMode
 0002:00001B6A       modesw$ProtMode
 0002:00001B6A       ProtMode
 0002:00001B78       modesw$h_ProtModeICSub
 0002:00001B84       h_RealOnly
 0002:00001B86       RealOnly
 0002:00001BA4       h_ProtOnly
 0002:00001BA6       ProtOnly
 0002:00001BC4       h_TaskOnly
 0002:00001BC8       f_TaskOnly
 0002:00001BCA       TaskOnly
 0002:00001BEC       h_RealProcTaskOnly
 0002:00001BEE       RealProcTaskOnly
 0002:00001C0C       h_RealTaskOnly
 0002:00001C0E       RealTaskOnly
 0002:00001C18       h_ProtTaskOnly
 0002:00001C1A       ProtTaskOnly
 0002:00001C24       h_GoProtAll
 0002:00001C26       GoProtAll
 0002:00001C60       h_GoRealAll
 0002:00001C62       GoRealAll
 0002:00001C88       Reboot
 0002:00001C94       redircall1
 0002:00001C9A       redircall2
 0002:00001CA0       redirdisp1
 0002:00001CA4       redirdisp2
 0002:00001CA8       f_EvtWakeMuxWait16
 0002:00001CB0       SysWakeMuxWait
 0002:00001CB8       RamWakeMuxWait
 0002:00001CDB       muxsem$WakeMuxWait
 0002:00001D10       h_EnableNMI
 0002:00001D14       f_EnableNMI
 0002:00001D16       EnableNMI
 0002:00001D48       h_DisableNMI
 0002:00001D4C       f_DisableNMI
 0002:00001D4E       DisableNMI
 0002:00001D80       RASRST
 0002:00001FB4       dh_ModifyPriority
 0002:00002024       DOSISEMREQUEST
 0002:0000208C       dh_SemRequest
 0002:000020B0       h_SemRequest
 0002:000020B4       f_SemRequest
 0002:000020B6       SemRequest
 0002:000020BA       sem$h_SemRequestSub
 0002:000020BC       sem$SemRequestSub
 0002:000020FC       sem$SysSemRequest
 0002:00002174       sem$FreezeCheck
 0002:000021B8       DOSISYSSEMCLEAR
 0002:00002218       h_w_RamSemWake
 0002:0000221C       f_w_RamSemWake
 0002:0000221E       w_RamSemWake
 0002:00002240       sem$h_FARRamSemWake
 0002:00002244       dh_SemClear
 0002:00002260       h_IOSemClear
 0002:00002264       f_IOSemClear
 0002:00002266       IOSemClear
 0002:00002274       h_SemClear
 0002:00002278       f_SemClear
 0002:0000227A       SemClear
 0002:000022C8       sem$RamSemWakeSub
 0002:00002377       sem$SysSemClear
 0002:000023D0       sem$h_SysSemWait
 0002:000023D2       sem$SysSemWait
 0002:00002400       sem$h_RamSemWait
 0002:00002402       sem$RamSemWait
 0002:00002448       h_SemBlock
 0002:0000244A       SemBlock
 0002:000024AC       h_VerifyRamSemAddr
 0002:000024AE       VerifyRamSemAddr
 0002:00002518       PutRamSemID
 0002:00002534       h_SemProtFault
 0002:00002536       SemProtFault
 0002:00002570       h_dh_OpenEventSem
 0002:00002572       dh_OpenEventSem
 0002:000025B4       h_dh_CloseEventSem
 0002:000025B6       dh_CloseEventSem
 0002:000025F8       h_dh_PostEventSem
 0002:000025FA       dh_PostEventSem
 0002:0000263C       h_dh_PMPostEventSem
 0002:0000263E       dh_PMPostEventSem
 0002:00002680       h_dh_ResetEventSem
 0002:00002682       dh_ResetEventSem
 0002:000026C4       h_PostPending
 0002:000026C8       f_PostPending
 0002:000026CA       PostPending
 0002:000026FC       sig$PostPendingSub
 0002:00002734       h_SigActive
 0002:00002738       f_SigActive
 0002:0000273A       SigActive
 0002:0000276C       dh_SemHandle
 0002:00002784       h_SemHandle
 0002:00002788       f_SemHandle
 0002:0000278A       SemHandle
 0002:000027F8       h_GetSysSemPtrChk
 0002:000027FC       GetSysSemPtrChk
 0002:00002800       GetSysSemPtr
 0002:00002838       h_GetSysSemPtr
 0002:0000283C       syssem$ChkSysSemPtr
 0002:00002870       h_w_SetDateTime
 0002:00002874       f_w_SetDateTime
 0002:00002876       w_SetDateTime
 0002:0000290B       time$common_write_clock
 0002:00002960       h_Date16
 0002:00002964       f_Date16
 0002:00002966       Date16
 0002:0000298C       h_ReadTime
 0002:0000298E       ReadTime
 0002:000029B8       DSUM
 0002:000029C4       CheckTime
 0002:000029F0       h_Calc_Date
 0002:000029F4       f_Calc_Date
 0002:000029F6       Calc_Date
 0002:00002A30       get_day_count
 0002:00002A88       f_DemWriteClock
 0002:00002A90       Tick_Handler
 0002:00002AEC       h_w_GetDateTime
 0002:00002AEE       w_GetDateTime
 0002:00002B20       w_EntryChk
 0002:00002B6C       w_MakeEntry
 0002:00002BC0       dh_SetTimer
 0002:00002BEC       dh_ResetTimer
 0002:00002C24       dh_TickCount
 0002:00002C6C       f_CallDHHookHandler
 0002:00002C78       dh_AllocateCtxHook
 0002:00002D0C       dh_FreeCtxHook
 0002:00002D44       dh_ArmCtxHook
 0002:00002DA4       Gen16HookAny_Low
 0002:00002E58       h_DeviceHelpRM
 0002:00002E5D       h_DeviceHelpDM
 0002:000030E4       dhrouter$dh_SetIRQ
 0002:000030F0       dhrouter$dh_UnSetIRQ
 0002:000030FC       dhrouter$dh_EOI
 0002:00003108       dhrouter$dh_SetROMVector
 0002:00003114       dhrouter$dh_RegisterStackUsage
 0002:00003120       dhrouter$dh_Sec
 0002:0000312C       dh_KillProc
 0002:00003160       dh_QSysState
 0002:000031AC       dhrouter$dh_RegisterPDD
 0002:00003208       dhrouter$dh_RegisterDeviceClass
 0002:00003298       dhrouter$dh_RegisterKrnlExit
 0002:000032C4       dhrouter$dh_CreateInt13VDM
 0002:00003308       dhrouter$dh_AbiosStub
 0002:00003310       SchedAddr
 0002:00003318       devhlp$SchedRet
 0002:0000332C       PullRequest
 0002:00003350       PullParticular
 0002:0000338C       PushRequest
 0002:000033C0       SortRequest
 0002:00003440       QueueFlush
 0002:00003450       QueueWrite
 0002:00003478       QueueRead
 0002:000034A8       GetDOSVar
 0002:00003528       dh_Yield
 0002:0000353C       dh_YieldTC
 0002:00003560       dh_ProcBlock
 0002:00003574       dh_ProcRun
 0002:00003580       dh_ProcRun2
 0002:000035A0       h_dh_SendEvent
 0002:000035A2       dh_SendEvent
 0002:000035F1       saba
 0002:000036DC       dh_RegisterKDD
 0002:00003794       f_BootDos16
 0002:0000383C       f_hyberReboot16
 0002:000038B4       dh_RegisterPerfCtrs
 0002:000038EC       h_NWDEnableWatchdogNMI
 0002:00003924       h_NWDDisableWatchdogNMI
 0002:00003928       f_NWDDisableWatchdogNMI
 0002:0000392A       NWDDisableWatchdogNMI
 0002:0000393C       h_NWDRestoreWatchdogNMI
 0002:0000395C       h_ProcessFreeze
 0002:00003960       f_ProcessFreeze
 0002:00003962       ProcessFreeze
 0002:0000398C       h_ProcBlock
 0002:0000398E       ProcBlock
 0002:000039F8       h_ProcRun
 0002:000039FA       ProcRun
 0002:00003A40       h_ProcRun2
 0002:00003A42       ProcRun2
 0002:00003A54       DevWait
 0002:00003A6C       DevDone
 0002:00003A88       h_w_Get_Version
 0002:00003A8C       f_w_Get_Version
 0002:00003A8E       w_Get_Version
 0002:00003AAC       h_DosHlpErr
 0002:00003ABC       h__InternalError
 0002:00003AF0       _tkPanic
 0002:00003AF7       subr$_tkPanicMsgLen
 0002:00003C2C       subr$ErrPrnt
 0002:00003C80       subr$DisplayAddress
 0002:00003CD8       subr$DisplayFmt
 0002:00003D20       subr$DisplayDecimal
 0002:00003D3C       subr$DisplayMsg
 0002:00003D5C       subr$DisplayAux
 0002:00003DB8       h_DisplayCrLf
 0002:00003DBA       DisplayCrLf
 0002:00003DC8       subr$FwordToAscii
 0002:00003DE8       h_IntToDecAscii
 0002:00003DEC       f_IntToDecAscii
 0002:00003DEE       IntToDecAscii
 0002:00003E3C       h_WrtToScrnClr
 0002:00003E40       f_WrtToScrnClr
 0002:00003E42       WrtToScrnClr
 0002:00003E54       h_WrtToScrn16
 0002:00003E5C       h_WrtToScrn
 0002:00003E60       f_WrtToScrn
 0002:00003E62       WrtToScrn
 0002:00003E74       subr$test_xga
 0002:00003F84       h_ClearAllInts
 0002:00003F88       f_ClearAllInts
 0002:00003F8A       ClearAllInts
 0002:00003FB0       h_ByteToScrnDM
 0002:00003FB4       f_ByteToScrnDM
 0002:00003FB6       ByteToScrnDM
 0002:000040D0       h_HexToAscii
 0002:000040D2       HexToAscii
 0002:000040DB       h_ByteToAscii
 0002:000040DD       ByteToAscii
 0002:000040E5       subr$NibbleToAscii
 0002:000040F4       h_StrLen
 0002:000040F8       f_StrLen
 0002:000040FA       StrLen
 0002:00004108       h_StrLen32
 0002:0000410C       f_StrLen32
 0002:0000410E       StrLen32
 0002:00004124       h_DStrLen
 0002:00004130       h_XCHGP
 0002:00004132       XCHGP
 0002:0000413C       h_SysServWake
 0002:00004140       f_SysServWake
 0002:00004142       SysServWake
 0002:0000414C       f_SysServQueueEvent
 0002:0000414E       SysServQueueEvent
 0002:000041CC       h_SysServChkDaemon
 0002:000041F8       tkmisc$CallRedir
 0002:00004210       tkmisc$h___panic
 0002:0000422C       tkmisc$h___panicfn
 0002:0000426E       tkmisc$h___panicfnmsg
 0002:000042E0       f___panic
 0002:000042E4       __panicfnmsgRM
 0002:00004310       h___panicsprintf
 0002:00004344       __panicLOW
 0002:0000434C       __panicRM
 0002:00004354       __panicfnLOW
 0002:0000435C       __panicfnmsgLOW
 0002:00004364       h_SchedClock
 0002:00004448       h_TCYield
 0002:0000444A       TCYield
 0002:00004478       h_Yield
 0002:0000447A       Yield
 0002:0000447C       h_SchedNext
 0002:0000447E       SchedNext
 0002:000044A4       far_dprintfRM
 0002:000044A8       far_doutcharRM
 0002:000044AC       h_dbtest
 0002:000044AE       dbtest
 0002:000044CE       h_DPRINTF
 0002:000044D0       DPRINTF
 0002:000044EC       h_dputs
 0002:000044EE       dputs
 0002:000044FF       h_dputchar
 0002:00004501       dputchar
 0002:00004517       dputcharnl
 0002:0000453C       f_Debug_BreakDM
 0002:0000453C       Debug_BreakDM
 0002:00004554       f_fdputs
 0002:00004556       fdputs
 0002:0000455C       dh_GetLIDEntry
 0002:0000455C       _StartABIOSCODE
 0002:0000455C       _EndCODE
 0002:00004568       h_GetLIDEntry
 0002:0000456A       GetLIDEntry
 0002:00004574       GetLID
 0002:0000468C       dh_FreeLIDEntry
 0002:00004698       h_FreeLIDEntry
 0002:0000469A       FreeLIDEntry
 0002:000046A4       FreeLID
 0002:000046F4       dh_ABIOSCall
 0002:00004700       h_ABIOSCall
 0002:00004702       ABIOSCall
 0002:0000470C       ABIOSEntry
 0002:000047B4       dh_ABIOSCommonEntry
 0002:00004850       dh_GetDeviceBlock
 0002:000048B4       dh_ABIOSGetParms
 0002:0000493C       IBMEnableNMI
 0002:00004964       IBMDisableNMI
 0002:0000498C       f_IntNMI
 0002:000049AC       _EndABIOSCODE
 0002:000049AC       dh_RegisterTmrDD
 0002:000049AC       _StartINITCODE
 0002:000049EC       MFSH_CALLRM
 0002:00004A88       MFSH_DOVOLIO
 0002:00004B8C       MFSH_INTERR
 0002:00004BA0       MFSH_SEGALLOC
 0002:00004C38       MFSH_SEGFREE
 0002:00004C6C       MFSH_SEGREALLOC
 0002:00004CBC       MFSH_SETBOOTDRIVE
 0002:00004CF0       MFSH_LOCK
 0002:00004D58       MFSH_PHYSTOVIRT
 0002:00004DBC       MFSH_UNLOCK
 0002:00004DE4       MFSH_UNPHYSTOVIRT
 0002:00004DF8       MFSH_VIRT2PHYS
 0002:00004E4C       f_w16_OpenPageFile
 0002:00004FE4       h_FS_EM_OpenPageFile
 0002:00005118       InitDiskTable
 0002:00005140       Get_Diskette_Data
 0002:00005198       Get_Disk_Data
 0002:00005214       h_InitDisk
 0002:00005228       dskinit$Get_IRQs
 0002:00005250       h_Get_Machine_Info
 0002:00005252       Get_Machine_Info
 0002:00005298       inicpu$CpuAbort
 0002:000052C4       CpuStepping
 0002:00005394       inicpu$CheckB1
 0002:000053BC       inicpu$Int6
 0002:000053C4       inicpu$CheckD1
 0002:000053F8       inicpu$Int1
 0002:00005408       inicpu$MulTest
 0002:00005418       inicpu$MulProc
 0002:00005438       h_syiPauseOnError
 0002:0000543A       syiPauseOnError
 0002:0000548C       h_syiSetVideoMode
 0002:0000554C       h_syiResetVideoMode
 0002:0000554E       syiResetVideoMode
 0002:000055D4       h_syiBMPDoCopyright
 0002:00005648       h_syiBMPStandBy
 0002:0000564C       f_syiBMPStandBy
 0002:0000564E       syiBMPStandBy
 0002:000056E8       h_w_GlobalSeg
 0002:000056EA       w_GlobalSeg
 0002:00005858       RealModeIC
 0002:000058DC       ProtModeIC
 0002:0000592C       h_syiABiosRealInit
 0002:00005C7C       LoadRAMPatch
 0002:00005F64       CheckRAMPatch
 0002:0000605C       h_DisplayLoadMsg
 0002:00006118       SYIInitOS2
 0002:0000621C       h_syiSwapDiskette
 0002:0000621E       syiSwapDiskette
 0002:00006398       syiDetermineHardwareConfigurati
 0002:0000642C       h_syiCheckForAltF1
 0002:00006510       h_syiProcessALTF1File
 0002:00006512       syiProcessALTF1File
 0002:0000687C       h_syiDMQS
 0002:0000694C       h_syiAPM
 0002:00006A38       h_GetBPB
 0002:00006A3A       GetBPB
 0002:00006A44       h_SYIReadSectors
 0002:00006A46       SYIReadSectors
 0002:00006B3C       syiPreInitSIFS
 0002:00006B78       SELInitRM
 0002:00006D24       ArenaSelToSeg
 0002:00006D70       selinit$GDTMapInit
 0002:00006E94       selinit$GDTMapAlloc
 0002:00006ED4       selinit$GDTAllocInit
 0002:00006F14       GDTInitTab
 0002:00006F44       TRAPInitRM
 0002:00006F90       DebugInitializeRM
 0002:00007030       h_DebugInitializeDM
 0002:00007032       DebugInitializeDM
 0002:0000706C       h_DebugMovedGDTIDT
 0002:00007070       f_DebugMovedGDTIDT
 0002:00007072       DebugMovedGDTIDT
 0002:00007098       h_DebugReInitialize
 0002:0000709A       DebugReInitialize
 0002:000071DC       dosinit$h_DebugInitialize
 0002:000071DE       dosinit$DebugInitialize
 0002:00007274       h_DebugLoadSymSysInitFS
 0002:00007278       f_DebugLoadSymSysInitFS
 0002:0000727A       DebugLoadSymSysInitFS
 0002:00007358       h_DebugRemoveSymMTE
 0002:0000735C       f_DebugRemoveSymMTE
 0002:0000735E       DebugRemoveSymMTE
 0003:00000000       _StartDCODE
 0003:00000004       _disasm
 0003:0000012F       _decodeop
 0003:000011D1       _fmtaddr
 0003:00001430       _cvkDStuffSum
 0003:000014E8       _cvkDUnStuffSum
 0003:000015DA       _cvkNSend
 0003:00001663       _cvkNReceive
 0003:0000173C       _cvkTSend
 0003:00001799       _cvkTReceive
 0003:000017FF       _KDPRawOutput
 0003:000018A9       _KDPEventNotify
 0003:00001B50       _KDPMain
 0003:00002882       _KDPRawInput
 0003:00002891       _KDPCharInput
 0003:000028B0       __sprntf
 0003:00002AB2       _sprintf
 0003:00002AC4       _sprintflc
 0003:00002AE8       _BreakPoint
 0003:00002AF2       _BreakShow
 0003:00002DD7       _BreakEna
 0003:00002F0C       _ChangeBPTaskNum
 0003:00002F7D       _Vector
 0003:0000308A       _VectorSet
 0003:0000312D       _ChangeDefCmd
 0003:00003177       _ExecuteIfTrue
 0003:000031B0       _BadCommandLine
 0003:000031C7       _ParseString
 0003:00003207       _CheckString
 0003:0000320E       _SetTmpBP
 0003:00003239       _SetGoBP
 0003:0000326A       _CheckDRBP
 0003:000032BF       _CheckDRhit
 0003:000032D9       _ChkBPaddr
 0003:00003328       _PutBPoints
 0003:00003438       _RestoreBPoints
 0003:000034C0       _ErrBreak
 0003:000034C9       _RCmdBreak
 0003:00003504       _perr
 0003:00003510       _perror
 0003:00003533       _CmdBreak
 0003:00003563       _command
 0003:000035EB       _DoCommand
 0003:00003693       _ExecSubr
 0003:000036AB       _KDPEvent
 0003:000036D8       _KDPRaw
 0003:000036F6       _KDPReadMem
 0003:0000371C       _KDPWriteMem
 0003:0000373B       _KDPGetAccAtr
 0003:00003E64       _DumpStack
 0003:00003E7A       _DumpStack2
 0003:00003ED6       _PrintStack
 0003:00004001       _GetEOL
 0003:0000400C       _ScanP
 0003:0000401C       _SkipB
 0003:00004024       _GetChr
 0003:0000402E       _GetChrI
 0003:0000404D       _IsSeparator
 0003:0000405D       _PeekChr
 0003:00004068       _EOLchk
 0003:0000406F       _SetDefaults
 0003:00004090       _Dump
 0003:000047B4       _EvalRange
 0003:000047E3       _EvalLength
 0003:0000482E       _EvalAddr
 0003:00004883       _EvalDword
 0003:00004896       _EvalWord
 0003:000048AE       _EvalByte
 0003:000048C2       _EvalExpr
 0003:00004ADE       _INDoprx
 0003:00004B97       _IsTrue
 0003:00004C52       _GetExprS
 0003:00004C65       _GetArgValue
 0003:00004DDB       _ScanAtom
 0003:00004E27       _HexChk
 0003:00004E3E       _ProtModeDS
 0003:00004E48       _Debug_Entry
 0003:000050BF       _KDPEnable
 0003:000050CA       _Debug_Break
 0003:000050D8       _Debug_Break32
 0003:000050E6       _Debug_Command
 0003:00005109       _Debug_Exit
 0003:00005112       _DebExit
 0003:00005192       _GetDebuggerDS
 0003:000051B0       _Debug_CtrlC
 0003:000051F5       f__Debug_CtrlC32
 0003:000051F5       _Debug_CtrlC32
 0003:00005280       _EndCtrlC32
 0003:000052AC       _DebCallOut
 0003:000052C8       _LowerCaseOn
 0003:000052D6       _LowerCaseOff
 0003:000052DC       _inbuf
 0003:00005313       _StrUpr
 0003:0000533A       _upper
 0003:00005345       _lower
 0003:000053E0       _prtstr
 0003:000053F1       _rprbuf
 0003:00005408       _OutAddrOff
 0003:0000542C       _OutAddrS
 0003:0000545E       _OutColonDword
 0003:0000547C       _Out32
 0003:00005488       _Out24
 0003:00005494       _Out20
 0003:000054A0       _out16
 0003:000054AD       _hex
 0003:000054BA       _OutHex
 0003:000054C6       _OutRadix
 0003:00005500       _fmtnum
 0003:00005597       _CrLfColOne
 0003:000055A2       _crlf
 0003:000055AF       _backup
 0003:000055BC       _tab
 0003:000055C2       _blank
 0003:000055CA       _putchar
 0003:000055F4       _putcharl
 0003:00005620       _InitComPort
 0003:000056DB       _GetEchoChr
 0003:000056F5       _waitchr
 0003:00005735       _inchr
 0003:00005745       _ungetc
 0003:00005749       _EnableNMI
 0003:0000574F       _EnableA20
 0003:00005755       _RestoreA20Status
 0003:0000575B       _KDPDSend
 0003:000057A7       _KDPDReceive
 0003:00005800       _Debug_Task
 0003:00005812       _KDPPageIn
 0003:00005889       _GetRMIDTaddr
 0003:00005896       _GetPMIDTaddr
 0003:000058A8       _GetGdtAddr
 0003:000058BA       _GetLdtAddr
 0003:000058E0       _GetCSIPaddr
 0003:000058F1       _GetDSaddr
 0003:000058FE       _FillDataAddr
 0003:00005919       _FillDefAddr
 0003:00005937       _FillSelAddr
 0003:00005953       _FillLinAddr
 0003:0000596E       _FillPhyAddr
 0003:00005989       _FillAddr
 0003:000059CA       _CompareAddr
 0003:00005A0A       _CompareLinAddr
 0003:00005A5D       _CopyAddr
 0003:00005A77       _AddAddr
 0003:00005A8F       _SubtractAddr
 0003:00005AE7       _CheckAddr
 0003:00005B06       _PrintMemErr
 0003:00005B5C       _geterrmessage
 0003:00005B74       _PutByteOff
 0003:00005B97       _PutByte
 0003:00005BB0       _PutWord
 0003:00005BB8       _PutWordOff
 0003:00005BD6       _PutDword
 0003:00005BDE       _PutDwordOff
 0003:00005BFF       _PutBuff
 0003:00005C07       _PutBuffOff
 0003:00005C51       _GetCache
 0003:00005C59       _GetCacheOff
 0003:00005C7F       _GetMem
 0003:00005C87       _GetMemOff
 0003:00005CEA       _GetByteOff
 0003:00005D0B       _GetByte
 0003:00005D22       _GetWord
 0003:00005D2A       _GetWordOff
 0003:00005D4A       _GetDword
 0003:00005D52       _GetDwordOff
 0003:00005D75       _GetBuff
 0003:00005D7D       _GetBuffOff
 0003:00005DF7       _AddrToPhy
 0003:00005E18       _AddrToLin
 0003:00005E56       _SelOffToLin
 0003:00005E9A       _GetAddrInfo
 0003:00005FEC       _GetPDE
 0003:0000603A       _GetPTE
 0003:000061E1       _EnterMem
 0003:0000632B       _ExitMem
 0003:00006373       _GetAddrType
 0003:0000637E       _GetAddrTask
 0003:00006389       _GetCurrTask
 0003:0000639A       _IsPagingEnabled
 0003:000063A2       _WhatIsClientMode
 0003:000063BB       _IsDebProtMode
 0003:000063C3       _Is286
 0003:000063CD       _PopFlags
 0003:000063CE       _KDPSelToLin
 0003:000063F1       _KDPGetSelInfo
 0003:00006424       _OpInterpret
 0003:000066BF       _GetInStr
 0003:000066F0       _SearchString
 0003:00006766       _shlaxdx
 0003:00006773       _shraxdx
 0003:000067A0       _reg
 0003:000067D7       _DispReg
 0003:00006840       _KDPLink
 0003:00006866       _KDPUnlink
 0003:0000688C       _Debug_Sym32
 0003:0000688C       f__Debug_Sym32
 0003:00006891       _Debug_Sym
 0003:00006B8B       _getsymbuf
 0003:00006BA4       _GetSymbolBuf
 0003:00006E1A       _GetSymbolVal
 0003:00006FA8       _WithMap
 0003:00007024       _Lists
 0003:000070E6       _PrintNearSym
 0003:0000717A       _PrintMapName
 0003:00007471       _EachMap
 0003:0000750B       _UpdateWinOS2Maps
 0003:000075D1       _EachGroup
 0003:00007643       _EachAbsSym
 0003:00007682       _EachAbsSym32
 0003:000076C1       _EachSym
 0003:0000772F       _EachSym32
 0003:0000779D       _EachSegDef
 0003:00007A6E       f__Debug_Trap32
 0003:00007A6E       _Debug_Trap32
 0003:00007AFB       _Debug_Trap
 0003:00007B04       _BreakEntry
 0003:00007CDA       f__Debug_Fatal
 0003:00007CFC       f__Debug_Fatal_User
 0003:00007D1E       _ExEnterDebugIRET
 0003:00007D3B       _ExEnterDebugRETF
 0003:00007D5D       _EnterDebugRETFD
 0003:00007DA2       _EnterDebugIRETD
 0003:00007E54       _EnterDebugRETF
 0003:00007E62       _EnterDebugINIT
 0003:00007E8F       _EnterDebugIRET
 0003:00007F83       _PrintTrapMsg
 0003:0000802B       _Go
 0003:0000807D       _KDPGo
 0003:00008096       _Ptrace
 0003:0000814F       _Trace
 0003:000081BD       _KDPTrace
 0003:00008588       _ExitDebug
 0003:0000858D       _ExitDebugNoBP
 0003:000085AF       _ExitDebugIRET
 0003:00008609       _ExitDebugIRETD
 0003:000089CF       _SetIdtEntry
 0003:00008ABB       _RestAllIdt
 0003:00008ACC       _RestIdtEntry
 0003:00008B7B       _GetTrapTblEntry
 0003:00008B90       _CheckCtrlC
 0003:00008BC8       _unassem
 0003:00008C0B       _disasln
 0003:00008C49       _checkbp
 0003:00008C63       _getmemc
 0003:00008C81       _getbuffc
 0003:00008CA8       _regval
 0003:00008CD4       _segregval
 0003:00008CEB       _getdbit
 0003:00008D1B       _lowercase
 0003:00008D3A       _strlen
 0003:00008D52       _strcpylc
 0003:00008D77       _strcpy
 0003:00008DA0       _prntf
 0003:00008DC7       ___aNlshl
 0003:00008DD3       ___aNlshr
 0003:00008DDF       ___aNulshr
 0003:00009129       _DebCallOutRoutine
 0003:00009146       _ExtCmdRoutine
 0003:00009779       _GetMTEName
 0003:00009944       _DebDRAlloc
 0003:0000996A       _DebDRFree
 0003:00009994       _SaveContext
 0003:000099A9       _CompareContext
 0003:000099BE       _ZeroGoTime
 0003:000099D9       _CheckGoTime
 0003:00009A04       _MarkGoTime
 0003:00009A49       _DisplayGoTime
 0003:00009AE9       _ShowTimeStamps
 0003:00009BBD       _TimeStampBP
 0003:00009C42       _ClearTimeStamps
 0003:00009C5C       _DumpCDA
 0003:00009D58       _DumpMem
 0003:0000A4F7       _DOAPrintLock
 0003:0000ACF3       _GetObjectAddr
 0003:0000AD4C       _GetPseudoObjectAddr
 0003:0000AFE4       InitComPort
 0003:0000AFED       _OEMInitCom
 0003:0000AFF8       _SetBaudCmd
 0003:0000B034       _RebootCmd
 0003:0000B046       _RebootEntry
 0003:0000B046       _KDPRebootEntry
 0003:0000B05E       _KDPReboot
 0003:0000B060       _SysdumpCmd
 0003:0000B072       _SysdumpEntry
 0003:0000B07F       _OEMOutputChar
 0003:0000B0AB       _OEMBreakChk
 0003:0000B0C6       _OEMScanChar
 0003:0000B101       _OEMEnableNMI
 0003:0000B111       _OEMEnableA20
 0003:0000B112       _OEMRestoreA20
 0003:0000B113       _OEMBeep
 0003:0000B149       _KDDComm
 0003:0000B244       _KDPTaskNew
 0003:0000B269       _KDPTaskEnd
 0003:0000B286       _MakePresentCmd
 0003:0000B69F       _DumpUserStack
 0003:0000B787       _ProcessStatus
 0003:0000BFE2       _RegisterSlot
 0003:0000C19C       _ChangeCurrTask
 0003:0000C286       _DebEntryRoutine
 0003:0000C295       _DebExitRoutine
 0003:0000C2EB       _DebGetCurrTask
 0003:0000C2EF       _DebGetCurrHobPTDA
 0003:0000C307       _DebGetDescInfo
 0003:0000C3A9       _DebGetPDE
 0003:0000C45F       _DebGetFrame
 0003:0000C4A1       _GetPTDAaddr
 0003:0000C54F       _InvalidHandle
 0003:0000C5CF       _KDPMemUtil
 0003:0000C638       _KDPNextModule
 0003:0000C681       _KDPhmte2pmte
 0003:0000C6C5       _KDPpmte2name
 0003:0000C76E       _KDPObjInfo
 0003:0000C957       _KDPObjCount
 0003:0000CA02       _KDPObjInfo2
 0003:0000CB4F       _KDPQueryThread
 0003:0000CC23       _KDPGetRegs
 0003:0000CD6D       _KDPPutRegs
 0003:0000CE89       _KDPGetNPX
 0003:0000CF27       _KDPPutNPX
 0003:0000CFBC       _DumpTraceBuffer
 0004:00000000       _DebSASTable
 0004:00000000       _StartDFIRST
 0004:0000008A       _EndDFIRST
 0004:0000008A       _StartDDATA
 0004:00001BBA       _BPcount
 0004:000028C0       _DebData
 0004:000028FA       _InDebugger
 0004:000028FB       _DisAddr
 0004:00002905       _DumpAddr
 0004:0000290F       _EnterAddr
 0004:00002919       _DefMode
 0004:0000291A       _DefType
 0004:0000291C       _KDDCDisabled
 0004:0000291D       _KDDCDisabledCause
 0004:0000291E       _KDDCActive
 0004:0000291F       _KDDCFlushSend
 0004:00002920       _KDDCInput
 0004:00002921       _KDDCTKSSBase
 0004:00002925       _fKDPEnabled
 0004:00002926       _fKDPPacketStop
 0004:00002927       _fKDPPacketMode
 0004:00002928       _fKDPRaw
 0004:00002929       _fKDPReceived
 0004:0000292A       _fKDPTaskNotifyEnable
 0004:0000292B       _KDPhMTE
 0004:0000292D       _KDPpMTE
 0004:00002931       _KDPSlot
 0004:00002935       _KDPPageinCount
 0004:00002937       _KDPPageinTable
 0004:00003137       _KDPPageHMTE
 0004:00003139       _KDPPageAddr
 0004:00003149       _InitCmdBuffer
 0004:000031E9       _CmdInputBuffer
 0004:00003289       _DefaultCmd
 0004:00003329       _pTXTstart
 0004:0000332B       _pTXT
 0004:0000332D       _CommandScriptAddrS
 0004:00003337       _CommandScriptSize
 0004:00003339       _TraceCallsStack
 0004:00003721       _TraceCallsDepth
 0004:00003723       _TraceCallsFirst
 0004:00003725       _TraceCallsSecond
 0004:00003727       _sbrtab
 0004:00003E12       _pRegSA
 0004:00003E14       _RegSA
 0004:00003E94       _LoadAllSav
 0004:00003EFA       _MemCache
 0004:000040FA       _DebStackFence
 0004:000050FC       _StackTop
 0004:000050FE       _AXmsg
 0004:00005102       _EAXmsg
 0004:00005107       _BXmsg
 0004:0000510B       _EBXmsg
 0004:00005110       _CXmsg
 0004:00005114       _ECXmsg
 0004:00005119       _DXmsg
 0004:0000511D       _EDXmsg
 0004:00005122       _SPmsg
 0004:00005126       _ESPmsg
 0004:0000512B       _BPmsg
 0004:0000512F       _EBPmsg
 0004:00005134       _SImsg
 0004:00005138       _ESImsg
 0004:0000513D       _DImsg
 0004:00005141       _EDImsg
 0004:00005146       _CSmsg
 0004:0000514A       _DSmsg
 0004:0000514E       _ESmsg
 0004:00005152       _SSmsg
 0004:00005156       _IPmsg
 0004:0000515A       _EIPmsg
 0004:0000515F       _GDTRmsg
 0004:00005165       _IDTRmsg
 0004:0000516B       _GDTBmsg
 0004:00005171       _GDTLmsg
 0004:00005177       _IDTBmsg
 0004:0000517D       _IDTLmsg
 0004:00005183       _TRmsg
 0004:00005187       _LDTRmsg
 0004:0000518D       _IOPLmsg
 0004:00005193       _MSWmsg
 0004:00005198       _CR0msg
 0004:0000519D       _CR2msg
 0004:000051A2       _CR3msg
 0004:000051A7       _CR4msg
 0004:000051AC       _Fmsg
 0004:000051AF       _EFmsg
 0004:000051B3       _FSmsg
 0004:000051B7       _GSmsg
 0004:000051BB       _DR0msg
 0004:000051C0       _DR1msg
 0004:000051C5       _DR2msg
 0004:000051CA       _DR3msg
 0004:000051CF       _TR6msg
 0004:000051D4       _TR7msg
 0004:000051D9       _DR6msg
 0004:000051DE       _DR7msg
 0004:00005943       _AtomBuf
 0004:00005B9F       _header
 0004:00005BB8       _cpumsg
 0004:00005BE2       _CursorColumn
 0004:00005BE6       _LoadallSaved
 0004:00006849       _PrtMSW
 0004:00006871       _PrtFlags
 0004:000068D5       _PrtRFVM
 0004:00006CDC       _TrapNumber
 0004:00006CDC       _TrapNumber32
 0004:00006CE0       _ErrorCode
 0004:00006CE2       _fRegDisp
 0004:00006CE3       _fExecTrap
 0004:00006CE4       _Tcount
 0004:00006CE6       _TraceAddr
 0004:00006CF0       _fTraceAddr
 0004:00006CF1       _fTraceCount
 0004:00006CF2       _fDoTraceBad
 0004:00006CF3       _fTraceSpecial
 0004:00006CF4       _fTraceSpecial2
 0004:00006CF5       _InstCount
 0004:00006CF9       _fDoGoSpecial
 0004:00006EFE       TrapTbl
 0004:000071B6       _opbuf
 0004:0000740C       _btatab
 0004:00007448       _ContextStartAddr
 0004:00007452       _ContextEndAddr
 0004:0000745C       _ContextEndAddr2
 0004:0000936A       _li_pvmli
 0004:0000936E       _li_cs
 0004:00009370       _li_eip
 0004:00009374       _li_phlock
 0004:00009378       _li_address
 0004:0000937C       _li_flg
 0004:0000937E       _li_hptda
 0004:00009380       _li_npages
 0004:00009382       _li_hob
 0004:00009384       _li_sig
 0004:00009386       _li_csig
 0004:00009388       _DosLinAddr
 0004:0000A32A       CurrTask
 0004:0000A4F1       _VDMmsg
 0004:0000A51B       _SYIthreadmsg
 0004:0000A524       _JITthreadmsg
 0004:0000AA38       _EndDCONST
 0004:0000AA38       _StartDBSS
 0004:0000AA38       _StartDCONST
 0004:0000AA38       _EndDDATA
 0005:00000000       _StartTASKDUMMY
 0005:0000F994       ptda_start
 0005:0000F994       pPTDAParent
 0005:0000F994       _EndTASKDUMMY
 0005:0000F994       _StartTASKDATA
 0005:0000F998       pPTDASelf
 0005:0000F99C       pPTDAFirstChild
 0005:0000F9A0       pPTDAExecChild
 0005:0000F9A4       pPTDANextZombie
 0005:0000F9A4       pPTDANextSibling
 0005:0000F9A8       pPTDAPrevZombie
 0005:0000F9A8       pPTDAPrevSibling
 0005:0000F9AC       ptda_pszproc
 0005:0000F9B0       ptda_pTCBHole
 0005:0000F9B4       ptda_pTCB1
 0005:0000F9B4       ptda_pTCBHead
 0005:0000F9B8       ptda_cTCB
 0005:0000F9BA       ptda_ctib
 0005:0000F9BC       ptda_avatib
 0005:0000F9D8       ptda_flDbgEnabled
 0005:0000F9DC       ptda_flDbg
 0005:0000F9E0       ptda_ah
 0005:0000FA20       ptda_pgdata
 0005:0000FA46       ptda_environ
 0005:0000FA48       ptda_pBeginLIBPATH
 0005:0000FA50       ptda_pgpc
 0005:0000FC90       ptda_pPVDBPrc
 0005:0000FC94       ptda_pSGSList
 0005:0000FC98       ptda_pexllist
 0005:0000FCA0       WFP_Start
 0005:0000FCA2       Ren_WFP
 0005:0000FCA4       WFP_Path_End
 0005:0000FCA6       Curr_Dir_End
 0005:0000FCA8       CDS_Handle
 0005:0000FCDC       OEMPtr
 0005:0000FCDE       Fgnd
 0005:0000FCDF       FgndOnly
 0005:0000FCE0       ptda_pTCBCritSec
 0005:0000FCE4       ptda_pTCBPriQCritSec
 0005:0000FCE8       ptda_cCritSec
 0005:0000FCEA       CurrentPDB
 0005:0000FCEC       DTAddr
 0005:0000FCF0       seltss
 0005:0000FCF2       VolID
 0005:0000FCF3       NoSetDir
 0005:0000FCF4       SpaceFlag
 0005:0000FCF5       VerFlg
 0005:0000FCF6       LCurDrv
 0005:0000FCF7       PCurDrv
 0005:0000FCF8       Creating
 0005:0000FCF9       DelAll
 0005:0000FCFA       FoundDel
 0005:0000FCFB       Found_dev
 0005:0000FCFC       fSplice
 0005:0000FCFD       ClusFac
 0005:0000FCFE       cMeta
 0005:0000FCFF       PathNameType
 0005:0000FD00       DevPt
 0005:0000FD04       DirSec
 0005:0000FD08       DirStart
 0005:0000FD0A       NxtClusNum
 0005:0000FD0C       EntFree
 0005:0000FD0E       EntLast
 0005:0000FD10       LastEnt
 0005:0000FD12       ProcFlag
 0005:0000FD14       ptda_ForcedActions
 0005:0000FD18       ptda_ulExitCode
 0005:0000FD1C       ptda_ulExitType
 0005:0000FD20       ptda_ulExitTID
 0005:0000FD24       ThisCDS
 0005:0000FD28       ptda_pCDS
 0005:0000FD2A       CDSsize
 0005:0000FD2C       Sattrib
 0005:0000FD2E       sPCB
 0005:0000FD30       ptda_pPCB
 0005:0000FD34       JFN_Max
 0005:0000FD36       NextSrchH
 0005:0000FD38       SrchRmp
 0005:0000FD3C       FNotifyLocal_First
 0005:0000FD3E       FNotifyLocal_Count
 0005:0000FD40       Sig_ignf
 0005:0000FD42       Sig_hndf
 0005:0000FD44       Sig_errf
 0005:0000FD46       Sig_attempted
 0005:0000FD48       Sig_arg
 0005:0000FD5A       HoldSigCnt
 0005:0000FD5E       JFN_Table
 0005:0000FD86       JFN_Flags
 0005:0000FD9A       ptda_rasflag
 0005:0000FD9C       SysSemPTDATbl
 0005:0000FE9C       SavedHardErr
 0005:0000FEA0       ptda_ptdasem
 0005:0000FEAC       ptda_DLMsem
 0005:0000FEBE       Csid
 0005:0000FEC0       Behav_bit
 0005:0000FEC2       MSW
 0005:0000FEC4       ptda_rsrclist
 0005:0000FEC8       ptda_pldrdldHead
 0005:0000FECC       pPrSemTbl
 0005:0000FED0       ulPrTblSize
 0005:0000FED4       ulPrTotUsed
 0005:0000FED8       ulPrNextFree
 0005:0000FEDC       hksPrTbl
 0005:0000FEE0       pShSemBmp
 0005:0000FEE4       ulShBmpSize
 0005:0000FEE8       hksShBmp
 0005:0000FEEC       ulMtxOwned
 0005:0000FEF0       ShareRetriesLeft
 0005:0000FEF2       RetryCount
 0005:0000FEF4       RetryLoop
 0005:0000FEF6       ptda_pSrchBuf
 0005:0000FEFA       ptda_pOpenBuf
 0005:0000FF24       Cons_Loc
 0005:0000FF2E       SysCallSfcn
 0005:0000FF2F       SysCall
 0005:0000FF30       KBD_Mode
 0005:0000FF31       ptda_NewFiles
 0005:0000FF32       AutoFail
 0005:0000FF33       Name1
 0005:0000FF33       DevFCB
 0005:0000FF4C       DESTSTART
 0005:0000FF53       CP_Flgs
 0005:0000FF54       Sig_vec
 0005:0000FF74       Exc_vec
 0005:0000FF94       Attrib
 0005:0000FF96       ExtFCB
 0005:0000FF97       ptda_extsig
 0005:0000FF9C       ptda_lanman_sec
 0005:0000FFA0       SigFTerm
 0005:0000FFA2       ptda_ppgdata
 0005:0000FFA4       ptda_child
 0005:0000FFA6       ptda_childalias
 0005:0000FFA8       ptda_handle
 0005:0000FFAA       ptda_module
 0005:0000FFAC       ptda_ldthandle
 0005:0000FFAE       ptda_ldtpgmap
 0005:0000FFB0       ptda_ldtaddr
 0005:0000FFB4       CP_CaseMapTbl
 0005:0000FFB8       codepage_tag
 0005:0000FFBA       JFN_Length
 0005:0000FFBC       JFN_pTable
 0005:0000FFC0       JFN_Flg_Ptr
 0005:0000FFC4       Joins
 0005:0000FFC5       ExtErr_Locus
 0005:0000FFC6       ExtErr
 0005:0000FFC8       ExtErr_Action
 0005:0000FFC9       ExtErr_Class
 0005:0000FFCA       ptda_infoseg
 0005:0000FFCA       Pid
 0005:0000FFCC       Ppid
 0005:0000FFD4       ProcStatus
 0005:0000FFD8       ProcType
 0005:0000FFEE       ptda_vme
 0005:0000FFF0       CurrTCB
 0005:0000FFF2       CurrTSD
 0005:0000FFF4       ThisPTDA
 0005:0000FFF6       ptda_NPX_em_cs
 0005:0000FFF8       ptda_NPX_em_eip
 0005:0000FFFE       ptda_signature
 0006:00000000       _StartGDTSTART
 0006:00000000       GDT
 0006:00000008       GDT_GDT
 0006:00000010       GDT_TSS
 0006:00000018       GDT_IDT
 0006:00000020       GDT_RM_IDT
 0006:00000028       GDT_LDT
 0006:00000030       GDT_PTDA
 0006:00000038       GDT_FPEM
 0006:00000040       GDT_ROMDATA
 0006:00000048       GDT_R2DS
 0006:00000050       GDT_R3DS
 0006:00000058       GDT_R3CS
 0006:00000060       GDT_R3PDS
 0006:00000068       GDT_R3THKDS
 0006:00000070       GDT_SAS
 0006:00000078       GDT_DOSALIAS
 0006:00000080       GDT_SYSINFOSEG
 0006:00000088       GDT_DFTSS
 0006:00000090       GDT_DFSTACK
 0006:00000098       GDT_VPB
 0006:000000A0       GDT_RDR1
 0006:000000A8       GDT_Buffers
 0006:000000B0       GDT_Unused
 0006:000000B8       GDT_RLR
 0006:000000C0       GDT_SFT
 0006:000000C8       GDT_FSC
 0006:000000D0       GDT_mFSD
 0006:000000D8       GDT_RIPL
 0006:000000E0       GDT_NULLIDT
 0006:000000E8       GDT_INTSTACK
 0006:000000F0       GDT_RMCODE
 0006:000000F8       GDT_RMDATA
 0006:00000100       GDT_POOL
 0006:00001508       GDT_POOLEND
 0006:00001508       GDT_TIB
 0006:00001510       _EndGDTSTART
 0006:00001510       _StartGDTCGSEG
 0006:00001D20       GDT_DOSALLOCSEG
 0006:00001D20       _StartGDTPUBSEG
 0006:00001D20       _EndGDTCGSEG
 0006:00001D28       GDT_DOSALLOCPROTSEG
 0006:00001D30       GDT_DOSDYNAMICTRACE
 0006:00001D38       GDT_DOSERROR
 0006:00001D40       GDT_DOSFREERESOURCE
 0006:00001D48       GDT_DOSQUERYABIOSSUPPORT
 0006:00001D50       GDT_DOS16LDRDIRTYWORKER
 0006:00001D58       GDT_DOSFREESEG
 0006:00001D60       GDT_DOSGETPROCADDR
 0006:00001D68       GDT_DOSIEXECPGM
 0006:00001D70       GDT_DOSIQAPPTYPE
 0006:00001D78       GDT_DOSISEMWAIT
 0006:00001D80       GDT_DOSLOADMODULE
 0006:00001D88       GDT_DOSMAKEPIPE
 0006:00001D90       GDT_DOSREALLOCSEG
 0006:00001D98       GDT_DOSSICG
 0006:00001DA0       GDT_PANICWRITE
 0006:00001DA8       GDT_DOSSETPRTY
 0006:00001DB0       GDT_DOSLOGMODE
 0006:00001DB8       GDT_DOSSETCP
 0006:00001DC0       GDT_DOSGLOBALSEG
 0006:00001DC8       GDT_DOSCREATETHREAD
 0006:00001DD0       GDT_DOSEXIT
 0006:00001DD8       GDT_DOSEXITLIST
 0006:00001DE0       GDT_DOSFREEMODULE
 0006:00001DE8       GDT_DOSRESUMETHREAD
 0006:00001DF0       GDT_DOSSLEEP
 0006:00001DF8       GDT_DOSSUSPENDTHREAD
 0006:00001E00       GDT_DOSLIBINIT
 0006:00001E08       GDT_REDIR
 0006:00001E10       GDT_DOSCHGFILEPTR
 0006:00001E18       GDT_DOSPROTECTCHGFILEPTR
 0006:00001E20       GDT_DOSCLOSE
 0006:00001E28       GDT_DOSPROTECTCLOSE
 0006:00001E30       GDT_DOSDELETE
 0006:00001E38       GDT_DOSDEVIOCTL
 0006:00001E40       GDT_DOSDEVIOCTL2
 0006:00001E48       GDT_DOSDUPHANDLE
 0006:00001E50       GDT_DOSICOPY
 0006:00001E58       GDT_DOSIREAD
 0006:00001E60       GDT_DOSIPROTECTREAD
 0006:00001E68       GDT_DOSISETRELMAXFH
 0006:00001E70       GDT_DOSIWRITE
 0006:00001E78       GDT_DOSIPROTECTWRITE
 0006:00001E80       GDT_DOSMOVE
 0006:00001E88       GDT_DOSOPEN
 0006:00001E90       GDT_DOSSETMAXFH
 0006:00001E98       GDT_MSSTACK
 0006:00001EA0       GDT_OS2LDR
 0006:00001EA8       GDT_NWDTSS
 0006:00001EB0       GDT_NWDSTACK
 0006:00001EB8       GDT_R0CSC
 0006:00001EC0       _StartGDTEND
 0006:00001EC0       _EndGDTPUBSEG
 0007:00000000       _StartINITDATA
 0007:00000002       CodeLockInitInfo
 0007:0000004A       fscNameList
 0007:000003B6       mfscNameList
 0007:000003FA       Disk_DD_Parameter_List
 0007:00000404       CFG_AutoCheck
 0007:0000041E       CFG_Break
 0007:0000041F       CFG_Dos_Flags
 0007:00000420       CFG_Buffers
 0007:00000422       CFG_DiskCache
 0007:00000426       CFG_DiskThresh
 0007:00000428       CFG_LazyWrite
 0007:00000429       CFG_FCBCount
 0007:0000042B       CFG_FCBKeep
 0007:0000042D       CFG_FILESCount
 0007:0000042F       CFG_Prompt
 0007:00000430       CFG_PrtBufSize
 0007:00000436       CFG_ProtectOnly
 0007:00000437       CFG_RMSize
 0007:00000439       CFG_LastDrive
 0007:0000043A       CFG_ReserveDriveLetter
 0007:000004DB       cdibseg
 0007:00000574       _CacheToAlloc
 0007:0000057C       sicg_packet_6
 0007:0000057E       sicg_packet_6_d
 0007:00000587       sicg_packet_D
 0007:00000589       sicg_packet_D_d
 0007:000005A3       sicg_packet_16
 0007:000005A5       sicg_packet_16_d
 0007:000005AB       sicg_packet_1A
 0007:000005AD       sicg_packet_1A_d
 0007:000005B3       pDosAllocSeg
 0007:000005B7       pDosClose
 0007:000005BB       pDosChgFilePtr
 0007:000005BF       pDosCreateThread
 0007:000005CB       pDosExit
 0007:000005CF       pDosFreeModule
 0007:000005D3       pDosFreeSeg
 0007:000005D7       pDosGetProcAddr
 0007:000005DB       pDosGlobalSeg
 0007:000005DF       pDosLoadModule
 0007:000005E7       pDosOpen
 0007:000005EB       pDosDevIOCtl
 0007:000005EF       pDosDevIOCtl2
 0007:000005F3       pDosMove
 0007:000005F7       pDosDelete
 0007:000005FB       pDosReallocSeg
 0007:000005FF       pDosRead
 0007:00000603       pDosWrite
 0007:00000607       pDosSemWait
 0007:0000060B       pDosSetCp
 0007:00000613       pPanicWrite
 0007:00000617       pDosIQAppType
 0007:0000061B       pSICG
 0007:00000641       pDosExecPgm
 0007:00000649       pDosGetMessage
 0007:00000651       pDosPutMessage
 0007:00000659       pDosCloseMessageFile
 0007:00000661       pKbdFlushBuffer
 0007:00000669       pKbdStringIn
 0007:00000671       pKbdCharIn
 0007:00000679       pKbdSetCp
 0007:00000681       pVioSetCp
 0007:000006A1       pDosSMSysInitSem
 0007:000006D8       tbl_prompt
 0007:000006DC       tbl_lost_messages
 0007:000006E4       tbl_system_stopped
 0007:000006E8       tbl_mFSD_failure
 0007:000006EC       tbl_mFSD_failure_2
 0007:000006F0       tbl_syi_boot_err
 0007:000006F4       tbl_filesys_unavail
 0007:00000903       open_action
 0007:00000907       standard_output_handle
 0007:00000911       message_file_name
 0007:00000924       clock_name
 0007:0000096E       _DDwith24BitDMA
 0007:00000978       sicg_packet_3_d
 0007:000009DA       sicg_packet_1B
 0007:000009DC       sicg_packet_1B_d
 0007:00000CB6       tbl_syibanner
 0007:00000E93       MsgLoading
 0007:00000EE3       MsgLoadingLen
 0007:00000EE5       MsgDoneLoading
 0007:00000F35       MsgDoneLoadingLen
 0007:00000F37       CurrentDev
 0007:000013F5       tbl_kernel_message
 0007:0000145F       AltFxKeyPressed
 0007:00001460       AltF1Flags
 0007:00001461       AltF1CmdParms
 0007:00001478       AltF1Parm
 0007:0000147A       AltF1xCmdParms
 0007:00001492       AltF1SecCmdParms
 0007:00001504       SIFSRoutines
 0007:00001520       _DebBreakChar
 0007:0000158C       _StartINITTABLE
 0007:0000158C       Config_AutoFail
 0007:0000158C       _EndINITDATA
 0007:00001598       Config_DLLBasing
 0007:000015A4       Config_VME
 0007:000015B0       Config_NWD
 0007:000015BA       Config_Reipl
 0007:000015C6       Config_PvwQSize
 0007:000015D2       Config_Basedev
 0007:000015E2       Config_Break
 0007:000015EE       Config_Buffers
 0007:000015FA       Config_Call
 0007:0000160A       Config_CodePage
 0007:00001610       Config_Country
 0007:0000161A       Config_DeviceHigh
 0007:0000162C       Config_Device
 0007:0000163C       Config_DevInfo
 0007:00001648       Config_DiskCache
 0007:0000164C       Config_Dump
 0007:00001656       Config_Dos
 0007:00001668       Config_FCBs
 0007:0000167A       Config_COPROCFake
 0007:00001686       Config_GlobalJITRegister
 0007:00001696       Config_GlobalJITFlags
 0007:000016A2       Config_FILES
 0007:000016AE       Config_IFS
 0007:000016BE       Config_LastDrive
 0007:000016C4       Config_ReserveDriveLetter
 0007:000016CA       Config_Protect16
 0007:000016D0       Config_LibPath
 0007:000016DC       Config_MaxWait
 0007:000016E8       Config_MemMan
 0007:000016EE       Config_Priority
 0007:000016FA       Config_Prompt
 0007:00001706       Config_PrintBufSize
 0007:0000171E       Config_ProtectOnly
 0007:0000172A       Config_ProtShell
 0007:0000173A       Config_PrtyIO
 0007:00001746       Config_RMSize
 0007:00001752       Config_Run
 0007:00001762       Config_Set
 0007:0000176C       Config_Shell
 0007:0000177C       Config_SwapPath
 0007:00001786       Config_Threads
 0007:00001792       Config_Processes
 0007:0000179E       Config_TimeSlice
 0007:000017AA       Config_Trace
 0007:000017B4       Config_Strace
 0007:000017BA       Config_TraceBuf
 0007:000017C2       Config_DumpProcess
 0007:000017C8       Config_SuppressPopUps
 0007:000017CE       Config_RASKData
 0007:000017D8       Config_NullCommand
 0007:000017DE       Config_InvalidCommand
 0007:000017E2       CommandTable
 0007:000018B2       SizeTokenTable
 0007:000018BA       TraceBufKeyWdTable
 0007:000018C6       TraceBufSysDataTable
 0007:000018EE       TraceBufModeTable
 0007:00001926       TrapdumpTable
 0007:0000193A       DumpProcessTable
 0007:00001942       YesNoTable
 0007:0000194E       OnOffTable
 0007:0000195A       AbsDynTable
 0007:00001966       RomTable
 0007:0000196E       UMBTable
 0007:00001982       DevTypeTable
 0007:0000199E       MemManTable
 0007:000019CE       LWTable
 0007:000019D6       RASKDataTable
 0007:000019E6       StraceInitTable
 0007:000019EE       StraceEnableTable
 0007:000019FA       StraceInsertTable
 0007:00001A06       _EndINITTABLE
 0007:00001A06       ConfigSysFilename
 0007:00001A06       _StartINITSTRING
 0007:00001D24       _StartINITBSS
 0007:00001D24       PrepCPs
 0007:00001D24       _EndINITSTRING
 0007:00001D26       fscInitTemplate
 0007:00001DE6       mfscInitTemplate
 0007:00001DFE       InitCache_Parameter_List
 0007:00001F08       CFG_TraceBuf
 0007:00001F0A       CFG_TraceBits
 0007:00001F2A       CFG_LocalTraceBits
 0007:00001F4A       CFG_TraceBufMode
 0007:00001F4B       CFG_TraceBufMode2
 0007:00001F4C       CFG_TraceBufData
 0007:00001F50       CFG_STraceAction
 0007:00001F51       CFG_STraceBuf
 0007:00001F53       CFG_STraceBits
 0007:00001F73       CFG_STraceInsertBits
 0007:00001F93       CFG_LocalSubType
 0007:00001F9B       Config_Sys_Data
 0007:00001F9D       Config_Sys_File
 0007:00001FA7       CFG_Token
 0007:00002CEA       syiMessageSelector
 0007:00002CEC       syiSavedMessageIndicator
 0007:000030F5       error_messages_displayed
 0007:000030F6       tmp_msg_buffer
 0007:0000350E       message_buffer
 0007:00003D0E       message_length
 0007:00003D50       decimalascii
 0007:00003D5E       hsemSICGThreadDead
 0007:00003D62       hsemVDMMInitMessageBufferEmpty
 0007:00003D66       hsemVDMMInitErrorHandlerBusy
 0007:00003DBC       fVDMMInitComplete
 0007:00003DE2       command_string
 0007:0000500C       ABIOSSelTable
 0007:00005200       ABIOSSelTableEnd
 0007:000052CA       syiLostMessages
 0007:000052CC       syiLowMem
 0007:000052CE       syiHighMem
 0007:000052D0       HardDriveCount
 0007:000052D1       OEM_config
 0007:000052D3       pBanner
 0007:000053A0       mFSD_Handle
 0007:000053A7       syiCodeSelector
 0007:000053A9       syiEnvironSelector
 0007:000053B0       FSHelperModHdl
 0007:000053B2       _SELGDTLaddrTmp
 0007:000053B6       _vaArenaInfo
 0007:000053BA       MaxGDTDesc
 0007:000053BC       GDTFreeList
 0007:000053BE       pszzBaseVDDs
 0008:00000000       _StartINITR3CODE
 0008:00000004       InitFSCTemplateR3
 0008:0000007C       StrTransPathCharR3
 0008:00000090       syicpInit
 0008:00000178       inicp$syicpID
 0008:00000248       inicp$syicpCountry
 0008:000004A8       syicpValidateCountry
 0008:00000524       inicp$syicpData
 0008:0000069C       inicp$syicpFormat
 0008:00000700       inicp$syicpCollate
 0008:00000764       inicp$syicpCasemap
 0008:000007C8       inicp$syicpDBCS
 0008:00000838       inicp$syicpDevInfo
 0008:0000096C       inicp$syicpFatal
 0008:00000984       inicp$syicpWarning
 0008:0000099C       inicp$syicpError
 0008:000009BC       inicp$syicpAscii
 0008:000009D0       inicp$syicpInt2Ascii
 0008:000009EC       syiSaveData
 0008:00000A30       syicpActivate
 0008:00000AFC       syiDisplaySavedMessagesR3
 0008:00000B98       syiDisplayMessageR3
 0008:00000BD0       syiRetrieveMessageR3
 0008:00000C24       syiShowMessageR3
 0008:00000C70       syiAbortR3
 0008:00000C7C       syiWordToDecR3
 0008:00000CB8       syiPauseOnErrorR3
 0008:00000D14       syiSaveMessageR3
 0008:00000D20       inimsg3$syiSICGMessageR3
 0008:00000D3C       h_syiProcess
 0008:00000E38       syiOpenFiles
 0008:00000E94       syiCheckFatDrive
 0008:00000F14       syiCloseFiles
 0008:00000F2C       syiGetLoadableEntries
 0008:00000FA8       iniproc1$syiInitStdErrIntercept
 0008:00000FD0       iniproc1$syiBeginStdErrIntercep
 0008:00001054       iniproc1$syiStdErrIntercept
 0008:000010D0       iniproc1$syiEndStdErrIntercept
 0008:00001190       iniproc1$syiTerminateStdErrInte
 0008:000011D0       syiQuery16MBDevices
 0008:00001200       syiQuery16MBDevice
 0008:0000127C       syiCheckFileSys
 0008:0000132C       syiInstallDeviceDrivers
 0008:000015CC       syiInstallDeviceDriver
 0008:000016C0       syiInstallFileSysDriver
 0008:00001828       syiLoadDeviceFileSysDriver
 0008:00001898       syiInitializeDeviceDriver
 0008:00001A90       syiStartDOSMode
 0008:00001BC8       iniproc2$syiReceiveVDMMErrors
 0008:00001BEC       syiConvertErrorCode
 0008:00001C0C       syiRegisterJITDebug
 0008:00001D7C       syiStartDaemonProcesses
 0008:00001E3C       syi2StartDaemonProcesses
 0008:00001EC4       syiStartShell
 0008:00001F04       syiStartProgram
 0008:00001FB0       syiCopyConfigSysData
 0008:00001FE8       syiConstructCommandLine
 0008:00002014       syiInitEnvironment
 0008:00002070       syiModifyEnvironment
 0008:000020C4       syiParseEnvironmentString
 0008:00002138       syiScanEnvironment
 0008:00002170       syiExcludeExtLIBPATH
 0008:000021BC       syiRemoveEnvironmentString
 0008:000021FC       syiAddEnvironmentString
 0008:00002240       syiFATAutoCheck
 0008:0000232C       syiStartAltF1Process
 0008:00002394       RMNotifyR3
 0008:000023B4       _VerifySignature
 0008:0000277C       _RunningLocked
 0008:00002800       _LockProblem
 0008:0000280C       _VerifyDDLoaded
 0008:00002868       _StartLockProgram
 0008:000028B4       __panicINITR3
 0008:000028F0       __panicfnmsgINITR3
 0009:00000000       _sftFCB
 0009:00000000       _StartMVDMINSTDATA
 0009:00000002       FCBLRU
 0009:00000006       _KeepCount
 0009:00000110       _pvheVDM
 0009:00000114       _ulCurrentClass
 0009:00000118       _acPriorityReference
 0009:00000130       _alPriorityLevel
 0009:00000148       _aulPriorityClassOrder
 0009:00000160       _vdmid_mphvdmptcb
 0009:00000164       _vdmid_mphvdmpptda
 0009:00000168       _vdmid_VDMSIG
 0009:0000016C       _vdmid_mi
 0009:0000017C       _vdmid_HVDM
 0009:00000180       _vdmid_ulFreezeCnt
 0009:00000184       _vdmid_hpfh
 0009:0000018C       _vdmid_hla
 0009:00000190       _vdmid_flVDM
 0009:00000194       _hksemPropertyValues
 0009:00000198       _pprinList
 0009:0000019C       _hookheadSTIH
 0009:000001A4       _pvsfFrameBase
 000A:00000000       _aseldemTemp
 000A:00000000       _StartSWAPINSTDATA
 000A:0000000C       _segV86Kernel
 000A:0000001C       _pV86CurrentPDB
 000A:00000020       _vpDosDDHead
 000A:00000024       flPrefix
 000A:00000028       pOffset
 000A:0000002C       selClient
 000A:00000034       _pFaultHandler
 000A:00000038       _lidtV86IDT
 000A:0000003E       _ulVSFEAX
 000A:00000042       _ulVSFEBX
 000A:00000046       _V86SelSWInfo
 000A:0000004E       _flVdmStatus
 000A:00000052       _pdhdHostData
 000A:00000056       _pdhdHostLast
 000A:0000005A       _pvpmData
 000A:0000005E       _flVpmIRQHooks
 000A:00000062       _cVPMExecution
 000A:00000066       _cVPMHWInt
 000A:0000006A       _hhookV86ReflectionHook
 000A:0000006E       _hhookVPMReflectionHook
 000A:00000072       _hhookVPMExcRetHook
 000A:00000076       _hhookGetPSPRetHook
 000A:0000007A       _hhookV86Int23Hook
 000A:0000007E       _pVPMBP
 000A:00000082       _selVPMBP
 000A:00000084       _papfnVPMBP
 000A:00000088       _vpVPMSwitchAddr
 000A:0000008C       _vpV86Int23vect
 000A:00000090       _vpOurV86Int23vect
 000A:00000094       _usEIPincr
 000A:00000098       _vdmid_phpFixed
 000A:0000009C       _vdmid_phpSwap
 000A:000000A0       _vdmid_apfnUndo
 000A:000000C8       _vdmid_RMSIZE
 000A:000000CC       _vdmid_achTitle
 000A:000000DC       _vdmid_DosHeap
 000A:000000E8       _vdmid_fFgnd
 000A:000000EC       _vdmid_vpicBases
 000A:000000F0       _vdmid_aLSV
 000A:00000168       _pfntrapD
 000A:0000016C       _flrestart
 000A:00000170       _pszV86KernelSpec
 000A:00000274       _pVerInfoHeadLocal
 000A:00000278       _demStartSession_CDS_lowmem
 000A:000002BC       _demAllocBlkVMKHBI
 000A:000002CE       _demSS_us
 000A:000002D2       _demVDMStartCount
 000A:000002D6       _demFindFirstHack_head
 000A:000002DA       _demVDMStartDoneHndl
 000A:000002DE       _demVDMStartDoneSem
 000A:000002F3       _pFCBSFT
 000A:000002F7       _pszV86KernelName
 000A:000002FB       _flVDMDEM
 000A:00000304       _apiop
 000A:00001304       _appha
 000A:00001384       _apinthHead
 000A:00001784       _apvdmbp
 000A:00001984       _ivdmbpFreeListHead
 000A:00001988       _cbvdmbp
 000A:0000198C       _vpVdmBpArpl
 000A:00001990       _ptss
 000A:00001994       _cbtss
 000A:00001998       _pMapMemLockList
 000A:0000199C       _pVAPIList
 000A:000019A0       _pswIntBitmap
 000B:00000000       _StartCINIT_DATA
 000B:0000003A       dologo
 000B:000000DC       _vmdhAllocAccess
 000B:000000E8       _pAccessList
 000B:000000EC       _hmteCur
 000B:000000EE       _pmhGlobal
 000B:000000F2       _pmhLocal
 000B:000000F6       _ppddepHead
 000B:000000FA       _pfnVbiosPostInit
 000B:000000FE       _pszVPIC
 000B:00000104       _ahpi
 000B:00000144       _aobj
 000B:00000194       SysInitProc
 000B:0000019C       _pgTrueEndBound
 000B:000001A8       _pgHighMemHeadppf
 000B:000001AC       _pgHighMemHeadframe
 000B:000001B0       _pgHighMemTailppf
 000B:000001B4       _pgHighMemTailframe
 000B:000001B8       _baseladdr
 000B:000001BC       _paPend
 000B:000001C0       _paVend
 000B:000001C4       _pgTruePhysMax
 000B:000001C8       _pa1M
 000B:000001CC       _pgHighInitPending
 000B:000001D0       _szDefaultApps
 000B:00000304       _StartTHUNKINIT_DATA
 000B:00000304       _EndCINIT_DATA
 000B:00000753       _ThunkTable
 000B:00001774       _StartCSWAP_DATA
 000B:00001774       _EndTHUNKINIT_DATA
 000B:00001774       _vmApiF0
 000B:000017B4       _vmApiF1
 000B:000017F4       _vmAPIF2
 000B:0000180C       apfnOpcode
 000B:00001C0C       mpivsf
 000B:00001C60       _fVpmInitOK
 000B:00001C64       _pfndpmInt31Rte
 000B:00001C68       _pfndpmCreateTask
 000B:00001C6C       _pfndpmEndTask
 000B:00001C70       _apfnHighDispatchTable
 000B:00001C98       _hksemHFault
 000B:00001C9C       _PS2POSRegs
 000B:00001CF0       _hksemHLock
 000B:00001CF4       _System_config_table
 000B:00001CFE       _nVDMCreated
 000B:00001D02       _pVDDFixedInstStart
 000B:00001D06       _pVDDSwapInstStart
 000B:00001D0A       _pKrnlInstance
 000B:00001D0E       _pKrnlFixed
 000B:00001D12       _pKrnlSwap
 000B:00001D16       _pKrnlInstSwap
 000B:00001D1A       _lockentryhead
 000B:00001D22       _pBlackHole
 000B:00001D26       _cbBlackHole
 000B:00001D2A       _pbphHead
 000B:00001D2E       _hksemHVDD
 000B:00001D32       _aeh
 000B:00001DE6       _pPS2POSRegs
 000B:00001DEA       _pSystem_config_table
 000B:00001DEE       _nevents
 000B:00001DF2       _ulMachineType
 000B:00001DF6       _cbKrnlInstance
 000B:00001DFA       _cbKrnlInstSwap
 000B:00001DFE       _plockentryhead
 000B:00001E02       _phdlVddHead
 000B:00001E06       _pvddepHead
 000B:00001E0A       _aGSV
 000B:00001F34       _hprinCreateVDM
 000B:00001F38       _pszDemCurrDir
 000B:00001F3C       _pszProgCreateVDM
 000B:00001F40       _pszArgsCreateVDM
 000B:00001F44       _szFailureCause
 000B:00002044       _szEMSLowMem
 000B:0000205C       _ahp
 000B:000020FC       _pdhdBeforeHWInt
 000B:00002100       _apvtbn_cpu
 000B:00002130       _pvtbh_cpu
 000B:00002160       _apvtbn_mem
 000B:000021E4       _pvtbh_mem
 000B:00002214       _apvtbn_fbc
 000B:0000225C       _pvtbh_fbc
 000B:0000228C       _apvtbn_fil
 000B:000022D4       _pvtbh_fil
 000B:00002304       _apvtbn_thd
 000B:0000234C       _pvtbh_thd
 000B:0000237C       _apvtbn_spr
 000B:0000246C       _pvtbh_spr
 000B:0000249C       _apvtbn_cal
 000B:000024CC       _pvtbh_cal
 000B:000024FC       _apvtbn_instance
 000B:00002538       _pvtbh_instance
 000B:00002568       _fdynCodeLocked
 000B:00002D90       _demStartSession_CDS
 000B:00002DD4       _demStartSession_data
 000B:000031D4       _szAutoexec
 000B:000031E1       _szFakeVersion
 000B:000031ED       _szLastDrive
 000B:000031FB       _szDOSFiles
 000B:00003205       _vpboundDOSFiles
 000B:0000320B       _pVerInfoHeadGlobal
 000B:0000320F       _szRealTime
 000B:0000321D       _szVPICName
 000B:00003222       _hvddVPIC
 000B:00003226       _pfnSlaveRequest
 000B:0000322A       _szAutoexecSpec
 000B:0000323A       _demSS_next
 000B:0000323E       _demSS_curr
 000B:00003244       _iopDefault
 000B:00003280       _iopIgnore
 000B:000032D6       _pvdmArpl
 000B:000032DA       _vpvdmIRet
 000B:000032E0       _Start_DATA
 000B:000032E0       _toeBeep
 000B:000032E0       _EndCSWAP_DATA
 000B:000032F4       _fPreemptBeep
 000B:000032F8       _fSerialBeep
 000B:000032FC       _ulBeepTaskID
 000B:00003300       _ulSerialBeepFreq
 000B:00003304       _ulSerialBeepDoneTime
 000B:00003308       _f32pfnPTDBeep
 000B:00003310       _fBeepOwned
 000B:00003314       _f32pfnCLKFreq
 000B:00003394       ulTmrFreq
 000B:00003398       _fsTmrStatus
 000B:0000339A       _usTmrSem
 000B:0000339C       _pfnTMR16AddTime
 000B:000033A0       _pfnTMR16SubTime
 000B:00003508       _KEXBugBug
 000B:0000350C       _pKExitListHead
 000B:000037EC       CADHandlerActive
 000B:000037F0       _HardErrSem
 000B:000037F1       _HardErrTCB
 000B:000037F5       _SwapFullPTDA
 000B:000037FC       _IOShutdownState
 000B:00003800       _pVPB_BMP
 000B:00003844       _BufHashTable
 000B:00007844       _GFB_Sem
 000B:00007848       _FileDirtyMsk
 000B:0000784C       _fAsyncReadRunning
 000B:00007850       _AsyncReadHeadSel
 000B:00007854       _AsyncReadHeadOff
 000B:00007858       _AsyncReadTailSel
 000B:0000785C       _AsyncReadTailOff
 000B:00007860       _cBufs
 000B:00007864       _cbufLWLock
 000B:00007868       _LWBufWanted
 000B:0000786C       _fGFBActive
 000B:00007870       _pGFBWaitChain
 000B:00007874       _FLWReqListSel
 000B:00007878       _LWData
 000B:00007890       _aBufa
 000B:00007910       _semLW
 000B:00007914       _semLR
 000B:00007918       _semLRWait
 000B:0000791C       _msLastDiskWrite
 000B:00007920       _cbufDirty
 000B:00007924       _abDirtOrd
 000B:00007934       _abDirtBits
 000B:00007938       _abDirtBits2
 000B:0000793C       _ByteBitMasks
 000B:00007944       _FreeBufs
 000B:00007AA0       _PextattrIndex
 000B:00007AA4       _FextattrIndex
 000B:00007AA8       _FFirstWordIndex
 000B:00007AAC       _PFirstWordIndex
 000B:00007B94       _abMustRead
 000B:00007BA4       _LWAsyncSem
 000B:00007E3C       _szHotFixFile
 000B:00007EAC       _fSec
 000B:00007EB0       _fImport
 000B:00007EB4       _fImportPDF
 000B:00007EB8       _fImportAV
 000B:00007EBC       _fReentrant
 000B:00007EC0       _pSecIm_list_head
 000B:00007F0C       _GlobalNWD
 000B:00007F40       _TempBufSels
 000B:00007F84       _cSwapperResizing
 000B:000084AC       _ERROR_BLOCK_cnt
 000B:000085B4       _abBitMask
 000B:000085BC       _abFirstBit
 000B:000086C8       _SELDiscSegRmpSem
 000B:0000870C       _SMCompNextIndex
 000B:00008710       _smcLastErrorFence
 000B:00008714       _smfBackedOffFence
 000B:00008718       _SMInHardError
 000B:0000871C       _smTcbResizing
 000B:00008720       _smHardErrPID
 000B:00008724       _smMinSwapFile
 000B:00008728       _smcGrowFails
 000B:0000872C       _SMcDFInuse
 000B:00008730       _SMcInMemFile
 000B:00008734       _SMpInMemFile
 000B:00008738       _SMSwapSpace
 000B:0000873C       _smbmDF
 000B:00008740       _smFileSize
 000B:00008744       _smSizeHistory
 000B:00008748       _smDFMac
 000B:0000874C       _smcBrokenDF
 000B:00008750       _SMMinFree
 000B:00008754       _smPendingShrink
 000B:00008755       _smInitialized
 000B:00008756       _smParanoid
 000B:00008758       _smToe
 000B:0000876C       _SMPageSemHeld
 000B:00008834       _smSFNarr
 000B:00008838       _smSFTmap
 000B:0000883C       _SMMaxPageCmds
 000B:0000888C       _smSFTOwner
 000B:00008920       _vmOffGSR
 000B:00008924       _vmcpgLDTSkew
 000B:00008928       _vmcpgGDTSkew
 000B:0000892C       _vmcpgPTOVSkew
 000B:00008930       _vmcpgPTOGSkew
 000B:000089B4       _hkhCurrMax
 000B:000089B8       _vmkhGflags
 000B:000089BC       _vmLogFlags
 000B:000089C0       _atvm
 000B:00008B44       _vmdhL_Flags
 000B:00008C2C       _vmdhA_Flags
 000B:00008E0C       _vmInitFlags
 000B:00008E20       _vmNamShrSem
 000B:00008E4C       _aulvmAlignMask
 000B:00008E5C       _vmSGSFl
 000B:00008F1C       _ackrhsInit
 000B:00008F30       _khbaFree
 000B:00008F38       _pkhbaFree
 000B:00008F3C       _khbaLast
 000B:00008F44       _pkhbaLast
 000B:00008F48       _khbaBusy
 000B:00008F50       _pkhbaBusy
 000B:00008F54       _khbaDBusy
 000B:00008F5C       _pkhbaDBusy
 000B:000092B8       _fIsMVDMPresent
 000B:000092BC       _fIsInitTime
 000B:000092C0       _anpfnVPL
 000B:000092D0       _pszVpl
 000B:000092D4       _ulPICMaskState
 000B:000094CC       _pTempBlockHead
 000B:00009D94       _ppropList
 000B:00009F30       _fIsMarkOn
 000B:00009FBC       _INT10TCBNumber
 000B:00009FC0       _VDMINT10
 000B:0000A048       _V86CurrentPDB
 000B:0000A04C       _iINT10Creation
 000B:0000A070       _hKSEMPerf
 000B:0000A074       _fPerfview
 000B:0000A078       _pbPvwMsgQ
 000B:0000A07C       _cusPvwKInitRef
 000B:0000A080       _flPvwFlags
 000B:0000A084       _pbhPvwRPD
 000B:0000A088       _pbhPvwCfg
 000B:0000A08C       _pPvwRPDHead
 000B:0000A090       _bidPvwLastRPD
 000B:0000A094       _ked_pers
 000B:0000A0F8       _ked_tran
 000B:0000A140       _ppmb
 000B:0000A144       _f32pfnPTTimer0
 000B:0000A398       _qsFunc
 000B:0000A3C4       _gl_flag
 000B:0000A3C8       _pPtrRec
 000B:0000A3CC       _qsPSList
 000B:0000A9D8       _DBGBugBug
 000B:0000A9DC       _pdcbHead
 000B:0000A9E0       _pSemListHead
 000B:0000B314       _DYNNullResetPoint
 000B:0000B318       _pbDYNResetPoint
 000B:0000B31C       _dynsemTrap
 000B:0000B320       _dynselDTB
 000B:0000B324       _pbdynTraceAlias
 000B:0000B328       _pptedynTraceAlias
 000B:0000B32C       _pbdynTraceIntAlias
 000B:0000B330       _pptedynTraceIntAlias
 000B:0000B334       _DYNSavedUserFlags
 000B:0000B338       _DYNOldUserFlags
 000B:0000B33C       _fDYNActive
 000B:0000B340       _pdtoHeadScan
 000B:0000B344       _cdtoDetached
 000B:0000B348       _cdtoLoading
 000B:0000B3D4       _criISF
 000B:0000B42C       _criTSF
 000B:0000B484       _criVSF
 000B:0000B4DC       _criSEF
 000B:0000B534       _criPASCALSEF
 000B:0000B58C       _criSSF
 000B:0000B5E4       _criDHF
 000B:0000B63C       _aerg
 000B:0000B680       _hookheadGlobal
 000B:0000B6B4       _MSladdr
 000B:0000B6B8       _MSpte
 000B:0000B6BC       _MSpde
 000B:0000B6C0       _fB1NPX
 000B:0000B6C4       _pErrata17Hook
 000B:0000B6D4       pemulahndlr
 000B:0000B6D8       _FPEMDataSize
 000B:0000B6DC       _FPEMHandler
 000B:0000B6DC       FPEMHandler
 000B:0000B6E0       _FPEMpfnHandler
 000B:0000B718       runner
 000B:0000B71C       _FgndSGID
 000B:0000B71E       _tkFgndPID
 000B:0000B720       fIdle
 000B:0000B721       _fTKUsesR2
 000B:0000B722       _papTCBSlots
 000B:0000B7A0       _flArmed
 000B:0000B7A4       _pFiredTimerQueue
 000B:0000B864       _pPTDACur
 000B:0000B868       _pTCBCur
 000B:0000B86C       _pTKTSDs
 000B:0000B870       _pTSDCur
 000B:0000B874       _TKSSBase
 000B:0000B878       _TKTCBBias
 000B:0000B87C       _pfntkSuBuff
 000B:0000B880       _JITDbgeeSesPTDA
 000B:0000B884       _ulPLDTrapData
 000B:0000B938       _TKLibiCur
 000B:0000BAD8       _LibiDispatcher
 000B:0000BADC       _LibiDispatcher16
 000B:0000BAE0       _LibiDispatcher32
 000B:0000BD10       _pafnDoscall1
 000B:0000BD74       _pptdaTKEvap
 000B:0000BD78       _ctkScanners
 000B:0000BD7C       _ctkScannerOwner
 000B:0000BDA0       _ctcbTKInUse
 000B:0000BE14       _ctomTick
 000B:0000BE18       _ctom32hz
 000B:0000BE1C       _ctom128hz
 000B:0000BE20       _ctomCancel
 000B:0000BE24       _ctomSetFire
 000B:0000BE28       _ctomSet8msRes
 000B:0000BE2C       _ctomSet32msRes
 000B:0000BE30       _cSetOrderForever
 000B:0000BE34       _ctomStartMigration
 000B:0000BE38       _ctomMigrateAll
 000B:0000BE3C       _ctomMigrate
 000B:0000BE40       _ctomFire
 000B:0000BE44       _cMigrateHiRes
 000B:0000BE84       _cMigrateNext8
 000B:0000BE88       _cMigrateNext32
 000B:0000BE8C       _cMigrateOrder0
 000B:0000BE90       _cMigrateOrder1
 000B:0000BE94       _cMigrateOrder2
 000B:0000BE98       _cMigrateOrder3
 000B:0000BE9C       _cMigrateOrder4
 000B:0000BEA0       _cMigrateOrder5
 000B:0000BEA4       _ctomFiredEarly
 000B:0000BEA8       _ctomMaxEarly
 000B:0000BEAC       _ctomMax8Late
 000B:0000BEB0       _ctomMax32Late
 000B:0000BEB4       _TOMapfn
 000B:0000BED8       _cmsecTomTime
 000B:0000BEDC       _tomHiResPending
 000B:0000BEE0       _atowHash
 000B:0000C248       _toeTimeslice
 000B:0000C28C       _pPLDGlobal
 000B:0000C2E4       _pPSA
 000B:0000C2E8       _cProcessors
 000B:0000C2EC       _curProcNum
 000B:0000C30C       _ulTraceActive
 000B:0000C32C       _ki_enabled
 000B:0000C3DC       p6_events
 000B:0000C5D1       XLATab
 000B:0000C6D4       dhooks_maj13
 000B:0000C714       _fpfnINTKernelExit
 000B:0000C71A       _fpfnINTVDMIRQRouter
 000B:0000C720       airqi
 000B:0000C720       _airqi
 000B:0000C830       fpOldStack
 000B:0000C836       _cpuRatingFlag
 000B:0000C848       cIRQ
 000B:0000C84C       NPX_IRQ
 000B:0000C850       HardwareInterruptTable
 000B:0000C8B0       os2Stack
 000B:0000C8C0       privateStack
 000B:0000C8C4       _fpfnDHKernelExit
 000B:0000C8CC       _KDDC
 000B:0000CA48       _pNonResNamTbl
 000B:0000CA4C       _cNonResNamTbl
 000B:0000CA50       _program_h
 000B:0000CA54       _program_l
 000B:0000CA58       _global_h
 000B:0000CA5C       _global_l
 000B:0000CA60       _specific_h
 000B:0000CA64       _specific_l
 000B:0000CA68       _swapping
 000B:0000CA6C       _do_gcollect
 000B:0000CA70       _LDRLieList
 000B:0000CA74       _pldrOpen
 000B:0000CA78       _pldrReadAt
 000B:0000CA7C       _pldrClose
 000B:0000CA80       _pIOSftTransPath
 000B:0000CA84       _pldrGetMedia
 000B:0000CA88       _ldrMiniFileIOFlag
 000B:0000CA8C       _mptbl
 000B:0000CAD0       _validatetbl
 000B:0000CAE4       _HeaderInfoTbl
 000B:0000CB14       _HeaderInfoSTE
 000B:0000CB3C       _objflags
 000B:0000CB74       _selflags
 000B:0000CB94       _objmem
 000B:0000CBB4       _pgstatechg
 000B:0000CBBC       RsrcHead
 000B:0000CBC0       _ldrErr
 000B:0000CBD0       _pDosModMte
 000B:0000CBD4       _pPortHoleMte
 000B:0000CBD8       _pPHMtePath
 000B:0000CBE6       _pPHMteResNam
 000B:0000CBF2       _pPHMteObjTab
 000B:0000CC0A       _BasicHWConfig
 000B:0000CC3C       _pldrdldHeadKernel
 000B:0000CC40       _ldrDoGCollect
 000B:0000D014       _PGSCNLocals
 000B:0000D018       _PGSCLocalsInit
 000B:0000D01C       _pGDTThreadCopy
 000B:0000D020       _pGDTTaskCopy
 000B:0000D024       _pGDTTIBCopy
 000B:0000D028       _clDescTaskCopy
 000B:0000D02C       _clDescThreadCopy
 000B:0000D030       _clDescTIBOffset
 000B:0000D034       InfoSegsValid
 000B:0000D140       _PGTestPage1
 000B:0000D144       _PGTestPage2
 000B:0000D1C0       _pgpSavePF
 000B:0000D1C4       _pgPhysPages
 000B:0000D1C8       _pgSwappablePages
 000B:0000D1CC       _pgResidentPages
 000B:0000D1D0       _pgDiscardablePages
 000B:0000D1D4       _pgShortLockPages
 000B:0000D1D8       _pgMaxResPages
 000B:0000D1DC       _pgResidentWanted
 000B:0000D1E0       _pgResPT
 000B:0000D1E4       _pgDiscardableInmem
 000B:0000D1E8       _PGGlobalFlags
 000B:0000D1EC       _pgcPageFaults
 000B:0000D1F0       _pgcPageFaultsActive
 000B:0000D1F4       _pgPhysMax
 000B:0000D1F8       _pgFlagMask
 000B:0000D1FC       _pgAgeRateTable
 000B:0000D258       _pgCurAgeRate
 000B:0000D25C       _ApuOwner
 000B:0000D264       _MonApp
 000B:0000D26C       _MonSys
 000B:0000D274       _pResInfBuf
 000B:0000D278       _cbRIB
 000B:0000D27C       _fRegistered
 000B:0000D280       _pgHighPages
 000B:0000D284       _pgHighPagesUsed
 000B:0000D438       _SELGDTLaddr
 000B:0000D43C       _SELGDTHandle
 000B:0000D43E       _SELMaxGDT
 000B:0000D440       _SELGDTFreeList
 000B:0000D442       _R0DS
 000B:0000D444       _R0CS
 000B:0000D446       _R2DS
 000B:0000D448       _R2CS
 000B:0000D44A       _R3DS
 000B:0000D44C       _R3PDS
 000B:0000D44E       _R3CS
 000B:0000D450       _R3THKDS
 000B:0000D452       _R0CSC
 000B:0000D454       _R3TIB
 000B:0000D478       _pfnDLLTermDisp32
 000B:0000D5C4       _ichain_print
 000B:0000D604       _TypLenTbl
 000B:0000D670       _FlatSelTbl
 000B:0000D6B8       _ldrOrdinalMap
 000B:0000D811       _ldrfromLdrRun
 000B:0000D814       _ldrWLOTbl
 000B:0000D830       _ldrSysTbl
 000B:0000DB38       _pVMLIHead
 000B:0000DB3C       _LogLockInfo
 000B:0000DB40       _cvmltMax
 000B:0000DB44       _cvmltUsed
 000B:0000DC04       _selGDT_PTDA
 000B:0000DE8C       _ppbPvwMtHook
 000B:0000DE90       fbPvwPatch
 000B:0000DE91       _Pvwptcblast
 000B:0000E0B4       _DBGlmskDR7system
 000B:0000E0B8       _DBGlmskDR7reserved
 000B:0000E298       CallGate_Debug_SymWinOS2
 000B:0000E29A       _pDevHead
 000B:0000E359       __acrtused
 000B:0000E3E4       _cbTKMaxStackUsed
 000B:0000E408       _pgfaultboost
 000B:0000E40C       _tkTSDSwapRateMax
 000B:0000E410       _tkMaxSlice
 000B:0000E414       _tkMinSlice
 000B:0000E418       _tkMaxWait
 000B:0000E41C       _cmsecStarveLength
 000B:0000E420       _tkAllowedStateTrans
 000B:0000E438       _schPriClassTbl
 000B:0000E538       _ksctalc
 000B:0000E53C       _ksctalcblk
 000B:0000E540       _fpfnTRAPKernelExit
 000B:0000E546       _fpfnVDMKernelExit
 000B:0000E98A       fTrapToScreen
 000B:0000E98E       _NMIPhysAddr
 000B:0000E992       _NMIPTDA
 000B:0000EAF8       _PTBugBug
 000B:0000FDC8       _GlobalJITDbg
 000B:0000FDCC       _GlobalJITParms
 000B:0000FDD0       _GlobalJITDbgFlgs
 000B:0000FDD4       _JITDBGOveride
 000B:00017E9C       GoTimeL
 000B:00017EA0       GoTimeH
 000B:00017EA4       DBGOveride
 000B:00017EB8       NESymHead
 000B:0001FEE5       _KDBNesting
 000B:0001FEE9       _PICMask
 000B:0001FEF0       _pprintfbuf
 000B:0001FEF4       _cprintfbuf
 000B:0001FF30       _DosModMte
 000B:0001FF30       _StartDOSMTE
 000B:0001FF30       _End_DATA
 000B:0001FF58       _DosModMteSwappable
 000B:0001FFDA       dcm_ote_start
 000B:00020172       _EndDOSMTE
 000B:00020172       _StartDOSMTEMID
 000B:00020172       _StartDOSMTENAME
 000B:00020172       _EndDOSMTENAME
 000B:00020173       dcm_length
 000B:00020173       dcm_entrytblstart
 000B:00020175       _EndDOSMTEMID
 000B:00020175       _StartDOSMTEENTRY
 000B:00020E5C       _ldrMteAux
 000B:00020E5C       _EndDOSMTEENTRY
 000B:00020E5C       _StartDOSMTEAUX
 000B:00020E74       _FSHModMte
 000B:00020E74       _StartFSHMTE
 000B:00020E74       _EndDOSMTEAUX
 000B:00020E9C       FSHModMteSwappable
 000B:00020F36       _EndFSHMTE
 000B:00020F36       _StartFSHMTEMID
 000B:00020F36       _StartFSHMTENAME
 000B:00020F36       _EndFSHMTENAME
 000B:00020F37       _EndFSHMTEMID
 000B:00020F37       fsh_entrytblstart
 000B:00020F37       _StartFSHMTEENTRY
 000B:00021013       _VDDModMte
 000B:00021013       _EndFSHMTEENTRY
 000B:00021013       _StartVDDMTE
 000B:0002103B       VDDModMteSwappable
 000B:000210CD       _EndVDDMTE
 000B:000210CD       _StartVDDMTEMID
 000B:000210CD       _StartVDDMTENAME
 000B:000210CD       _EndVDDMTENAME
 000B:000210CE       vdd_length
 000B:000210CE       vdd_entrytblstart
 000B:000210D0       _EndVDDMTEMID
 000B:000210D0       _StartVDDMTEENTRY
 000B:00021368       _EndVDDMTEENTRY
 000B:00021368       _StartPANICMSG
 000B:000269F8       _EndCONST
 000B:000269F8       _StartCONST
 000B:000269F8       _Start_BSS
 000B:000269F8       _EndPANICMSG
 000B:00026B30       _hyberStat
 000B:00026B30       _End_BSS
 000B:00026B30       _Startc_common
 000B:00026B34       _pRecStart
 000B:00026B38       _pobvmZero
 000B:00026B3C       _pSec32Worker
 000B:00026B40       _DBGapgwpcb
 000B:00026B50       _pSec16Worker
 000B:00026B54       _pgpAgerTCB
 000B:00026B58       _LDRLibPath
 000B:00026B5C       _pgVPBasePg
 000B:00026B60       _parRWBasedSearchStart
 000B:00026B64       _pheaderbuf
 000B:00026B68       _DBGpdcbCur
 000B:00026B6C       _smpHeapEnd
 000B:00026B70       _pgAliasPte
 000B:00026B74       _laGlobalMap
 000B:00026B80       _pg64Kerrata
 000B:00026B84       _aErrorCode
 000B:00026C08       _fHotFixing
 000B:00026C0C       _pgbmSegBuf
 000B:00026C10       _pgpPageDir
 000B:00026C14       _pBeginCache
 000B:00026C18       _DiskThresh
 000B:00026C1C       _pResLibRec
 000B:00026C20       _DBGaDRowner
 000B:00026C30       _ldrQATCache
 000B:00026C3C       _pageTKTSDs
 000B:00026C40       _aptcbSleep
 000B:00027044       _pgFreeList
 000B:0002705C       _pgIdleList
 000B:00027074       _BufLRUHead
 000B:000271C8       _pHyberInfo
 000B:000271CC       _pgSysPtHOB
 000B:000271D0       _FFirstWord
 000B:00027360       _TKBitBucket
 000B:00027364       _pKStackBase
 000B:00027368       _VMPackedMem
 000B:0002736C       _SMpCompTbl
 000B:00027370       _smDelaySwap
 000B:00027374       _parProtectSearchStart
 000B:00027378       _FextattrRBA
 000B:00027698       _smpHeapComp
 000B:0002769C       _PGFaultCnt
 000B:000276A0       _PFirstWord
 000B:00027830       _pgErrCdMask
 000B:00027834       _pgSegBufPte
 000B:000278F4       _pPTDAFirst
 000B:000278F8       _ResExLibRec
 000B:0002791E       _smSwapDisk
 000B:00027920       _pVMTempBuf
 000B:00027924       _pResPtrRec
 000B:00027928       _PextattrRBA
 000B:00027C48       _pPhysLRBuf
 000B:00027C4C       _hPvwMtLock
 000B:00027C58       _pgCommitSem
 000B:00027C64       _HotFixKsem
 000B:00027C70       _pgAliasLaddr
 000B:00027C74       _pgTSDStart
 000B:00027C78       _hMteDoscall1
 000B:00027C7C       _BufFreeList
 000B:00027DD0       _SMpCompBase
 000B:00027DD4       _aulSysInfo
 000B:00027E40       _pgbmContext
 000B:00028040       _pmteDoscall1
 000B:00028044       _ulShTotUsed
 000B:00028048       _ulShTblSize
 000B:0002804C       _palVMAliases
 000B:00028050       _ulkdbAddrLDT
 000B:00028054       _pgListCount
 000B:00028058       _hookheadTIMH
 000B:00028060       _pgAgerAsleep
 000B:00028064       _pgShrCRPtHOB
 000B:00028068       _pEndStateBuf
 000B:0002806C       _vmladdrMinKH
 000B:00028070       _pCurStateBuf
 000B:00028074       _pgListHeadVP
 000B:00028080       _StartupData
 000B:00028194       _vmladdrMaxKH
 000B:00028198       _BufDirtyHead
 000B:000282EC       _ptcbPriQTSD
 000B:000282F0       _hyberPhysPT
 000B:000282F4       _pgflPinFault
 000B:000282F8       _pfntkDosExit
 000B:000282FC       _hyberInfoHob
 000B:00028300       _ulShNextFree
 000B:00028304       _AsyncReadSem
 000B:00028308       _pPLDDynTrace
 000B:0002830C       _pkshdVMDescs
 000B:00028310       _SMSwapperSem
 000B:0002831C       _hyberPhysHob
 000B:00028320       _pShSemStrTbl
 000B:00028324       _pgPageablePAI
 000B:00028350       _hyberOpCount
 000B:00028354       _PGSegBufLaddr
 000B:00028358       _BaseSavedMTEs
 000B:000283A0       _ldrDebugFlags
 000B:000283A4       _PGSwapEnabled
 000B:000283A8       _LDRLibPathLen
 000B:000283AC       _DBGlDR7global
 000B:000283B0       _pPLDRing0Trap
 000B:000283B4       _phookCodeLock
 000B:000283B8       _ldrcDLLDetach
 000B:000283BC       _MiniVDMCreate
 000B:000283C0       _MonLockHandle
 000B:000283CC       _pgAllocBufHob
 000B:000283D0       _aSharedBuffer
 000B:00028BD0       _VDMInt13IRQCS
 000B:00028BD4       _hNonResNamTbl
 000B:00028BD8       _vmPackedLBDRY
 000B:00028BDC       _tkcPriUpdates
 000B:00028BE0       _PLDQuiesceSem
 000B:00028BEC       _pageTKTSDsEnd
 000B:00028BF0       _vmPackedUBDRY
 000B:00028BF4       _pgSegBufOwner
 000B:00028BFC       _tkcPriChanges
 000B:00028C2C       _pgResidentPAI
 000B:00028C58       _pHyberInfoHdr
 000B:00028C5C       _pgZeroFillPte
 000B:00028C60       _pgLdrBufOwner
 000B:00028C80       _pgcPtePresent
 000B:00029180       _pgpZeroFillVP
 000B:00029184       _parGlobalShrSearchStart
 000B:00029188       _tkcStateTrans
 000B:000293C8       _ptcbPriQReady
 000B:000293CC       _SMCompactSlot
 000B:000293D0       _pft
 000B:000293D4       _pfntkDos32Exit
 000B:000293D8       _apfi
 000B:000294D8       _apkh
 000B:00029520       _pgSegBufWanted
 000B:00029521       _Int13TCBNumber
 000B:00029523       _pgLdrBufWanted
 000B:00029524       _pgbmLdrPageBuf
 000B:00029528       _paTCB
 000B:0002952C       _ichain_cphyspg
 000B:00029530       _pfnSigDispatch
 000B:00029534       _VDMInt13IRQEIP
 000B:00029538       _ldrpFileNameBuf
 000B:0002953C       _VDMInt13CurIRQ
 000B:00029540       _GFBActiveThread
 000B:00029544       _FextattrRBAcnt
 000B:000296D4       _ppteKStackBase
 000B:000296D8       _pgSwapAddrType
 000B:000296DC       _fLWIO
 000B:000296E0       _pgcPteResident
 000B:00029BE0       _pgcPteAllocated
 000B:0002A0E0       _SMpFreeCompDFs
 000B:0002A0E4       _pgHiResBoundfr
 000B:0002A0E8       _pslhLockHandles
 000B:0002A0EC       _SelShrPackedEnd
 000B:0002A0F0       _nrbuf
 000B:0002A1F4       _pgLoResBoundfr
 000B:0002A1F8       _pgSwapBufOwner
 000B:0002A238       _dynlh
 000B:0002A244       _ulFreeMuxCount
 000B:0002A248       _QsSem
 000B:0002A254       _pgpCRPageTables
 000B:0002A258       _VMProtectedMem
 000B:0002A25C       _mte_h
 000B:0002A260       _ptcbPriQDelayed
 000B:0002A264       _pvmlt
 000B:0002A268       _ptcbtkTSDDaemon
 000B:0002A26C       _pgbmSwapPageBuf
 000B:0002A270       _pPLDHotKeyHook
 000B:0002A274       _pgSwapBufWanted
 000B:0002A278       _pgHiResBoundppf
 000B:0002A27C       _DBGmpclwpcbcptda
 000B:0002A284       _pgLoResBoundppf
 000B:0002A288       _S2_RW_RQPKT_SIZE
 000B:0002A28C       _vmGlobalShrLBDRY
 000B:0002A290       _vmGlobalShrUBDRY
 000B:0002A294       _ldr16pFileNameBuf
 000B:0002A298       _ptcbPriQRunner
 000B:0002A29C       _ptcbPriQBadStack
 000B:0002A2A0       _pgpSysPageTables
 000B:0002A2A4       _pPTDAFirstZombie
 000B:0002A2A8       _hyberMaxPageCmds
 000B:0002A2AC       _ptcbPriQGetStack
 000B:0002A2B0       _pgcShrPtePresent
 000B:0002A2F0       _syncTSInitTout
 000B:0002A2F4       _pfnXcptFRestore32
 000B:0002A2F8       _pgLdrPageBufLaddr
 000B:0002A2FC       _paPTDA
 000B:0002A300       _pgShortLockWanted
 000B:0002A304       _pgData
 000B:0002A32C       _cmsecHiResTomTime
 000B:0002A330       _DBGckDR
 000B:0002A334       _hmapid
 000B:0002A33C       _hksemPropertyBits
 000B:0002A340       _pgcShrPteResident
 000B:0002A380       _gl_pid
 000B:0002A384       _LdrSem
 000B:0002A390       _SelShrPackedStart
 000B:0002A394       _ahtimer
 000B:0002A398       _dynDTB
 000B:0002B418       _smpHeap
 000B:0002B41C       _ulShSemStrTblUsed
 000B:0002B420       _fpregs
 000B:0002B48C       _ahvmShr
 000B:0002B4CC       _ulShSemStrTblSize
 000B:0002B4D0       _FLWKsem
 000B:0002B4DC       _pSigGCH
 000B:0002B4E0       _pgVPHob
 000B:0002B4E4       _smPCarr
 000B:0002B4F4       _pgLDTva
 000B:0002B4F8       _ahvmSys
 000B:0002B538       _PSAVARS
 000B:0002B598       _tmplist
 000B:0002B59C       _ntimers
 000B:0002B5A0       _cDLLTerm
 000B:0002B5A4       _pgVPHead
 000B:0002B5B0       _pgTSDEnd
 000B:0002B5B4       _qsElist
 000B:0002B5B8       _palvmIal
 000B:0002B5BC       _timhTail
 000B:0002B5E4       _pgpVPEnd
 000B:0002B5E8       _parvmOne
 000B:0002B5EC       _pFreeMux
 000B:0002B5F0       _pcovmOne
 000B:0002B5F4       _pfnXcptDispatcher32
 000B:0002B5F8       _smbmComp
 000B:0002B618       _PDumpSem
 000B:0002B624       _hksShTbl
 000B:0002B628       _pPLDInfo
 000B:0002B62C       _htimhook
 000B:0002B630       _pobvmOne
 000B:0002B634       _bCodeLockHookArmed
 000B:0002B638       _PopUpSem
 000B:0002B644       _msLastIO
 000B:0002B648       _BaseRememberedMTEs
 000B:0002B708       _pVDMInt13
 000B:0002B70C       _pEndCache
 000B:0002B710       _pgcShrPteAllocated
 000B:0002B750       _pCurCache
 000B:0002B754       _ResLibRec
 000B:0002B76C       _pDebugLoadSymDosFS
 000B:0002B770       _fLWDaemon
 000B:0002B774       _pgSwapPageBufLaddr
 000B:0002B778       _ulkdbAddr
 000B:0002B77C       _pgShrData
 000B:0002B7A2       _gl_hndmod
 000B:0002B7A4       _pgpVPBase
 000B:0002B7A8       _pgpShrCRPageTables
 000B:0002B7AC       _DosModHdl
 000B:0002B7B0       _hksSemRec
 000B:0002B7B4       _smHobheap
 000B:0002B7B8       _pgVPEndPg
 000B:0002B7BC       _pDebugLoadSymModule
 000B:0002B7C0       _pFPEMVMBH
 000B:0002B7C4       _DBGcSysDR
 000B:0002B7C8       _ResPtrRec
 000B:0002B7E8       _pgCRPtHOB
 000B:0002B7EC       _ShortName
 000B:0002B7F8       _pgBufSels
 000B:0002B804       _pLinLRBuf
 000B:0002B808       _pShSemTbl
 000B:0002B80C       _pgSysPtpg
 000B:0002B810       _hksStrTbl
 000B:0002B814       _parPackedSearchStart
 000B:0002B818       _parvmZero
 000B:0002B81C       _pcovmZero
 000B:0002B820       _uskdbSlot
 000C:00000000       _StartHIGH2CODE
 000C:00000004       h_AssertNoBufProc
 000C:00000006       AssertNoBufProc
 000C:00000038       checkfat
 000C:000000A8       h_w_DiskReset
 000C:000000AC       f_w_DiskReset
 000C:000000AE       w_DiskReset
 000C:000000B8       BufInvalidate
 000C:000000F0       BufInvalidate2
 000C:0000012C       h_BufFree
 000C:00000130       f_BufFree
 000C:00000132       BufFree
 000C:00000198       h_BufIncRef
 000C:0000021C       h_BufDecRef
 000C:0000022C       h_BufNext
 000C:00000268       ScanPlace
 000C:00000270       PlaceBufMRU
 000C:0000028C       PlaceBufLRU
 000C:000002A8       h_GetMRUBufSec
 000C:000002AC       f_GetMRUBufSec
 000C:000002AE       GetMRUBufSec
 000C:000002C0       buf$UnlinkBuf
 000C:000002F4       h_GetBuffrBP
 000C:000002F8       f_GetBuffrBP
 000C:000002FA       GetBuffrBP
 000C:00000300       h_GetBuffr
 000C:00000302       GetBuffr
 000C:0000030C       h_GetBuffrB
 000C:0000030E       GetBuffrB
 000C:000004F4       BufCacheRead
 000C:00000624       ChkBufPtr
 000C:00000654       buf$GetFreeBuffr
 000C:00000738       h_RlseBuffr
 000C:0000073C       f_RlseBuffr
 000C:0000073E       RlseBuffr
 000C:00000784       BufCacheWrite
 000C:00000874       buf$LockBuf_
 000C:000008C4       UnlockBuf
 000C:00000904       h_FlushBuf
 000C:00000906       FlushBuf
 000C:0000090B       FlushBufND
 000C:000009B4       h_FlushBuf2
 000C:000009B6       FlushBuf2
 000C:00000A78       h_FSD_FlushBuf
 000C:00000A7A       FSD_FlushBuf
 000C:00000B38       f_w16_FSD_FlushBuf
 000C:00000C44       buf$FlushFsdBuf
 000C:00000CC8       h_PointComp
 000C:00000CCA       PointComp
 000C:00000CDC       buf$WaitBuf
 000C:00000D14       h_BufWrite
 000C:00000D16       BufWrite
 000C:00000EA0       h_RemoveBufVPB
 000C:00000EA2       RemoveBufVPB
 000C:00000EBC       buf$ChkNoBuf
 000C:00000EC0       GetOverlapBuf
 000C:00000F50       h_FindMultiChar
 000C:00000F52       FindMultiChar
 000C:00000F94       ExmDBCS
 000C:00000FD8       CharTypeHIGH2
 000C:000010D8       h_w_16DevIOCtl
 000C:000010DC       f_w_16DevIOCtl
 000C:000010DE       w_16DevIOCtl
 000C:00001100       h_w_32DevIOCtl
 000C:00001104       f_w_32DevIOCtl
 000C:00001106       w_32DevIOCtl
 000C:0000116C       w_DevIOCtl
 000C:000015B4       sw_EjectPassT
 000C:000016AC       h_sw_DevIOCtlFar
 000C:000016C4       sw_DevIOCtl
 000C:00001894       devioctl$swioc_calldriver
 000C:00001910       h_EndTransfer
 000C:00001912       EndTransfer
 000C:00001978       h_FSD_Read
 000C:0000197C       f_FSD_Read
 000C:0000197E       FSD_Read
 000C:00001B04       h_FSD_Write_NT
 000C:00001B08       f_FSD_Write_NT
 000C:00001B0A       FSD_Write_NT
 000C:00001B12       disk$FSD_WriteNoSpool
 000C:00001B1B       h_FSD_Write
 000C:00001B1D       FSD_Write
 000C:00001D4C       SpoolWrite
 000C:00001DD8       SpoolFirstWrite
 000C:00001E70       SpoolWriteErr
 000C:00001E9C       SpoolXact
 000C:00001F04       Read_Lock_Violation
 000C:00001F64       Write_Lock_Violation
 000C:00001F8C       Network_Retry
 000C:00001FD4       dosfs$PhysClose
 000C:00002024       h_Byte13_PackName
 000C:00002078       h_FSD_Exit
 000C:0000207A       FSD_Exit
 000C:000020A0       h_FSD_Close
 000C:000020A4       f_FSD_Close
 000C:000020A6       FSD_Close
 000C:00002234       h_FSD_Commit
 000C:00002238       f_FSD_Commit
 000C:0000223A       FSD_Commit
 000C:00002294       dosfs$SetSFTTimes
 000C:000022E0       h_FSD_Delete
 000C:000022E2       FSD_Delete
 000C:000023D0       h_FSD_Move
 000C:000023D2       FSD_Move
 000C:0000257C       h_CheckPathSyntax
 000C:0000257E       CheckPathSyntax
 000C:000025DC       h_DOS_Abort
 000C:000025E0       f_DOS_Abort
 000C:000025E2       DOS_Abort
 000C:00002710       f_DOS_AbortVDM
 000C:00002794       dosfs$Ren_Check
 000C:00002814       h_w_FindClose
 000C:00002816       w_FindClose
 000C:0000283C       FSD_FindClose
 000C:00002948       h_w_32FindFirst
 000C:00002B20       h_w_FindFirst
 000C:00002B22       w_FindFirst
 000C:00002D84       FSD_FindFirst
 000C:00002DD4       dossrch$call_fsd_ff
 000C:00002E70       dossrch$GetSrchSel
 000C:00002E8C       h_w_32FindNext
 000C:00003318       h_w_FindNext
 000C:0000331C       f_w_FindNext
 000C:0000331E       w_FindNext
 000C:0000348C       wfn_FreeGDTSelector
 000C:000034A0       FSD_FindNext
 000C:000034E0       dossrch$call_fsd_fn
 000C:00003520       dossrch$GetNewHand
 000C:00003538       dossrch$GetSStruc
 000C:0000354C       dossrch$WrapInc
 000C:00003564       h_FindExit
 000C:00003590       h_w_FindFromName
 000C:00003594       f_w_FindFromName
 000C:00003596       w_FindFromName
 000C:000036D4       dossrch$FSD_FindFromName
 000C:00003740       h_CopyEANameString
 000C:000037B4       h_CheckEAName
 000C:00003820       h_MakeFcb
 000C:00003824       f_MakeFcb
 000C:00003826       MakeFcb
 000C:000038B7       fcb$NORMSCAN
 000C:000038EF       fcb$GETWORD
 000C:000038F5       fcb$MUSTGETWORD
 000C:00003968       fcb$Compatibility
 000C:000039BC       h_NameTrans
 000C:000039BE       NameTrans
 000C:00003A7C       fcb$GetLet
 000C:00003AAB       DELIM
 000C:00003AB0       SPCHK
 000C:00003AB8       h_api_Close
 000C:00003ABA       api_Close
 000C:00003AD4       h_w_Close
 000C:00003AD8       f_w_Close
 000C:00003ADA       w_Close
 000C:00003C30       fhandle$CloseSpooled
 000C:00003C7C       h_Wake_plock
 000C:00003C7E       Wake_plock
 000C:00003CD0       f_w_3xBufReset
 000C:00003CFC       f_ReadDo
 000C:00003D0C       h_w_Read
 000C:00003D10       f_w_Read
 000C:00003D12       w_Read
 000C:00003D2E       h_WriteDo
 000C:00003D30       WriteDo
 000C:00003D46       h_ReadDo
 000C:00003D48       ReadDo
 000C:00003DBC       h_w_Write
 000C:00003DC0       f_w_Write
 000C:00003DC2       w_Write
 000C:00003DD0       h_w_NewSize
 000C:00003DD4       f_w_NewSize
 000C:00003DD6       w_NewSize
 000C:00003EAC       f_FSD_NewSize
 000C:00003EAE       FSD_NewSize
 000C:00003F58       h_w_LSeek
 000C:00003F5C       f_w_LSeek
 000C:00003F5E       w_LSeek
 000C:00003FB0       h_sft_lseek
 000C:00003FB4       f_sft_lseek
 000C:00003FB6       sft_lseek
 000C:0000403C       h_FSD_ChgFilePtr
 000C:00004040       f_FSD_ChgFilePtr
 000C:00004042       FSD_ChgFilePtr
 000C:00004140       h_FileTimes
 000C:00004144       f_FileTimes
 000C:00004146       FileTimes
 000C:000041AC       h_w_Dup
 000C:000041B0       f_w_Dup
 000C:000041B2       w_Dup
 000C:00004218       h_w_Dup2
 000C:0000421A       w_Dup2
 000C:0000427C       h_api_Dup
 000C:0000427E       api_Dup
 000C:00004294       h_w_QFHandState
 000C:00004298       f_w_QFHandState
 000C:0000429A       w_QFHandState
 000C:00004360       h_w_SetFHandState
 000C:00004362       w_SetFHandState
 000C:00004424       h_w_QHandType
 000C:00004428       f_w_QHandType
 000C:0000442A       w_QHandType
 000C:0000449C       h_is_device
 000C:0000449E       is_device
 000C:000044B8       h_PhysHandle
 000C:000044BC       f_PhysHandle
 000C:000044BE       PhysHandle
 000C:000044D4       f_Ext_Information
 000C:000045AC       f_EAOP_selector_free
 000C:000045B4       h_EAOP_selector_alloc
 000C:000045B8       f_EAOP_selector_alloc
 000C:000045BA       EAOP_selector_alloc
 000C:000045EF       h_EAOP_selector_free
 000C:000045F1       EAOP_selector_free
 000C:00004610       h_api_OpenCreate
 000C:00004612       api_OpenCreate
 000C:000046D8       h_w_OpenCreate
 000C:000046DC       f_w_OpenCreate
 000C:000046DE       w_OpenCreate
 000C:00004A58       file$OpenSpooled
 000C:00004BA0       h_TransactSpooler
 000C:00004BA2       TransactSpooler
 000C:00004BD0       file$SetPhysDiskSFT
 000C:00004C08       h_w_Creat
 000C:00004C0A       w_Creat
 000C:00004C0F       w_CreateNew
 000C:00004C12       AccessSet
 000C:00004C24       f_w_3xCreateNew
 000C:00004C26       w_3xCreateNew
 000C:00004C30       f_w_CreateTempFile
 000C:00004CDC       h_DoOpenCreate
 000C:00004CE0       f_DoOpenCreate
 000C:00004CE2       DoOpenCreate
 000C:00004D30       h_w_ChMod
 000C:00004D34       f_w_ChMod
 000C:00004D36       w_ChMod
 000C:00004DFC       h_w_Unlink
 000C:00004E00       f_w_Unlink
 000C:00004E02       w_Unlink
 000C:00004E5C       h_w_StoreFile
 000C:00004E60       f_w_StoreFile
 000C:00004E62       w_StoreFile
 000C:00004E98       h_w_StoreFile3x
 000C:00004E9C       f_w_StoreFile3x
 000C:00004E9E       w_StoreFile3x
 000C:00004ECC       h_w_Rename
 000C:00004ED0       f_w_Rename
 000C:00004ED2       w_Rename
 000C:00004FBC       file$SetAttrib
 000C:00004FE0       file$Check_Access_AX
 000C:00005008       CheckNotPipeDir
 000C:00005040       h_FSD_QFileMode
 000C:00005042       FSD_QFileMode
 000C:000050B8       FSD_SetFileMode
 000C:00005168       f_SFT_SetFileInfo
 000C:00005170       h_w_SetFileInfo
 000C:00005172       w_SetFileInfo
 000C:000051ED       h_SFT_SetFileInfo
 000C:000051EF       SFT_SetFileInfo
 000C:00005304       FSD_QFileInfo
 000C:00005364       f_SFT_QFileInfo
 000C:0000536C       h_w_QFileInfo
 000C:00005370       f_w_QFileInfo
 000C:00005372       w_QFileInfo
 000C:000053F8       h_w_QPathInfo
 000C:000053FC       f_w_QPathInfo
 000C:000053FE       w_QPathInfo
 000C:00005438       h_w_SetPathInfo
 000C:0000543A       w_SetPathInfo
 000C:000054F0       finfo$DoPathInfo
 000C:00005724       f_w_3xEnumAttrib
 000C:000057EC       f_w_BigOper16
 000C:000059C0       h_fscNext
 000C:000059C2       fscNext
 000C:000059DC       h_fscFind
 000C:000059DE       fscFind
 000C:000059F8       fsc$fscStrCmp
 000C:00005A44       Share_Violation
 000C:00005A57       Violation_Delay_Retry
 000C:00005A90       FSH_SEGALLOC
 000C:00005B10       FSH_SEGFREE
 000C:00005B38       FSH_SEGREALLOC
 000C:00005B70       FSH_FORCENOSWAP
 000C:00005B94       FSH_SEMSET
 000C:00005BB4       FSH_SEMSETWAIT
 000C:00005BDC       FSH_SEMWAIT
 000C:00005C04       FSH_PROBEBUF
 000C:00005C38       FSH_EXTENDTIMESLICE
 000C:00005C4C       FSH_GETPRIORITY
 000C:00005C78       FSH_IOBOOST
 000C:00005CA4       FSH_QUERYSERVERTHREAD
 000C:00005CC0       FSH_QUERYOPLOCK
 000C:00005CFC       FSH_FLUSHBUF
 000C:00005D3C       FSH_CRITERROR
 000C:00005DBC       CritErrPause
 000C:00005E38       FSH_DEVIOCTL
 000C:00005E88       FSH_GETVOLPARM
 000C:00005EE0       FSH_FINDDUPHVPB
 000C:00005F20       FSH_DOVOLIO
 000C:00006160       FSH_DOVOLIO2
 000C:000061A0       FSH_ADDSHARE
 000C:00006250       FSH_REMOVESHARE
 000C:00006268       FSH_ISCURDIRPREFIX
 000C:00006294       FSH_LOADCHAR
 000C:000062D4       FSH_PREVCHAR
 000C:00006318       FSH_STORECHAR
 000C:00006354       FSH_GETOVERLAPBUF
 000C:00006394       FSH_WILDMATCH
 000C:00006538       FSH_FINDCHAR
 000C:00006568       FSH_CANONICALIZE
 000C:00006628       FSH_QSYSINFO
 000C:000066CC       FSH_NAMEFROMSFN
 000C:00006730       FSH_UPPERCASE
 000C:00006768       FSH_CHECKEANAME
 000C:000067BC       FSH_CALLDRIVER
 000C:00006820       FSH_SETVOLUME
 000C:00006880       FSH_STACKSPACE
 000C:000068A4       FSH_REGISTERPERFCTRS
 000C:000068CC       h_w_SetFSInfo
 000C:000068D0       f_w_SetFSInfo
 000C:000068D2       w_SetFSInfo
 000C:00006960       fsinfo$cook_label
 000C:00006A00       h_FSD_SetFSInfo
 000C:00006A02       FSD_SetFSInfo
 000C:00006A98       h_w_QFsInfo
 000C:00006A9C       f_w_QFsInfo
 000C:00006A9E       w_QFsInfo
 000C:00006B98       h_GetVolLabel
 000C:00006C5C       h_w_SetVerify
 000C:00006C60       f_w_SetVerify
 000C:00006C62       w_SetVerify
 000C:00006C74       h_w_QVerify
 000C:00006C7C       h_w_Get_Drive_Freespace
 000C:00006C80       f_w_Get_Drive_Freespace
 000C:00006C82       w_Get_Drive_Freespace
 000C:00006D24       h_w_QCurDisk
 000C:00006D88       h_w_SelectDisk
 000C:00006DA4       h_w_Set_Default_Drive
 000C:00006DA8       f_w_Set_Default_Drive
 000C:00006DAA       w_Set_Default_Drive
 000C:00006DF0       w_Get_Default_Drive
 000C:00006DF8       h_w_GetInfoSeg
 000C:00006E00       h_w_R0GetInfoSeg
 000C:00006E18       h_w_DevConfig
 000C:00006E48       h_w_GetMachineMode
 000C:00006E4C       h_w_Error
 000C:00006E80       h_w_QSysInfo
 000C:00006EA8       h_MFTclose
 000C:00006EAC       f_MFTclose
 000C:00006EAE       MFTclose
 000C:00006F98       h_AddShare
 000C:00006F9A       AddShare
 000C:00006FE0       h_RemoveShare
 000C:00006FE2       RemoveShare
 000C:0000700C       f_ASC
 000C:0000700E       ASC
 000C:000070E4       CUC
 000C:00007174       CSI
 000C:0000718C       h_RSC
 000C:0000718E       RSC
 000C:00007200       CPS
 000C:0000729C       cpj
 000C:000072D4       SFM
 000C:000072E8       h_ShChk
 000C:000072FC       h_ShSave
 000C:00007314       ShCloseFile
 000C:00007430       h_ShSU
 000C:00007432       ShSU
 000C:0000754C       f_w_JSA
 000C:0000756C       joinsbst$w_Join
 000C:0000777C       joinsbst$w_Subst
 000C:000079B8       h_ListCDSText
 000C:000079BC       f_ListCDSText
 000C:000079BE       ListCDSText
 000C:000079E8       joinsbst$DriveBusy
 000C:000079F4       joinsbst$PathErr
 000C:00007A88       joinsbst$CheckDirPath
 000C:00007B84       h_w_LockOper
 000C:00007B88       f_w_LockOper
 000C:00007B8A       w_LockOper
 000C:00007C34       Lock_Violation
 000C:00007C6C       h_w_FileLocks
 000C:00007C6E       w_FileLocks
 000C:00007D38       FLK_Get_Parms
 000C:00007D70       h_Lock_list
 000C:00007D72       Lock_list
 000C:00007DDC       Lckl_Unlock
 000C:00007DFC       h_Unlock_list
 000C:00007DFE       Unlock_list
 000C:00007E44       f_Set_Block
 000C:00007E46       Set_Block
 000C:000080A8       h_LockBlock
 000C:000080AA       LockBlock
 000C:00008104       f_Clr_Block
 000C:00008106       Clr_Block
 000C:00008210       clp
 000C:00008234       f_CheckRange
 000C:00008236       CheckRange
 000C:00008264       Chk_Block
 000C:000082A8       f_ScanLock
 000C:000082AA       ScanLock
 000C:00008380       h_LockAlloc
 000C:00008382       LockAlloc
 000C:0000839C       ClrSFLock
 000C:00008458       f_w_NameTrans
 000C:000084A4       h_AsgCheckDrive
 000C:000084A6       AsgCheckDrive
 000C:00008520       macro$h_acd_proc
 000C:00008522       macro$acd_proc
 000C:00008544       h_Find_DPB
 000C:00008548       f_Find_DPB
 000C:0000854A       Find_DPB
 000C:00008568       h_InitCDS
 000C:0000856A       InitCDS
 000C:000085EC       h_GetVisDrv
 000C:000085F0       f_GetVisDrv
 000C:000085F2       GetVisDrv
 000C:00008614       macro$GetThisDrvSrv
 000C:00008623       h_GetThisDrv
 000C:00008625       GetThisDrv
 000C:000086A8       h_GetCDSFromDrv
 000C:000086AA       GetCDSFromDrv
 000C:00008754       h_GetCDS
 000C:00008756       GetCDS
 000C:00008778       h_NextCDS
 000C:0000877A       NextCDS
 000C:00008790       macro$GetNextCDS
 000C:000087C8       h_DupCDS
 000C:000087CC       f_DupCDS
 000C:000087CE       DupCDS
 000C:000087F4       h_AddGlobalCDS
 000C:000087F6       AddGlobalCDS
 000C:000087FC       h_AddCDS
 000C:000087FE       AddCDS
 000C:00008824       h_DelCDS
 000C:00008826       DelCDS
 000C:0000886C       h_TransFCB
 000C:00008870       f_TransFCB
 000C:00008872       TransFCB
 000C:0000890C       h_ChkVal
 000C:0000890E       ChkVal
 000C:00008954       ConvertPathChars
 000C:00008998       h_TransPath
 000C:0000899C       f_TransPath
 000C:0000899E       TransPath
 000C:000089A4       h_TransPathCnvPathChars
 000C:000089A8       f_TransPathCnvPathChars
 000C:000089AA       TransPathCnvPathChars
 000C:000089BF       h_TransPathNoJoinIfSame
 000C:000089C1       TransPathNoJoinIfSame
 000C:000089C6       TransPathNoJoin
 000C:000089CD       h_TransPathNoPCName
 000C:000089CF       TransPathNoPCName
 000C:000089D4       TransPathNoErrNMP
 000C:000089DC       h_TransPath2
 000C:000089DE       TransPath2
 000C:00008BF8       macro$transfile
 000C:00008C64       macro$transdev
 000C:00008CD8       h_canpath
 000C:00008CDA       canpath
 000C:00008D64       macro$transNMP
 000C:00008DA0       macro$UNCTest
 000C:00008DB8       macro$transUNC
 000C:00008E1C       macro$GetUncFsdFromPath
 000C:00008E70       h_Canonicalize
 000C:00008E72       Canonicalize
 000C:00008E7A       UNC_Canonicalize
 000C:00008FB8       macro$RemoveLeadDots
 000C:00009000       h_SkipBack
 000C:00009002       SkipBack
 000C:0000902C       macro$CopyComponent
 000C:0000914C       ValidateCDS
 000C:000092D4       macro$Join
 000C:000093BC       h_DriveFromText
 000C:000093C0       f_DriveFromText
 000C:000093C2       DriveFromText
 000C:000093E4       h_TextFromDrive
 000C:000093E6       TextFromDrive
 000C:000093ED       TextFromDrive1
 000C:000093F4       h_PathPref
 000C:000093F6       PathPref
 000C:00009450       h_ScanPathChar
 000C:00009452       ScanPathChar
 000C:00009488       h_w_Canon
 000C:0000948C       f_w_Canon
 000C:0000948E       w_Canon
 000C:00009568       h_ScanCDS
 000C:0000956A       ScanCDS
 000C:000095C4       h_FSCFromCDS
 000C:000095C6       FSCFromCDS
 000C:00009638       macro$FSD_ProcessName
 000C:0000970A       CheckLastComponent
 000C:00009828       macro$Truncpath
 000C:000098D0       h_FindPathEnd
 000C:000098D4       f_FindPathEnd
 000C:000098D6       FindPathEnd
 000C:000098F4       Trunc8dot3
 000C:0000998C       macro$IsRiplDrive
 000C:000099B0       h_QueryDriveLetter
 000C:000099B4       f_QueryDriveLetter
 000C:000099B6       QueryDriveLetter
 000C:000099E4       h_AllocateDriveLetter
 000C:000099E8       f_AllocateDriveLetter
 000C:000099EA       AllocateDriveLetter
 000C:00009A1C       h_FreeDriveLetter
 000C:00009A20       f_FreeDriveLetter
 000C:00009A22       FreeDriveLetter
 000C:00009A44       h_w_EditName
 000C:00009A48       f_w_EditName
 000C:00009A4A       w_EditName
 000C:00009B54       h_MetaEdit
 000C:00009B56       MetaEdit
 000C:00009D20       last_delimeter
 000C:00009D38       CompactExpression
 000C:00009DE0       metachar$SearchForChar
 000C:00009E00       metachar$CopyOneComponent
 000C:00009E60       h_PackName
 000C:00009E62       PackName
 000C:00009E98       h_UnpackName
 000C:00009E9A       UnpackName
 000C:00009EC4       h_MetaMatch
 000C:00009EC6       MetaMatch
 000C:00009FDC       h_w_BufReset
 000C:00009FDE       w_BufReset
 000C:0000A060       h_w_GetDPB
 000C:0000A064       f_w_GetDPB
 000C:0000A066       w_GetDPB
 000C:0000A148       h_VPBContext32
 000C:0000A14C       f_VPBContext32
 000C:0000A14E       VPBContext32
 000C:0000A15C       h_FNotify_Handle_Wake
 000C:0000A15E       FNotify_Handle_Wake
 000C:0000A160       h_FNotify_Path_Wake
 000C:0000A162       FNotify_Path_Wake
 000C:0000A164       h_CNotify_Path_Wake
 000C:0000A166       CNotify_Path_Wake
 000C:0000A190       h_FSD_OpenCreate
 000C:0000A194       f_FSD_OpenCreate
 000C:0000A196       FSD_OpenCreate
 000C:0000A648       h_SHARE_ERROR
 000C:0000A64A       SHARE_ERROR
 000C:0000A6AC       f_w16_AllocatePageSpace
 000C:0000A71C       h_FS_EM_AllocatePageSpace
 000C:0000A770       f_w16_DoPageIO
 000C:0000A800       h_FS_EM_DoPageIO
 000C:0000A8D8       h_w_Current_Dir
 000C:0000A8DC       f_w_Current_Dir
 000C:0000A8DE       w_Current_Dir
 000C:0000A984       h_w_RmDir
 000C:0000A988       f_w_RmDir
 000C:0000A98A       w_RmDir
 000C:0000AA84       FSD_RmDir
 000C:0000AB04       h_w_ChDir
 000C:0000AB08       f_w_ChDir
 000C:0000AB0A       w_ChDir
 000C:0000AD90       h_w_MkDir
 000C:0000AD94       f_w_MkDir
 000C:0000AD96       w_MkDir
 000C:0000AE4C       FSD_MkDir
 000C:0000AED8       FSD_ChDir
 000C:0000AFE8       FSD_ChDirFree
 000C:0000B0A4       h_w_MakePipe
 000C:0000B0A6       w_MakePipe
 000C:0000B114       pipe$palloc
 000C:0000B1C4       pipe$aps
 000C:0000B1F8       h_ClosePipe
 000C:0000B1FA       ClosePipe
 000C:0000B264       pipe$pfree
 000C:0000B28C       h_ReadPipe
 000C:0000B2F4       pipe$readiob
 000C:0000B32C       pipe$rcb
 000C:0000B374       h_WritePipe
 000C:0000B3DC       pipe$writeiob
 000C:0000B410       pipe$wcb
 000C:0000B474       pipe$SBlk
 000C:0000B478       pipe$SWait
 000C:0000B4A8       pipe$SSig
 000C:0000B4C0       h_FNDCLUS
 000C:0000B504       h_SKPCLP
 000C:0000B506       SKPCLP
 000C:0000B5D8       h_CMSkip
 000C:0000B5DA       CMSkip
 000C:0000B66C       CMSize
 000C:0000B68C       CMAlloc
 000C:0000B754       CMCheckFail
 000C:0000B78C       f_CMAttendSwapper
 000C:0000B814       CMFill
 000C:0000B854       CMRequestShared
 000C:0000B890       CMRequestExclusiveWait
 000C:0000B89E       CMRequestExclusive
 000C:0000B8DC       CMRelease
 000C:0000B8F8       h_CMKill
 000C:0000B8FC       f_CMKill
 000C:0000B8FE       CMKill
 000C:0000B909       h_CMShrink
 000C:0000B90B       CMShrink
 000C:0000B990       BufSec
 000C:0000BA38       h_BufRd
 000C:0000BAE0       h_BufWrt
 000C:0000BAE4       f_BufWrt
 000C:0000BAE6       BufWrt
 000C:0000BBD4       h_BigBufRd
 000C:0000BEB4       f_Dir_Search_First
 000C:0000BFE0       search$StoreDirEntry
 000C:0000C01C       h_Do_3xSearch_First
 000C:0000C01E       Do_3xSearch_First
 000C:0000C0AC       f_Dir_Search_Next
 000C:0000C1EC       h_Do_3xSearch_Next
 000C:0000C1EE       Do_3xSearch_Next
 000C:0000C224       h_w_3xFindFirst
 000C:0000C228       f_w_3xFindFirst
 000C:0000C22A       w_3xFindFirst
 000C:0000C43C       h_w_3xFindNext
 000C:0000C440       f_w_3xFindNext
 000C:0000C442       w_3xFindNext
 000C:0000C570       search$IFS_3xFindFirst
 000C:0000C694       search$IFS_3xFindNext
 000C:0000C774       search$QFSInfoDisp
 000C:0000C788       QFSInfoDisp2
 000C:0000C828       search$CopyDirEntry
 000C:0000C850       Grow3xSrchBmp
 000C:0000C898       search$Get3xSrchSel
 000C:0000C918       search$SaveSrchInfo
 000C:0000C96C       search$Alloc3xSrchStruc
 000C:0000C9C0       search$Free3xSrchStruc
 000C:0000C9F8       search$GetSrchInfo
 000C:0000CA88       search$InsertSrchStruc
 000C:0000CAB4       search$RemoveSrchStruc
 000C:0000CAE8       h_w_3xFind_Close
 000C:0000CAF1       h_w_3xDir_Search_Close
 000C:0000CB38       search$Find3xClose
 000C:0000CBA8       h_FFCB3xClose
 000C:0000CBAA       FFCB3xClose
 000C:0000CBD8       search$Get3xSrchStruc
 000C:0000CC1C       h_Find3xExit
 000C:0000CC1E       Find3xExit
 000C:0000CC68       ShutdownCheck
 000C:0000CCC8       WakeShutdownThread
 000C:0000CCDC       ShutdownBlock
 000C:0000CCF4       SDWriteFilter
 000C:0000CD00       SDFSInfoFilter
 000C:0000CD0C       SDChgFPtrFilter
 000C:0000CD18       SDReadFilter
 000C:0000CD24       h_pJFNFromHandle
 000C:0000CD28       f_pJFNFromHandle
 000C:0000CD2A       pJFNFromHandle
 000C:0000CD58       h_SFFromHandle
 000C:0000CD5C       f_SFFromHandle
 000C:0000CD5E       SFFromHandle
 000C:0000CD80       h_SFFromHandleLock
 000C:0000CD82       SFFromHandleLock
 000C:0000CD98       h_SFFromSFN
 000C:0000CD9C       f_SFFromSFN
 000C:0000CD9E       SFFromSFN
 000C:0000CDA0       h_SFFromSFNNoRefChk
 000C:0000CDA4       f_SFFromSFNNoRefChk
 000C:0000CDA6       SFFromSFNNoRefChk
 000C:0000CDF0       SFWaitIdle
 000C:0000CE2C       h_SFLock
 000C:0000CE30       f_SFLock
 000C:0000CE32       SFLock
 000C:0000CE51       h_SFLockNoSD
 000C:0000CE53       SFLockNoSD
 000C:0000CEB0       h_SFUnlock
 000C:0000CEB4       f_SFUnlock
 000C:0000CEB6       SFUnlock
 000C:0000CF24       h_JFNFindFree
 000C:0000CF26       JFNFindFree
 000C:0000CF44       h_ScanJFN
 000C:0000CF46       ScanJFN
 000C:0000CF60       CheckSFTRef
 000C:0000CF94       h_SFLinkFree
 000C:0000CF98       f_SFLinkFree
 000C:0000CF9A       SFLinkFree
 000C:0000D05C       h_SFNAlloc
 000C:0000D060       f_SFNAlloc
 000C:0000D062       SFNAlloc
 000C:0000D164       h_GetSFT
 000C:0000D166       GetSFT
 000C:0000D19C       h_GrowSFT
 000C:0000D19E       GrowSFT
 000C:0000D204       h_DoGrowSFT
 000C:0000D206       DoGrowSFT
 000C:0000D254       util$GrowSFTLastSeg
 000C:0000D338       h_InitSFE
 000C:0000D33A       InitSFE
 000C:0000D378       h_doshlp_RedirDev
 000C:0000D394       h_DRead
 000C:0000D398       f_DRead
 000C:0000D39A       DRead
 000C:0000D3C8       h_DWrite
 000C:0000D3CC       f_DWrite
 000C:0000D3CE       DWrite
 000C:0000D460       h_DskRead
 000C:0000D462       DskRead
 000C:0000D474       h_DskWrite
 000C:0000D476       DskWrite
 000C:0000D490       RawDiskIO
 000C:0000D4AD       h_DiskIO
 000C:0000D4AF       DiskIO
 000C:0000D580       volio$DiskHE
 000C:0000D59E       DiskHE2
 000C:0000D5E4       DoVolIO
 000C:0000D7E8       DoVolIO2
 000C:0000D8E0       volio$DiskCall
 000C:0000D91C       h_ProbeChange
 000C:0000D91E       ProbeChange
 000C:0000D978       h_ResetMedia
 000C:0000D97A       ResetMedia
 000C:0000D9AC       h_FatSecRd
 000C:0000D9B0       f_FatSecRd
 000C:0000D9B2       FatSecRd
 000C:0000DA04       h_ReadBoot
 000C:0000DA06       ReadBoot
 000C:0000DA2C       h_BuildBPB
 000C:0000DA2E       BuildBPB
 000C:0000DB08       volio$ValidateBPB
 000C:0000DB30       h_Volume_Access_Lock
 000C:0000DB32       Volume_Access_Lock
 000C:0000DB8C       h_Volume_Access_Unlock
 000C:0000DB8E       Volume_Access_Unlock
 000C:0000DBE0       h_Volume_Alloc_Lock
 000C:0000DBE2       Volume_Alloc_Lock
 000C:0000DC58       h_Volume_Alloc_Unlock
 000C:0000DC5A       Volume_Alloc_Unlock
 000C:0000DCBC       h_RequestVPBSem
 000C:0000DCC0       f_RequestVPBSem
 000C:0000DCC2       RequestVPBSem
 000C:0000DCD4       h_ReleaseVPBSem
 000C:0000DCD8       f_ReleaseVPBSem
 000C:0000DCDA       ReleaseVPBSem
 000C:0000DCEC       h_IncVPBRef
 000C:0000DCEE       IncVPBRef
 000C:0000DD14       h_DecVPBRef
 000C:0000DD16       DecVPBRef
 000C:0000DD20       h_DecVPBRefInv
 000C:0000DD22       DecVPBRefInv
 000C:0000DDB4       h_PathIncVPBRef
 000C:0000DDB6       PathIncVPBRef
 000C:0000DDE8       h_PathDecVPBRef
 000C:0000DDEA       PathDecVPBRef
 000C:0000DE04       IncVPBSearch
 000C:0000DE2C       h_DecVPBSearch
 000C:0000DE2E       DecVPBSearch
 000C:0000DE58       h_VPBAllocCopy
 000C:0000DE5A       VPBAllocCopy
 000C:0000DE7C       h_VPBFree
 000C:0000DE7E       VPBFree
 000C:0000DEE4       h_VPBLink
 000C:0000DEE6       VPBLink
 000C:0000DF14       h_VPBFind
 000C:0000DF16       VPBFind
 000C:0000DF58       h_WaitVPB
 000C:0000DF5A       WaitVPB
 000C:0000DF88       h_WaitDPB
 000C:0000DF8A       WaitDPB
 000C:0000DFB0       h_LockVBuf
 000C:0000DFB2       LockVBuf
 000C:0000DFDC       h_WakeVPB
 000C:0000DFDE       WakeVPB
 000C:0000DFFC       h_WakeDPB
 000C:0000DFFE       WakeDPB
 000C:0000E010       h_UnlockVBuf
 000C:0000E012       UnlockVBuf
 000C:0000E02C       ToggleRequest
 000C:0000E0A0       volsubr$Hysteresis
 000C:0000E0F0       h_UnreadableVPB
 000C:0000E0F2       UnreadableVPB
 000C:0000E12C       h_CRC
 000C:0000E130       f_CRC
 000C:0000E132       CRC
 000C:0000E14C       WPTLockBuf
 000C:0000E174       WPTUnlockBuf
 000C:0000E18C       h_fVolumeWriteable
 000C:0000E18E       fVolumeWriteable
 000C:0000E238       h_FatDirtyBitToggle
 000C:0000E23C       f_FatDirtyBitToggle
 000C:0000E23E       FatDirtyBitToggle
 000C:0000E30C       h_ResetCurrency
 000C:0000E30E       ResetCurrency
 000C:0000E360       chkvselhdprc
 000C:0000E3B8       h_DWrite2
 000C:0000E464       h_DRead2
 000C:0000E494       DRWIO
 000C:0000E73C       drw_waker
 000C:0000E794       h_DiskHE3
 000C:0000E796       DiskHE3
 000C:0000E7E0       h_SuByteNF
 000C:0000E7E2       SuByteNF
 000C:0000E804       h_SuByte
 000C:0000E808       f_SuByte
 000C:0000E80A       SuByte
 000C:0000E848       h_SuWordNF
 000C:0000E84C       f_SuWordNF
 000C:0000E84E       SuWordNF
 000C:0000E870       h_SuWord
 000C:0000E872       SuWord
 000C:0000E8B0       h_SuDWord
 000C:0000E8B2       SuDWord
 000C:0000E8F0       h_FuByteNF
 000C:0000E8F4       f_FuByteNF
 000C:0000E8F6       FuByteNF
 000C:0000E918       h_FuByte
 000C:0000E91A       FuByte
 000C:0000E958       h_FuWordNF
 000C:0000E95C       f_FuWordNF
 000C:0000E95E       FuWordNF
 000C:0000E980       h_FuWord
 000C:0000E982       FuWord
 000C:0000E9C0       h_FuStrLen
 000C:0000E9C4       f_FuStrLen
 000C:0000E9C6       FuStrLen
 000C:0000EA0C       h_FuStrLenZ
 000C:0000EA10       f_FuStrLenZ
 000C:0000EA12       FuStrLenZ
 000C:0000EAB4       h_SuBuff
 000C:0000EAB8       f_SuBuff
 000C:0000EABA       SuBuff
 000C:0000EB00       h_FuBuffNF
 000C:0000EB02       FuBuffNF
 000C:0000EB24       h_FuBuff
 000C:0000EB28       f_FuBuff
 000C:0000EB2A       FuBuff
 000C:0000EB6A       setfetum$SuFuBuff
 000C:0000EC38       h_SuBuffz
 000C:0000EC3C       f_SuBuffz
 000C:0000EC3E       SuBuffz
 000C:0000EC84       h_FuBuffzNF
 000C:0000EC86       FuBuffzNF
 000C:0000ECA8       h_FuBuffz
 000C:0000ECAA       FuBuffz
 000C:0000ECEA       setfetum$SuFuBuffz
 000C:0000ED0C       h_ProbeBuff
 000C:0000ED0E       ProbeBuff
 000C:0000EE40       setfetum$TrapExit
 000C:0000EE5A       setfetum$TrapExitNF
 000C:0000EE70       Gen16Hook0_High2
 000C:0000EEAC       Gen16HookAny_High2
 000C:0000EF44       f_w_KillProcessPD
 000C:0000EF4C       __panicHIGH2
 000C:0000EF54       __panicfnHIGH2
 000C:0000EF5C       __panicfnmsgHIGH2
 000D:00000000       _StartHIGH3CODE
 000D:00000004       h_CharHard
 000D:00000006       CharHard
 000D:00000009       CharHardAllowed
 000D:00000024       Dev_OC_SFT
 000D:000000F0       h_Dev_Open_SFT
 000D:000000F2       Dev_Open_SFT
 000D:000000FC       h_Dev_Close_SFT
 000D:000000FE       Dev_Close_SFT
 000D:00000108       h_w_DevWOHandle
 000D:0000010C       f_w_DevWOHandle
 000D:0000010E       w_DevWOHandle
 000D:00000178       h_FindDevName
 000D:0000017C       f_FindDevName
 000D:0000017E       FindDevName
 000D:00000228       h_Check_valid_cp
 000D:0000022A       Check_valid_cp
 000D:00000274       h_Check_valid_CC
 000D:00000276       Check_valid_CC
 000D:000002A0       h_w_CopyName
 000D:000002A2       w_CopyName
 000D:000002DC       h_w_CopyCty
 000D:000002DE       w_CopyCty
 000D:00000334       h_w_DosProfile
 000D:00000336       w_DosProfile
 000D:00000350       flagToPCB
 000D:00000370       SetPCB
 000D:0000038C       ProfOff
 000D:000003C4       ProfOn
 000D:00000408       ProfClear
 000D:000004A4       ProfAlloc
 000D:000005B0       BuildSelList
 000D:0000066C       initKProf
 000D:00000758       AddProcLDTs
 000D:0000079C       AddLibLDTs
 000D:000007B0       ProfFree
 000D:00000828       ProfTerm
 000D:0000083C       ProfDump
 000D:00000924       flatDump
 000D:00000A34       h_SelToName
 000D:00000A36       SelToName
 000D:00000A9C       GDTSelToName
 000D:00000AD0       LDTSelToName
 000D:00000B00       MTEFindSel
 000D:00000B54       findSel
 000D:00000BB8       MTEHandleToPtr
 000D:00000BD4       SetTimer0
 000D:00000BF0       h_TMR16AddTime
 000D:00000C50       h_TMR16SubTime
 000D:00000CA0       W_DOSDELETE
 000D:00000E78       _GetVars
 000D:00000FC8       _StoreFile
 000D:0000104C       _CreateDeletePath
 000D:000010EA       _GetEnvVars
 000D:00001232       _GetFileFromPath
 000D:00001278       _CreateDeleteRecord
 000D:000013BA       _MakeRoom
 000D:000014DE       _EraseOverflow
 000D:0000161A       _strstrf
 000D:00001694       _atol
 000D:00001732       _ltoa
 000D:00001794       _power10
 000D:000017E4       _strlenfc
 000D:000017FC       _strcmpfc
 000D:00001828       _strncmpfc
 000D:00001864       _ulongmulc
 000D:0000187C       _ushortmulc
 000D:00001888       _udivc
 000D:000018AC       _strcpyfc
 000D:000018E4       _memsetfc
 000D:00001914       _DOSFORCEDELETE
 000D:00001930       _DOSMKDIR
 000D:00001954       _DOSMOVE
 000D:00001978       _DOSQCURDISK
 000D:000019A0       _DOSQCURDIR
 000D:000019D4       P_DOSFINDFIRST
 000D:00001A08       _DOSFINDCLOSE
 000D:00001A24       _modify_fSharing
 000D:00001A5C       P_DOSOPEN
 000D:00001A90       _DOSCHGFILEPTR
 000D:00001AC8       _DOSPWRITE
 000D:00001AF8       _DOSCLOSE
 000D:00001B20       _DOSREAD
 000D:00001B50       _DOSNEWSIZE
 000D:00001B7C       _DOSSETFILEMODE
 000D:00001BA0       _DOSQPATHINFO
 000D:00001BC8       _DOSGETDATETIME
 000D:00001BE8       _DOSALLOCSEG
 000D:00001C1C       _DOSFREESEG
 000D:00001C38       P_DOSQFSATTACH
 000D:00001C60       _SEM_REQUEST
 000D:00001C80       _SEM_RELEASE
 000D:00001CA0       h_AddCharDevEntry
 000D:00001CA2       AddCharDevEntry
 000D:00001D90       h_RemCharDevEntry
 000D:00001D92       RemCharDevEntry
 000D:00001DCC       h_SetCharDevFields
 000D:00001DF4       h_FindCharDevEntry
 000D:00001DF6       FindCharDevEntry
 000D:00001E2C       h_GetCharDevEntry
 000D:00001E2E       GetCharDevEntry
 000D:00001EAC       IsThisADevice
 000D:00001ED4       chardd$MakeRecordEntry
 000D:00001F18       h_CheckThisDevice
 000D:00001F1C       f_CheckThisDevice
 000D:00001F1E       CheckThisDevice
 000D:00001F90       f_GetDeviceName
 000D:00001F92       GetDeviceName
 000D:00001FF8       h_GetDevEntry
 000D:00001FFA       GetDevEntry
 000D:00002010       h_AddSpoolDevEntry
 000D:00002012       AddSpoolDevEntry
 000D:000020A4       h_RemSpoolDevEntry
 000D:000020A6       RemSpoolDevEntry
 000D:000020C4       h_FindSpoolDevEntry
 000D:000020C6       FindSpoolDevEntry
 000D:00002104       h_CheckSpoolDevice
 000D:00002140       h_w_SetCp
 000D:00002144       f_w_SetCp
 000D:00002146       w_SetCp
 000D:00002194       Check_val_cp
 000D:000021CC       h_w_GetCp
 000D:000021D0       f_w_GetCp
 000D:000021D2       w_GetCp
 000D:000021E4       h_w_GetCp2
 000D:000021E6       DosGetCp_PreTrace
 000D:000021E6       w_GetCp2
 000D:000021F1       DosGetCp_PostTrace
 000D:000021F4       w_GetCp_All
 000D:00002244       Get_val_cp
 000D:000022AC       h_SpoolIOCtl
 000D:000025FC       h_wdi_BeginFormat
 000D:000025FE       wdi_BeginFormat
 000D:00002668       h_wdi_updateVPB
 000D:0000266A       wdi_updateVPB
 000D:000026B8       h_Spindle_Lock
 000D:00002810       h_Spindle_Unmount
 000D:00002938       h_Spindle_Unlock
 000D:00002978       h_ErrorTriage
 000D:0000297A       ErrorTriage
 000D:000029AC       h_GetDriveInfo
 000D:000029B0       f_GetDriveInfo
 000D:000029B2       GetDriveInfo
 000D:000029F0       h_GetHandleInfo
 000D:000029F4       f_GetHandleInfo
 000D:000029F6       GetHandleInfo
 000D:00002A24       h_GetHandleSFT
 000D:00002A26       GetHandleSFT
 000D:00002A50       devioctl$Update_SFT_size
 000D:00002A90       h_DupJFN
 000D:00002A94       f_DupJFN
 000D:00002A96       DupJFN
 000D:00002ABC       dosfs$DupPMJFN
 000D:00002B44       dosfs$CopyJFNTab
 000D:00002B58       dosfs$Dup1Handle
 000D:00002B80       dosfs$CopyJFNFlag
 000D:00002B90       h_w_SetRelMaxFH
 000D:00002C44       h_w_SetMaxFH
 000D:00002C48       f_w_SetMaxFH
 000D:00002C4A       w_SetMaxFH
 000D:00002C84       fhandle$GrowJFNSeg
 000D:00002D74       fhandle$MovJFNToSeg
 000D:00002DBC       AllocJFNSeg
 000D:00002E24       h_FreeJFNSeg
 000D:00002E26       FreeJFNSeg
 000D:00002E68       fhandle$ShrinkJFNs
 000D:00002ECC       fhandle$FindNewJFNMax
 000D:00002F04       h_w_EnumAttribute
 000D:00003114       h_w_ProtectEnumAttribute
 000D:00003324       f_HardError
 000D:00003326       h_HardError
 000D:00003354       h_S2HardError
 000D:00003534       h_S3HardError
 000D:00003644       harderr$GenErrCode
 000D:000036C8       harderr$CopyTemplate
 000D:000036DC       h_ChkHEDaemon
 000D:000036DE       ChkHEDaemon
 000D:000036EC       harderr$FillHEPacket
 000D:000038FC       harderr$GetHEResponse
 000D:00003924       harderr$ProcessHE
 000D:000039F0       h_HEAction
 000D:00003A4C       harderr$SetLogicalDrive
 000D:00003A74       harderr$VDMHardError
 000D:00003BE0       h_Bmp_SetGrowFunction
 000D:00003BE2       Bmp_SetGrowFunction
 000D:00003BF4       Bmp_DefaultGrowFunction
 000D:00003C14       h_Bmp_Get
 000D:00003C16       Bmp_Get
 000D:00003D28       h_Bmp_CheckOffset
 000D:00003D4C       h_Bmp_Free
 000D:00003D50       f_Bmp_Free
 000D:00003D52       Bmp_Free
 000D:00003D9C       h_Bmp_QueryFree
 000D:00003DA0       f_Bmp_QueryFree
 000D:00003DA2       Bmp_QueryFree
 000D:00003DB4       h_GetTempBuffer
 000D:00003DB8       f_GetTempBuffer
 000D:00003DBA       GetTempBuffer
 000D:00003E0C       h_FreeTempBuffer
 000D:00003E10       f_FreeTempBuffer
 000D:00003E12       FreeTempBuffer
 000D:00003E6C       h_Bmp_Init
 000D:00003E6E       Bmp_Init
 000D:00003E9C       h_Rmp_Wait
 000D:00003E9E       Rmp_Wait
 000D:00003ECC       rmp$Rmp_Req
 000D:00003EDC       rmp$Rmp_Clr
 000D:00003EFC       h_Rmp_Alloc
 000D:00003F00       f_Rmp_Alloc
 000D:00003F02       Rmp_Alloc
 000D:00003FC4       rmp$rmprealloc
 000D:00004004       h_Rmp_Free
 000D:00004030       h_Rmp_Add
 000D:00004034       f_Rmp_Add
 000D:00004036       Rmp_Add
 000D:00004114       rmp$Rmp_Srch
 000D:00004148       rmp$Rmp_Comp
 000D:000041C0       rmp$Rmp_Move
 000D:000041E8       rmp$Rmp_Link
 000D:00004258       h_Rmp_Rem
 000D:0000425C       f_Rmp_Rem
 000D:0000425E       Rmp_Rem
 000D:00004314       h_Rmp_Find
 000D:00004318       f_Rmp_Find
 000D:0000431A       Rmp_Find
 000D:00004334       h_Rmp_FindN
 000D:00004338       f_Rmp_FindN
 000D:0000433A       Rmp_FindN
 000D:000043B8       h_MemMapAlias
 000D:000043BA       MemMapAlias
 000D:000043E0       h_MemUnmapAlias
 000D:000043E2       MemUnmapAlias
 000D:0000440C       h_GDTAlloc
 000D:0000440E       GDTAlloc
 000D:00004450       h_GDTFree
 000D:00004452       GDTFree
 000D:00004478       selmap$GDTInvalidate
 000D:000044BC       SetDescInfo
 000D:000044C0       h_SetDescInfo
 000D:00004504       h_GetDescInfo
 000D:00004506       GetDescInfo
 000D:00004550       h_DescInvalidate
 000D:00004554       f_DescInvalidate
 000D:00004556       DescInvalidate
 000D:00004574       h_HandleGetSelector
 000D:00004576       HandleGetSelector
 000D:000045C8       h_PhysToGDTSel
 000D:000045CA       PhysToGDTSel
 000D:00004764       h_UVirtToPhys
 000D:00004766       UVirtToPhys
 000D:000047E8       h_VirtToLin
 000D:000047EC       f_VirtToLin
 000D:000047EE       VirtToLin
 000D:00004850       h_LinToGDTSel
 000D:00004852       LinToGDTSel
 000D:00004958       h_SegAlloc
 000D:00004980       f_SegAlloc2
 000D:000049A4       h_SegRealloc
 000D:000049A6       SegRealloc
 000D:000049C4       h_SegFree
 000D:000049C6       SegFree
 000D:000049CA       h_ifs_SegFree
 000D:000049CC       ifs_SegFree
 000D:000049DC       f_SegFree2
 000D:000049F0       selseg$SegLockSub
 000D:00004A58       h_SegLock
 000D:00004A5A       SegLock
 000D:00004C50       selseg$SegUnlockSub
 000D:00004C70       h_SegUnlock
 000D:00004C72       SegUnlock
 000D:00004D14       h_SegGetInfo
 000D:00004DAC       h_SegMapVirt
 000D:00004DFC       h_w_AllocProtSeg
 000D:00004E04       h_w_AllocSeg
 000D:00004E18       h_w_ReallocSeg
 000D:00004E1A       w_ReallocSeg
 000D:00004E2C       h_w_FreeSeg
 000D:00004E2E       w_FreeSeg
 000D:00004F04       h_w_GiveSeg2
 000D:00004F0B       h_w_GiveSeg
 000D:00004F30       h_w_GetSeg
 000D:00004F54       h_w_LockSeg
 000D:00004F64       h_w_UnlockSeg
 000D:00004F74       h_w_AllocProtHuge
 000D:00004F7C       h_w_AllocHuge
 000D:00004F90       h_w_ReallocHuge
 000D:00004FA0       h_w_GetHugeShift
 000D:00004FAC       h_w_CreateCSAlias
 000D:00004FBC       h_w_MemAvail
 000D:00005070       h_w_SizeSeg
 000D:00005130       h_w_AllocShrProtSeg
 000D:00005132       w_AllocShrProtSeg
 000D:0000513E       h_w_AllocShrSeg
 000D:00005140       w_AllocShrSeg
 000D:000051A4       h_w_GetShrSeg
 000D:000051A6       w_GetShrSeg
 000D:000051D8       demsvc$f_DosHlpProtGetMessage
 000D:000051E4       DOSALLOCHUGE
 000D:000051F5       preDOSALLOCHUGE
 000D:00005206       postDOSALLOCHUGE
 000D:00005210       DOSALLOCSEG
 000D:0000521B       preDOSALLOCSEG
 000D:0000522C       postDOSALLOCSEG
 000D:00005234       DOSALLOCSHRSEG
 000D:0000524E       preDOSALLOCSHRSEG
 000D:0000525F       postDOSALLOCSHRSEG
 000D:00005268       DOSALLOCPROTHUGE
 000D:00005279       preDOSALLOCPROTHUGE
 000D:0000528A       postDOSALLOCPROTHUGE
 000D:00005294       DOSALLOCPROTSEG
 000D:0000529F       preDOSALLOCPROTSEG
 000D:000052B0       postDOSALLOCPROTSEG
 000D:000052B8       DOSALLOCSHRPROTSEG
 000D:000052D2       preDOSALLOCSHRPROTSEG
 000D:000052E3       postDOSALLOCSHRPROTSEG
 000D:000052EC       DOSCLOSESEM
 000D:000052F7       preDOSCLOSESEM
 000D:00005300       postDOSCLOSESEM
 000D:00005308       DOSCREATECSALIAS
 000D:00005310       preDOSCREATECSALIAS
 000D:00005321       postDOSCREATECSALIAS
 000D:0000532C       DOSCREATESEM
 000D:00005346       preDOSCREATESEM
 000D:0000535A       postDOSCREATESEM
 000D:00005360       DOSCWAIT
 000D:0000536E       preDOSCWAIT
 000D:0000538D       postDOSCWAIT
 000D:00005398       DOSDEVCONFIG
 000D:000053A3       preDOSDEVCONFIG
 000D:000053B4       postDOSDEVCONFIG
 000D:000053BC       DOSDYNAMICTRACE
 000D:000053E8       DOSERROR
 000D:000053F0       preDOSERROR
 000D:000053F9       postDOSERROR
 000D:00005404       DOSFLAGPROCESS
 000D:00005415       preDOSFLAGPROCESS
 000D:0000541E       postDOSFLAGPROCESS
 000D:00005428       DOSFREERESOURCE
 000D:00005435       preDOSFREERESOURCE
 000D:0000543E       postDOSFREERESOURCE
 000D:00005448       DOSQUERYABIOSSUPPORT
 000D:00005460       DOS16LDRDIRTYWORKER
 000D:00005480       DOSFREESEG
 000D:0000548D       preDOSFREESEG
 000D:00005496       postDOSFREESEG
 000D:000054A0       DOSGETENV
 000D:000054CC       DOSGETHUGESHIFT
 000D:000054EC       DOSGETINFOSEG
 000D:00005518       R0DOSGETINFOSEG
 000D:00005544       DOSGETMACHINEMODE
 000D:00005564       DOSGETMODHANDLE
 000D:0000557B       preDOSGETMODHANDLE
 000D:0000558C       postDOSGETMODHANDLE
 000D:00005594       DOSGETMODNAME
 000D:000055AE       preDOSGETMODNAME
 000D:000055B7       postDOSGETMODNAME
 000D:000055C0       DOSGETPID
 000D:000055C5       preDOSGETPID
 000D:000055DC       postDOSGETPID
 000D:000055E4       DOSGETPPID
 000D:000055EF       preDOSGETPPID
 000D:00005600       postDOSGETPPID
 000D:00005608       DOSGETPROCADDR
 000D:00005629       preDOSGETPROCADDR
 000D:0000563D       postDOSGETPROCADDR
 000D:00005644       DOSGETRESOURCE
 000D:00005655       preDOSGETRESOURCE
 000D:00005668       postDOSGETRESOURCE
 000D:00005670       DOSGETRESOURCE2
 000D:00005681       preDOSGETRESOURCE2
 000D:00005698       postDOSGETRESOURCE2
 000D:000056A0       DOSGETSEG
 000D:000056A8       preDOSGETSEG
 000D:000056B1       postDOSGETSEG
 000D:000056BC       DOSGETSHRSEG
 000D:000056D3       preDOSGETSHRSEG
 000D:000056E4       postDOSGETSHRSEG
 000D:000056EC       DOSGETVERSION
 000D:000056F1       preDOSGETVERSION
 000D:00005702       postDOSGETVERSION
 000D:0000570C       DOSGIVESEG
 000D:00005717       preDOSGIVESEG
 000D:00005728       postDOSGIVESEG
 000D:00005730       DOSICANONICALIZE
 000D:00005774       DOSIEXECPGM
 000D:000057CB       preDOSIEXECPGM
 000D:000057DF       postDOSIEXECPGM
 000D:000057E8       DOSIQAPPTYPE
 000D:00005818       DOSIRAMSEMREQUEST
 000D:00005840       DOSIRAMSEMWAKE
 000D:00005860       DOSISEMWAIT
 000D:00005884       DOSKILLPROCESS
 000D:0000588F       preDOSKILLPROCESS
 000D:00005898       postDOSKILLPROCESS
 000D:000058A0       DOSLOADMODULE
 000D:000058C5       preDOSLOADMODULE
 000D:000058D6       postDOSLOADMODULE
 000D:000058E0       DOSLOCKSEG
 000D:000058FC       DOSMAKEPIPE
 000D:00005907       preDOSMAKEPIPE
 000D:00005923       postDOSMAKEPIPE
 000D:0000592C       DOSMEMAVAIL
 000D:00005950       DOSOPENSEM
 000D:00005967       preDOSOPENSEM
 000D:0000597B       postDOSOPENSEM
 000D:00005984       DOSPHYSICALDISK
 000D:00005995       preDOSPHYSICALDISK
 000D:0000599E       postDOSPHYSICALDISK
 000D:000059A8       DOSPROFILE
 000D:000059EC       DOSPTRACE
 000D:00005A0C       DOSR2STACKREALLOC
 000D:00005A14       preDOSR2STACKREALLOC
 000D:00005A1D       postDOSR2STACKREALLOC
 000D:00005A28       DOSQPROCSTATUS
 000D:00005A50       DOSREALLOCHUGE
 000D:00005A5E       preDOSREALLOCHUGE
 000D:00005A67       postDOSREALLOCHUGE
 000D:00005A70       DOSREALLOCSEG
 000D:00005A7B       preDOSREALLOCSEG
 000D:00005A84       postDOSREALLOCSEG
 000D:00005A8C       DOSSEMSETWAIT
 000D:00005A9D       preDOSSEMSETWAIT
 000D:00005AA6       postDOSSEMSETWAIT
 000D:00005AB0       DOSSENDSIGNAL
 000D:00005ABB       preDOSSENDSIGNAL
 000D:00005AC4       postDOSSENDSIGNAL
 000D:00005ACC       DOSSETSIGHANDLER
 000D:00005ADD       preDOSSETSIGHANDLER
 000D:00005B19       postDOSSETSIGHANDLER
 000D:00005B24       DOSSETVEC
 000D:00005B32       preDOSSETVEC
 000D:00005B46       postDOSSETVEC
 000D:00005B50       DOSSICG
 000D:00005B74       DOSSIZESEG
 000D:00005B98       DOSSYSTEMSERVICE
 000D:00005BB5       preDOSSYSTEMSERVICE
 000D:00005BBE       postDOSSYSTEMSERVICE
 000D:00005BC8       DOSUNLOCKSEG
 000D:00005BE4       PANICWRITE
 000D:00005C0C       DYNAM_API_0
 000D:00005C18       DYNAM_API_1
 000D:00005C24       DYNAM_API_2
 000D:00005C30       DYNAM_API_3
 000D:00005C3C       DYNAM_API_4
 000D:00005C48       DYNAM_API_5
 000D:00005C54       DYNAM_API_6
 000D:00005C60       DYNAM_API_7
 000D:00005C6C       DYNAM_API_8
 000D:00005C78       DYNAM_API_9
 000D:00005C84       DYNAM_API_A
 000D:00005C90       DYNAM_API_B
 000D:00005C9C       DYNAM_API_C
 000D:00005CA8       DYNAM_API_D
 000D:00005CB4       DYNAM_API_E
 000D:00005CC0       DYNAM_API_F
 000D:00005CCC       h_Dynam_API_DevHlp
 000D:00005DA0       dyn_locateSlot
 000D:00005DB8       dynam_sci
 000D:00005E58       h_w_dynam_API
 000D:00005F0C       DOSSETDATETIME
 000D:00005F17       preDOSSETDATETIME
 000D:00005F20       postDOSSETDATETIME
 000D:00005F28       DOSGETDATETIME
 000D:00005F33       preDOSGETDATETIME
 000D:00005F3C       postDOSGETDATETIME
 000D:00005F44       DOSSETPRTY
 000D:00005F55       preDOSSETPRTY
 000D:00005F5E       postDOSSETPRTY
 000D:00005F68       DOSGETPRTY
 000D:00005F73       preDOSGETPRTY
 000D:00005F84       postDOSGETPRTY
 000D:00005F8C       DOSSETFGND
 000D:00005FA8       DOSBEEP
 000D:00005FB3       preDOSBEEP
 000D:00005FBC       postDOSBEEP
 000D:00005FC4       DOSSGSWITCH
 000D:00005FE4       DOSSGSWITCHME
 000D:00006000       DOSSGSWITCHPROC2
 000D:00006020       DOSSTRUCHECK
 000D:00006038       DOSSTRURESUPDATE
 000D:00006068       DOSGETSTDA
 000D:0000608C       DOSSETTRACEINFO
 000D:0000609D       preDOSSETTRACEINFO
 000D:000060A9       postDOSSETTRACEINFO
 000D:000060AC       DOSLOGENTRY
 000D:000060D0       DOSGETLOGBUFFER
 000D:000060D8       DOSLOGMODE
 000D:000060E0       DOSISETCP
 000D:000060EB       preDOSISETCP
 000D:000060F4       postDOSISETCP
 000D:000060FC       DOSGETCP
 000D:0000610F       preDOSGETCP
 000D:00006120       postDOSGETCP
 000D:00006128       DOSGLOBALSEG
 000D:0000615C       DOSCLIACCESS
 000D:00006161       preDOSCLIACCESS
 000D:0000616A       postDOSCLIACCESS
 000D:00006174       DOSPORTACCESS
 000D:00006185       preDOSPORTACCESS
 000D:0000618E       postDOSPORTACCESS
 000D:00006198       h_w_portacc
 000D:0000619A       w_portacc
 000D:000061B4       h_w_zeroax
 000D:000061B6       w_zeroax
 000D:000061BC       DOSSYSTRACE
 000D:000061F8       DOSENTERCRITSEC
 000D:00006203       preDOSENTERCRITSEC
 000D:00006206       post2DOSENTERCRITSEC
 000D:00006248       DOSEXITCRITSEC
 000D:000062DD       preDOSEXITCRITSEC
 000D:000062E0       post2DOSEXITCRITSEC
 000D:0000638C       DOS32ISETFHSTATE
 000D:000063A4       preDOS32ISETFHSTATE
 000D:000063AD       postDOS32ISETFHSTATE
 000D:000063B4       DOS32IQUERYFHSTATE
 000D:000063C6       preDOS32IQUERYFHSTATE
 000D:000063DA       postDOS32IQUERYFHSTATE
 000D:000063E0       DOS32IPROTECTSETFHSTATE
 000D:000063FA       preDOS32IPROTECTSETFHSTATE
 000D:00006403       postDOS32IPROTECTSETFHSTATE
 000D:0000640C       DOS32IPROTECTQUERYFHSTATE
 000D:00006420       preDOS32IPROTECTQUERYFHSTATE
 000D:00006434       postDOS32IPROTECTQUERYFHSTATE
 000D:0000643C       DOSBUFRESET
 000D:00006444       preDOSBUFRESET
 000D:0000644D       postDOSBUFRESET
 000D:00006458       DOSCHDIR
 000D:00006478       preDOSCHDIR
 000D:00006481       postDOSCHDIR
 000D:00006488       DOSCHGFILEPTR
 000D:000064A0       preDOSCHGFILEPTR
 000D:000064B4       postDOSCHGFILEPTR
 000D:000064BC       DOSPROTECTCHGFILEPTR
 000D:000064D6       preDOSPROTECTCHGFILEPTR
 000D:000064EA       postDOSPROTECTCHGFILEPTR
 000D:000064F0       DOSCLOSE
 000D:000064FF       preDOSCLOSE
 000D:00006508       postDOSCLOSE
 000D:00006510       DOSPROTECTCLOSE
 000D:00006521       preDOSPROTECTCLOSE
 000D:0000652A       postDOSPROTECTCLOSE
 000D:00006530       DOSCLOSECHANGENOTIFY
 000D:00006538       preDOSCLOSECHANGENOTIFY
 000D:00006541       postDOSCLOSECHANGENOTIFY
 000D:0000654C       DOSDELETE
 000D:0000656C       preDOSDELETE
 000D:00006575       postDOSDELETE
 000D:0000657C       DOSDEVIOCTL
 000D:000065A5       preDOSDEVIOCTL
 000D:000065AE       postDOSDEVIOCTL
 000D:000065B8       DOSDEVIOCTL2
 000D:0000660A       preDOSDEVIOCTL2
 000D:00006613       postDOSDEVIOCTL2
 000D:0000661C       DOSDUPHANDLE
 000D:0000662F       preDOSDUPHANDLE
 000D:00006640       postDOSDUPHANDLE
 000D:00006648       DOSEDITNAME
 000D:00006686       preDOSEDITNAME
 000D:0000668F       postDOSEDITNAME
 000D:00006698       DOSENUMATTRIBUTE
 000D:000066D0       preDOSENUMATTRIBUTE
 000D:000066D9       postDOSENUMATTRIBUTE
 000D:000066E0       DOSPROTECTENUMATTRIBUTE
 000D:0000671A       preDOSPROTECTENUMATTRIBUTE
 000D:00006723       postDOSPROTECTENUMATTRIBUTE
 000D:0000672C       DOSFILEIO
 000D:00006746       preDOSFILEIO
 000D:0000674F       postDOSFILEIO
 000D:00006758       DOSPROTECTFILEIO
 000D:00006777       preDOSPROTECTFILEIO
 000D:00006780       postDOSPROTECTFILEIO
 000D:00006788       DOSFILELOCKS
 000D:000067B1       preDOSFILELOCKS
 000D:000067BA       postDOSFILELOCKS
 000D:000067C0       DOSPROTECTFILELOCKS
 000D:000067EB       preDOSPROTECTFILELOCKS
 000D:000067F4       postDOSPROTECTFILELOCKS
 000D:000067FC       DOSFINDCLOSE
 000D:00006807       preDOSFINDCLOSE
 000D:00006810       postDOSFINDCLOSE
 000D:00006818       DOSFINDFIRST
 000D:00006842       preDOSFINDFIRST
 000D:0000685E       postDOSFINDFIRST
 000D:00006864       DOSFINDFIRST2
 000D:0000688E       preDOSFINDFIRST2
 000D:000068AA       postDOSFINDFIRST2
 000D:000068B0       DOSIFINDFIRST
 000D:000068E8       DOSFINDFROMNAME
 000D:00006907       preDOSFINDFROMNAME
 000D:00006918       postDOSFINDFROMNAME
 000D:00006920       DOSFINDNEXT
 000D:00006944       preDOSFINDNEXT
 000D:00006955       postDOSFINDNEXT
 000D:0000695C       DOSIFINDNEXT
 000D:0000697C       DOSFINDNOTIFYCLOSE
 000D:00006984       preDOSFINDNOTIFYCLOSE
 000D:0000698D       postDOSFINDNOTIFYCLOSE
 000D:00006998       DOSFINDNOTIFYFIRST
 000D:000069CA       preDOSFINDNOTIFYFIRST
 000D:000069E6       postDOSFINDNOTIFYFIRST
 000D:000069F0       DOSFINDNOTIFYNEXT
 000D:00006A18       preDOSFINDNOTIFYNEXT
 000D:00006A29       postDOSFINDNOTIFYNEXT
 000D:00006A34       DOSFORCEDELETE
 000D:00006A54       preDOSFORCEDELETE
 000D:00006A5D       postDOSFORCEDELETE
 000D:00006A64       DOSFSATTACH
 000D:00006A9C       preDOSFSATTACH
 000D:00006AA5       postDOSFSATTACH
 000D:00006AAC       DOSFSCTL
 000D:00006ADF       preDOSFSCTL
 000D:00006AE8       postDOSFSCTL
 000D:00006AF0       DOSICOPY
 000D:00006B33       preDOSICOPY
 000D:00006B3C       postDOSICOPY
 000D:00006B44       DOSIDEVIOCTL
 000D:00006B58       preDOSIDEVIOCTL
 000D:00006B61       postDOSIDEVIOCTL
 000D:00006B6C       DOSIREAD
 000D:00006B8E       preDOSIREAD
 000D:00006BA6       postDOSIREAD
 000D:00006BB0       DOSIPROTECTREAD
 000D:00006BD2       preDOSIPROTECTREAD
 000D:00006BE3       postDOSIPROTECTREAD
 000D:00006BEC       DOSISETFILEINFO
 000D:00006C11       preDOSISETFILEINFO
 000D:00006C1A       postDOSISETFILEINFO
 000D:00006C20       DOSIPROTECTSETFILEINFO
 000D:00006C47       preDOSIPROTECTSETFILEINFO
 000D:00006C50       postDOSIPROTECTSETFILEINFO
 000D:00006C58       DOSISETPATHINFO
 000D:00006CA2       preDOSISETPATHINFO
 000D:00006CAB       postDOSISETPATHINFO
 000D:00006CB4       DOSISETRELMAXFH
 000D:00006CD1       preDOSISETRELMAXFH
 000D:00006CDA       postDOSISETRELMAXFH
 000D:00006CE0       DOSIWRITE
 000D:00006D02       preDOSIWRITE
 000D:00006D1A       postDOSIWRITE
 000D:00006D24       DOSIPROTECTWRITE
 000D:00006D46       preDOSIPROTECTWRITE
 000D:00006D57       postDOSIPROTECTWRITE
 000D:00006D60       DOSMKDIR
 000D:00006D84       preDOSMKDIR
 000D:00006D8D       postDOSMKDIR
 000D:00006D94       DOSMKDIR2
 000D:00006DC9       preDOSMKDIR2
 000D:00006DD2       postDOSMKDIR2
 000D:00006DD8       DOSMOVE
 000D:00006E18       preDOSMOVE
 000D:00006E21       postDOSMOVE
 000D:00006E28       DOSNEWSIZE
 000D:00006E3D       preDOSNEWSIZE
 000D:00006E46       postDOSNEWSIZE
 000D:00006E4C       DOSPROTECTNEWSIZE
 000D:00006E63       preDOSPROTECTNEWSIZE
 000D:00006E6C       postDOSPROTECTNEWSIZE
 000D:00006E74       DOSOPEN
 000D:00006E99       preDOSOPEN
 000D:00006EB5       postDOSOPEN
 000D:00006EBC       DOSOPEN2
 000D:00006EE4       preDOSOPEN2
 000D:00006F00       postDOSOPEN2
 000D:00006F08       DOSOPEN2COMPT
 000D:00006F30       preDOSOPEN2COMPT
 000D:00006F4C       postDOSOPEN2COMPT
 000D:00006F54       DOSPROTECTOPEN
 000D:00006F7C       preDOSPROTECTOPEN
 000D:00006FA4       postDOSPROTECTOPEN
 000D:00006FAC       DOSOPENCHANGENOTIFY
 000D:00006FCC       preDOSOPENCHANGENOTIFY
 000D:00006FDD       postDOSOPENCHANGENOTIFY
 000D:00006FE8       DOSOPLOCKRELEASE
 000D:00006FF9       preDOSOPLOCKRELEASE
 000D:00007002       postDOSOPLOCKRELEASE
 000D:0000700C       DOSOPLOCKSHUTDOWN
 000D:00007024       DOSOPLOCKWAIT
 000D:00007043       preDOSOPLOCKWAIT
 000D:0000704C       postDOSOPLOCKWAIT
 000D:00007054       DOSQCURDIR
 000D:00007070       preDOSQCURDIR
 000D:00007081       postDOSQCURDIR
 000D:00007088       DOSQCURDISK
 000D:00007090       preDOSQCURDISK
 000D:000070AF       postDOSQCURDISK
 000D:000070B8       DOSQFHANDSTATE
 000D:000070C9       preDOSQFHANDSTATE
 000D:000070DA       postDOSQFHANDSTATE
 000D:000070E0       DOSPROTECTQFHANDSTATE
 000D:000070F3       preDOSPROTECTQFHANDSTATE
 000D:00007104       postDOSPROTECTQFHANDSTATE
 000D:0000710C       DOSQFILEINFO
 000D:0000712F       preDOSQFILEINFO
 000D:00007138       postDOSQFILEINFO
 000D:00007140       DOSPROTECTQFILEINFO
 000D:00007165       preDOSPROTECTQFILEINFO
 000D:0000716E       postDOSPROTECTQFILEINFO
 000D:00007174       DOSQFILEMODE
 000D:00007196       preDOSQFILEMODE
 000D:000071A7       postDOSQFILEMODE
 000D:000071B0       DOSQFSATTACH
 000D:000071E3       preDOSQFSATTACH
 000D:000071F4       postDOSQFSATTACH
 000D:000071FC       DOSQFSINFO
 000D:00007219       preDOSQFSINFO
 000D:00007222       postDOSQFSINFO
 000D:00007228       DOSQHANDTYPE
 000D:00007233       preDOSQHANDTYPE
 000D:0000724F       postDOSQHANDTYPE
 000D:00007258       DOSQPATHINFO
 000D:00007290       preDOSQPATHINFO
 000D:00007299       postDOSQPATHINFO
 000D:000072A0       DOSQSYSINFO
 000D:000072B1       preDOSQSYSINFO
 000D:000072BA       postDOSQSYSINFO
 000D:000072C4       DOSQVERIFY
 000D:000072C9       preDOSQVERIFY
 000D:000072DA       postDOSQVERIFY
 000D:000072E4       DOSRESETCHANGENOTIFY
 000D:00007304       preDOSRESETCHANGENOTIFY
 000D:0000730D       postDOSRESETCHANGENOTIFY
 000D:00007318       DOSRMDIR
 000D:00007338       preDOSRMDIR
 000D:00007341       postDOSRMDIR
 000D:00007348       DOSSELECTDISK
 000D:00007353       preDOSSELECTDISK
 000D:0000735C       postDOSSELECTDISK
 000D:00007364       DOSSETFHANDSTATE
 000D:00007378       preDOSSETFHANDSTATE
 000D:00007381       postDOSSETFHANDSTATE
 000D:00007388       DOSPROTECTSETFHANDSTATE
 000D:0000739E       preDOSPROTECTSETFHANDSTATE
 000D:000073A7       postDOSPROTECTSETFHANDSTATE
 000D:000073B0       DOSSETFILEINFO
 000D:000073D5       preDOSSETFILEINFO
 000D:000073DE       postDOSSETFILEINFO
 000D:000073E4       DOSPROTECTSETFILEINFO
 000D:0000740B       preDOSPROTECTSETFILEINFO
 000D:00007414       postDOSPROTECTSETFILEINFO
 000D:0000741C       DOSSETFILEMODE
 000D:00007442       preDOSSETFILEMODE
 000D:0000744B       postDOSSETFILEMODE
 000D:00007454       DOSSETFSINFO
 000D:00007470       preDOSSETFSINFO
 000D:00007479       postDOSSETFSINFO
 000D:00007480       DOSSETMAXFH
 000D:0000748B       preDOSSETMAXFH
 000D:00007494       postDOSSETMAXFH
 000D:0000749C       DOSSETPATHINFO
 000D:000074E5       preDOSSETPATHINFO
 000D:000074EE       postDOSSETPATHINFO
 000D:000074F4       DOSSETVERIFY
 000D:000074FC       preDOSSETVERIFY
 000D:00007505       postDOSSETVERIFY
 000D:00007510       DOSSHUTDOWN
 000D:00007534       DOSMAKENMPIPE
 000D:00007580       preDOSMAKENMPIPE
 000D:00007591       postDOSMAKENMPIPE
 000D:00007598       DOSCALLNMPIPE
 000D:000075E0       preDOSCALLNMPIPE
 000D:000075F1       postDOSCALLNMPIPE
 000D:000075FC       DOSCONNECTNMPIPE
 000D:00007604       preDOSCONNECTNMPIPE
 000D:0000760D       postDOSCONNECTNMPIPE
 000D:00007618       DOSDISCONNECTNMPIPE
 000D:00007620       preDOSDISCONNECTNMPIPE
 000D:00007629       postDOSDISCONNECTNMPIPE
 000D:00007634       DOSPEEKNMPIPE
 000D:00007648       preDOSPEEKNMPIPE
 000D:00007664       postDOSPEEKNMPIPE
 000D:0000766C       DOSQNMPHANDSTATE
 000D:00007674       preDOSQNMPHANDSTATE
 000D:00007685       postDOSQNMPHANDSTATE
 000D:00007690       DOSQNMPIPEINFO
 000D:000076A4       preDOSQNMPIPEINFO
 000D:000076AD       postDOSQNMPIPEINFO
 000D:000076B8       DOSRAWREADNMPIPE
 000D:000076C9       preDOSRAWREADNMPIPE
 000D:000076DA       postDOSRAWREADNMPIPE
 000D:000076E4       DOSRAWWRITENMPIPE
 000D:000076F5       preDOSRAWWRITENMPIPE
 000D:00007706       postDOSRAWWRITENMPIPE
 000D:00007710       DOSSETNMPHANDSTATE
 000D:0000771B       preDOSSETNMPHANDSTATE
 000D:00007724       postDOSSETNMPHANDSTATE
 000D:0000772C       DOSTRANSACTNMPIPE
 000D:00007743       preDOSTRANSACTNMPIPE
 000D:00007754       postDOSTRANSACTNMPIPE
 000D:0000775C       DOSWAITNMPIPE
 000D:00007785       preDOSWAITNMPIPE
 000D:0000778E       postDOSWAITNMPIPE
 000D:00007798       DOSSETNMPIPESEM
 000D:000077A9       preDOSSETNMPIPESEM
 000D:000077B2       postDOSSETNMPIPESEM
 000D:000077BC       DOSQNMPIPESEMSTATE
 000D:000077D0       preDOSQNMPIPESEMSTATE
 000D:000077D9       postDOSQNMPIPESEMSTATE
 000D:000077E4       h_w_DynamicTrace
 000D:00007814       h_w_ExecPgm
 000D:00007820       h_w_DosSGSwitch
 000D:0000785C       h_w_DosSGSwitchMe
 000D:000078A4       h_w_DosSGSwitchProc2
 000D:00007948       KSGKillProcess
 000D:00007974       ksg$ksgTaskSearch
 000D:000079E4       ksg$ksgValidate
 000D:00007A10       DOSMUXSEMWAIT
 000D:00007AA4       postDOSMUXSEMWAIT2
 000D:00007B14       postDOSMUXSEMWAIT
 000D:00007B1C       muxsem$ScanMuxList
 000D:00007C34       h_w_MuxSemWait
 000D:00007C40       h_MuxSemWait
 000D:00007C42       MuxSemWait
 000D:00007C4B       muxsem$MuxSemWaitSub
 000D:00007CA0       muxsem$h_GetMuxListCount
 000D:00007CA2       muxsem$GetMuxListCount
 000D:00007D00       muxsem$GetFreeList
 000D:00007D24       muxsem$SetupMuxList
 000D:00007E9C       muxsem$MuxWait
 000D:00007ECC       muxsem$RemActiveList
 000D:00007EEC       muxsem$h_RamGetMuxSemID
 000D:00007EEE       muxsem$RamGetMuxSemID
 000D:00007F84       h_NPX16_Interrupt
 000D:00007F88       f_NPX16_Interrupt
 000D:00007F8A       NPX16_Interrupt
 000D:00007FA8       h_w_DosQProcStatus
 000D:00007FD8       f_w_EnterCritSec
 000D:00007FDA       w_EnterCritSec
 000D:00007FDF       DosEnterCritSec_PreTrace
 000D:00008010       DosEnterCritSec_PostTrace
 000D:00008028       f_w_ExitCritSec
 000D:0000802A       w_ExitCritSec
 000D:0000802F       DosExitCritSec_PreTrace
 000D:0000809D       DosExitCritSec_PostTrace
 000D:000080A0       h_w_GetPrty
 000D:000080A2       w_GetPrty
 000D:000080B5       DosGetPrty_PreTrace
 000D:0000814B       DosGetPrty_PostTrace
 000D:00008154       h_w_SetFgnd
 000D:00008158       f_w_SetFgnd
 000D:0000815A       w_SetFgnd
 000D:00008208       h_w_SetPrty
 000D:0000820A       w_SetPrty
 000D:00008226       DosSetPrty_PreTrace
 000D:00008347       DosSetPrty_PostTrace
 000D:00008378       pre_sci
 000D:000083B4       sci
 000D:00008488       to_farcall
 000D:000084B6       fc01
 000D:00008504       h_AdjustError
 000D:00008508       f_AdjustError
 000D:0000850A       AdjustError
 000D:00008520       to_getusrbufz3
 000D:00008524       to_getusrbufz206
 000D:00008529       to_getusrbufz
 000D:000085DC       UsrArgError
 000D:000085E4       sci$UsrFaultHandler
 000D:000085F4       CleanUpReturn
 000D:00008604       to_return
 000D:000086E1       to_enterfscrit
 000D:00008726       to_exitfscrit
 000D:00008768       SCIReturn0
 000D:0000876C       SCIReturn2
 000D:00008774       SCIReturn4
 000D:0000877C       SCIReturn6
 000D:00008784       SCIReturn8
 000D:0000878C       SCIReturn10
 000D:00008794       SCIReturn12
 000D:0000879C       SCIReturn14
 000D:000087A4       SCIReturn16
 000D:000087AC       SCIReturn18
 000D:000087B4       SCIReturn20
 000D:000087BC       SCIReturn22
 000D:000087C4       SCIReturn24
 000D:000087CC       SCIReturn26
 000D:000087D4       SCIReturn28
 000D:000087DC       SCIReturn30
 000D:000087E4       SCIReturn32
 000D:000087EC       SCIReturn34
 000D:000087F4       SCIReturn36
 000D:000087FC       _ausSCIReturn
 000D:00008822       _fpfnSCIKernelExit
 000D:00008828       h_Take_Kernel_Sem
 000D:0000882A       Take_Kernel_Sem
 000D:0000885C       h_Clear_Kernel_Sem
 000D:0000885E       Clear_Kernel_Sem
 000D:00008890       h_w_RamSemRequest
 000D:00008894       f_w_RamSemRequest
 000D:00008896       w_RamSemRequest
 000D:000088CC       sem$h_w_SemRequest
 000D:000088DC       h_w_SemSetWait
 000D:000088E8       h_SemSetWait
 000D:000088EC       f_SemSetWait
 000D:000088EE       SemSetWait
 000D:00008904       DOSISYSSEMSET
 000D:00008980       h_SemSet
 000D:00008984       f_SemSet
 000D:00008986       SemSet
 000D:0000899C       sem$SysSemSet
 000D:000089D0       h_w_SemWait
 000D:000089D4       f_w_SemWait
 000D:000089D6       w_SemWait
 000D:000089E0       h_SemWait
 000D:000089E4       f_SemWait
 000D:000089E6       SemWait
 000D:00008A14       sem$SemStampRPL
 000D:00008A8C       DOSHOLDSIGNAL
 000D:00008AA8       preDOSHOLDSIGNAL
 000D:00008AD4       post2DOSHOLDSIGNAL
 000D:00008B18       postDOSHOLDSIGNAL
 000D:00008B20       h_w_HoldSignal
 000D:00008B22       w_HoldSignal
 000D:00008B24       sig$HoldSignal
 000D:00008BF0       h_w_SendSignal
 000D:00008BF4       f_w_SendSignal
 000D:00008BF6       w_SendSignal
 000D:00008C38       sig$FindSigProc
 000D:00008C64       h_w_FlagProcess
 000D:00008C80       h_w_SetSigHandler
 000D:00008CE8       sig$f_SetSignal
 000D:00008CEA       sig$SetSignal
 000D:00008E4C       sig$f_ResetSigFocus
 000D:00008E4E       sig$ResetSigFocus
 000D:00008F0C       f_ResetSignals
 000D:00008F80       h_POST_SIGNAL
 000D:00008F82       POST_SIGNAL
 000D:00008FE4       h_psig16
 000D:00008FE6       psig16
 000D:000090A0       h_PostSigFocus
 000D:000090A2       PostSigFocus
 000D:000090E8       h_CreateSem
 000D:000090E8       h_w_CreateSem
 000D:00009120       h_CreateAnonSem
 000D:00009122       CreateAnonSem
 000D:00009140       h_OpenSem
 000D:00009140       h_w_OpenSem
 000D:00009170       h_w_CloseSem
 000D:00009172       w_CloseSem
 000D:0000917B       h_CloseSem
 000D:0000917D       CloseSem
 000D:000091FC       syssem$FindSysSemName
 000D:0000925C       syssem$AddSysSemName
 000D:000092E0       h_CanonBuf
 000D:000092E4       f_CanonBuf
 000D:000092E6       CanonBuf
 000D:00009330       FreeSysSem
 000D:0000933C       syssem$FreeSysSemWorker
 000D:00009380       f_SysSemExitList
 000D:00009390       syssem$SysSemExitListWorker
 000D:000093B4       f_SysSemOwnerDied
 000D:000093C4       syssem$SysSemOwnerDiedWorker
 000D:00009400       syssem$EachSysSem
 000D:00009448       syssem$CleanUpSysSemName
 000D:00009494       syssem$h_RemSysSemName
 000D:00009496       syssem$RemSysSemName
 000D:000094C0       syssem$GetSysSemPTDAIndex
 000D:000094E8       syssem$GetSysSemEntry
 000D:00009530       ScanTasks
 000D:00009590       h_ScanTasks
 000D:000095A8       f_Scan16
 000D:000095C0       h_EnterCritSecHoldSig
 000D:000095C4       f_EnterCritSecHoldSig
 000D:000095C6       EnterCritSecHoldSig
 000D:000095E0       h_ExitCritSecUnHoldSig
 000D:000095E4       f_ExitCritSecUnHoldSig
 000D:000095E6       ExitCritSecUnHoldSig
 000D:000095F8       h_w_GetPid
 000D:0000960C       h_w_GetPPID
 000D:0000965C       h_w_GetEnv
 000D:00009678       h_w_R2StackRealloc
 000D:00009700       DOSICALLBACK
 000D:000098E2       wcb3
 000D:00009900       DOSRETFORWARD
 000D:00009AA9       wrf3
 000D:00009AC8       Gen16Hook0
 000D:00009B00       Gen16Hook1
 000D:00009B50       Gen16HookV16
 000D:00009BA4       Gen16HookAny
 000D:00009C84       int$f_Call16bitDD
 000D:00009C8C       f_Call16bitKrnlExitDD
 000D:00009C94       INTProtMode
 000D:00009CA0       INTRealMode
 000D:00009CAC       sicg$sicgf2rest
 000D:00009D20       f_is_path
 000D:00009D22       is_path
 000D:00009D48       h_CheckModName
 000D:00009D4C       f_CheckModName
 000D:00009D4E       CheckModName
 000D:00009D88       h_w_loadmodule
 000D:00009D94       h_w_QAppType
 000D:00009DDC       h_w_getprocaddr
 000D:00009E48       h_w_getmodhandle
 000D:00009E4C       f_w_getmodhandle
 000D:00009E4E       w_getmodhandle
 000D:00009F64       h_w_getmodname
 000D:00009F68       f_w_getmodname
 000D:00009F6A       w_getmodname
 000D:0000A094       CheckModHandle
 000D:0000A0B8       h_w_QueryABIOSSupport
 000D:0000A0BC       f_w_QueryABIOSSupport
 000D:0000A0BE       w_QueryABIOSSupport
 000D:0000A0D4       h_w_ldrDirtyWorker
 000D:0000A0F8       h_ldrIncRefCount
 000D:0000A0FC       f_ldrIncRefCount
 000D:0000A0FE       ldrIncRefCount
 000D:0000A150       h_w_getresource
 000D:0000A1DC       f_GetRsrcSel
 000D:0000A300       ldrrsrc$RsrcPreload
 000D:0000A338       f_ldrRsrcAlloc
 000D:0000A33A       ldrRsrcAlloc
 000D:0000A3A8       h_w_FreeResource
 000D:0000A4C0       DOSQTRACEINFO
 000D:0000A4E0       h_w_QTraceInfo
 000D:0000A4F4       ProcessKill
 000D:0000A62D       TCBUnlink1_StartHook
 000D:0000A637       TCBUnlink1_EndHook
 000D:0000A65C       f_DHGetMessage16
 000D:0000A668       h_OutMessage
 000D:0000A66C       f_OutMessage
 000D:0000A66E       OutMessage
 000D:0000A6A4       h_StrCmp32
 000D:0000A6A8       f_StrCmp32
 000D:0000A6AA       StrCmp32
 000D:0000A704       h_StrCpy32
 000D:0000A708       f_StrCpy32
 000D:0000A70A       StrCpy32
 000D:0000A760       h_w_SystemService
 000D:0000A7C0       SysServVDM
 000D:0000A880       SysServSM
 000D:0000A90E       f_SysServReboot
 000D:0000A90E       h_SysServReboot
 000D:0000A92C       SysServHE
 000D:0000A964       SysServJIT
 000D:0000A9C0       SysServJIT2
 000D:0000AA04       SysServPS
 000D:0000AA0C       sysserv$SysServWait
 000D:0000AA44       sysserv$SysServWaitQ
 000D:0000AAC4       SysServVP
 000D:0000ABA0       Sys_FreezeThaw
 000D:0000ABF0       f_ProcessTerminate
 000D:0000AD14       h_w_KillProcess
 000D:0000AD19       h_w_KillProc
 000D:0000AD44       h_w_CWait
 000D:0000AD6C       CookedKBD
 000D:0000ADD4       h___TKSetSSBase
 000D:0000AE34       __panicHIGH3
 000D:0000AE3C       __panicfnHIGH3
 000D:0000AE44       __panicfnmsgHIGH3
 000D:0000AE4C       h_w_SetVec
 000D:0000AEA0       Exc_Lookup
 000D:0000AEE8       h_UsrArgFault
 000D:0000AEEC       f_UsrArgFault
 000D:0000AEEE       UsrArgFault
 000D:0000AF24       h_UsrArgFaultMsg
 000D:0000AF26       UsrArgFaultMsg
 000D:0000B088       trap286$FormatRegDump
 000D:0000B09C       trap286$FormatLimAccDump
 000D:0000B0DC       f_DelayHardErrTrap2
 000D:0000B0DE       DelayHardErrTrap2
 000D:0000B0E8       f_DelayHardErr
 000D:0000B0EA       DelayHardErr
 000D:0000B100       DelayHardErrSub
 000D:0000B2AC       h_ChkDelayHardErr
 000D:0000B2AE       ChkDelayHardErr
 000D:0000B430       h_w_Ptrace
 000D:0000B448       dosinit$f_KDPLink
 000D:0000B450       dosinit$f_KDPUnlink
 000D:0000B458       dosinit$f_KDPEnable
 000D:0000B460       dosinit$f_KDPPageIn
 000D:0000B468       f_DebugThreadOneStarting
 000D:0000B470       f_DebugThreadNDying
 000D:0000B48E       h_DebugThreadOneDying
 000D:0000B4C0       dosinit$h_GetSymName
 000D:0000B4C4       dosinit$f_GetSymName
 000D:0000B4C6       dosinit$GetSymName
 000E:00000000       _StartHIGH4CODE
 000E:00000004       h_DISK_INFO
 000E:00000006       DISK_INFO
 000E:00000038       dinfo$DISK_INFO_NoCDS
 000E:000000A4       f_DISK_INFO_NoCDS
 000E:000000AC       DiskFreeSpace
 000E:00000190       CountClusters
 000E:000001D4       FindEntry
 000E:0000024B       Srch
 000E:00000274       NEXTENT
 000E:0000046C       NextEntry
 000E:00000520       GETENTRY
 000E:00000544       GETENT
 000E:0000056A       SetEntry
 000E:00000584       SetDirSrch
 000E:000005E3       SetRootSrch
 000E:00000638       h_GetPath
 000E:0000063A       GetPath
 000E:00000660       GetPathNoSet
 000E:000006D8       dir$ROOTPATH
 000E:0000070A       dir$FINDPATH
 000E:00000840       StartSrch
 000E:00000884       h_MatchAttributes
 000E:00000886       MatchAttributes
 000E:000008B4       dir$Build_device_ent
 000E:00000904       dir$CheckForDevice
 000E:00000950       h_fValidFATDisk
 000E:00000952       fValidFATDisk
 000E:0000097C       h_DOS_Read
 000E:0000097E       DOS_Read
 000E:00000A68       disk$ReadDev
 000E:00000A94       disk$DevRWRaw
 000E:00000BAC       disk$EndReadDev
 000E:00000BB4       disk$CRDFERR
 000E:00000BD0       h_DOS_Write
 000E:00000BD2       DOS_Write
 000E:00000CE4       WriteDev
 000E:00000D14       EndWriteDev
 000E:00000D34       DirRead
 000E:00000DC6       FirstCluster
 000E:00000DE8       SET_BUF_AS_DIR
 000E:00000DFC       h_SetupForIO
 000E:00000E00       f_SetupForIO
 000E:00000E02       SetupForIO
 000E:00000E06       SetupForIO_EA
 000E:00000ED4       disk$BreakDown
 000E:00000F08       disk$DiskRead
 000E:00000F74       DoDiskRead
 000E:00001260       disk$AdjustPageList
 000E:00001284       disk$FATReadInit
 000E:00001294       h_InitTCBVars
 000E:00001298       f_InitTCBVars
 000E:0000129A       InitTCBVars
 000E:000012DC       disk$FATRWLockMem
 000E:00001330       FATDevLockMem
 000E:0000146C       DoCPDiskRead
 000E:00001638       disk$AdjPgLstBefIO
 000E:00001660       disk$h_SetAccessDenied
 000E:00001662       disk$SetAccessDenied
 000E:00001674       disk$SetSFT
 000E:000016B8       disk$DiskWrite
 000E:0000172C       DiskUpdateFileSize
 000E:000018F4       DoDiskWrite
 000E:00001C6C       disk$DoCPDiskWrite
 000E:00001D94       disk$FATWriteInit
 000E:00001DD0       disk$FileGrowth
 000E:00001F84       disk$WrtErr
 000E:00001FA0       h_Setup_PhysIO
 000E:00001FA4       f_Setup_PhysIO
 000E:00001FA6       Setup_PhysIO
 000E:00002000       f_ABSDRDWRT
 000E:00002090       disk$AbsSetup
 000E:000020D8       disk$XAbsSetup
 000E:00002110       disk$GetVPB
 000E:000021AC       h_DOS_Close
 000E:000021D4       DirFromSFT
 000E:00002244       h_DOS_Commit
 000E:00002246       DOS_Commit
 000E:000022B0       FileCommit
 000E:000023E0       h_DOS_ChDir
 000E:0000245C       h_DOS_Dup
 000E:00002460       f_DOS_Dup
 000E:00002462       DOS_Dup
 000E:00002480       dossrch$FindEdit
 000E:00002558       dossrch$FEFixDate
 000E:00002598       dossrch$FEFixTime
 000E:000025D0       h_IsEOF
 000E:000025D4       f_IsEOF
 000E:000025D6       IsEOF
 000E:000025EC       h_UnPack
 000E:000025F0       f_UnPack
 000E:000025F2       UnPack
 000E:0000268C       h_Pack
 000E:00002690       f_Pack
 000E:00002692       Pack
 000E:0000278C       fat$MapCluster
 000E:00002894       CheckExtent
 000E:00002988       h_DOS_Search_First
 000E:0000298A       DOS_Search_First
 000E:00002A64       h_DOS_Search_Next
 000E:00002A66       DOS_Search_Next
 000E:00002B14       h_HogEAFile
 000E:00002BB0       h_UnHogEAFile
 000E:00002C48       EA_EnterShare
 000E:00002D1C       h_DOS_QFileMode
 000E:00002D6C       h_DOS_SetFileMode
 000E:00002DF0       h_DOS_SetInfo
 000E:00002DF2       DOS_SetInfo
 000E:00002E14       SetInfoForFile
 000E:00002EE0       ValidateTmDt
 000E:00002F24       h_DOS_QInfo
 000E:00002F26       DOS_QInfo
 000E:00002F50       GetInfoForFile
 000E:00003034       bytesToClusters
 000E:00003060       f_Call32FSDLock
 000E:00003084       f_Call32FSDCancelLock
 000E:0000309C       h_DOS_QFsInfo
 000E:000030FC       fsinfo$GetpFSInfo
 000E:0000312C       f_GSetMediaID
 000E:00003284       f_Call32FSD
 000E:0000329C       h_DOS_Get_Drive_Freespace
 000E:0000329E       DOS_Get_Drive_Freespace
 000E:000032BC       LockMFTShar
 000E:000032C1       LockMFT
 000E:00003320       UnlockMFT
 000E:00003378       h_DosIOAllowed
 000E:0000337A       DosIOAllowed
 000E:0000339C       RetryLockedDrive
 000E:000033D8       h_CheckPipeDir
 000E:000033DA       CheckPipeDir
 000E:000033FC       h_w_OpLockRelease
 000E:0000346C       FillSFTFromDirEnt
 000E:00003500       FillDeviceSFT
 000E:00003590       GetBufBack
 000E:000035E8       h_NextSec
 000E:000035EC       f_NextSec
 000E:000035EE       NextSec
 000E:00003654       Optimize
 000E:00003748       h_FigRec
 000E:0000374C       f_FigRec
 000E:0000374E       FigRec
 000E:00003780       Allocate
 000E:00003784       AllocateEA
 000E:000039A5       postAllocate
 000E:000039A8       h_WriteFATOrdered
 000E:000039AC       f_WriteFATOrdered
 000E:000039AE       WriteFATOrdered
 000E:00003A78       h_Release
 000E:00003A7C       f_Release
 000E:00003A7E       Release
 000E:00003A85       RelBlks
 000E:00003AA8       preRelease
 000E:00003B84       AllocateEAVL
 000E:00003B9C       h_AllocateHotFix
 000E:00003BA0       f_AllocateHotFix
 000E:00003BA2       AllocateHotFix
 000E:00003BA8       ReleaseVL
 000E:00003BDC       GetEOF
 000E:00003BF4       DeleteVID
 000E:00003C10       UpdateVID
 000E:00003C28       h_Find_VPB
 000E:00003C2C       f_Find_VPB
 000E:00003C2E       Find_VPB
 000E:00003C6C       h_Req_List_Init
 000E:00003C70       f_Req_List_Init
 000E:00003C72       Req_List_Init
 000E:00003CFC       ReqListNotifyRtn
 000E:00003D50       h_Req_List_Add_Req
 000E:00003D54       f_Req_List_Add_Req
 000E:00003D56       Req_List_Add_Req
 000E:00003EE4       h_Req_List_Add_Extent
 000E:00003EE8       f_Req_List_Add_Extent
 000E:00003EEA       Req_List_Add_Extent
 000E:00003FBC       h_Req_List_Read
 000E:00003FC0       f_Req_List_Read
 000E:00003FC2       Req_List_Read
 000E:00004034       h_Req_List_Write
 000E:00004038       f_Req_List_Write
 000E:0000403A       Req_List_Write
 000E:000040C0       h_Req_List_Add_SG
 000E:000040C4       f_Req_List_Add_SG
 000E:000040C6       Req_List_Add_SG
 000E:000041BC       h_Req_List_Exec
 000E:000041C0       f_Req_List_Exec
 000E:000041C2       Req_List_Exec
 000E:000043A8       h_GetReqList
 000E:000043AC       f_GetReqList
 000E:000043AE       GetReqList
 000E:000043C0       h_FreeReqList
 000E:000043C4       f_FreeReqList
 000E:000043C6       FreeReqList
 000E:000043D0       h_UseCache
 000E:000043D4       f_UseCache
 000E:000043D6       UseCache
 000E:00004434       h_Init_VPB_Cache
 000E:00004436       Init_VPB_Cache
 000E:000044A8       strat2$GetPageBreakInfo
 000E:00004558       h_FSGetPriorityInfo
 000E:0000455A       FSGetPriorityInfo
 000E:00004584       strat2$FatDirtyBitSet
 000E:000045D0       FatDirtyBitClear
 000E:00004624       Gen16HookAny_High4
 000E:000046BC       __panicHIGH4
 000E:000046C4       __panicfnHIGH4
 000E:000046CC       __panicfnmsgHIGH4
 000E:000046D4       _EndHIGH4CODE
 000E:000046D4       _StartHIGH4SWAPCODE
 000E:000046D4       _StartFSSWAPCODE
 000E:000046D4       _EndHIGH4SWAPCODE
 000E:000046D4       h_w_PhysicalDisk
 000E:000046D4       _StartPHYSDSKGROUP
 000E:000046D8       f_w_PhysicalDisk
 000E:000046DA       w_PhysicalDisk
 000E:000047AC       h_DevLockPhysDrive
 000E:000047AE       DevLockPhysDrive
 000E:00004878       h_DevUnlockPhysDrive
 000E:0000487A       DevUnlockPhysDrive
 000E:000048F8       devphys$DevReturnHandle
 000E:000049D8       h_DevQueryHandle
 000E:000049DA       DevQueryHandle
 000E:00004A1C       h_DevReleaseHandle
 000E:00004A1E       DevReleaseHandle
 000E:00004AA0       devphys$LockPhysDrv
 000E:00004B68       devphys$UnlockPhysDrv
 000E:00004BC8       h_DOS_FindFirst
 000E:00004BC8       _StartSRCHGROUP
 000E:00004BC8       _EndPHYSDSKGROUP
 000E:00004C24       h_DOS_FindNext
 000E:00004C26       DOS_FindNext
 000E:00004C48       dossrch$DoFindlp
 000E:00004C56       dossrch$DoFindLpGotOne
 000E:00004CB0       dossrch$DoFind
 000E:00004E30       dossrch$Find_GetFEAList
 000E:00004EC0       dossrch$FillTempSFTForObject
 000E:00004F60       dossrch$CopyInfoToUserBuf
 000E:00004F94       h_DOS_FindFromName
 000E:00004FD0       _EndSRCHGROUP
 000E:00004FD0       h_DOS_PathInfo
 000E:00005188       fatdirop$FillSFTForRootDir
 000E:000051AC       h_DOS_Delete
 000E:000051AE       DOS_Delete
 000E:00005360       h_DOS_RmDir
 000E:000055AC       h_SaveFCBInfo
 000E:000055B0       f_SaveFCBInfo
 000E:000055B2       SaveFCBInfo
 000E:000055F8       ResetLRU
 000E:00005624       f_SetOpenAge
 000E:00005626       SetOpenAge
 000E:00005648       f_LRUFCB
 000E:0000564A       LRUFCB
 000E:00005728       FCBRegen
 000E:0000573C       f_BlastSFT
 000E:0000573E       BlastSFT
 000E:000057B4       f_CheckFCB
 000E:000057B6       CheckFCB
 000E:00005810       h_SFTFromFCB
 000E:00005814       f_SFTFromFCB
 000E:00005816       SFTFromFCB
 000E:00005858       f_FCBHardErr
 000E:0000585A       FCBHardErr
 000E:00005878       fcbio$FindSFT
 000E:000058F8       f_w_FCB_Delete
 000E:00005A8C       f_w_FCB_Rename
 000E:00005C7C       f_w_Get_FCB_File_Length
 000E:00005D10       h_ChkIFSVol
 000E:00005D14       f_ChkIFSVol
 000E:00005D16       ChkIFSVol
 000E:00005D64       h_w_FCB_VolId
 000E:00005D68       f_w_FCB_VolId
 000E:00005D6A       w_FCB_VolId
 000E:00005EA0       h_SetDeviceFont
 000E:00005EF4       h_w_Copy
 000E:00006008       h_DOS_OpenCreate
 000E:00006008       _StartNODEGROUP
 000E:0000600A       DOS_OpenCreate
 000E:0000649C       h_DOS_MkDir
 000E:00006784       h_DOS_SetFSInfo
 000E:000068DC       h_DOS_Rename
 000E:00006C10       mknode$BuildDir
 000E:00006C94       NewDir
 000E:00006D60       mknode$SetDotEnt
 000E:00006DB4       mknode$MakeNode
 000E:00006E48       mknode$NewEntry
 000E:0000702C       mknode$AttribOk
 000E:0000704C       mknode$FillDirectBlockDeviceSFT
 000E:000070BC       mknode$NeedEASPresent
 000E:000071E4       mknode$BlanksBeforeDot
 000E:0000722C       mknode$GET_SOURCE
 000E:0000727C       h_w_FindNotifyClose
 000E:0000727C       _EndNODEGROUP
 000E:0000727C       _StartNOTIFYGROUP
 000E:0000727E       w_FindNotifyClose
 000E:000072E0       h_w_FindNotifyNext
 000E:000072E2       w_FindNotifyNext
 000E:00007344       h_w_FindNotifyFirst
 000E:00007346       w_FindNotifyFirst
 000E:000074AC       FSD_FindNotifyFirst
 000E:00007558       DOS_FindNotifyClose
 000E:000075DC       DOS_FindNotifyFirst
 000E:00007768       DOS_FindNotifyNext
 000E:000078B4       FNotify_AllocDirHandle
 000E:00007914       FNotify_FreeDirHandle
 000E:0000796C       FNotify_AllocFatHandle
 000E:00007990       FNotify_ChkDirHandle
 000E:000079D0       Find_RMPFNYRec
 000E:000079E4       h_FNotifyExit
 000E:00007A18       h_w_OpenChangeNotify
 000E:00007A1A       w_OpenChangeNotify
 000E:00007AA0       h_w_ResetChangeNotify
 000E:00007AA2       w_ResetChangeNotify
 000E:00007BA4       h_w_CloseChangeNotify
 000E:00007BA6       w_CloseChangeNotify
 000E:00007BDC       CNotifySemGet
 000E:00007BFC       CNotifySemRel
 000E:00007C1C       CNotify_AllocStruc
 000E:00007C64       CNotify_FreeStruct
 000E:00007C8C       h_CNotify_PWake
 000E:00007CBC       h_CNotify_ADWake
 000E:00007D1C       notify$CNotify_Wake
 000E:00007DD0       h_CNotifyExit
 000E:00007DF0       _EndNOTIFYGROUP
 000E:00007DF0       h_w_Shutdown
 000E:00007DF4       f_w_Shutdown
 000E:00007DF6       w_Shutdown
 000E:0000807C       shutdown$NotifyDevs
 000E:000080D8       shutdown$GetNextDev
 000E:00008100       shutdown$FlushAllSFTs
 000E:00008154       shutdown$FlushVDMfcbSFTs
 000E:0000816C       shutdown$SetSDFlags
 000E:000081C4       shutdown$DisableFSDs
 000E:00008258       shutdown$IsSwapFSC
 000E:000082A4       GetFEAInfo
 000E:000082A4       _StartFATEASWAPCODE
 000E:000082A4       _EndFSSWAPCODE
 000E:00008454       SetFEAInfo
 000E:000084AC       DoSetFEAInfo
 000E:00008620       extattr$DeleteFEA
 000E:00008670       extattr$AppendFEA
 000E:000086F0       extattr$GetFEAsizes
 000E:00008714       extattr$UpdateFEAlist
 000E:000087CC       extattr$FindGEAbyFEA
 000E:000088A8       extattr$FindFEAbyGEA
 000E:0000892C       extattr$FindFEAbyFEA
 000E:000089CC       extattr$GetFEAFromGEAlist
 000E:00008AD4       extattr$MakeDummyFEA
 000E:00008B38       GetFEAlistSize
 000E:00008B74       EASerialize
 000E:00008B98       EAUnserialize
 000E:00008BC8       EAWait
 000E:00008BF0       WakeEAWaiters
 000E:00008C04       DiskReadFEAlist
 000E:00008D08       SetupFatEA
 000E:00008F64       EAFileSane
 000E:00008F84       CountHandle
 000E:00008FD4       EZ_DRead
 000E:00009030       EZ_DCommit
 000E:00009074       EZ_DWrite
 000E:000090C8       IsSFT
 000E:00009138       GenNullEAFile
 000E:000091F8       FreeNullEAFile
 000E:00009200       EZ_DOpen
 000E:00009320       EAHandleToOffset
 000E:00009418       DiskWriteFEAlist
 000E:00009478       AddEA
 000E:000095E8       SetEADataHeader
 000E:00009628       CreateEAData
 000E:000096EC       WriteEADataHeader
 000E:00009728       UpdateEADataHandle
 000E:00009774       ClustersFromBytes
 000E:00009794       ClusterToBytes
 000E:000097A4       AllocEAHandle
 000E:00009834       CreateNewHandles
 000E:000098A4       FillCluster
 000E:000098F8       FindFreeEAHandle
 000E:00009A48       MarkHandleAllocated
 000E:00009C14       MarkEAHandleFree
 000E:00009C68       GetEADataInfo
 000E:00009D14       GetEAFileSector
 000E:00009D54       ChangeEAHandle
 000E:00009DE4       DeleteEA
 000E:00009EE4       ReleaseEA
 000E:00009FF4       SwapClusterChain
 000E:0000A128       DoClusterSwap
 000E:0000A360       SetLog
 000E:0000A3E0       DoPack
 000E:0000A3F4       DoSKPCLP
 000E:0000A424       FixBaseOffTables
 000E:0000A494       AdjustTableBlock
 000E:0000A568       OffsetToClusSec
 000E:0000A590       _EndMONLOCKCODE
 000E:0000A590       h_w_FileIO
 000E:0000A590       _EndMONSWAPCODE
 000E:0000A590       _StartNMPIPESWAPCODE
 000E:0000A590       _EndFATEASWAPCODE
 000E:0000A590       _StartFILEIOGROUP
 000E:0000A590       _StartMONLOCKCODE
 000E:0000A590       _StartMONSWAPCODE
 000E:0000A592       w_FileIO
 000E:0000A6A4       fhandle$FileIORouter
 000E:0000A870       CmdPktCopy
 000E:0000A884       _EndFILEIOGROUP
 000E:0000A884       _StartFSCTLGROUP
 000E:0000A884       h_w_FSAttach
 000E:0000A954       SpoolAttachDetach
 000E:0000AA20       AttachToFSD
 000E:0000AAB8       fsctl$AttachDrive
 000E:0000ABA8       fsctl$AttachDevice
 000E:0000AC5C       fsctl$detach_rem_drive
 000E:0000ACA8       fsctl$DetachFromFSD
 000E:0000AD0C       fsctl$DetachDevice
 000E:0000AD84       fsctl$DetachDrive
 000E:0000AE1C       call_attach_fsd
 000E:0000AE44       h_DelDerefDrive
 000E:0000AE46       DelDerefDrive
 000E:0000AE78       h_ddd_etsk
 000E:0000AE98       h_w_qFSAttach
 000E:0000AE9C       f_w_qFSAttach
 000E:0000AE9E       w_qFSAttach
 000E:0000AF44       q_dev_drv
 000E:0000AFF8       fillin_dev
 000E:0000B098       fillin_drv
 000E:0000B170       q_ord_dev
 000E:0000B1C4       q_ord_drv
 000E:0000B204       call_query_fsd
 000E:0000B2CC       ord_FindCharDevEntry
 000E:0000B2F8       ord_FindDrive
 000E:0000B320       load_2_fields
 000E:0000B354       load_3_fields
 000E:0000B3BC       fill_fields_0
 000E:0000B3F0       fill_fields_FAT
 000E:0000B468       update_drv
 000E:0000B498       fsctl$Path_Check
 000E:0000B53C       h_w_FSCtl
 000E:0000B53C       _EndFSCTLGROUP
 000E:0000B540       f_w_FSCtl
 000E:0000B542       w_FSCtl
 000E:0000B658       fsctl$handle_route
 000E:0000B688       path_route
 000E:0000B6C8       fsd_route
 000E:0000B6DC       call_control_fsd
 000E:0000B71C       FSD_FSCtl
 000E:0000B798       h_DOS_FSCtl
 000E:0000B79A       DOS_FSCtl
 000E:0000B808       _StartDRVLOCKGROUP
 000E:0000B808       DirectIOAllowed
 000E:0000B880       h_LockDrive
 000E:0000B882       LockDrive
 000E:0000B96C       h_UnlockDrive
 000E:0000B96E       UnlockDrive
 000E:0000B9C8       _EndDRVLOCKGROUP
 000E:0000B9C8       _StartNMPIPEGROUP
 000E:0000B9CB       PipeDir
 000E:0000B9D4       h_w_MakeNmPipe
 000E:0000BC30       nampipe1$npm_chk_buf_size
 000E:0000BC54       nampipe1$npm_memalloc
 000E:0000BCE8       nampipe1$npcr_initbuf
 000E:0000BD00       h_w_ConnectNmPipe
 000E:0000BE3C       h_w_DisconnectNmPipe
 000E:0000BF54       h_w_WaitNmPipe
 000E:0000BF58       f_w_WaitNmPipe
 000E:0000BF5A       w_WaitNmPipe
 000E:0000C068       nampipe1$CopyName
 000E:0000C084       nampipe1$wnp_sub
 000E:0000C0D8       nampipe1$check_server_mode
 000E:0000C128       nampipe1$flushpipe
 000E:0000C1B0       h_NmPipeOpen
 000E:0000C1B2       NmPipeOpen
 000E:0000C478       NmPipeClose
 000E:0000C570       nampipe1$npcl_dealloc_all
 000E:0000C588       nampipe1$npcl_dealloc_buf
 000E:0000C5D4       nampipe1$npcl_detach_spooled
 000E:0000C644       h_w_QNmPHandState
 000E:0000C648       f_w_QNmPHandState
 000E:0000C64A       w_QNmPHandState
 000E:0000C6E0       h_w_SetNmPHandState
 000E:0000C6E4       f_w_SetNmPHandState
 000E:0000C6E6       w_SetNmPHandState
 000E:0000C7C4       nampipe1$sphs_check_pmode
 000E:0000C7DC       nampipe1$sphs_check_block
 000E:0000C7F4       h_w_QNmPipeInfo
 000E:0000C7F8       f_w_QNmPipeInfo
 000E:0000C7FA       w_QNmPipeInfo
 000E:0000C9B0       nampipe1$npqi_bufsize
 000E:0000C9C4       h_w_CallNmPipe
 000E:0000C9C8       f_w_CallNmPipe
 000E:0000C9CA       w_CallNmPipe
 000E:0000CBC0       h_w_SetNmPipeSem
 000E:0000CCB4       nampipe1$snps_sem_deref
 000E:0000CD20       h_w_QNmPipeSemState
 000E:0000CE28       nampipe1$qnps_xfer_rec
 000E:0000CE48       nampipe1$qnps_check_space
 000E:0000CF84       nampipe1$np_handle_chk
 000E:0000CFC0       nampipe1$findpipe
 000E:0000CFFC       nampipe1$get_next_instance
 000E:0000D010       nampipe1$get_free_npn
 000E:0000D0AC       nampipe1$find_npn
 000E:0000D0E8       nampipe1$get_free_np
 000E:0000D148       nampipe1$dealloc_np
 000E:0000D200       startofnampipe2
 000E:0000D200       nampipe2$np_handle_io
 000E:0000D200       endofnampipe1
 000E:0000D209       np_sft_io
 000E:0000D25C       h_w_PeekNmPipe
 000E:0000D260       f_w_PeekNmPipe
 000E:0000D262       w_PeekNmPipe
 000E:0000D354       h_w_RawReadNmPipe
 000E:0000D358       f_w_RawReadNmPipe
 000E:0000D35A       w_RawReadNmPipe
 000E:0000D3F8       h_NmPipeRead
 000E:0000D3FA       NmPipeRead
 000E:0000D424       nampipe2$nmpipe_read_peek
 000E:0000D498       nampipe2$readiob
 000E:0000D524       nprcb
 000E:0000D5C4       rd_chk_avail
 000E:0000D5D4       nampipe2$chk_buf_wrap
 000E:0000D5DD       nampipe2$chk_buf_wrap1
 000E:0000D5FC       h_w_TransactNmPipe
 000E:0000D600       f_w_TransactNmPipe
 000E:0000D602       w_TransactNmPipe
 000E:0000D6C8       np_trans_sft
 000E:0000D7B0       h_w_RawWriteNmPipe
 000E:0000D7B4       f_w_RawWriteNmPipe
 000E:0000D7B6       w_RawWriteNmPipe
 000E:0000D854       h_NmPipeWrite
 000E:0000D856       NmPipeWrite
 000E:0000D880       nampipe2$nmpipe_write_raw
 000E:0000D8F4       h_NmPipeCommit
 000E:0000D8F6       NmPipeCommit
 000E:0000D950       nampipe2$writeiob
 000E:0000DA44       wrt_chk_avail
 000E:0000DAA4       npwcb
 000E:0000DB14       nampipe2$get_lock_sem
 000E:0000DB28       nampipe2$np_sem_blk
 000E:0000DB2B       np_sem_wait
 000E:0000DBDC       np_sem_sig
 000E:0000DBEC       np_sem_clear
 000E:0000DC40       nampipe2$np_poke_user_sem
 000E:0000DC64       h_w_OpLockWait
 000E:0000DC64       _EndNMPIPEGROUP
 000E:0000DC64       _StartOPLOCKGROUP
 000E:0000DD64       h_OpLockCleanUp
 000E:0000DD68       f_OpLockCleanUp
 000E:0000DD6A       OpLockCleanUp
 000E:0000DECC       oplock$GetOpLockThread
 000E:0000DF04       h_w_OpLockShutDown
 000E:0000DF38       _EndNMPIPESWAPCODE
 000E:0000DF38       _EndOPLOCKGROUP
 000E:0000DF38       _StartENDHIGH4CODE
 000F:00000000       _StartHIGH5CODE
 000F:00000004       VPBGrow
 000F:0000004C       h_WhatVolumePercFar
 000F:00000050       h_WhatVolume
 000F:00000052       WhatVolume
 000F:00000064       WhatVolumePerc
 000F:0000006A       h_WhatVolumeCheck
 000F:0000006C       WhatVolumeCheck
 000F:00000083       h_WhatVolumeForce
 000F:00000085       WhatVolumeForce
 000F:00000210       volmount$GenhVPB
 000F:000005FC       Check_if_FAT
 000F:000006BC       Check_if_FAT_Check
 000F:000006D8       Check_if_FAT_Init
 000F:000006F4       h_GenRemotehVPB
 000F:00000768       volmount$FSMountVolume
 000F:0000086C       h_FSDMount
 000F:0000086E       FSDMount
 000F:00000894       volmount$FindVID
 000F:00000924       h_ForceMount
 000F:00000926       ForceMount
 000F:00000B60       h_RedetermineMedia
 000F:00000B62       RedetermineMedia
 000F:00000D6C       h_SecReadPre
 000F:00000D9C       h_SecReadPost
 000F:00000DC8       h_SecWritePre
 000F:00000DE4       h_SecWritePost
 000F:00000E08       h_SecNewSize
 000F:00000E24       $TJMP
 000F:00000E28       h_$TJMP
 000F:00000E48       h_PathChrCmp
 000F:00000E4A       PathChrCmp
 000F:00000E54       h_StrCmp
 000F:00000E56       StrCmp
 000F:00000EA0       h_StrCpy
 000F:00000EA4       f_StrCpy
 000F:00000EA6       StrCpy
 000F:00000EEC       h_FStrCpy
 000F:00000EF0       f_FStrCpy
 000F:00000EF2       FStrCpy
 000F:00000F24       h_FStrCpy32
 000F:00000F28       f_FStrCpy32
 000F:00000F2A       FStrCpy32
 000F:00000F68       h_UCase
 000F:00000F6C       f_UCase
 000F:00000F6E       UCase
 000F:00000F90       __panicHIGH5
 000F:00000F98       __panicfnHIGH5
 000F:00000FA0       __panicfnmsgHIGH5
 000F:00000FA8       f_K_F_Systrace
 000F:00000FB0       dosinit$f_DebugLoadSymDosFS
 000F:00000FB2       dosinit$DebugLoadSymDosFS
 000F:00001124       _StartHIGH5SWAPCODE
 000F:00001124       h_SecOpenPre
 000F:00001124       _EndHIGH5CODE
 000F:00001140       h_SecOpenPost
 000F:000011B0       h_SecMovePre
 000F:000011E4       h_SecMovePost
 000F:00001230       h_SecDeletePre
 000F:00001258       h_SecDeletePost
 000F:00001298       h_SecChgFilePtr
 000F:0000130C       h_SecQueryFileInfo
 000F:00001328       h_SecSetFileInfo
 000F:00001350       h_SecSetFileMode
 000F:00001388       h_SecSetPathInfo
 000F:000013D4       h_SecClose
 000F:000013E8       h_SecFindFirst
 000F:0000141C       h_Sec3xFindFirst
 000F:00001444       h_Sec3xFindFirstNext
 000F:00001458       h_Sec3xFindClose
 000F:0000146C       h_SecFindNext
 000F:000014A4       h_SecFindClose
 000F:000014BC       h_SecMakeDir
 000F:000014EC       h_SecChangeDir
 000F:00001518       h_SecRemoveDir
 000F:00001540       h_SecSetDateTime
 000F:00001574       h_SecDevIoctl
 000F:00001628       h_Sec16Router
 000F:0000163C       _StartLOGSWAPCODE
 000F:0000163C       h_w_LogEntry
 000F:0000163C       _EndHIGH5SWAPCODE
 000F:0000163E       w_LogEntry
 000F:000016D0       RAS_dh_GetLIDEntry
 000F:000016D0       _EndLOGSWAPCODE
 000F:000016D0       _EndLOGLOCKCODE
 000F:000016D0       _StartLOGLOCKCODE
 000F:000016D0       _StartRASLOCKCODE
 000F:00001718       RAS_dh_GetDeviceBlock
 000F:00001718       RAS_dh_FreeLIDEntry
 000F:00001744       RAS_dh_ABIOSCall
 000F:00001788       RAS_dh_ABIOSCommonEntry
 000F:000017CC       RAS_dh_ABIOSCall_post
 000F:000017CC       RAS_dh_ABIOSCommonEntry_post
 000F:000017CC       RAS_dh_FreeLIDEntry_post
 000F:000017CC       RAS_CFparameters_post
 000F:000017F0       RAS_dh_GetLIDEntry_post
 000F:000017F0       RAS_CFAxparameters_post
 000F:00001814       RAS_dh_GetDeviceBlock_post
 000F:0000183C       RAS_Yield
 000F:0000183C       RAS_dh_SetROMVector
 000F:0000183C       RAS_dh_RegisterStackUsage
 000F:0000183C       RAS_dh_UnPhysToVirt
 000F:0000183C       RAS_DevDone
 000F:0000183C       RAS_dh_AttachDD
 000F:0000183C       RAS_dh_DynamicAPI
 000F:0000183C       RAS_AllocReqPacket
 000F:0000183C       RAS_dh_SetTimer
 000F:0000183C       RAS_dh_ResetTimer
 000F:0000183C       RAS_dh_InternalError
 000F:0000183C       RAS_dvh39
 000F:0000183C       RAS_Noparms
 000F:0000183C       RAS_dh_YieldTC
 000F:0000183C       RAS_SchedAddr
 000F:00001850       RAS_FreePhysDM
 000F:00001850       RAS_SegUnlockDM
 000F:00001850       RAS_ProcRun2
 000F:00001850       RAS_dh_SemClear
 000F:00001850       RAS_AxBxparms
 000F:00001850       RAS_dh_DeRegister
 000F:00001850       RAS_dh_PhysToVirt
 000F:00001850       RAS_ProcRun
 000F:0000186C       RAS_dh_RegisterTmrDD
 000F:0000186C       RAS_CxDiparms
 000F:0000186C       RAS_dh_RegisterBeep
 000F:0000188C       RAS_BxCxparms
 000F:0000188C       RAS_dh_Beep
 000F:000018A8       RAS_AllocPhysDM
 000F:000018A8       RAS_AxBxDhparms
 000F:000018A8       RAS_dh_SemHandle
 000F:000018DC       RAS_BxDhparms
 000F:000018DC       RAS_dh_ModifyPriority
 000F:0000190C       RAS_dh_AllocGDTSelector
 000F:0000190C       RAS_EsDiCxparms
 000F:00001930       RAS_dh_RegisterKrnlExit
 000F:00001930       RAS_dh_PhysToGDTSelector
 000F:00001930       RAS_AxBxCxSiparms
 000F:00001950       RAS_dh_RegisterPerfCtrs
 000F:00001950       RAS_SiAxDiBxCxparms
 000F:00001970       RAS_EsDiDsSiparms
 000F:00001970       RAS_dh_RegisterPDD
 000F:00001990       RAS_AxBxDiCxparms
 000F:00001990       RAS_dh_SemRequest
 000F:000019B0       RAS_dh_PhysToUVirt
 000F:000019B0       RAS_AxBxCxDhparms
 000F:000019E4       RAS_AxBxDiCxDhparms
 000F:000019E4       RAS_ProcBlock
 000F:00001A1C       RAS_DsBxAlparms
 000F:00001A1C       RAS_QueueWrite
 000F:00001A48       RAS_SegLockDM
 000F:00001A48       RAS_AxBhBlparms
 000F:00001A68       RAS_PushPullpartSortPacket
 000F:00001A68       RAS_SortRequest
 000F:00001A68       RAS_PushRequest
 000F:00001A68       RAS_PullParticular
 000F:00001A98       RAS_PullRequest
 000F:00001A98       RAS_VirtToPhysDM
 000F:00001A98       RAS_DsSiparms
 000F:00001A98       RAS_dh_RealToProt
 000F:00001A98       RAS_dh_ProtToReal
 000F:00001AC4       RAS_EsBxparms
 000F:00001AC4       RAS_FreeReqPacket
 000F:00001AE4       RAS_QueueRead
 000F:00001AE4       RAS_QueueInit
 000F:00001AE4       RAS_QueueFlush
 000F:00001AE4       RAS_QueueTrace
 000F:00001B10       RAS_dh_FreeGDTSelector
 000F:00001B10       RAS_dh_MonFlush
 000F:00001B10       RAS_dh_GetDescInfo
 000F:00001B10       RAS_Axparms
 000F:00001B2C       RAS_Bxparms
 000F:00001B2C       RAS_dh_UnSetIRQ
 000F:00001B2C       RAS_dh_TickCount
 000F:00001B2C       RAS_dh_SetIRQ
 000F:00001B48       RAS_dh_MonWrite
 000F:00001B90       RAS_dh_MonitorCreate
 000F:00001BC0       RAS_dh_Register
 000F:00001BF8       RAS_dh_SendEvent
 000F:00001BF8       RAS_Ahparms
 000F:00001C1C       RAS_dh_VerifyAccess
 000F:00001C54       RAS_dh_VMLock
 000F:00001C80       RAS_dh_VMUnlock
 000F:00001CBC       RAS_dh_VMAlloc
 000F:00001CE4       RAS_EAXparms
 000F:00001CE4       RAS_dh_OpenEventSem
 000F:00001CE4       RAS_dh_VMFree
 000F:00001CE4       RAS_dh_PostEventSem
 000F:00001CE4       RAS_dh_FreeCtxHook
 000F:00001CE4       RAS_dh_CloseEventSem
 000F:00001D04       RAS_EAXECXDHSIparms
 000F:00001D04       RAS_dh_PhysToGDTSel
 000F:00001D3C       RAS_dh_VMProcessToGlobal
 000F:00001D3C       RAS_dh_VMGlobalToProcess
 000F:00001D3C       RAS_dh_VMSetMem
 000F:00001D3C       RAS_dh_ArmCtxHook
 000F:00001D3C       RAS_EAXEBXECXparms
 000F:00001D60       RAS_dh_AllocateCtxHook
 000F:00001D60       RAS_EAXEBXparms
 000F:00001D80       RAS_EAXEDIparms
 000F:00001D80       RAS_dh_ResetEventSem
 000F:00001DB0       RAS_dh_VirtToLin
 000F:00001DB0       RAS_AxEsiparms
 000F:00001DD0       RAS_dh_LinToGDTSelector
 000F:00001DF4       RAS_dh_LinToPageList
 000F:00001E1C       RAS_dh_PageListToLin
 000F:00001E40       RAS_dh_PageListToGDTSelector
 000F:00001E7C       RAS_dh_RAS
 000F:00001E7C       RAS_NoTrace
 000F:00001E7C       RAS_Save_Message
 000F:00001E7C       RAS_dh_LogEntry
 000F:00001E7C       RAS_dh_VideoPause
 000F:00001E80       RAS_dh_ABIOSGetParms
 000F:00001EAC       RAS_dh_ROMCritSection
 000F:00001EAC       RAS_dh_EOI
 000F:00001EAC       RAS_GetDOSVar
 000F:00001EAC       RAS_Alparms
 000F:00001ED0       RAS_dh_RegisterBeep_post
 000F:00001ED0       RAS_dh_SetROMVector_post
 000F:00001ED0       RAS_FreePhysDM_post
 000F:00001ED0       RAS_dh_DynamicAPI_post
 000F:00001ED0       RAS_dh_YieldTC_post
 000F:00001ED0       RAS_dh_RegisterPDD_post
 000F:00001ED0       RAS_DevDone_post
 000F:00001ED0       RAS_dh_ROMCritSection_post
 000F:00001ED0       RAS_dh_ModifyPriority_post
 000F:00001ED0       RAS_Noparms_post
 000F:00001ED0       RAS_ProcRun_post
 000F:00001ED0       RAS_ProcRun2_post
 000F:00001ED0       RAS_SortRequest_post
 000F:00001ED0       RAS_SchedAddr_post
 000F:00001ED0       RAS_QueueFlush_post
 000F:00001ED0       RAS_PushRequest_post
 000F:00001ED0       RAS_dvh39_post
 000F:00001ED0       RAS_QueueInit_post
 000F:00001ED0       RAS_ProcBlock_post
 000F:00001EE4       RAS_VirtToPhysDM_post
 000F:00001EE4       RAS_CFAxBxparms_post
 000F:00001F08       RAS_CFbasedAxBxparms_post
 000F:00001F08       RAS_AllocPhysDM_post
 000F:00001F08       RAS_SegLockDM_post
 000F:00001F08       RAS_dh_SemHandle_post
 000F:00001F2C       RAS_dh_PhysToUVirt_post
 000F:00001F2C       RAS_PullRequest_post
 000F:00001F2C       RAS_AllocReqPacket_post
 000F:00001F2C       RAS_CFEsBxparms_post
 000F:00001F54       RAS_dh_RegisterTmrDD_post
 000F:00001F54       RAS_DiBxDiCxparms_post
 000F:00001F78       RAS_dh_RegisterPerfCtrs_post
 000F:00001F78       RAS_dh_MonFlush_post
 000F:00001F78       RAS_dh_Register_post
 000F:00001F78       RAS_dh_Beep_post
 000F:00001F78       RAS_AXparms_post
 000F:00001F78       RAS_dh_FreeGDTSelector_post
 000F:00001F78       RAS_dh_MonWrite_post
 000F:00001F94       RAS_dh_DeRegister_post
 000F:00001F94       RAS_dh_MonitorCreate_post
 000F:00001F94       RAS_CFAXparms_post
 000F:00001FB8       RAS_CFAlparms_post
 000F:00001FB8       RAS_QueueRead_post
 000F:00001FDC       RAS_SegUnlockDM_post
 000F:00001FDC       RAS_dh_SendEvent_post
 000F:00001FDC       RAS_dh_VerifyAccess_post
 000F:00001FDC       RAS_dh_UnPhysToVirt_post
 000F:00001FDC       RAS_PullParticular_post
 000F:00001FDC       RAS_dh_TickCount_post
 000F:00001FDC       RAS_Yield_post
 000F:00001FDC       RAS_dh_RealToProt_post
 000F:00001FDC       RAS_dh_ProtToReal_post
 000F:00001FDC       RAS_FreeReqPacket_post
 000F:00001FDC       RAS_QueueWrite_post
 000F:00001FDC       RAS_dh_PhysToVirt_post
 000F:00001FDC       RAS_dh_AttachDD_post
 000F:00001FDC       RAS_CFparms_post
 000F:00001FDC       RAS_dh_ResetTimer_post
 000F:00001FDC       RAS_dh_EOI_post
 000F:00001FDC       RAS_dh_UnSetIRQ_post
 000F:00001FDC       RAS_dh_SetIRQ_post
 000F:00001FDC       RAS_dh_SetTimer_post
 000F:00001FDC       RAS_GetDOSVar_post
 000F:00002000       RAS_dh_VMFree_post
 000F:00002000       RAS_dh_AllocateCtxHook_post
 000F:00002000       RAS_dh_LinToGDTSelector_post
 000F:00002000       RAS_dh_ArmCtxHook_post
 000F:00002000       RAS_dh_LinToPageList_post
 000F:00002000       RAS_dh_FreeCtxHook_post
 000F:00002000       RAS_dh_VMUnlock_post
 000F:00002000       RAS_EAXparms_post
 000F:00002000       RAS_dh_PageListToGDTSelector_po
 000F:00002000       RAS_dh_VMLock_post
 000F:0000202C       RAS_CFbasedEAXparms_post
 000F:0000202C       RAS_dh_VMProcessToGlobal_post
 000F:0000202C       RAS_dh_VMGlobalToProcess_post
 000F:0000202C       RAS_dh_OpenEventSem_post
 000F:0000202C       RAS_dh_VMSetMem_post
 000F:0000202C       RAS_dh_VMAlloc_post
 000F:0000202C       RAS_dh_VirtToLin_post
 000F:0000202C       RAS_dh_PageListToLin_post
 000F:0000202C       RAS_dh_CloseEventSem_post
 000F:0000202C       RAS_dh_PostEventSem_post
 000F:00002058       RAS_dh_ResetEventSem_post
 000F:00002058       RAS_CFbasedEAXEDIparms_post
 000F:00002094       RAS_dh_AllocGDTSelector_post
 000F:00002094       RAS_AXCFbasedparms_post
 000F:00002094       RAS_dh_PhysToGDTSelector_post
 000F:00002094       RAS_dh_SemClear_post
 000F:00002094       RAS_dh_RegisterStackUsage_post
 000F:00002094       RAS_dh_SemRequest_post
 000F:00002094       RAS_dh_ABIOSGetParms_post
 000F:00002094       RAS_dh_RegisterKrnlExit_post
 000F:00002094       RAS_dh_PhysToGDTSel_post
 000F:000020B8       RAS_dh_GetDescInfo_post
 000F:000020E8       RAS_dh_InternalError_post
 000F:000020E8       RAS_dh_VideoPause_post
 000F:000020E8       RAS_NoTrace_post
 000F:000020E8       RAS_dh_RAS_post
 000F:000020E8       RAS_Save_Message_post
 000F:000020E8       RAS_dh_LogEntry_post
 000F:000020EC       RAS_dh_RegisterKDD_post
 000F:000020EC       RAS_dh_RegisterFreq_post
 000F:000020EC       RAS_dh_CreateInt13VDM_post
 000F:000020EC       RAS_dh_CreateInt13VDM
 000F:000020EC       RAS_dh_ReallocSeg_post
 000F:000020EC       RAS_dh_KillProc_post
 000F:000020EC       RAS_dh_RegisterDeviceClass_post
 000F:000020EC       RAS_dh_RegisterDeviceClass
 000F:000020EC       RAS_dh_KillProc
 000F:000020EC       RAS_dvhe_post
 000F:000020EC       RAS_dh_RegisterFreq
 000F:000020EC       RAS_dh_QSysState
 000F:000020EC       RAS_dh_ReallocSeg
 000F:000020EC       RAS_dh_QSysState_post
 000F:000020EC       RAS_dh_RegisterKDD
 000F:000020EC       RASStubProc
 000F:000020EC       RAS_dvhe
 000F:000020F4       h_w_systrace
 000F:000020F6       w_systrace
 000F:000021CC       h_K_D_Systrace
 000F:000021CE       K_D_Systrace
 000F:000021EC       h_K_T_Systrace
 000F:000021EE       K_T_Systrace
 000F:00002242       h_K_F_Systrace
 000F:00002244       K_F_Systrace
 000F:00002260       h_K_S_Systrace
 000F:00002262       K_S_Systrace
 000F:0000227A       strp_common
 000F:00002914       f_K_S_Systrace
 000F:0000291C       f_K_D_Systrace
 000F:00002924       h_w_GetSTDA
 000F:00002928       f_w_GetSTDA
 000F:0000292A       w_GetSTDA
 000F:00002D50       RASDevHlpFuncDisp
 000F:00003170       h_RASPreTraceRouter
 000F:00003188       h_RASPostTraceRouter
 000F:000031A4       _EndRASLOCKCODE
 000F:000031A4       h_w_strucheck
 000F:000031A4       _StartRASSWAPCODE
 000F:000031A6       w_strucheck
 000F:000031C8       h_w_struresupdate
 000F:000031CA       w_struresupdate
 000F:0000333C       h_w_SetTraceInfo
 000F:0000333E       w_SetTraceInfo
 000F:0000335D       w_SetTraceInfoExit
 000F:000033AC       rasstru$SetEndTimeStamp
 000F:000033D8       rasstru$SuspendRasTrace
 000F:00003418       rasstru$ResumeRasTrace
 000F:000034A8       rasstru$ClearRasTrace
 000F:00003520       rasstru$TraceTilError
 000F:00003580       rasstru$TraceTilErrorOff
 000F:000035E0       rasstru$IncErrorCount
 000F:00003648       rasstru$PIDTraceOn
 000F:000036D4       h_SetOnePid
 000F:000036DC       rasstru$PIDTraceOnAll
 000F:0000378C       rasstru$PIDTraceOff
 000F:000037F4       rasstru$PIDTraceOffAll
 000F:000038B4       rasstru$WrapBufOn
 000F:00003948       rasstru$WrapBufOff
 000F:00003994       rasstru$SYSDATAOn
 000F:00003A60       rasstru$SYSDATAOff
 000F:00003B2C       rasstru$calcsysdatalen
 000F:00003BBC       rasstru$AllocSTDA
 000F:00003D0C       rasstru$FreeSTDA
 000F:00003DB4       rasstru$ProcTraceOn
 000F:00003F14       h_SetNamedPid
 000F:00003F40       rasstru$ProcTraceOff
 000F:0000404C       f_RASAttach
 000F:000040F0       f_RASSuspend
 000F:00004108       f_RASResume
 000F:00004120       f__RASQuiesce
 000F:00004184       f__RASUnQuiesce
 000F:000041F8       rasstru$SynchGSTDAOn
 000F:00004274       h_ValOnePid
 000F:00004278       rasstru$SynchGSTDAOff
 000F:000042FC       rasstru$QueuedTraceOn
 000F:0000434C       rasstru$QueuedTraceOff
 000F:00004384       rasstru$DynNoIPI
 000F:0000438C       rasstru$DynUseIPI
 000F:00004394       rasstru$h_SetRasSem
 000F:00004396       rasstru$SetRasSem
 000F:000043AC       rasstru$h_FreeRasSem
 000F:000043AE       rasstru$FreeRasSem
 000F:000043BC       _EndRASSWAPCODE
 000F:000043BC       _StartHIGHINITCODE
 000F:000043BC       InitLIDTable
 000F:00004484       InitReqPackets
 000F:00004530       h_InitDeviceRes
 000F:00004538       InitDevice
 000F:0000458C       h_RMNotifyWork
 000F:000045D0       InitDeviceMgr
 000F:0000471C       h_SetDPBRemovFlag
 000F:00004768       devphys$BuildPhysDiskTable
 000F:00004818       ReinitDDs
 000F:00004878       InitKbd
 000F:00004898       MONINIT
 000F:000048D4       BufInit
 000F:0000492C       buf$BufAlloc
 000F:00004978       buf$BufSize
 000F:00004990       buf$BufLinkUp
 000F:00004A1C       CharDevTabInit
 000F:00004A74       SetPMCharDevEntries
 000F:00004A94       chardd$TransDevName
 000F:00004AE4       h_AddRecFromDevHdr
 000F:00004AE6       AddRecFromDevHdr
 000F:00004B40       InitKernelCountryData
 000F:00004B64       InitKernelDBCS
 000F:00004BE8       DBCSTableInit
 000F:00004C10       InitCharTypeHIGH2
 000F:00004C4C       h_Install_ExtDrive
 000F:00004C84       fscInit
 000F:00004CE0       fscAdd
 000F:00004DB0       fscCheck
 000F:00004E20       InitFSCTemplate
 000F:00004EA0       InitFileSystem
 000F:00005114       f_FSD_SetSwap
 000F:0000513C       RLRInit
 000F:00005170       StrTransPathChar
 000F:00005184       NmpInit
 000F:000051F4       QueryPipe
 000F:00005214       SFTInit
 000F:00005284       VPBInit
 000F:00005300       syiConfigParse
 000F:000054C8       h_Int2Ascii
 000F:000054CC       f_Int2Ascii
 000F:000054CE       Int2Ascii
 000F:000054F4       Config_Init
 000F:00005590       Config_LinkPacket
 000F:000055D0       Config_GetToken
 000F:00005748       Config_ScanTable
 000F:0000577C       Config_CompareStrings
 000F:00005788       Config_RangeCheck
 000F:000057C0       Config_NextLine
 000F:000057CC       inicfg$Config_GetChar
 000F:000057CC       Config_GetChar
 000F:000057E4       Config_GetNumber
 000F:000057F0       Config_GetLongNumber
 000F:000057FC       Config_wNumber
 000F:00005894       Config_GetEqualSign
 000F:000058B8       Config_GetComma
 000F:000058D4       Config_GetOpenParen
 000F:000058F8       Config_GetCloseParen
 000F:0000591C       Config_GetEndOfLine
 000F:0000594C       Config_VerifyToken
 000F:0000594C       inicfg$Config_VerifyToken
 000F:00005960       Config_GetTrapdump
 000F:0000596C       Config_GetRASKData
 000F:00005978       Config_GetYesNo
 000F:00005984       Config_GetOnOff
 000F:00005990       Config_GetDosFlags
 000F:0000599C       Config_GetMemManToken
 000F:000059A8       Config_GetAbsDyn
 000F:000059B4       Config_GetCodePage
 000F:000059C4       Config_GetCountry
 000F:000059E4       Config_GetDiskThresh
 000F:000059FC       Config_GetLazyWrite
 000F:00005A08       Config_GetAutoCheck
 000F:00005A94       Config_GetRom
 000F:00005AA0       Config_GetDevType
 000F:00005AAC       Config_GetSubType
 000F:00005ACC       Config_GetStraceInit
 000F:00005AD8       Config_GetStraceEnable
 000F:00005AE4       Config_GetStraceInsert
 000F:00005AF0       Config_GetHexNumber
 000F:00005B90       Config_ProcessCommand
 000F:00005BD4       inicmd$Config_SetParmValue1
 000F:00005BDC       inicmd$Config_SetParmValue2
 000F:00005BE4       inicmd$Config_SetParmValue3
 000F:00005BEC       inicmd$Config_GetParmString
 000F:00005BF4       inicmd$Config_GetParmList
 000F:00005BFC       inicmd$Config_GetString
 000F:00005C58       inicmd$Config_CMD_AutoFail
 000F:00005C68       inicmd$Config_CMD_DLLBasing
 000F:00005C78       inicmd$Config_CMD_VME
 000F:00005C88       inicmd$Config_CMD_NWD
 000F:00005CA0       inicmd$Config_CMD_Reipl
 000F:00005CB0       inicmd$Config_CMD_PvwQSize
 000F:00005CE4       Config_CMD_Basedev
 000F:00005D3C       inicmd$Config_CMD_Break
 000F:00005D48       Config_CMD_Buffers
 000F:00005D6C       Config_CMD_Call
 000F:00005DBC       Config_CMD_CodePage
 000F:00005E48       Config_CMD_Country
 000F:00005EA8       Config_GetSizeToken
 000F:00005ECC       Config_CMD_Device_IFS
 000F:00005ECC       Config_CMD_Device
 000F:00005ED0       Config_CMD_IFS
 000F:00005F2C       Config_CMD_DevInfo
 000F:00006094       Config_CMD_DiskCache
 000F:00006314       inicmd$Config_CMD_Dump
 000F:000063F4       inicmd$Config_CMD_Dos
 000F:00006404       Config_CMD_FCBs
 000F:0000643C       Config_CMD_COPROCFake
 000F:00006450       Config_CMD_GlobalJITRegister
 000F:000064AC       Config_CMD_GlobalJITFlags
 000F:000064FC       Config_CMD_FILES
 000F:00006520       Config_CMD_LastDrive
 000F:00006554       Config_CMD_ReserveDriveLetter
 000F:00006588       Config_CMD_Protect16
 000F:00006630       Config_CMD_LibPath
 000F:00006674       Config_CMD_MaxWait
 000F:00006698       Config_CMD_MemMan
 000F:00006754       Config_CMD_Priority
 000F:00006764       Config_CMD_Prompt
 000F:00006770       Config_CMD_PrintBufSize
 000F:000067B4       Config_CMD_ProtectOnly
 000F:000067CC       Config_CMD_ProtShell
 000F:00006820       Config_CMD_PrtyIO
 000F:00006830       Config_CMD_RMSize
 000F:00006850       Config_CMD_Run
 000F:000068A0       Config_CMD_Set
 000F:000068E4       Config_CMD_Shell
 000F:00006938       Config_CMD_SwapPath
 000F:00006A08       Config_CMD_Threads
 000F:00006A30       Config_CMD_Processes
 000F:00006A54       Config_CMD_TimeSlice
 000F:00006AA4       Config_CMD_Trace
 000F:00006B64       Config_CMD_Strace
 000F:00006C74       Config_CMD_TraceBuf
 000F:00006E8C       Config_CMD_DumpProcess
 000F:00007044       Config_CMD_SuppressPopUps
 000F:0000708C       inicmd$Config_CMD_RASKData
 000F:000070BC       Config_CMD_NullCommand
 000F:000070C0       Config_CMD_InvalidCommand
 000F:000070C8       h_syiDisplayMessage
 000F:000070CA       syiDisplayMessage
 000F:000070F0       h_syiRetrieveMessage
 000F:000070F2       syiRetrieveMessage
 000F:0000716C       h_syiShowMessage
 000F:0000716E       syiShowMessage
 000F:00007188       h_SYISaveMessage
 000F:0000718C       f_SYISaveMessage
 000F:0000718E       SYISaveMessage
 000F:0000724C       f_SYISaveMessageID
 000F:0000724E       SYISaveMessageID
 000F:00007264       syiDisplaySavedMessages
 000F:000072D0       h_SYIAbort
 000F:000072D2       SYIAbort
 000F:000072F4       syiWordToDec
 000F:00007330       syiFillColor
 000F:000073B8       syiSetupPMPallete
 000F:00007460       syiEnableVideo
 000F:00007480       syiProcessLogoFile
 000F:000075C8       syiBlastLogo
 000F:000076A0       h_syiSetupForBMP
 000F:000076A4       f_syiSetupForBMP
 000F:000076A6       syiSetupForBMP
 000F:000076C8       h_syiBMPRestoreBIOSData
 000F:000076CA       syiBMPRestoreBIOSData
 000F:0000772C       f_syiBMPGetSelector
 000F:0000772E       syiBMPGetSelector
 000F:00007760       syiBMPFreeSelector
 000F:00007770       InitPRT
 000F:000077A0       InitTempBuffers
 000F:00007890       PhysToVirtInit
 000F:00007900       PhysToVirtReinit
 000F:00007968       IBMInitNMI
 000F:00007A58       InitNMI
 000F:00007A84       RASSTIP
 000F:00007BD4       InitSem
 000F:00007C20       INTMaskAllInterrupts
 000F:00007C38       h_syiABiosInit
 000F:00007C48       SYIAllocSel
 000F:00007D40       SYIFreeSel
 000F:00007D80       h_Get_Patch_Mem
 000F:00007E0C       h_SystemOwner
 000F:00007E6C       h_ABIOSPatchOwner
 000F:00007E90       strncmp
 000F:00007E9C       syiABiosProtInit
 000F:000080FC       GetSelector
 000F:00008164       EditFTT
 000F:00008190       EditFTTEntry
 000F:000081EC       InitBaseDDs
 000F:00008210       InitBaseList
 000F:00008344       InitBASEDEVs
 000F:0000848C       devlbdd$BaseDevLoad
 000F:0000856C       BaseDevInit
 000F:0000877C       BaseDevConstructCommandLine
 000F:000087C8       OrderBASEDEVs
 000F:00008868       RelinkBASEDEVs
 000F:000088C8       h_RMNotify
 000F:00008904       ToUpperEDX
 000F:00008920       h_SYIInitOS2_Part2
 000F:00008A80       syiDiscardDosHlp
 000F:00008B7C       syiInitDataStructures
 000F:00008EA8       inidin2$syiMiniFSD
 000F:00008F64       inidin2$syiCheckMemorySize
 000F:00008FBC       syiInitOS2Components
 000F:000093A0       syiInitInt13Thread
 000F:000093D0       syiInitProcess
 000F:0000960C       inidin2$f_SysInitThread3
 000F:00009660       syiSetCharDevTable
 000F:00009670       syiCreateEnvironment
 000F:000096DC       syiR0ParseEnvironmentString
 000F:00009750       syiProcExtLIBPATH
 000F:000097C8       syiDosHlpFix32
 000F:0000995C       syiReinitAdds
 000F:000099F4       syiOS2VER
 000F:00009A8C       h_w_SICG
 000F:00009AB0       sicg$sicgf0
 000F:00009AC4       sicg$sicgf1
 000F:00009ACC       sicg$sicgf2
 000F:00009B3C       sicgf3
 000F:00009BD4       sicg$sicgf4
 000F:00009C28       sicgf5
 000F:00009C90       sicg$sicgf5sub
 000F:00009CAC       sicg$sicgf6
 000F:00009CB8       sicg$sicgf7
 000F:00009DD0       sicg$sicg7realloc
 000F:00009DF4       sicg$sicg7reallocsub
 000F:00009E28       sicg$sicgf8
 000F:00009E50       sicg$sicgf9
 000F:00009E84       sicg$sicgfA
 000F:00009E90       sicg$sicgfB
 000F:00009EF8       sicg$sicgfC
 000F:00009F94       sicg$sicgfD
 000F:00009F9C       sicg$sicgfE
 000F:0000A01C       sicg$sicgf10
 000F:0000A020       sicg$sicgf11
 000F:0000A030       sicg$sicgf12
 000F:0000A064       sicg$sicgf13
 000F:0000A07C       sicg$sicgf14
 000F:0000A090       sicg$sicgf15
 000F:0000A098       sicg$sicgf16
 000F:0000A0C0       sicg$sicgf17
 000F:0000A0C4       sicg$sicgf18
 000F:0000A0E0       sicg$sicgf19
 000F:0000A0F0       sicg$sicgf1A
 000F:0000A108       sicg$sicgf1B
 000F:0000A1D8       Cluster2Sector
 000F:0000A1FC       GetDir
 000F:0000A2AC       GetFAT
 000F:0000A410       GetNextCluster
 000F:0000A44C       h_syiInitSIFS
 000F:0000A44E       syiInitSIFS
 000F:0000AB60       h_SYIOpenFile
 000F:0000AB64       f_SYIOpenFile
 000F:0000AB66       SYIOpenFile
 000F:0000AD88       ParseFilespec
 000F:0000AE28       DriveCheck
 000F:0000AE54       ReadClusters
 000F:0000AE84       h_SYIReadFile
 000F:0000AE88       f_SYIReadFile
 000F:0000AE8A       SYIReadFile
 000F:0000B018       h_syiReadAtFile
 000F:0000B01C       f_syiReadAtFile
 000F:0000B01E       syiReadAtFile
 000F:0000B344       h_SYICloseFile
 000F:0000B348       f_SYICloseFile
 000F:0000B34A       SYICloseFile
 000F:0000B370       h_syiReInitSIFS
 000F:0000B372       syiReInitSIFS
 000F:0000B374       h_syiTermSIFS
 000F:0000B376       syiTermSIFS
 000F:0000B490       ValidateCluster
 000F:0000B4A8       Check_U_ModName
 000F:0000B4D0       RsrcInit
 000F:0000B524       h_GDTAllocN
 000F:0000B526       GDTAllocN
 000F:0000B54C       SELReinitDPL
 000F:0000B614       _panicsicg
 000F:0000B638       ProcInit
 000F:0000B674       ProcDataResize
 000F:0000B758       _EndHIGHINITCODE
 000F:0000B758       _StartENDHIGH5CODE
 0010:00000000       _StartTHUNK_TEXT
 0010:00001DDC       DevWOHandle
 0010:00001DDC       _EndTHUNK_TEXT
 0010:00001DDC       _StartHIGH32CODE
 0010:00001DE4       g_CodeLockProc
 0010:00001DE9       CodeLockProc
 0010:00001EDC       g_CodeUnlockProc
 0010:00001EE1       CodeUnlockProc
 0010:00001F4C       _FSAbortVDM
 0010:00001F64       FS32IREAD
 0010:00001F70       FS32IWRITE
 0010:00001F7C       w_Big32IO
 0010:00001FEC       w_SetFileLocks
 0010:00001FF4       w_ProtectSetFileLocks
 0010:00001FFC       w_CancelFileLocks
 0010:00002004       w_realSetFileLocks
 0010:00002358       w_realProtectSetFileLocks
 0010:00002648       w_realCancelFileLocks
 0010:00002864       _SetupPhysIO
 0010:000028D8       _FigRec
 0010:00002928       _ReqListAdd_REQ
 0010:00002964       _ReqListAdd_Extent
 0010:0000299C       _ReqListAdd_SG
 0010:000029D0       _ReqListExecute
 0010:00002A0C       _ReqListAlloc
 0010:00002A38       _ReqListInit
 0010:00002A64       _ReqListLnkPtr
 0010:00002A90       _ReqList_GetNextRead
 0010:00002AC0       _ReqList_GetReadAheadData
 0010:00002AE4       _ReqList_SetNextRead
 0010:00002B20       _IsEOF
 0010:00002B54       _NextSec
 0010:00002B90       _DRead
 0010:00002BC0       _DWrite
 0010:00002BF4       _FreeDosBuffer
 0010:00002C1C       _WriteDosBuffer
 0010:00002C44       _IsDriveLocked
 0010:00002C74       _GetVIDSector
 0010:00002C94       _UpdateVID
 0010:00002D18       AllocCluster
 0010:000031E4       FreeCluster
 0010:00003238       InitVPBCacheData
 0010:00003598       Get12BitBadSectors
 0010:000036C0       FreeVPBCacheData
 0010:0000371C       _IsRBABad
 0010:00003798       _IsRBAInSysArea
 0010:000037C4       _IsRBAForFAT
 0010:000037F4       _CheckFATSector
 0010:0000387C       _FreeReqList
 0010:000038A0       _SetupForIO
 0010:000038D8       _FATReadInit
 0010:00003900       _FindNonChar
 0010:00003934       _BufFillFromBitMap
 0010:0000399C       _SaveFatTCBInfo
 0010:000039B8       _RestoreFatTCBInfo
 0010:000039D4       _AllocateClus
 0010:00003A20       _FreeCluster
 0010:00003A50       _FindClusInfo
 0010:00003B1C       _ReLinkClus
 0010:00003BAC       _RBAToClus
 0010:00003C10       _GetDriveLetterFromhVPB
 0010:00003C38       _GetBuf
 0010:00003CE0       _ReleaseBuf
 0010:00003CF8       _HotFixHardError
 0010:00003D44       _GetClusterSize
 0010:00003D78       CacheFlush
 0010:00003DA8       _fReqListFree
 0010:00003E04       _IOGetDiskSpaceInfo
 0010:00003EFC       g_MFT_Enter
 0010:00003F01       MFT_Enter
 0010:00004078       g_FNM
 0010:0000407D       FNM
 0010:000040DC       g_RMN
 0010:000040E1       RMN
 0010:0000415C       MFT_KeyLen
 0010:00004184       MFT_KeyAlloc
 0010:00004244       MFT_KeyFree
 0010:000042B8       MFT_GetKey
 0010:000042E8       g_FreeMFTSem
 0010:000042ED       FreeMFTSem
 0010:00004310       g_GetMFTSem
 0010:00004315       GetMFTSem
 0010:00004360       VDMINT24HANDLER
 0010:00004450       _PathCharTrans
 0010:00004498       _IOGetMediaInfo
 0010:00004530       _IOSftOpen
 0010:000047F4       _IOSftReadAt
 0010:000047FB       _IOSftWriteAt
 0010:00004998       IO_Read
 0010:000049A0       IO_Write
 0010:000049A8       _IOSftClose
 0010:00004A40       _IOSftTransPath
 0010:00004B18       g_ioSaveTCB
 0010:00004B1D       ioSaveTCB
 0010:00004B40       g_ioRestoreTCB
 0010:00004B45       ioRestoreTCB
 0010:00004B68       _SftFileSize
 0010:00004BE4       _Canon
 0010:00004C20       _SDSetVDMFlags
 0010:00004C4C       _SDFlushVDMSFTs
 0010:00004CBC       CADHandler
 0010:00004CDC       Sec32Router
 0010:00004CEC       _SecHook32CG
 0010:00004D1C       _SecHook16CG
 0010:00004D4C       TurnOffPageProtection
 0010:00004D64       TurnOnPageProtection
 0010:00004D7C       g_SecDevRoute
 0010:00004E78       _ChgFilePtr
 0010:00004F1C       _SFTFromSFN
 0010:00004F50       _FindNextHlp
 0010:00004F88       _FindNextHlp2
 0010:00004FE8       _VMGetTempBuffer
 0010:000050CC       _vmTempBuffToSelOff
 0010:000050F0       _VMFreeTempBuffer
 0010:00005198       _AllocBit
 0010:000051F8       _AllocBitGroup
 0010:0000527C       _FreeBit
 0010:0000529C       _HighestBit
 0010:00005304       _strncmp
 0010:00005330       _xchg
 0010:00005340       _selGetLDTAddr
 0010:000053B4       _SELAllocGDT
 0010:000054DC       _selFreeGDTSub
 0010:00005560       _SELFreeGDT
 0010:00005574       selmgra$selCheckFreeList
 0010:000055CC       selmgra$selConvertToExpandUp
 0010:00005614       selmgra$selConvertToExpandDown
 0010:00005630       _SELVirtToLin
 0010:00005698       _SELGetDescInfo
 0010:00005760       _SELSetDescInfo
 0010:000058D0       _selEachDesc
 0010:000059F4       selmgra$selGate
 0010:00005A2C       _selSwitchLDTsub
 0010:00005A54       selmgra$selGDTall
 0010:00005AA0       selmgra$selGDTlimit
 0010:00005AF0       selmgra$selSDMatch
 0010:00005B38       _SELConvertToSelOff
 0010:00005B58       _SELConvertToSelector
 0010:00005C00       _SELConvertToLaddr
 0010:00005C18       _SELConvertToLinear
 0010:00005C58       _SELSelToLa
 0010:00005CB4       tci_Fault0
 0010:00005CD8       _SELLaToSel
 0010:00005DCA       tci_Fault1
 0010:00005E08       g_PhysToUVirt
 0010:00005FF4       _TranslateRAS
 0010:000060B8       _apdemSVC
 0010:00006214       DEMDispatch
 0010:000062F8       demSVCNOP
 0010:000062FC       demVDMInt13Request
 0010:00006308       demVDMInt10Request
 0010:00006314       EM86DispatchSTIHooks
 0010:00006360       VDHRESETEVENTSEM
 0010:0000636C       VDHPOSTEVENTSEM
 0010:00006378       VDHQUERYSEM
 0010:00006388       VDHVIEWHANDLE
 0010:00006414       VDHJFNFROMHANDLE
 0010:00006484       VDHReleaseNPX
 0010:0000648C       VDHNPXRegisterVDD
 0010:000064A4       VDHNPXClearBusy
 0010:000064B8       VDHNPXReset
 0010:000064CC       PROIntProfile
 0010:0000654C       KMEnterKmodeThunkSEF
 0010:000065E0       KMEnterKmodeSEF
 0010:00006654       KMEnterKmodePASCALSEF
 0010:000066C8       KMExitKmodeSEF
 0010:0000674C       KMExitKmodePASCALSEF
 0010:000067C8       KMExitKmodeSEF0
 0010:000067D0       KMExitKmodeSEF4
 0010:000067DC       KMExitKmodeSEF8
 0010:000067E8       KMExitKmodeSEF12
 0010:000067F4       KMExitKmodeSEF16
 0010:00006800       KMExitKmodeSEF20
 0010:0000680C       KMExitKmodeSEF24
 0010:00006818       KMExitKmodeSEF28
 0010:00006824       KMExitKmodeSEF32
 0010:00006830       KMExitKmodeSEF36
 0010:0000683C       KMExitKmodePASCALSEF0
 0010:00006844       KMExitKmodePASCALSEF4
 0010:00006850       KMExitKmodePASCALSEF8
 0010:0000685C       KMExitKmodePASCALSEF12
 0010:00006868       KMExitKmodePASCALSEF16
 0010:00006874       KMExitKmodePASCALSEF20
 0010:00006880       KMExitKmodePASCALSEF24
 0010:0000688C       KMExitKmodePASCALSEF28
 0010:00006898       KMExitKmodePASCALSEF32
 0010:000068A4       KMExitKmodePASCALSEF36
 0010:000068B0       _afpfnReturnSEF
 0010:00006900       _afpfnReturnPASCALSEF
 0010:00006970       g_KMEnterKmodeEvents
 0010:00006975       KMEnterKmodeEvents
 0010:000069EC       g_KMExitKmodeEvents
 0010:000069F1       KMExitKmodeEvents
 0010:00006AEC       kmodea$kmCheckForceFlags
 0010:00006BC4       kmCheckSigHandler
 0010:00006CB4       kmodea$kmDispatchLocalContextHo
 0010:00006CC4       _kmCTXHDaemon
 0010:00006CDC       kmodea$kmDispatchGlobalContextH
 0010:00006CF4       KMDispatchHook
 0010:00006DA0       KMARMHOOK
 0010:00006DE4       muxsem$g_semRamGetMuxSemIDSub
 0010:00006E18       _semEventWakeMuxWait
 0010:00006E38       SwitchNPX
 0010:00006F0C       SaveNPX
 0010:00006F74       WaitNPX
 0010:00006F8C       g__ReleaseNPX
 0010:00006F91       _ReleaseNPX
 0010:00006FFC       g_NPX_Interrupt_Handler
 0010:00007058       NPX_Error_Handler
 0010:000070E8       Con_CS_IP
 0010:0000710C       NPXRegisterVDD
 0010:00007148       NPXClearBusy
 0010:00007150       NPXReset
 0010:00007170       _NPXReadContext
 0010:0000720C       _NPXWriteContext
 0010:00007380       B1NPX_Errata_02
 0010:000078A8       g_B1NPX_Errata_17
 0010:000079E4       B1NPX_Errata_17HookFn
 0010:00007A10       forceEMHandler
 0010:00007A50       _schMapPid
 0010:00007A6C       _schMapTid
 0010:00007A88       _schForceExitCritSec
 0010:00007ABC       _schSetKbdLocus
 0010:00007BA4       _schSetThreadKbdLocus
 0010:00007BD4       _schSetScreenGroupFgnd
 0010:00007C40       _schSetProcessFgnd
 0010:00007C88       _schFgndBoost
 0010:00007CC0       _schFgndDiskIO
 0010:00007CF0       _schSetProcPrty
 0010:00007D0C       _schSetThreadPrty
 0010:00007D2C       _SuBuff386
 0010:00007D74       _FuBuff386
 0010:00007DB1       setfetum$SuFuBuff386
 0010:00007E8C       SIGPOSTPENDINGHOOK
 0010:00007E9C       VR32IExitMustComplete
 0010:00007ED0       _SIGPsig
 0010:00008068       Sig_Proc
 0010:0000814C       _SigResetSigFocus
 0010:0000816C       _SigReset
 0010:000081F0       _SigResetAPTERM
 0010:00008224       _SIGApiSendSignalException
 0010:00008258       TIMSEMHANDLE
 0010:000082B0       TIMSEMCLEAR
 0010:000082D8       TIMGSETHTIMER
 0010:00008354       _DHContextHook
 0010:00008384       _SoftTraceGetTimeStamp
 0010:00008394       _SoftTraceGetStackULONG
 0010:000083D0       _UpdatePerformanceMEC
 0010:00008458       _StraceBufToDumpFmt
 0010:00008464       _KIEnable
 0010:000084B4       _KIEnableInit
 0010:00008554       _KIDisable
 0010:000085B8       _KILatch
 0010:0000860C       _StartCPURating
 0010:00008638       ReadSysCPUClocks
 0010:0000865C       ComputeCPURate
 0010:000086C0       _GetSyncTimeStamp_up
 0010:000086D8       _ictrace_on
 0010:0000882C       monitor_on
 0010:0000892F       init_loop_done
 0010:000089A0       ictrace_hotkey
 0010:00008A68       _ictrace_off
 0010:00008AE4       _ictrace_reset
 0010:00008AFC       ictrace_trapcount_handler
 0010:00008AFC       ictrace_count
 0010:00008B59       do_count
 0010:00008B62       delay_pause
 0010:00008B86       shared
 0010:00008B8C       ct_inst
 0010:00008BA7       do_count_loop
 0010:00008BC3       got_a_tbl
 0010:00008BCA       final_count
 0010:00008BD9       no_cachef
 0010:00008BDD       same_table
 0010:00008BE0       do_srch
 0010:00008BF2       srch_entry
 0010:00008C14       got_entry
 0010:00008C22       hint_set
 0010:00008C2E       ct_no_room
 0010:00008C3D       zero_hint
 0010:00008C43       new_tbl
 0010:00008C64       final_table_ov
 0010:00008C70       final_table
 0010:00008C7B       ft_common
 0010:00008CA4       overflow
 0010:00008CBC       find_pid
 0010:00008CC2       pid_chain
 0010:00008CC8       pid_loop
 0010:00008CD9       add_a_pid
 0010:00008CE3       got_a_pid
 0010:00008CFA       hit_pid
 0010:00008D01       set_pid
 0010:00008D0D       pid_overflow
 0010:00008D18       get_new_pid_tbl
 0010:00008D34       refill_pid_stack
 0010:00008D4F       new_seg
 0010:00008DC8       selector_to_base
 0010:00008DD2       not_v86
 0010:00008DFD       gdt_seg
 0010:00008E08       ldt_seg
 0010:00008E19       initiate_pause
 0010:00008E35       pause_now
 0010:00008E6C       simulate_inst
 0010:00008E73       decode_loop
 0010:00008E87       jmp_prefix66
 0010:00008E87       jmp_base
 0010:00008E8E       jmp_other_prefix
 0010:00008E91       jmp_iret
 0010:00008E96       jmp_popf
 0010:00008E9B       jmp_load_seg
 0010:00008EA0       suspend_ictrace
 0010:00008EBA       suspend_final
 0010:00008EC8       jmp_cli
 0010:00008EDA       enter_blkout
 0010:00008EDE       ictrace_exit
 0010:00008EF3       ictrace_fault_handler
 0010:00008F35       ictrace_irqcommon_handler
 0010:00008F9C       irq_active
 0010:00008FCC       ictrace_pgflt_handler
 0010:00009016       ictrace_postblkout_handler
 0010:00009030       ictrace_setup_handler
 0010:00009030       ictrace_flow
 0010:00009090       ictrace_trapflow_handler
 0010:000090DA       do_ictrace
 0010:000090ED       seg_done
 0010:0000910A       pid_return
 0010:0000913E       too_big
 0010:0000914A       pos_offset
 0010:0000914F       one_byte
 0010:00009154       logging_done
 0010:000091A9       suspended
 0010:00009213       log_sel_susp
 0010:0000924E       new_pid
 0010:00009270       ictrace_monitor
 0010:00009270       ictrace_monitor_handler
 0010:000092C3       ictrace_idle_handler
 0010:000092D6       ictrace_intr_end_intr_handler
 0010:000092F2       ictrace_busy_handler
 0010:00009308       ictrace_spurious_handler
 0010:00009320       do_monitor
 0010:00009365       code_32
 0010:0000936C       do_pd_ctrs
 0010:00009402       setup_next_event
 0010:0000942E       set_p6_control_reg
 0010:000094AC       mon_buffer_full
 0010:000094B3       simulate_ls
 0010:000094DF       simulate_popf
 0010:000094ED       simulate_iret
 0010:0000950F       iret_small
 0010:00009518       get_user_stack
 0010:0000953D       big_stack
 0010:00009540       ring0
 0010:00009550       _GenSTraceHook
 0010:00009874       Gen32Hook0
 0010:000098B4       Gen32Hook1
 0010:00009900       Gen32HookV32
 0010:0000995C       Gen32HookAny
 0010:00009A58       _DHookSwitch
 0010:00009A60       g_INTDHSetIRQ
 0010:00009A60       DHookAll
 0010:00009A94       g_INTSetIRQ
 0010:00009A99       INTSetIRQ
 0010:00009B80       INTSetVDMIRQ
 0010:00009BD4       g_INTDHUnSetIRQ
 0010:00009C54       INTUnsetVDMIRQ
 0010:00009CAC       int$intFreeDIRQ
 0010:00009CF0       int$intSearchDIRQ
 0010:00009D24       g_INTDHEOI
 0010:00009D40       INTEOIVDMIRQ
 0010:00009D60       INTSHUTOFFVDMIRQ
 0010:00009D80       g_INTDHSetROMVector
 0010:00009D84       g_INTDHRegisterStackUsage
 0010:00009E00       intIRQRouter
 0010:00009E1C       HookKI_intr_begin_entry
 0010:00009E2B       HookKI_intr_begin_gettmr
 0010:00009E51       phook_irq_fixup
 0010:00009E56       HookKI_intr_begin_exit
 0010:00009E56       phook_irq_resume
 0010:00009EAA       cpu_int
 0010:0000A02E       cpu_stint
 0010:0000A0F9       cpu_etint
 0010:0000A12B       HookKI_intr_end_entryintr
 0010:0000A12F       HookKI_intr_end_gettmrintr
 0010:0000A15B       phook_intr_end_intr_fixup
 0010:0000A160       phook_intr_end_intr_resume
 0010:0000A162       HookKI_intr_end_exitintr
 0010:0000A28E       int$intKernelExit
 0010:0000A2A4       PrivateStackExit
 0010:0000A2F8       intSwitchStack
 0010:0000A350       int$intShutOffIRQ
 0010:0000A374       g_num_to_object
 0010:0000A3A8       _ldrRead
 0010:0000A494       ldrGetMTESem
 0010:0000A514       ldrClrMTESem
 0010:0000A56C       _ldrAscToOrd
 0010:0000A5A0       _ldrUCaseString
 0010:0000A5D8       _ldrFindChar
 0010:0000A638       _pgEnablePaging
 0010:0000A670       _pgFlushTLB
 0010:0000A67C       _lldt
 0010:0000A6C4       _PGVerifyInfoSegs
 0010:0000A6DC       _PGSwitchContext
 0010:0000A8A0       ictrace_blkout1
 0010:0000A8CB       ictrace_blkout2
 0010:0000A921       pgSwitchRet
 0010:0000A921       phook_postblkout_fixup
 0010:0000A926       phook_postblkout_resume
 0010:0000AA0C       Block
 0010:0000AA28       Wakeup
 0010:0000AA44       _pgwTrap2FindPage
 0010:0000AAD0       _pgGetErrorLogFrame
 0010:0000AAEC       _int3
 0010:0000AAF0       _ldrProcessImports
 0010:0000AE03       _ldrRecordMTE
 0010:0000AF3C       _ldrDirtyWorkerThunk
 0010:0000AF48       _LDRGetLibName
 0010:0000AFC8       ldrGetLibNameSub
 0010:0000AFF0       ldrGetRsrcTypeName
 0010:0000B098       ldrIsBaseRsrc
 0010:0000B0CC       ldrrsrc$g_RsrcFindLocal
 0010:0000B0D1       ldrrsrc$RsrcFindLocal
 0010:0000B100       _LDRIsResource
 0010:0000B178       _vdmmEnterV86Mode
 0010:0000B1CC       _vdmmInt13SVCCode
 0010:0000B1E4       _vdmmInt10SVCCode
 0010:0000B1FC       _vdmmInt13BufferAlloc
 0010:0000B26C       _vdmmInt13BufferFree
 0010:0000B28C       _vdmmReadABIOSSelTbl
 0010:0000B304       vdmma$Int2Ascii
 0010:0000B324       vdmma$_nulroutine
 0010:0000B328       NWDHandler
 0010:0000B480       NWDEditTss
 0010:0000B588       NWDAccessTSS
 0010:0000B5AC       _tkSysFrzThwWrkr
 0010:0000B5F4       _TKTermTask
 0010:0000B610       _TKTermThread
 0010:0000B834       TCBUnlink2_StartHook
 0010:0000B840       TCBUnlink2_EndHook
 0010:0000B868       _tkCheckStackUsage
 0010:0000B8B4       g__TKSetSSBase
 0010:0000B8B9       _TKSetSSBase
 0010:0000B918       _tkStop
 0010:0000B924       _TKTestPause
 0010:0000B930       _TKGetProtTSS
 0010:0000B938       _TKsetjmp
 0010:0000B958       _TKlongjmp
 0010:0000B960       tkmisc$tkLongJmp
 0010:0000B97C       _TKCatchFault
 0010:0000B9DC       _TKClrFault
 0010:0000BA20       tkmisc$tkFaultHandler
 0010:0000BA4C       _AssertDSESFlat
 0010:0000BB23       alignesp
 0010:0000BB2C       __panicsprintf
 0010:0000BB64       __panicHIGH32
 0010:0000BB78       __panicfnHIGH32
 0010:0000BB8C       __panicfnmsgHIGH32
 0010:0000BBA0       __panic
 0010:0000BBB4       __panicfn
 0010:0000BBF2       __panicfnmsg
 0010:0000BC1A       __panicfmt
 0010:0000BC40       VR32Redir
 0010:0000BC4B       tkmisc$VR32RedirReturn
 0010:0000BC4C       _VR32ForceSystemDump
 0010:0000BCCC       tkForceSystemDump
 0010:0000BCD4       _KSEMRequestMutex
 0010:0000BDE8       _KSEMReleaseMutex
 0010:0000BE48       _KSEMQueryMutex
 0010:0000BEA0       _KSEMRequestExclusive
 0010:0000BFF4       _KSEMRequestShared
 0010:0000C11C       _KSEMRelease
 0010:0000C1B4       _KSEMCreate
 0010:0000C1CC       _KSEMInit
 0010:0000C1E0       _KSEMDestroy
 0010:0000C1EC       _KSEMQuery
 0010:0000C1FC       _KSEMAlloc
 0010:0000C218       _KSEMResetEvent
 0010:0000C224       _KSEMPostEvent
 0010:0000C230       _KSEMWaitEvent
 0010:0000C240       ksemovie
 0010:0000C253       ksemsigie
 0010:0000C266       ksemownie
 0010:0000C279       szKSEM
 0010:0000C27C       ksemAlloc
 0010:0000C2C6       ksemInit
 0010:0000C30C       ksemCreate
 0010:0000C344       ksemDestroy
 0010:0000C398       ksemResetEvent
 0010:0000C3BC       ksemPostEvent
 0010:0000C3FC       ksemWaitEvent
 0010:0000C47C       ksemRequestMutex
 0010:0000C524       ksemReleaseMutex
 0010:0000C574       ksemQuery
 0010:0000C5C4       trap00
 0010:0000C5E0       trap$ReadDR0
 0010:0000C5E4       trap$ReadDR1
 0010:0000C5E8       trap$ReadDR2
 0010:0000C5EC       trap$ReadDR3
 0010:0000C5F0       trap$UserCSEIPToLaddr
 0010:0000C5F6       trap$CSEIPToLaddr
 0010:0000C650       DR6NotBn
 0010:0000C670       trap01
 0010:0000C670       phook_trap01_fixup
 0010:0000C675       phook_trap01_resume
 0010:0000C830       trap03
 0010:0000C8BC       trap04
 0010:0000C8C8       trap05
 0010:0000C8D4       trap06
 0010:0000C96C       trap07
 0010:0000C978       trap08
 0010:0000C9BC       trap09
 0010:0000C9CC       trap0a
 0010:0000C9D4       trap0b
 0010:0000C9DC       trap0c
 0010:0000C9E4       trap0d
 0010:0000C9E6       trap$VDMDispatchOpcode
 0010:0000CCA0       trap0e
 0010:0000CCA0       phook_trap0e_fixup
 0010:0000CCA5       phook_trap0e_resume
 0010:0000CCAC       trap0f
 0010:0000CCB4       trap10
 0010:0000CCBC       trap11
 0010:0000CCC4       trap1f
 0010:0000CCCC       TRAPCommonFaultEntry
 0010:0000CCCC       trap$CommonFaultEntry
 0010:0000CCDC       phook_fault_fixup
 0010:0000CCE1       phook_fault_resume
 0010:0000CD05       trap$OS2PMFaultEntry
 0010:0000CDB1       trap$OS2PMFaultExit
 0010:0000CE1C       trap$V86FaultEntry
 0010:0000CE50       trap$VPMFaultEntry
 0010:0000CE9A       trap$VDMFaultExit
 0010:0000CF08       trap$KernelFaultEntry
 0010:0000D000       trap$UserTraceFault
 0010:0000D0C8       trap$UserBPFault
 0010:0000D158       trap$UserInvalidTSSFault
 0010:0000D208       trap$UserNPXNAFault
 0010:0000D274       trap$UserSegmentNPFault
 0010:0000D32C       trap$UserStackFault
 0010:0000D360       UserPageFault
 0010:0000D498       trap$KernelTraceFault
 0010:0000D514       trap$NMIFault
 0010:0000D854       trap$KernelInvalidTSSFault
 0010:0000D890       KernelSegmentNPFault
 0010:0000D978       SegmentNPFaultFindMTE
 0010:0000D9B8       trap$KernelGPFault
 0010:0000DA90       trap$KernelPageFault
 0010:0000DB60       trap$ProcessFatalFault
 0010:0000DB80       _TRAPProcessFatalFault
 0010:0000DC88       trap$SystemFatalFault
 0010:0000DCC0       TRAPDebugFault
 0010:0000E00C       trap$_FormatRegisters
 0010:0000E070       _UserFatalDebugBreakIn
 0010:0000E098       FormatRegDump
 0010:0000E0CC       FormatLimAccDump
 0010:0000E12C       trap$FormatControlRegs
 0010:0000E160       trap$CallGateFault
 0010:0000E218       trap$DecodeCallAddress
 0010:0000E2BC       trap$QueryOverrides
 0010:0000E328       trap$RebuildStackFrame
 0010:0000E458       _TRAPCheckExcept16Handler
 0010:0000E478       TRAPCheckExceptHandler
 0010:0000E490       _TRAPArmExcept16Handler
 0010:0000E4A0       TRAPArmExceptHandler
 0010:0000E5A0       g_Int13exit
 0010:0000E604       _TRAPGetCR0CR2
 0010:0000E620       _TRAPSetCR2
 0010:0000E630       trap$_trapQueryRegister
 0010:0000E66C       trap$_trapSetRegister
 0010:0000E69C       trapPreTrace
 0010:0000E750       XCPTFormatAndSendException
 0010:0000E773       trap$xcptSimple
 0010:0000E781       trap$xcptPanic
 0010:0000E794       trap$xcptInOp
 0010:0000E7E3       trap$xcptStackFault
 0010:0000E803       trap$xcptAccessViolation
 0010:0000E820       trap$xcptGPFault
 0010:0000E8C0       trap$xcptPageFault
 0010:0000E904       g_VR2_Ptrace
 0010:0000E9C8       _PTModifyDesc
 0010:0000E9F0       _TKTCYield
 0010:0000EA08       _TKYieldTimeslice
 0010:0000EA24       _TKResched
 0010:0000EA64       _tkSchedNextRet
 0010:0000EA6C       _TKYield
 0010:0000EA7C       _tkSchedNext
 0010:0000EAE1       HPTDispatch
 0010:0000EDA9       NTDispatch
 0010:0000EDB7       HookKI_goidle_entry
 0010:0000EDBB       HookKI_goidle_gettmr
 0010:0000EDF3       phook_idle_fixup
 0010:0000EDF8       phook_idle_resume
 0010:0000EDF8       HookKI_goidle_exit
 0010:0000EE7D       HaltInst
 0010:0000EE7D       sch20a
 0010:0000EE7E       sch20b
 0010:0000EE98       HookKI_gobusy_entry
 0010:0000EE9C       HookKI_gobusy_gettmr
 0010:0000EED4       phook_busy_fixup
 0010:0000EED9       phook_busy_resume
 0010:0000EED9       HookKI_gobusy_exit
 0010:0000F004       postSchedNext
 0010:0000F0D8       SchedNextRet
 0010:0000F0E7       SchedNextRet2
 0010:0000F158       DebugLoadSymDosFS_Stub
 0010:0000F160       _KDPEnableCVK
 0010:0000F16C       _DebugPageLoaded
 0010:0000F188       _DebugLoadSymMTE
 0010:0000F1E9       EndDebugLoadSymMTE
 0010:0000F1EC       _DebugUnLinkSymMTE
 0010:0000F24C       DebugLoadSymModule
 0010:0000F360       _DebugLoadSymV86Krnl
 0010:0000F3E0       _DebugFreeSymV86Krnl
 0010:0000F41C       _Debug_SymWinOS2
 0010:0000F76C       _Debug_ForceSymWinOS2
 0010:0000F810       dosinit$g_DebAllocMem
 0010:0000F83C       dosinit$g_DebFreeMem
 0010:0000F84C       g_KDDCEnter
 0010:0000F97C       g_KDDCExit
 0010:0000F9FC       _EndHIGH32CODE
 0010:0000F9FC       _Start_TEXT
 0010:0000F9FC       _BeepPreempt
 0010:0000FB22       _BeepTom
 0010:0000FB64       _BeepClose
 0010:0000FBB8       _FreqSet
 0010:0000FBCC       _Head
 0010:0000FBD4       _TMR32QueryTime_DW
 0010:0000FBE8       _TMR32QueryTime_CQW
 0010:0000FC34       _TMR32AddTime
 0010:0000FC80       _TMR32SubTime
 0010:0000FCC0       TMR32AddTime
 0010:0000FD04       TMR32SubTime
 0010:0000FD3C       TMR32ClrTime
 0010:0000FD44       tmr32NTimes
 0010:0000FD7C       TMR32AddNTimes
 0010:0000FDC0       TMR32SubNTimes
 0010:0000FDF8       _VR32TmrQueryFreq
 0010:0000FE4C       _VR32TmrQueryTime
 0010:0000FEBC       _ioBeginTransfer
 0010:00010001       _FAT_DOPAGEIO
 0010:000102CC       _FSTomCodeUnlock
 0010:00010300       _CodeLockHook
 0010:0001039C       _FFNWalk
 0010:000109CC       _PackGEA
 0010:00010A80       _UnpackGEA
 0010:00010BA0       _memmove
 0010:00010C58       _SetRBA_Count
 0010:00010D0D       _BufReadError
 0010:00010D6B       _BufReadComplete
 0010:00010E35       _BufReadExecute
 0010:00010E8E       _BufAddToReqList
 0010:00010F66       _BufReadPartial
 0010:000112FD       _BufCopyUserExtent
 0010:000113F2       _BufAddReadExtent
 0010:000114A2       _BufRead
 0010:000122E0       _BufAlloc
 0010:00012324       _BufFind
 0010:000123CC       _PlaceBuf
 0010:00012448       _BufWrt
 0010:00012601       _GFBWait
 0010:0001262B       _GFB
 0010:0001287C       _AddHash
 0010:00012906       _HashFind
 0010:00012947       _RemoveHash
 0010:0001297D       _BufUnlink
 0010:000129D8       _diskw_read
 0010:00012A40       _BufWritePartial
 0010:00012F12       _BufWrite
 0010:00013810       _msNow
 0010:0001381A       _LWWakeUp
 0010:0001382D       _LWForceWakeUp
 0010:00013855       _fBufWritable
 0010:000138F8       _LazyRead
 0010:00013B54       _LazyReadIODone
 0010:00013C0D       _LWAsync
 0010:00014059       _LazyWriter
 0010:00014276       _AddLW
 0010:000142F9       _BufFree
 0010:0001437C       _BufLock
 0010:000143B4       _BufWaitUnLock
 0010:000143CE       _BufUnLock
 0010:0001441C       _BufIODone
 0010:000144AD       _FLW
 0010:00014515       _BufDiscard
 0010:00014568       _BufPreWrt
 0010:000145F9       _BufPreWrt2
 0010:0001465A       _BufFlush
 0010:000146A2       _BufFlushAll
 0010:000146E2       _BufFlushAll2
 0010:00014724       _BufFlushFATDir
 0010:00014764       _BufFlushFAT
 0010:000147B4       _StartReadAhead
 0010:00014B81       _AsyncRead
 0010:00014D85       _QueueAsyncRead
 0010:00014DE8       _CCH
 0010:00014E28       _WriteHotFixData
 0010:00014EE1       _HotFix
 0010:000157F8       _PGAgeLoop
 0010:00015A64       _pgAgePt
 0010:00015E6D       _pgIllegalWrite
 0010:00015F6E       _PGMarkNP
 0010:00016090       _pgIdle
 0010:00016197       _pgAgeRate
 0010:0001621B       _pgTestSMCompress
 0010:0001639A       _pgSMFreeDF
 0010:0001644C       _pgwFree
 0010:00016727       _pgCommit
 0010:000169F6       _pgCommitFree
 0010:00016BD4       _pgShortLockCommit
 0010:00016C69       _pgShortLockCommitFree
 0010:00016CA8       _pgPinPt
 0010:00016E73       _pgPinForcePresent
 0010:000174C3       _pgUnpinPt
 0010:000175EF       _pgReleasePt
 0010:00017975       _pgDriver
 0010:00017F3C       _pgStrict
 0010:00018198       _pgDriver2
 0010:000188E0       _pgFrameToPF
 0010:00018984       _pgInsertPF
 0010:00018AE5       _pgDeletePF
 0010:00018C28       _PGPhysAvail
 0010:00018C60       _PGPhysPresent
 0010:00018C6C       _pgAllocPF
 0010:0001909B       _pgLockPF
 0010:00019448       _pgFindContig
 0010:00019682       _pgGetPF
 0010:00019971       _pgValidateContig
 0010:00019D05       _pgMovePF
 0010:0001A041       _pgFindFrame
 0010:0001A416       _pgMoveFrame
 0010:0001A7AC       _PGLock
 0010:0001AA99       _PGUnlock
 0010:0001ACA7       _pgLockTSD
 0010:0001AD4B       _pgTakeSem
 0010:0001AEB4       _pgClearSem
 0010:0001AF5C       _PGPageToPhys
 0010:0001B02E       _PGMapVirt
 0010:0001B0F3       _PGLinToPageList
 0010:0001B267       _PGPageListToLin
 0010:0001B38D       _PGPhysToHOB
 0010:0001B407       _pgPageToPte
 0010:0001B49A       _pgAliasTemp
 0010:0001B4E7       _PGMapTmpAlias
 0010:0001B59E       _PGAllocBuf
 0010:0001B909       _PGFreeBuf
 0010:0001BBBE       _PGKStackMap
 0010:0001BE09       _PGKStackRemap
 0010:0001BE55       _pgPageToPd
 0010:0001BEB4       _PGVerifyPermission
 0010:0001C0D0       _pgIsInCore
 0010:0001C16C       _PGReclaimCheck
 0010:0001C256       _PGGetDirty
 0010:0001C3E1       _qpuFindApp
 0010:0001C439       _qpuFAWorker
 0010:0001C526       _qpuGetPageInfo
 0010:0001C662       _qpuwScanPages
 0010:0001C6E4       _qpuSharedAndSize
 0010:0001C9C3       _qpuGetSize
 0010:0001CB38       _PTCreate
 0010:0001CBD3       _ptFindNode
 0010:0001CC37       _ptFindNodeStop
 0010:0001CCC4       _CountMatch
 0010:0001CCF0       _ptFirstDiff
 0010:0001CDE5       _PTInsert
 0010:0001D0EC       _PTFind
 0010:0001D19F       _PTFindFromPrefix
 0010:0001D259       _PTFindMaxPrefix
 0010:0001D381       _ptDeleteNode
 0010:0001D4D3       _PTDelete
 0010:0001D5E0       _PTDestroy
 0010:0001D5E8       _ptWalkWorker
 0010:0001D5FE       _PTWalk
 0010:0001D64A       _ptWalkNodeWorker
 0010:0001D709       _PTWalkNode
 0010:0001D745       _PTInsert_16
 0010:0001D77C       _PTFind_16
 0010:0001D7B3       _PTFindFromPrefix_16
 0010:0001D7EA       _PTFindMaxPrefix_16
 0010:0001D821       _PTDelete_16
 0010:0001D855       _ptCheckTree
 0010:0001D870       _ptCheckNode
 0010:0001D938       _SELGetOd
 0010:0001D9FF       _SELLdrDesc
 0010:0001DA3D       _SELMapVirt
 0010:0001DA9F       _SELGetSelector
 0010:0001DAEB       _SELSetAccess
 0010:0001DB74       _smSetSwapFlags
 0010:0001DBC8       _smClearSwapFlags
 0010:0001DC90       _smAllocSFT
 0010:0001DCF4       _smHardError
 0010:0001DD30       _SMPrintFatalMsg
 0010:0001DD64       _smFreeSFT
 0010:0001DDAC       _vmFreeAlias
 0010:0001DE78       _vmCheckAlias
 0010:0001DEE2       _vmIsPrivLoadOb
 0010:0001DF4B       _VMMapVDM
 0010:0001E6B5       _vmIsBusyAliasRec
 0010:0001E6C8       _vmLinkOb
 0010:0001E6EA       _VMReserve
 0010:0001E89D       _vmReserveSub
 0010:0001F1ED       _vmRecalcShrBound
 0010:0001F2ED       _vmFreeSearchUp
 0010:0001F43A       _vmFreeSearchDown
 0010:0001F57A       _vmMoveSentinelUp
 0010:0001F76E       _vmMoveSentinelDown
 0010:0001F8A6       _vmAllocTLBAdjust
 0010:0001F918       _VR32SetMem
 0010:0001FA78       _vmErrorSub
 0010:0001FA82       _VMGetOd
 0010:000202AF       _vmRecordOd
 0010:00020824       _vmEraseOd
 0010:00020B85       _vmLinkArena
 0010:00020C35       _vmUnlinkArena
 0010:00020CB0       _bmpUpdateLastBusy
 0010:00020CEA       _vmRebuildBMPFreeList
 0010:00020D19       _bmpShrink
 0010:00020E25       _BMPDestroy
 0010:00020E54       _BMPFree
 0010:00020F30       _BMPGet
 0010:0002105A       _BMPGet2
 0010:000210B2       _vmBmpGet
 0010:00021136       _bmpIsBusy
 0010:0002113E       _vmBuildBMPFreeList
 0010:000211A0       _BMPHandleMap
 0010:000211DE       _vmInitBMPObject
 0010:0002124C       _dhw_VMLock
 0010:00021335       _dhw_VMUnlock
 0010:0002137E       _dhw_VMFree
 0010:000214A8       _VMLinToPhys
 0010:000214EC       _VMVirtFree
 0010:00021789       _VMFreeMemOd
 0010:00021A31       _vmFreeMemNotifyOd
 0010:00022214       _vmFreeMemCtxtOd
 0010:00022698       _vmSetObPermOd
 0010:00022758       _VMGetLaddr
 0010:000227AF       _VMTrap2FindArena
 0010:00022814       _VMObjHandleInfo
 0010:0002296B       _VMQueryArenaAvailMem
 0010:00022ABB       _VMQueryMem
 0010:00022E09       _VMIsPrivatized
 0010:00022E88       g__LDRClearSem
 0010:00022E93       g__PGPhysAvail
 0010:00022EA0       ReserveVM
 0010:00022ED8       _vmbmScan
 0010:00022FF8       _vmRetAddr
 0010:00022FFC       _VMHandleVerify
 0010:00023070       _VMHandleMap
 0010:000230A5       _VMGetSem
 0010:00023386       _VMGetPTDAAddr
 0010:000233D0       _VMGetHandle
 0010:00023459       _VMQueryMaxAlloc
 0010:00023544       _VMSGSControl
 0010:000235BE       _VMSGSValidate
 0010:000236C6       _vmSGSAdd
 0010:000237B7       _vmSGSRemove
 0010:00023894       _vmIsBusyArBMP
 0010:000238A6       _vmIsBusyObBMP
 0010:000238B8       _vmIsBusyCoBMP
 0010:000238CA       _VMGetOwner
 0010:00023957       _VMClearSem
 0010:00023A44       _vmLinkAr
 0010:00023AAB       _vmLinkCo
 0010:00023B2A       _vmFindArCo
 0010:00023D3F       _VMSearchRef
 0010:00023EBF       _VMIsAttached
 0010:00023F06       _vmEachMapCheck
 0010:00023F43       _vmEachMapSub
 0010:00024244       _VMEachMap
 0010:000243B1       _VMScanMaps
 0010:00024628       _VMAttach
 0010:00024AD4       _VMAllocKHB
 0010:000256CE       _VMReallocKHB
 0010:00025ACB       _VMFreeKHB
 0010:00025C7F       _VMShrinkKHB
 0010:000260FD       _VMGetKHBI
 0010:000262DC       _VMMoveKHB
 0010:00026441       _vmFindKRHB
 0010:000264B6       _vmCopyKHB
 0010:0002656B       _vmPhysCheckKRHB
 0010:00026615       _vmCreateKRHB
 0010:000267E9       _vmYieldKRHB
 0010:00026908       _vmCoalesceKRHB
 0010:00026EC5       _vmGrowKRHB
 0010:00026FA9       _vmCarveKRHB
 0010:00027024       _vmRelinkFreeKRHB
 0010:0002707C       _vmInsertFreeKRHB
 0010:00027273       _vmRemoveFreeKRHB
 0010:00027407       _vmCommitSubKRHB
 0010:000274AC       _vmCommitSubAllocKRHB
 0010:00027571       _vmDecommitKRHB
 0010:000275F8       _vmFirstPKRHS
 0010:00027619       _vmSizeToPKRHS
 0010:00027651       _VMSetReadOnlyUL
 0010:00027682       _VMSetReadOnlyUS
 0010:000276B7       _VMAddReadOnlyULNew
 0010:000276E8       _vmIsValidKRH
 0010:00027E9C       _VMFlagsKH
 0010:00027EDE       _vmSetOwnerKRHB
 0010:00027F38       _vmRoundReqKRHB
 0010:00027F6E       _vmSetAttrKRHB
 0010:00027FD6       _VMGetAttrKRHB
 0010:0002801D       _VMSelKHB
 0010:00028061       _VMOwnerKHB
 0010:000280A9       _VMGetInfoKHB
 0010:000280E7       _VMValidateKHBAddress
 0010:0002811D       _VMPrintKRH
 0010:000281A0       _VMRequestSems
 0010:0002820D       _VMReleaseSems
 0010:00028250       _vmAllocKSHB
 0010:00028694       _vmReallocKSHB
 0010:000287C4       _vmFreeKSHB
 0010:00028AB6       _vmShrinkKSHB
 0010:00028B60       _vmIsValidKSH
 0010:00028CAD       _vmFindKSHB
 0010:00028D39       _vmSetupSpecialKSHB
 0010:00028E64       _SELAllocKHB
 0010:00028F3C       _SELReallocKHB
 0010:0002902B       _SELFreeKHB
 0010:00029106       _SELMoveKHB
 0010:0002920B       _SELGetKHBI
 0010:00029289       _SELValidateKHBAddress
 0010:000292D8       _pgAllocVP
 0010:00029357       _pgFreeVP
 0010:0002944A       _pgResizeVP
 0010:00029597       _pgSavePF
 0010:00029600       _pgFindPF
 0010:000296FC       _a2n_getall_mte
 0010:00029815       _a2nexe_getAllmte
 0010:00029833       _a2ngexe_mtes
 0010:00029932       _a2nshr_mtes
 0010:0002996A       _a2n_process_mte
 0010:00029BA4       VDHSETPRIORITY
 0010:00029D3A       VDHFREEZEVDM
 0010:00029D8C       VDHTHAWVDM
 0010:00029DCA       VDHISVDMFROZEN
 0010:00029DE4       VDMMKILLVDM
 0010:00029E83       VDMMVDMTERMINATING
 0010:00029EC1       PFNUNDOHMAPID
 0010:00029F3A       VDMMDISPATCHINCONTEXT
 0010:00029FE8       VDMMDISPATCHPAGEFAULT
 0010:0002A133       VDMMSTRNCPYZ
 0010:0002A160       VDMMINITMAPID
 0010:0002A1D5       VDMMMARKVDM
 0010:0002A1F0       VDMMVDMCREATED
 0010:0002A228       VDHGETERROR
 0010:0002A25C       VDHSETERROR
 0010:0002A295       VDHHANDLEFROMSGID
 0010:0002A2C7       VDHENUMERATEVDMS
 0010:0002A300       VDHQUERYLIN
 0010:0002A340       VDHQUERYSYSVALUE
 0010:0002A436       GETVDMHANDLE
 0010:0002A49F       VDHDEVBEEP
 0010:0002A4C4       VDHARMTIMERHOOK
 0010:0002A62F       VDHDISARMTIMERHOOK
 0010:0002A6FD       VDMMPROCTICK
 0010:0002A88C       _VDMInt13Request
 0010:0002A957       VDMINT13TMRTICK
 0010:0002A97D       VDMINT13IRQREQUEST
 0010:0002A9D8       VDMINT13IRQSIMULATE
 0010:0002AA63       _VDMInt13IRQDone
 0010:0002AAC4       _VDMINT10CreateMiniVDM
 0010:0002AB7F       _VDMINT10CreateMiniVDMSub
 0010:0002AFA1       _VDMINT10IssueRequest
 0010:0002B211       _VDMINT10DestroyMiniVDM
 0010:0002B35B       _VDMInt10DispatchRequest
 0010:0002B38C       _VDMInt10Request
 0010:0002B491       _VDMINT10ThawRequest
 0010:0002B4C8       DOS32ALIASMEM
 0010:0002B4D0       preDOS32ALIASMEM
 0010:0002B4E1       postDOS32ALIASMEM
 0010:0002B4E8       DOS32ALIASPERFCTRS
 0010:0002B4F0       preDOS32ALIASPERFCTRS
 0010:0002B501       postDOS32ALIASPERFCTRS
 0010:0002B508       DOS32ALLOCMEM
 0010:0002B510       preDOS32ALLOCMEM
 0010:0002B521       postDOS32ALLOCMEM
 0010:0002B528       DOS32ALLOCPROTECTEDMEM
 0010:0002B530       preDOS32ALLOCPROTECTEDMEM
 0010:0002B541       postDOS32ALLOCPROTECTEDMEM
 0010:0002B548       DOS32ALLOCSHAREDMEM
 0010:0002B550       preDOS32ALLOCSHAREDMEM
 0010:0002B561       postDOS32ALLOCSHAREDMEM
 0010:0002B568       DOS32CANCELLOCKREQUEST
 0010:0002B570       preDOS32CANCELLOCKREQUEST
 0010:0002B581       postDOS32CANCELLOCKREQUEST
 0010:0002B588       DOS32CLOSEVDD
 0010:0002B590       preDOS32CLOSEVDD
 0010:0002B5A1       postDOS32CLOSEVDD
 0010:0002B5A8       DOS32CONFIGUREPERF
 0010:0002B5B0       preDOS32CONFIGUREPERF
 0010:0002B5C1       postDOS32CONFIGUREPERF
 0010:0002B5C8       DOS32CREATETHREAD
 0010:0002B5D0       preDOS32CREATETHREAD
 0010:0002B5E1       postDOS32CREATETHREAD
 0010:0002B5E8       DOS32KILLTHREAD
 0010:0002B5F0       preDOS32KILLTHREAD
 0010:0002B601       postDOS32KILLTHREAD
 0010:0002B608       DOSCREATETHREAD
 0010:0002B610       preDOSCREATETHREAD
 0010:0002B621       postDOSCREATETHREAD
 0010:0002B628       DOSCREATEVDM
 0010:0002B630       preDOSCREATEVDM
 0010:0002B641       postDOSCREATEVDM
 0010:0002B648       DOS32DECONPERF
 0010:0002B650       preDOS32DECONPERF
 0010:0002B661       postDOS32DECONPERF
 0010:0002B668       DOS32EXCEPTIONCALLBACK
 0010:0002B670       preDOS32EXCEPTIONCALLBACK
 0010:0002B681       postDOS32EXCEPTIONCALLBACK
 0010:0002B688       DOS32DEBUG
 0010:0002B690       preDOS32DEBUG
 0010:0002B6A1       postDOS32DEBUG
 0010:0002B6A8       DOS32DYNAMICTRACE
 0010:0002B6B0       preDOS32DYNAMICTRACE
 0010:0002B6C1       postDOS32DYNAMICTRACE
 0010:0002B6C8       DOSEXIT
 0010:0002B6D0       preDOSEXIT
 0010:0002B6DE       postDOSEXIT
 0010:0002B6E4       DOSEXITLIST
 0010:0002B6F4       preDOSEXITLIST
 0010:0002B702       postDOSEXITLIST
 0010:0002B708       DOS32EXITLIST
 0010:0002B710       preDOS32EXITLIST
 0010:0002B721       postDOS32EXITLIST
 0010:0002B728       DOS32FREEMEM
 0010:0002B730       preDOS32FREEMEM
 0010:0002B741       postDOS32FREEMEM
 0010:0002B748       DOSFREEMODULE
 0010:0002B758       preDOSFREEMODULE
 0010:0002B766       postDOSFREEMODULE
 0010:0002B76C       DOS32FREERESOURCE
 0010:0002B774       preDOS32FREERESOURCE
 0010:0002B785       postDOS32FREERESOURCE
 0010:0002B78C       DOS32GETNAMEDSHAREDMEM
 0010:0002B794       preDOS32GETNAMEDSHAREDMEM
 0010:0002B7A5       postDOS32GETNAMEDSHAREDMEM
 0010:0002B7AC       DOS32QUERYPROCADDR
 0010:0002B7B4       preDOS32QUERYPROCADDR
 0010:0002B7C5       postDOS32QUERYPROCADDR
 0010:0002B7CC       DOS32GETRESOURCE
 0010:0002B7D4       preDOS32GETRESOURCE
 0010:0002B7E5       postDOS32GETRESOURCE
 0010:0002B7EC       DOS32QUERYRESOURCESIZE
 0010:0002B7F4       preDOS32QUERYRESOURCESIZE
 0010:0002B805       postDOS32QUERYRESOURCESIZE
 0010:0002B80C       DOS32INITIALIZEPORTHOLE
 0010:0002B814       preDOS32INITIALIZEPORTHOLE
 0010:0002B825       postDOS32INITIALIZEPORTHOLE
 0010:0002B82C       DOS32QUERYHEADERINFO
 0010:0002B834       preDOS32QUERYHEADERINFO
 0010:0002B845       postDOS32QUERYHEADERINFO
 0010:0002B84C       DOS32QUERYPROCTYPE
 0010:0002B854       preDOS32QUERYPROCTYPE
 0010:0002B865       postDOS32QUERYPROCTYPE
 0010:0002B86C       DOS32GETSHAREDMEM
 0010:0002B874       preDOS32GETSHAREDMEM
 0010:0002B885       postDOS32GETSHAREDMEM
 0010:0002B88C       DOS32GIVESHAREDMEM
 0010:0002B894       preDOS32GIVESHAREDMEM
 0010:0002B8A5       postDOS32GIVESHAREDMEM
 0010:0002B8AC       DOS32OPENVDD
 0010:0002B8B4       preDOS32OPENVDD
 0010:0002B8C5       postDOS32OPENVDD
 0010:0002B8CC       DOS32QUERYDOSPROPERTY
 0010:0002B8D4       preDOS32QUERYDOSPROPERTY
 0010:0002B8E5       postDOS32QUERYDOSPROPERTY
 0010:0002B8EC       DOS32SETDOSPROPERTY
 0010:0002B8F4       preDOS32SETDOSPROPERTY
 0010:0002B905       postDOS32SETDOSPROPERTY
 0010:0002B90C       DOS32STARTTIMER
 0010:0002B914       preDOS32STARTTIMER
 0010:0002B925       postDOS32STARTTIMER
 0010:0002B92C       DOS32STOPTIMER
 0010:0002B934       preDOS32STOPTIMER
 0010:0002B945       postDOS32STOPTIMER
 0010:0002B94C       DOS32ASYNCTIMER
 0010:0002B954       preDOS32ASYNCTIMER
 0010:0002B965       postDOS32ASYNCTIMER
 0010:0002B96C       DOS32ISTARTTIMER
 0010:0002B974       preDOS32ISTARTTIMER
 0010:0002B985       postDOS32ISTARTTIMER
 0010:0002B98C       DOS32IASYNCTIMER
 0010:0002B994       preDOS32IASYNCTIMER
 0010:0002B9A5       postDOS32IASYNCTIMER
 0010:0002B9AC       DOS32SETFILELOCKS
 0010:0002B9B4       preDOS32SETFILELOCKS
 0010:0002B9C5       postDOS32SETFILELOCKS
 0010:0002B9CC       DOS32PROTECTSETFILELOCKS
 0010:0002B9D4       preDOS32PROTECTSETFILELOCKS
 0010:0002B9E5       postDOS32PROTECTSETFILELOCKS
 0010:0002B9EC       DOS32PROFILE
 0010:0002B9F4       preDOS32PROFILE
 0010:0002BA05       postDOS32PROFILE
 0010:0002BA0C       DOS32QUERYMEM
 0010:0002BA14       preDOS32QUERYMEM
 0010:0002BA25       postDOS32QUERYMEM
 0010:0002BA2C       DOS32QUERYMEMSTATE
 0010:0002BA34       preDOS32QUERYMEMSTATE
 0010:0002BA45       postDOS32QUERYMEMSTATE
 0010:0002BA4C       DOS32QUERYSYSINFO
 0010:0002BA54       preDOS32QUERYSYSINFO
 0010:0002BA65       postDOS32QUERYSYSINFO
 0010:0002BA6C       DOSQUERYRASINFO
 0010:0002BA74       preDOSQUERYRASINFO
 0010:0002BA85       postDOSQUERYRASINFO
 0010:0002BA8C       DOS32QUERYSYSSTATE
 0010:0002BA94       preDOS32QUERYSYSSTATE
 0010:0002BAA5       postDOS32QUERYSYSSTATE
 0010:0002BAAC       DOS32REGISTERPERFCTRS
 0010:0002BAB4       preDOS32REGISTERPERFCTRS
 0010:0002BAC5       postDOS32REGISTERPERFCTRS
 0010:0002BACC       DOSRESUMETHREAD
 0010:0002BADC       preDOSRESUMETHREAD
 0010:0002BAEA       postDOSRESUMETHREAD
 0010:0002BAF0       DOS32REQUESTVDD
 0010:0002BAF8       preDOS32REQUESTVDD
 0010:0002BB09       postDOS32REQUESTVDD
 0010:0002BB10       DOS32SETMEM
 0010:0002BB18       preDOS32SETMEM
 0010:0002BB29       postDOS32SETMEM
 0010:0002BB30       DOSSLEEP
 0010:0002BB38       preDOSSLEEP
 0010:0002BB46       postDOSSLEEP
 0010:0002BB4C       DOSSUSPENDTHREAD
 0010:0002BB5C       preDOSSUSPENDTHREAD
 0010:0002BB6A       postDOSSUSPENDTHREAD
 0010:0002BB70       DOS32TMRQUERYFREQ
 0010:0002BB78       preDOS32TMRQUERYFREQ
 0010:0002BB89       postDOS32TMRQUERYFREQ
 0010:0002BB90       DOS32TMRQUERYTIME
 0010:0002BB98       preDOS32TMRQUERYTIME
 0010:0002BBA9       postDOS32TMRQUERYTIME
 0010:0002BBB0       DOS32CREATEEVENTSEM
 0010:0002BBB8       preDOS32CREATEEVENTSEM
 0010:0002BBC9       postDOS32CREATEEVENTSEM
 0010:0002BBD0       DOS32OPENEVENTSEM
 0010:0002BBD8       preDOS32OPENEVENTSEM
 0010:0002BBE9       postDOS32OPENEVENTSEM
 0010:0002BBF0       DOS32CLOSEEVENTSEM
 0010:0002BBF8       preDOS32CLOSEEVENTSEM
 0010:0002BC09       postDOS32CLOSEEVENTSEM
 0010:0002BC10       DOS32RESETEVENTSEM
 0010:0002BC18       preDOS32RESETEVENTSEM
 0010:0002BC29       postDOS32RESETEVENTSEM
 0010:0002BC30       DOS32POSTEVENTSEM
 0010:0002BC38       preDOS32POSTEVENTSEM
 0010:0002BC49       postDOS32POSTEVENTSEM
 0010:0002BC50       DOS32WAITEVENTSEM
 0010:0002BC58       preDOS32WAITEVENTSEM
 0010:0002BC69       postDOS32WAITEVENTSEM
 0010:0002BC70       DOS32QUERYEVENTSEM
 0010:0002BC78       preDOS32QUERYEVENTSEM
 0010:0002BC89       postDOS32QUERYEVENTSEM
 0010:0002BC90       DOS32CREATEMUTEXSEM
 0010:0002BC98       preDOS32CREATEMUTEXSEM
 0010:0002BCA9       postDOS32CREATEMUTEXSEM
 0010:0002BCB0       DOS32OPENMUTEXSEM
 0010:0002BCB8       preDOS32OPENMUTEXSEM
 0010:0002BCC9       postDOS32OPENMUTEXSEM
 0010:0002BCD0       DOS32CLOSEMUTEXSEM
 0010:0002BCD8       preDOS32CLOSEMUTEXSEM
 0010:0002BCE9       postDOS32CLOSEMUTEXSEM
 0010:0002BCF0       DOS32REQUESTMUTEXSEM
 0010:0002BCF4       preDOS32REQUESTMUTEXSEM
 0010:0002BD3D       postDOS32REQUESTMUTEXSEM
 0010:0002BD54       DOS32RELEASEMUTEXSEM
 0010:0002BD58       preDOS32RELEASEMUTEXSEM
 0010:0002BD9D       postDOS32RELEASEMUTEXSEM
 0010:0002BDB4       DOS32QUERYMUTEXSEM
 0010:0002BDBC       preDOS32QUERYMUTEXSEM
 0010:0002BDCD       postDOS32QUERYMUTEXSEM
 0010:0002BDD4       DOS32CREATEMUXWAITSEM
 0010:0002BDDC       preDOS32CREATEMUXWAITSEM
 0010:0002BDED       postDOS32CREATEMUXWAITSEM
 0010:0002BDF4       DOS32OPENMUXWAITSEM
 0010:0002BDFC       preDOS32OPENMUXWAITSEM
 0010:0002BE0D       postDOS32OPENMUXWAITSEM
 0010:0002BE14       DOS32CLOSEMUXWAITSEM
 0010:0002BE1C       preDOS32CLOSEMUXWAITSEM
 0010:0002BE2D       postDOS32CLOSEMUXWAITSEM
 0010:0002BE34       DOS32WAITMUXWAITSEM
 0010:0002BE3C       preDOS32WAITMUXWAITSEM
 0010:0002BE4D       postDOS32WAITMUXWAITSEM
 0010:0002BE54       DOS32ADDMUXWAITSEM
 0010:0002BE5C       preDOS32ADDMUXWAITSEM
 0010:0002BE6D       postDOS32ADDMUXWAITSEM
 0010:0002BE74       DOS32DELETEMUXWAITSEM
 0010:0002BE7C       preDOS32DELETEMUXWAITSEM
 0010:0002BE8D       postDOS32DELETEMUXWAITSEM
 0010:0002BE94       DOS32QUERYMUXWAITSEM
 0010:0002BE9C       preDOS32QUERYMUXWAITSEM
 0010:0002BEAD       postDOS32QUERYMUXWAITSEM
 0010:0002BEB4       DOS32PMPOSTEVENTSEM
 0010:0002BEBC       preDOS32PMPOSTEVENTSEM
 0010:0002BECD       postDOS32PMPOSTEVENTSEM
 0010:0002BED4       DOS32PMWAITEVENTSEM
 0010:0002BEDC       preDOS32PMWAITEVENTSEM
 0010:0002BEED       postDOS32PMWAITEVENTSEM
 0010:0002BEF4       DOS32PMWAITMUXWAITSEM
 0010:0002BEFC       preDOS32PMWAITMUXWAITSEM
 0010:0002BF0D       postDOS32PMWAITMUXWAITSEM
 0010:0002BF14       DOS32PMREQUESTMUTEXSEM
 0010:0002BF78       DOS32PM16SEMCHK
 0010:0002BF80       preDOS32PM16SEMCHK
 0010:0002BF91       postDOS32PM16SEMCHK
 0010:0002BF98       DOS32PM16SEMRST
 0010:0002BFA0       preDOS32PM16SEMRST
 0010:0002BFB1       postDOS32PM16SEMRST
 0010:0002BFB8       DOS32WAITTHREAD
 0010:0002BFC0       preDOS32WAITTHREAD
 0010:0002BFD1       postDOS32WAITTHREAD
 0010:0002BFD8       DOS32QUERYPAGEUSAGE
 0010:0002BFE0       preDOS32QUERYPAGEUSAGE
 0010:0002BFF1       postDOS32QUERYPAGEUSAGE
 0010:0002BFF8       DOSQUERYMODFROMCS
 0010:0002C000       preDOSQUERYMODFROMCS
 0010:0002C011       postDOSQUERYMODFROMCS
 0010:0002C018       DOS32QUERYMODFROMEIP
 0010:0002C020       preDOS32QUERYMODFROMEIP
 0010:0002C031       postDOS32QUERYMODFROMEIP
 0010:0002C038       DOS32QUERYABIOSSUPPORT
 0010:0002C040       preDOS32QUERYABIOSSUPPORT
 0010:0002C051       postDOS32QUERYABIOSSUPPORT
 0010:0002C058       DOSLDRDIRTYWORKER
 0010:0002C060       preDOSLDRDIRTYWORKER
 0010:0002C071       postDOSLDRDIRTYWORKER
 0010:0002C078       DOSLIBINIT
 0010:0002C080       preDOSLIBINIT
 0010:0002C08E       postDOSLIBINIT
 0010:0002C094       DOS32DLLTERM
 0010:0002C09C       preDOS32DLLTERM
 0010:0002C0AD       postDOS32DLLTERM
 0010:0002C0B4       DOS32IREAD
 0010:0002C0BC       preDOS32IREAD
 0010:0002C0CD       postDOS32IREAD
 0010:0002C0D4       DOS32IWRITE
 0010:0002C0DC       preDOS32IWRITE
 0010:0002C0ED       postDOS32IWRITE
 0010:0002C0F4       DOS32IPROTECTREAD
 0010:0002C0FC       preDOS32IPROTECTREAD
 0010:0002C10D       postDOS32IPROTECTREAD
 0010:0002C114       DOS32IPROTECTWRITE
 0010:0002C11C       preDOS32IPROTECTWRITE
 0010:0002C12D       postDOS32IPROTECTWRITE
 0010:0002C134       DosRedir
 0010:0002C13C       preDosRedir
 0010:0002C14A       postDosRedir
 0010:0002C150       DOS32SETSIGNALEXCEPTIONFOC
 0010:0002C158       preDOS32SETSIGNALEXCEPTIONFOC
 0010:0002C169       postDOS32SETSIGNALEXCEPTIONFOC
 0010:0002C170       DOS32SENDSIGNALEXCEPTION
 0010:0002C178       preDOS32SENDSIGNALEXCEPTION
 0010:0002C189       postDOS32SENDSIGNALEXCEPTION
 0010:0002C190       DOS32IEXITMUSTCOMPLETE
 0010:0002C198       preDOS32IEXITMUSTCOMPLETE
 0010:0002C1A9       postDOS32IEXITMUSTCOMPLETE
 0010:0002C1B0       DOS32ICACHEMODULE
 0010:0002C1B8       preDOS32ICACHEMODULE
 0010:0002C1C9       postDOS32ICACHEMODULE
 0010:0002C1D0       DOS32FORCESYSTEMDUMP
 0010:0002C1D8       preDOS32FORCESYSTEMDUMP
 0010:0002C1E9       postDOS32FORCESYSTEMDUMP
 0010:0002C1F0       DOS32IRAISEEXCEPTION
 0010:0002C1F8       preDOS32IRAISEEXCEPTION
 0010:0002C209       postDOS32IRAISEEXCEPTION
 0010:0002C210       DOS32ACKNOWLEDGESIGNALEXC
 0010:0002C218       preDOS32ACKNOWLEDGESIGNALEXC
 0010:0002C229       postDOS32ACKNOWLEDGESIGNALEXC
 0010:0002C230       DOS32IMONWRITE
 0010:0002C238       preDOS32IMONWRITE
 0010:0002C249       postDOS32IMONWRITE
 0010:0002C250       DOS32IMONREAD
 0010:0002C258       preDOS32IMONREAD
 0010:0002C269       postDOS32IMONREAD
 0010:0002C270       DOS32DUMPPROCESS
 0010:0002C278       preDOS32DUMPPROCESS
 0010:0002C289       postDOS32DUMPPROCESS
 0010:0002C290       DOS32SUPPRESSPOPUPS
 0010:0002C298       preDOS32SUPPRESSPOPUPS
 0010:0002C2A9       postDOS32SUPPRESSPOPUPS
 0010:0002C2B0       DOS32ALLOCTHREADLOCALMEMORY
 0010:0002C2B8       preDOS32ALLOCTHREADLOCALMEMORY
 0010:0002C2C9       postDOS32ALLOCTHREADLOCALMEMORY
 0010:0002C2D0       DOS32FREETHREADLOCALMEMORY
 0010:0002C2D8       preDOS32FREETHREADLOCALMEMORY
 0010:0002C2E9       postDOS32FREETHREADLOCALMEMORY
 0010:0002C2F0       DOS32QUERYEXTLIBPATH
 0010:0002C2F8       preDOS32QUERYEXTLIBPATH
 0010:0002C309       postDOS32QUERYEXTLIBPATH
 0010:0002C310       DOS32SETEXTLIBPATH
 0010:0002C318       preDOS32SETEXTLIBPATH
 0010:0002C329       postDOS32SETEXTLIBPATH
 0010:0002C330       DOS32VERIFYPIDTID
 0010:0002C338       preDOS32VERIFYPIDTID
 0010:0002C349       postDOS32VERIFYPIDTID
 0010:0002C350       DOS32SYSCTL
 0010:0002C358       preDOS32SYSCTL
 0010:0002C369       postDOS32SYSCTL
 0010:0002C370       DOS32QUERYTHREADCONTEXT
 0010:0002C378       preDOS32QUERYTHREADCONTEXT
 0010:0002C389       postDOS32QUERYTHREADCONTEXT
 0010:0002C390       DOS32PERFSYSCALL
 0010:0002C398       preDOS32PERFSYSCALL
 0010:0002C3A9       postDOS32PERFSYSCALL
 0010:0002C3B0       _DbgThreadTerm
 0010:0002C4FC       _DbgLinkDCB
 0010:0002C560       g__TKTstnClrKernelSem
 0010:0002C565       _TKTstnClrKernelSem
 0010:0002C5A0       KMALLOCCONTEXTHOOK
 0010:0002C5BC       KMARMCONTEXTHOOK
 0010:0002C641       KMALLOCHOOK
 0010:0002C6F4       KMFREEHOOK
 0010:0002C77F       KMDISARMHOOK
 0010:0002C7E9       KMTHREADTERMINATE
 0010:0002C837       KMREBUILDSTACKFRAME
 0010:0002CAE3       KMQUERYALLCLIENTREGISTERS
 0010:0002CB27       KMSETALLCLIENTREGISTERS
 0010:0002CB6C       KMQUERYCLIENTREGISTER
 0010:0002CBB2       KMSETCLIENTREGISTER
 0010:0002CBFD       KMQUERYCSEIPLADDR
 0010:0002CC7D       KMQUERYSSESPLADDR
 0010:0002CC9B       KMQUERYRETURNESPLADDR
 0010:0002CD4E       KMQUERYCLIENTRETURNESP
 0010:0002CDB6       KMSETCLIENTRETURNESP
 0010:0002CE0F       KMSETFLATDISPATCH
 0010:0002CF77       KMPUSHCLIENTSTACK
 0010:0002CFC3       KMPOPCLIENTSTACK
 0010:0002D1A0       _schWindowBoost
 0010:0002D22C       sched$GetNextRunner
 0010:0002D242       _SCHGetNextRunner
 0010:0002D298       DispLatency_TCreschedFF
 0010:0002D2A4       _schInitTCB
 0010:0002D334       _SCHSlotSetPriority
 0010:0002D390       _SCHSetPriority
 0010:0002D3E0       _SEMInitPTDA
 0010:0002D4F0       _SEMMarkOwnerDied
 0010:0002D735       _semWakeAllMtxNMux
 0010:0002D76F       _SEMCleanProcDying
 0010:0002DAF4       _SEMTerminatePTDA
 0010:0002DC04       _semChkSharedHdl
 0010:0002DCDE       _semChkPrivateHdl
 0010:0002DD18       _semChkHdl
 0010:0002DD68       _semGetTblHdl
 0010:0002DE09       _semGetType
 0010:0002DEAA       _semSlotToPidTid
 0010:0002DF18       _semGetOpenQNode
 0010:0002DF60       _semSrchSnglForPid
 0010:0002DFA6       _semSrchMuxForPid
 0010:0002DFFF       _semChkSigInMux
 0010:0002E055       _semChkSRInMux
 0010:0002E1AC       _semChkDupHandle
 0010:0002E20C       _semIfHdlInSR
 0010:0002E25A       _semIfAllEvtsPosted
 0010:0002E2D2       _semIfAllMtxFree
 0010:0002E34E       _semOwnMtxInSR
 0010:0002E419       _semAddToMuxQ
 0010:0002E45F       _semDelFromMuxQ
 0010:0002E4EE       _semUpdateAllMuxQ
 0010:0002E51D       _semDelAllMuxQ
 0010:0002E555       _semUpdateFreeMuxQ
 0010:0002E5AD       _semFreeMuxQList
 0010:0002E5DA       _semHash
 0010:0002E63D       _semGetStr
 0010:0002E70F       _semStoreStr
 0010:0002E7F1       _semStrTblSrch
 0010:0002E990       _semStrTblInsert
 0010:0002EB41       _semStrTblDelete
 0010:0002EC6F       _semValidateName
 0010:0002EDFF       _SEMMuxWait16
 0010:0002EE5A       _SEMFindType
 0010:0002EF0C       _SIGInitContextHook
 0010:0002EF28       _SIGGetMustComplete
 0010:0002EFC3       _SIGSetMustCompleteFlag
 0010:0002F056       _TKApiSetSignalExceptionFocus
 0010:0002F194       _VR32SetSignalExceptionFocus
 0010:0002F1DB       _VR32SendSignalException
 0010:0002F1FF       _VR32AcknowledgeSignalException
 0010:0002F254       _VR32StartTimer
 0010:0002F2AE       _VR32StopTimer
 0010:0002F2D0       _VR32AsyncTimer
 0010:0002F32B       _VR32IStartTimer
 0010:0002F36F       _VR32IAsyncTimer
 0010:0002F3C8       _timArmTimer
 0010:0002F4C2       _timDisarmTimer
 0010:0002F59F       _timLinkTimer
 0010:0002F5D2       _timUnlinkTimer
 0010:0002F623       _timQueryTimer
 0010:0002F659       _TIMTomClear
 0010:0002F6AE       TIMCONTEXTHOOK
 0010:0002F7C5       _timProcTerminate
 0010:0002F8C4       _TKForceTask
 0010:0002F8FE       _TKForceThread
 0010:0002F98F       _TKEachThread
 0010:0002F9CD       _TKTidTo_pTCB
 0010:0002FA02       _TKTidTo_iSlot
 0010:0002FA3D       _TKiSlotTo_pTCB
 0010:0002FA82       _tkAsyncPTERM
 0010:0002FAA9       _tkPostPTERMs
 0010:0002FAF6       _tkInnerExit
 0010:0002FB88       _TKDieSoonPTDA
 0010:0002FC35       _TKExit
 0010:0002FC69       _TKForceCritSec
 0010:0002FCA4       _tkIsTCBInUse
 0010:0002FCB5       _tkIsPTDAInUse
 0010:0002FCC8       _tkStartScan
 0010:0002FCF6       _tkStopScan
 0010:0002FD41       _tkWaitScan
 0010:0002FD80       _tkCheckPid
 0010:0002FDA7       _TKPidToPTDA
 0010:0002FE1E       _tkCheckCsid
 0010:0002FE40       _TKScanTasks
 0010:00030041       _TKLinkTask
 0010:00030098       _TKUnlinkTask
 0010:00030215       _TKAdoptTask
 0010:000302F0       _TKDescendant
 0010:00030361       _TKPidGetSem
 0010:000303A4       tkScanWorker
 0010:00030408       _TKUsrArgFault
 0010:0003041C       _TKDisable
 0010:00030420       _TKEnable
 0010:00030428       _tkGetTCBReqPkt
 0010:0003046C       _tkFreeTCBReqPkt
 0010:0003049C       _tkThreadStart
 0010:000304A1       thread_start
 0010:0003052C       _tkIThreadStart
 0010:00030560       _tkVerifyTCBLinks
 0010:00030641       _tkEvapAll
 0010:000306D8       _tkLinkTCB
 0010:0003078B       _tkUnlinkTCBSub
 0010:00030835       _TKWaitThread
 0010:00030999       _tkRunWaitThreads
 0010:00030A49       _tkAllocTCB
 0010:00030F02       _tkFreeTCB
 0010:0003104C       _tkUnlinkTCB
 0010:000310EC       _tkSuBuff386
 0010:00031218       _tkSuBuff486
 0010:000312FB       _TKSuFuBuff
 0010:00031414       _TKSuBuffz
 0010:00031478       _TKFuBuff
 0010:0003155B       _TKFuBuffz
 0010:00031644       _TKFuBufLen
 0010:00031706       _TKUsrMemPageFault
 0010:0003171C       _TKUsrMemGPFault
 0010:00031732       _tkUsrMemError
 0010:00031768       _TKCopyBuff
 0010:0003182C       _tkScanBuffz
 0010:00031888       _TKSuBuff
 0010:00031890       _TKSuByte
 0010:000318A0       _TKSuByteNF
 0010:000318AD       _TKSuWord
 0010:000318BD       _TKSuWordNF
 0010:000318CA       _TKSuDWord
 0010:000318DA       _TKSuDWordNF
 0010:00031900       _TKProbeBuff
 0010:000319E0       _tkBufferWithinUserDSLimit
 0010:00031A2C       _tomCheckFire
 0010:00031AEB       _TOMQuery
 0010:00031B12       _TOMSet
 0010:00031D97       _TOMCancel
 0010:00031E1C       _TOMTick
 0010:000320D7       _tomStartMigration
 0010:00032218       _tomMigrateAll
 0010:00032548       _VDMMTomHook
 0010:0003254C       _MakeSuffix
 0010:00032589       _PLD_OpenDump
 0010:000327A0       _VR32IPerfSysCall
 0010:000329FD       _InitPerfBuffer
 0010:00032B95       _FreePerfBuffer
 0010:00032BDE       _GetPerfBuffer
 0010:00032C59       _GetPerfBufferHeaders
 0010:00032CE4       _InfoPerfBuffer
 0010:00032D38       _DoClockSync
 0010:00032D50       _SoftTraceOn
 0010:00032E07       _SoftTraceStartup
 0010:00032F34       _SoftTraceGetMte
 0010:00033042       _SoftTraceOff
 0010:000330E1       _SoftTraceAllocBuffer
 0010:0003311B       _SoftTraceFreeBuffer
 0010:0003317A       _SoftTraceResetBuffer
 0010:00033205       _SoftTraceGetBuffer
 0010:000332C4       _SoftTraceQueryInfo
 0010:0003335A       _SoftTraceEnable
 0010:00033391       _PerfDoSSTime
 0010:000333DA       _PerfGetSSTime
 0010:00033484       _PerfDoCPURating
 0010:000334C8       _PerfGetCPURating
 0010:00033543       _SoftTraceUserLog
 0010:000335C4       _STrace0
 0010:000335DB       _STrace1
 0010:000335F5       _STrace2
 0010:00033612       _STrace3
 0010:00033632       _STrace4
 0010:00033655       _STraceData
 0010:00033675       _STraceDataSZ
 0010:000336A9       _STraceVData1
 0010:000336C6       _STraceVData2
 0010:000336E9       _STraceVData3
 0010:00033712       _STraceVData4
 0010:00033741       _STraceVDataSZ1
 0010:0003375B       _STraceVDataSZ2
 0010:00033778       _STraceVDataSZ3
 0010:00033798       _STraceVDataSZ4
 0010:000337BB       _SoftTracehook
 0010:00033B28       _PerfKIEnable
 0010:00033B30       _PerfKIDisable
 0010:00033B38       _PerfKIRdCnt
 0010:00033B7C       g_ldrGetObjOff
 0010:00033BB8       _PGPageFault
 0010:00034361       _pgForcePresent
 0010:00034537       _pgReloadFrame
 0010:00034871       _pgMapPte
 0010:00034A3E       _PGMakePresent
 0010:00034A72       _PGTrap2FindPage
 0010:00034D00       _PrintArena
 0010:00034DA4       _pgDeleteArena
 0010:00034DCE       _pgInsertArena
 0010:00034E04       _LDRNotifyLoadedModules
 0010:00034F34       _VMLockMem
 0010:0003585E       _vmAccessLongLockInfo
 0010:00035AB2       _vmLockHandleSig
 0010:00035AE5       _VMUnlock
 0010:00035DB8       VDHQUERYHOOKDATA
 0010:00035DF5       VDHARMCONTEXTHOOK
 0010:00035E74       VDHARMSTIHOOK
 0010:00035F74       pvwMt_Ct_mem_DemandLd_0
 0010:00035F80       pvwMt_Ct_mem_Reassigned_0
 0010:00035F8C       pvwMt_Ct_fbc_RdHit_0
 0010:00035F98       pvwMt_Ct_fbc_RdMiss_0
 0010:00035FA4       pvwMt_Ct_fbc_WrtHit_0
 0010:00035FB0       pvwMt_Ct_fbc_WrtMiss_0
 0010:00035FBC       g_pvwMt_Ct_fbc_WrtActiv_0
 0010:00035FD8       g_pvwMt_Ct_fbc_Bypass_0
 0010:00035FF4       g_pvwMt_ST_thd_FileIOWait_1
 0010:00035FF4       g_pvwMt_ST_thd_FileIOWait_0
 0010:00036044       g_pvwMt_ET_thd_FileIOWait_1
 0010:00036044       g_pvwMt_ET_thd_FileIOWait_0
 0010:000360C0       g_pvwMt_ST_thd_FileIOWait_2
 0010:000360C0       g_pvwMt_ST_thd_FileIOWait_3
 0010:00036110       g_pvwMt_ET_thd_FileIOWait_2
 0010:00036116       g_pvwMt_ET_thd_FileIOWait_3
 0010:00036190       g_pvwMt_ET_spr_Spare1_1
 0010:000361B8       g_pvwMt_ST_spr_Spare1_1
 0010:000361E0       g_pvwMt_CtST_spr_Spare1_1
 0010:0003620C       g_pvwMt_Ct_spr_Spare1_1
 0010:00036228       g_pvwMt_ET_spr_Spare2_1
 0010:00036250       g_pvwMt_ST_spr_Spare2_1
 0010:00036278       g_pvwMt_CtST_spr_Spare2_1
 0010:000362A4       g_pvwMt_Ct_spr_Spare2_1
 0010:000362C0       g_pvwMt_ET_spr_Spare3_1
 0010:000362E8       g_pvwMt_ST_spr_Spare3_1
 0010:00036310       g_pvwMt_CtST_spr_Spare3_1
 0010:0003633C       g_pvwMt_Ct_spr_Spare3_1
 0010:00036358       g_pvwMt_ET_spr_Spare4_1
 0010:00036380       g_pvwMt_ST_spr_Spare4_1
 0010:000363A8       g_pvwMt_CtST_spr_Spare4_1
 0010:000363D4       g_pvwMt_Ct_spr_Spare4_1
 0010:000363F0       g_pvwMt_ET_spr_Spare5_1
 0010:00036418       g_pvwMt_ST_spr_Spare5_1
 0010:00036440       g_pvwMt_CtST_spr_Spare5_1
 0010:0003646C       g_pvwMt_Ct_spr_Spare5_1
 0010:00036488       g_pvwMt_ET_spr_Spare6_1
 0010:000364B0       g_pvwMt_ST_spr_Spare6_1
 0010:000364D8       g_pvwMt_CtST_spr_Spare6_1
 0010:00036504       g_pvwMt_Ct_spr_Spare6_1
 0010:00036520       g_pvwMt_ET_spr_Spare7_1
 0010:00036548       g_pvwMt_ST_spr_Spare7_1
 0010:00036570       g_pvwMt_CtST_spr_Spare7_1
 0010:0003659C       g_pvwMt_Ct_spr_Spare7_1
 0010:000365B8       g_pvwMt_ET_spr_Spare8_1
 0010:000365E0       g_pvwMt_ST_spr_Spare8_1
 0010:00036608       g_pvwMt_CtST_spr_Spare8_1
 0010:00036634       g_pvwMt_Ct_spr_Spare8_1
 0010:00036650       g_pvwMt_ET_spr_Spare9_1
 0010:00036678       g_pvwMt_ST_spr_Spare9_1
 0010:000366A0       g_pvwMt_CtST_spr_Spare9_1
 0010:000366CC       g_pvwMt_Ct_spr_Spare9_1
 0010:000366E8       g_pvwMt_ET_spr_Spare10_1
 0010:00036714       g_pvwMt_ST_spr_Spare10_1
 0010:00036740       g_pvwMt_CtST_spr_Spare10_1
 0010:00036774       g_pvwMt_Ct_spr_Spare10_1
 0010:00036794       _PvwGetMFTName
 0010:000367F8       _PvwMtFilDataBlk
 0010:00036870       perfvwa$pvwAliasHook
 0010:000368A8       _PVWSetHook
 0010:000368D0       _PVWUnSetHook
 0010:000368F0       perfvwa$pvwPatchHook
 0010:00036956       perfvwa$pvwPatchHookA
 0010:00036958       _PvwPatch_Ct_cpu_Int_0
 0010:0003695F       _PvwPatch_Mt_cpu_STInt_STNotIdl
 0010:00036966       _PvwPatch_Mt_cpu_ETInt_ETNotIdl
 0010:0003696D       _PvwPatch_Ct_cpu_Sched_0
 0010:00036974       _PvwPatch_ST_cpu_NotIdle_0
 0010:0003697B       _PvwPatch_ET_cpu_NotIdle_0
 0010:00036982       _PvwPatch_Ct_mem_DemandLd_0
 0010:00036989       _PvwPatch_Ct_mem_Discard_0
 0010:00036990       _PvwPatch_Mt_mem_PageFault_0
 0010:00036997       _PvwPatch_Mt_mem_PageFault_1
 0010:0003699E       _PvwPatch_Ct_mem_SwapOut_0
 0010:000369A5       _PvwPatch_Ct_mem_SwapIn_0
 0010:000369AC       _PvwPatch_Ct_mem_Reassigned_0
 0010:000369B3       _PvwPatch_Ct_mem_Reassigned_1
 0010:000369BA       _PvwPatch_Ct_mem_Recovered_0
 0010:000369C1       _PvwPatch_Ct_mem_Idled_0
 0010:000369C8       _PvwPatch_EQ_mem_QUsed_0
 0010:000369CF       _PvwPatch_LQ_mem_QUsed_0
 0010:000369D6       _PvwPatch_EQ_mem_QFree_0
 0010:000369E0       _PvwPatch_LQ_mem_QFree_0
 0010:000369EA       _PvwPatch_EQ_mem_QCTResident_0
 0010:000369F4       _PvwPatch_LQ_mem_QCTResident_0
 0010:000369FE       _PvwPatch_ST_thd_FileIOWait_0
 0010:00036A08       _PvwPatch_ET_thd_FileIOWait_0
 0010:00036A12       _PvwPatch_ST_thd_FileIOWait_1
 0010:00036A1C       _PvwPatch_ET_thd_FileIOWait_1
 0010:00036A26       _PvwPatch_ST_thd_FileIOWait_2
 0010:00036A30       _PvwPatch_ET_thd_FileIOWait_2
 0010:00036A3A       _PvwPatch_ST_thd_FileIOWait_3
 0010:00036A44       _PvwPatch_ET_thd_FileIOWait_3
 0010:00036A4E       _PvwPatch_CtST_cal_Masm_0
 0010:00036A58       _PvwPatch_ET_cal_Masm_0
 0010:00036A62       _PvwPatch_CtST_cal_C_0
 0010:00036A6C       _PvwPatch_ET_cal_C_0
 0010:00036A76       _PvwPatch_Ct_fbc_RdHit_0
 0010:00036A80       _PvwPatch_Ct_fbc_RdMiss_0
 0010:00036A8A       _PvwPatch_Ct_fbc_WrtHit_0
 0010:00036A94       _PvwPatch_Ct_fbc_WrtMiss_0
 0010:00036A9E       _PvwPatch_Ct_fbc_WrtActiv_0
 0010:00036AA8       _PvwPatch_Ct_fbc_Bypass_0
 0010:00036AB2       _PvwPatch_ET_spr_Spare1_0
 0010:00036ABC       _PvwPatch_ST_spr_Spare1_0
 0010:00036AC6       _PvwPatch_CtST_spr_Spare1_0
 0010:00036AD0       _PvwPatch_Ct_spr_Spare1_0
 0010:00036ADA       _PvwPatch_ET_spr_Spare2_0
 0010:00036AE4       _PvwPatch_ST_spr_Spare2_0
 0010:00036AEE       _PvwPatch_CtST_spr_Spare2_0
 0010:00036AF8       _PvwPatch_Ct_spr_Spare2_0
 0010:00036B02       _PvwPatch_ET_spr_Spare3_0
 0010:00036B0C       _PvwPatch_ST_spr_Spare3_0
 0010:00036B16       _PvwPatch_CtST_spr_Spare3_0
 0010:00036B20       _PvwPatch_Ct_spr_Spare3_0
 0010:00036B2A       _PvwPatch_ET_spr_Spare4_0
 0010:00036B34       _PvwPatch_ST_spr_Spare4_0
 0010:00036B3E       _PvwPatch_CtST_spr_Spare4_0
 0010:00036B48       _PvwPatch_Ct_spr_Spare4_0
 0010:00036B52       _PvwPatch_ET_spr_Spare5_0
 0010:00036B5C       _PvwPatch_ST_spr_Spare5_0
 0010:00036B66       _PvwPatch_CtST_spr_Spare5_0
 0010:00036B70       _PvwPatch_Ct_spr_Spare5_0
 0010:00036B7A       _PvwPatch_ET_spr_Spare6_0
 0010:00036B84       _PvwPatch_ST_spr_Spare6_0
 0010:00036B8E       _PvwPatch_CtST_spr_Spare6_0
 0010:00036B98       _PvwPatch_Ct_spr_Spare6_0
 0010:00036BA2       _PvwPatch_ET_spr_Spare7_0
 0010:00036BAC       _PvwPatch_ST_spr_Spare7_0
 0010:00036BB6       _PvwPatch_CtST_spr_Spare7_0
 0010:00036BC0       _PvwPatch_Ct_spr_Spare7_0
 0010:00036BCA       _PvwPatch_ET_spr_Spare8_0
 0010:00036BD4       _PvwPatch_ST_spr_Spare8_0
 0010:00036BDE       _PvwPatch_CtST_spr_Spare8_0
 0010:00036BE8       _PvwPatch_Ct_spr_Spare8_0
 0010:00036BF2       _PvwPatch_ET_spr_Spare9_0
 0010:00036BFC       _PvwPatch_ST_spr_Spare9_0
 0010:00036C06       _PvwPatch_CtST_spr_Spare9_0
 0010:00036C10       _PvwPatch_Ct_spr_Spare9_0
 0010:00036C1A       _PvwPatch_ET_spr_Spare10_0
 0010:00036C24       _PvwPatch_ST_spr_Spare10_0
 0010:00036C2E       _PvwPatch_CtST_spr_Spare10_0
 0010:00036C38       _PvwPatch_Ct_spr_Spare10_0
 0010:00036C58       DbgWPScan
 0010:00036CD4       _DbgSetDRladdr
 0010:00036CFC       _DBGDRDisableVDM
 0010:00036D64       _DBGDREnableVDM
 0010:00036D9C       _DbgDRAlloc
 0010:00036F3B       _DbgDRFree
 0010:000370A0       _semSharedAlloc
 0010:0003731C       _semPrivateAlloc
 0010:00037480       _semOpenSharedAlloc
 0010:00037713       _semAllocWaitMuxQs
 0010:0003786C       _semSharedClose
 0010:000378F0       _semPrivateClose
 0010:00037967       _semOpenSem
 0010:00037BC0       _VR32CreateEventSem
 0010:00037D1C       _VR32OpenEventSem
 0010:00037DE3       _VR32CloseEventSem
 0010:00037E17       _VR32ResetEventSem
 0010:00037E83       _VR32PostEventSem
 0010:00037EB7       _VR32WaitEventSem
 0010:00037EE8       _VR32QueryEventSem
 0010:00037F54       _SEMApiCreateEventSem
 0010:000380B2       _SEMApiOpenEventSem
 0010:00038228       _dhw_OpenEventSem
 0010:00038243       _dhw_CloseEventSem
 0010:00038273       _dhw_PostEventSem
 0010:000382A3       _dhw_ResetEventSem
 0010:000382D6       _semCreateEventSem
 0010:00038466       _SEMCloseEventSem
 0010:0003878A       _SEMResetEventSem
 0010:000388BE       _SEMPostEventSem
 0010:00038BFF       _SEMWaitEventSem
 0010:00038D87       _SEMQueryEventSem
 0010:00038E60       _VR32CreateMuxWaitSem
 0010:00039062       _VR32OpenMuxWaitSem
 0010:0003911D       _VR32CloseMuxWaitSem
 0010:00039163       _VR32WaitMuxWaitSem
 0010:00039251       _VR32AddMuxWaitSem
 0010:000392EB       _VR32DeleteMuxWaitSem
 0010:000395B5       _VR32QueryMuxWaitSem
 0010:00039742       _SEMApiCreateMuxWaitSem
 0010:00039940       _SEMApiOpenMuxWaitSem
 0010:00039AB0       _SEMApiWaitMuxWaitSem
 0010:00039BE9       _SEMApiAddMuxWaitSem
 0010:00039E9F       _semCreateMuxWaitSem
 0010:0003A02F       _SEMCloseMuxWaitSem
 0010:0003A31D       _semWaitMuxWaitSem
 0010:0003A8FE       _semAddMuxWaitSem
 0010:0003AE5F       _SEMDeleteMuxWaitSem
 0010:0003B105       _SEMQueryMuxWaitSem
 0010:0003B300       _VR32CreateMutexSem
 0010:0003B444       _VR32OpenMutexSem
 0010:0003B4FF       _VR32CloseMutexSem
 0010:0003B53F       _VR32RequestMutexSem
 0010:0003B7FE       _VR32ReleaseMutexSem
 0010:0003BA32       _VR32QueryMutexSem
 0010:0003BB1F       _SEMApiCreateMutexSem
 0010:0003BC7D       _SEMApiOpenMutexSem
 0010:0003BDF6       _semCreateMutexSem
 0010:0003BF4C       _SEMCloseMutexSem
 0010:0003C3C5       _SEMRequestUnownedMutex
 0010:0003C5B1       _SEMRequestOwnedMutexWkr
 0010:0003C7E9       _SEMRequestOwnedMutex
 0010:0003C7F9       _SEMReleaseMutexSem
 0010:0003C834       _SEMReleaseUnwaitedMutex
 0010:0003C9E9       _SEMReleaseWaitedMutex
 0010:0003CC8C       _SEMQueryMutexSem
 0010:0003CE34       _pmSemIN
 0010:0003CE6C       _semPMPostEventSem
 0010:0003CF85       _VR32PMPostEventSem
 0010:0003CF98       _VR32PMWaitEventSem
 0010:0003D05C       _VR32PMRequestMutexSem
 0010:0003D0E6       _VR32PMWaitMuxWaitSem
 0010:0003D15B       _dhw_PMPostEventSem
 0010:0003D170       _VR32PM16SEMCHK
 0010:0003D1C6       _VR32PM16SEMRST
 0010:0003D204       HexToAscii32
 0010:0003D20D       ByteToAscii32
 0010:0003D217       subr$NibbleToAscii32
 0010:0003D224       _IntToDecAscii
 0010:0003D23C       _DHGetMessage32
 0010:0003D274       _SysServTerm
 0010:0003D298       _SysServWakeJIT
 0010:0003D2FC       _TKVSprintf
 0010:0003D70B       _TKDebugHardError
 0010:0003D804       g_KMTHREADTERMINATE
 0010:0003D80F       g__SEMInitShrTbl
 0010:0003D81A       g__SEMCleanProcDying
 0010:0003D825       g__semValidateName
 0010:0003D830       g__SIGInitContextHook
 0010:0003D83B       g__KIEnableInit
 0010:0003D846       g__SoftTraceEnable
 0010:0003D851       g__SoftTraceOn
 0010:0003D85C       g__SoftTraceAllocBuffer
 0010:0003D867       g__DHookSwitch
 0010:0003D874       _TKPriCalc
 0010:0003D8CE       _TKGetPriority
 0010:0003D8EB       _VRSleep
 0010:0003D938       _TKSleep
 0010:0003DC06       _TKWakeup
 0010:0003DF75       _TKWakeThread
 0010:0003DFBA       _TKQueryWakeup
 0010:0003E0D9       _TKDelayedWakeup
 0010:0003E104       _tkSleepQInsert
 0010:0003E3C0       _tkSleepQRemove
 0010:0003E3FF       _tkPriQRemoveChain
 0010:0003E5D2       _tkPriQInsert
 0010:0003E7B3       _tkPriQRemove
 0010:0003E9C0       _TKGetReadyThread
 0010:0003EA52       _TKIdleLoop
 0010:0003EA83       _TKUpdatePriority
 0010:0003EC18       _TKUpdateState
 0010:0003F0BE       _TKYieldNonIdle
 0010:0003F0DB       _tkTSDDaemon
 0010:0003F2C7       _TKIdleTSD
 0010:0003F34B       _TKNeedTSDDaemon
 0010:0003F356       _TKTomTimeslice
 0010:0003F470       _TKTomWake
 0010:0003F4D7       _TKTomStarve
 0010:0003F528       _TKExitInversion
 0010:0003F553       _TKDeclareInversion
 0010:0003F5CE       _tkKDBDaemon
 0010:0003F642       _TKMakePresentKDB
 0010:0003F6FC       g_CWait
 0010:0003F701       CWait
 0010:0003F7FC       tkCollectZomb
 0010:0003F854       _dputs
 0010:0003F86C       _printf
 0010:0003F888       _EP2_32_Decompress
 0010:0003F888       EP2_32_Decompress
 0010:0003F8C1       decomp32
 0010:0003FA20       _FSD_AllocatePageSpace
 0010:0003FA20       _StartSMLOCK_TEXT
 0010:0003FA20       _End_TEXT
 0010:0003FAA0       _FSD_DoPageIO
 0010:0003FB2C       _FSD_FlushBuf
 0010:0003FB54       _PGBuildGrpIOList
 0010:0003FD42       _pgFindDF
 0010:0003FDD0       _SMSwapOut
 0010:00040019       _SMSwapIn
 0010:000401AC       _smAllocDF
 0010:0004038D       _SMFreeDF
 0010:000404DA       _smGRPAllocDF
 0010:0004072F       _SMSetSwapSpace
 0010:0004084B       _SMSetSwapSpace2
 0010:00040922       _smIncreaseSpace
 0010:00040BD2       _smDecreaseSpace
 0010:00040C68       _SMTomHook
 0010:00040C84       _smPerformShrink
 0010:00040DA3       _SMTestSwapFile
 0010:00040F01       _SMQuerySwapSpace
 0010:00040F6E       _smCompress
 0010:00041035       _smDecompress
 0010:0004108C       _smSIOSwapIn
 0010:00041100       _smSIOResize
 0010:00041166       _smSIOSpaceQuery
 0010:000411D1       _smGrpSwpErrHandler
 0010:000413E0       _smRetrySwapOut
 0010:000414D1       _smSetCmd1
 0010:00041524       _SMCompact
 0010:0004195B       _SMFreeCompDFs
 0010:000419B8       _PLD_WriteSharedInstance
 0010:00041C14       _StartHIGH32SWAP_TEXT
 0010:00041C14       _dhw_32KrnlExit
 0010:00041C14       _EndSMLOCK_TEXT
 0010:00041D9E       _KrxAdd
 0010:00041F12       _KrxDelete
 0010:0004201C       _KrxQuery
 0010:000420CC       _StartLock32
 0010:000420CD       _AssertNoSwap
 0010:000420F5       _Sec32ReadPre
 0010:000421BD       _Sec32ReadPost
 0010:00042227       _Sec32WritePre
 0010:000422DC       _Sec32WritePost
 0010:00042344       _Sec32ChgFilePtr
 0010:000423E7       _Sec32NewSize
 0010:0004248D       _SaveTCB
 0010:000424AF       _SavePTDA
 0010:00042507       _RestorePTDA
 0010:0004255E       _RestoreTCB
 0010:00042580       _GetCurSFN
 0010:000425BA       _ExtractSFN
 0010:000425CF       _SecHlpTrustedPathNotify
 0010:0004261A       SecOpen
 0010:000426A7       SecPathFromSFN
 0010:00042705       SecSFFromSFN
 0010:00042741       SecWrite
 0010:00042787       SecRead
 0010:000427D0       SecClose
 0010:0004280A       SecQFileSize
 0010:00042847       SecChgFilePtr
 0010:00042888       _EndLock32
 0010:00042889       _Sec32OpenPre
 0010:00042963       _Sec32OpenPost
 0010:00042A83       _Sec32DeletePre
 0010:00042B1A       _Sec32DeletePost
 0010:00042B4D       _Sec32MovePre
 0010:00042C1E       _Sec32MovePost
 0010:00042C55       _Sec32GetModule
 0010:00042C9A       _Sec32Close
 0010:00042D11       _SecCreateVDM
 0010:00042D5A       _SecCreateVDMPost
 0010:00042D8F       _SecLdrOpen
 0010:00042DE8       _SecExec
 0010:00042E70       _SecExecPost
 0010:00042EBF       _Sec32QueryFileInfo
 0010:00042F3B       _Sec32SetFileInfo
 0010:00043003       _Sec32SetFileMode
 0010:000430CA       _Sec32SetPathInfo
 0010:000431C3       _Sec32FindFirst
 0010:0004331A       _Sec32FindFirst3x
 0010:000433B5       _Sec32FindFirstNext3x
 0010:0004347C       _Sec32FindClose3x
 0010:000434C1       _Sec32FindNext
 0010:00043603       _Sec32FindClose
 0010:00043632       _Sec32MakeDir
 0010:000436C9       _Sec32ChangeDir
 0010:00043760       _Sec32RemoveDir
 0010:000437F7       _Sec32SetDateTime
 0010:00043842       _Sec32DevIoctl
 0010:00043CD3       _ProbeIt
 0010:00043CFC       SecHlpFindNext
 0010:00043E31       _Sec32AuditHook
 0010:00044662       _Sec32GetInfo
 0010:00044729       _Sec32GetPPTDA
 0010:0004473C       _VMGetObPermOd
 0010:0004473C       _StartSWAP32_1
 0010:0004473C       _EndHIGH32SWAP_TEXT
 0010:0004473C       _StartTHUNKSWAP_TEXT
 0010:0004473C       _EndTHUNKSWAP_TEXT
 0010:000447D3       _VMSetMem
 0010:000449F8       _StartSWAP32_2
 0010:000449F8       _EndSWAP32_1
 0010:000449F8       _PGSetAccess
 0010:00044A5D       _pgwSetAccess
 0010:00044B44       _SELAddPermission
 0010:00044BCC       _VR32GetSharedMem
 0010:00044D08       _VR32VerifyPidTid
 0010:00044D64       _StartSWAP32_3
 0010:00044D64       _PGAlloc
 0010:00044D64       _EndSWAP32_2
 0010:000451AE       _pgwAlloc
 0010:00045270       _SELGetSize
 0010:00045414       _VMSetMemSub
 0010:000458EC       _PGFree
 0010:000458EC       _StartSWAP32_4
 0010:000458EC       _EndSWAP32_3
 0010:000459D4       _SELSetDescAll
 0010:00045A34       _SELAlloc
 0010:00045C00       _SELFree
 0010:00045CF0       _selFreeLDTSub
 0010:00045E84       _VMAllocMem
 0010:00046694       _vmCommitMemWrkr
 0010:0004685F       _VMFreeMem
 0010:0004691C       _ldrClearGraph
 0010:00046938       _LDRClearSem
 0010:000469C0       _ldrValidateMteHandle
 0010:000469E8       selmgra$selLDTall
 0010:000469E8       _StartSWAP32_5
 0010:000469E8       _EndSWAP32_4
 0010:00046A68       _selValidateLDT
 0010:00046BBD       _selAllocLDTSub
 0010:00046C4C       _ldrMarkTaskInGraph
 0010:00046CA9       _ldrMarkInGraph
 0010:00046CD4       _ldrFindGraph
 0010:00046D84       _LDRTstnSetSem
 0010:00046DCB       _ldrFindObject
 0010:00046E60       _ldrSetupResource
 0010:00046EE4       _ldrFindHmteInDLDRecord
 0010:00046F18       _ldrGetResource
 0010:000470BE       _VR32GetResource
 0010:00047134       _LDRCheckModHandle
 0010:00047162       _ldrGet32Rsrc
 0010:0004720A       _LDRFreeObject
 0010:00047438       _VR32FreeResource
 0010:000476B4       _ldrIncRefCount
 0010:000476DC       _ldrCheckForResource
 0010:000477A0       g_SELSegFree
 0010:000477A0       _EndSWAP32_5
 0010:000477A0       _StartSWAP32_6
 0010:0004785C       _VR32AllocMem
 0010:00047985       _VR32FreeMem
 0010:00047B59       _VMScanContext
 0010:00047CB9       _vmFreeMemContext
 0010:00047D13       _VMFreeAllContext
 0010:00047F08       _tkUpdateTIBPriority
 0010:00047F48       _LDRGetPage
 0010:00048358       _ldr32UnpackPage2
 0010:00048508       _ldrEnum32bitRelRecs
 0010:00048604       _StartSWAP32_7
 0010:00048604       _PGAttach
 0010:00048604       _EndSWAP32_6
 0010:0004869B       _pgwAttach
 0010:00048F38       _vmDecommitMemWrkr
 0010:00048FF4       _ldrSetVMflags
 0010:000490ED       _ldrAllocObject
 0010:00049480       _ldrRsrcAlloc
 0010:000494C4       _ldrRsrcFindGlobal
 0010:00049518       ldrrsrc$ldrRsrcFindGlobal
 0010:0004954C       ldrrsrc$ldrRsrcDeleteLocal
 0010:000495A8       ldrrsrc$ldrRsrcDeleteGlobal
 0010:000495F4       _StartSWAP32_8
 0010:000495F4       _PGQueryAccess
 0010:000495F4       _EndSWAP32_7
 0010:000496BC       selmgra$selLDTlimit
 0010:0004975C       _selReallocSub
 0010:00049830       selwrk$g_selReallocSeg
 0010:00049A2C       _vmQueryObject
 0010:00049BA0       _TKCreateThread
 0010:00049EB4       _tkInitThrdKStack
 0010:0004A179       _tkInitThrdUStack
 0010:0004A342       _tkAllocTIB
 0010:0004A4FE       _tkSetTIB
 0010:0004A5F0       _ldrOpen
 0010:0004A68C       _ldrGetMedia
 0010:0004A6D4       _ldrOpenNewExe
 0010:0004A87B       _ldrOpenPath
 0010:0004AA78       _pgwQueryAccess
 0010:0004AA78       _StartSWAP32_9
 0010:0004AA78       _EndSWAP32_8
 0010:0004AB04       _VR32QueryMem
 0010:0004ABD8       _VM32ApiQueryMem
 0010:0004AEC4       _VR32CreateThread
 0010:0004AF88       _ldrClose
 0010:0004AFAC       _ldrHashQATName
 0010:0004AFD8       _LDRQAppType
 0010:0004B26F       _ldrMungeFlags
 0010:0004B33C       _EndSWAP32_9
 0010:0004B33C       _ldrExpandHeader
 0010:0004B33C       _StartSWAP32_10
 0010:0004B3D0       _xcpt2Trap
 0010:0004B43B       _XCPTBuildR3DispatcherStack
 0010:0004BB83       _VR32ExceptionCallBack
 0010:0004BBED       _xcptExceptionCallBack
 0010:0004BD3F       _xcptDefaultAction
 0010:0004C018       _xcptRestoreXcptContext
 0010:0004C25F       _xcptCopyinXcptStruct
 0010:0004C2DC       _EndSWAP32_10
 0010:0004C2DC       _StartSWAP32_11
 0010:0004C2DC       _ldrNumToOte
 0010:0004C316       _ldrGetEntAddr
 0010:0004C96C       _ldrGetSelector
 0010:0004CA80       _ldrSkipEnts
 0010:0004CAF0       _StartSWAP32_12
 0010:0004CAF0       _EndSWAP32_11
 0010:0004CAF0       VDHSetFlags
 0010:0004CB40       em86opSTI
 0010:0004CB88       EM86ENABLEDINTERRUPTS
 0010:0004CBF8       EM86opARPL
 0010:0004CC0A       em86DispatchVDMBP
 0010:0004CC67       EM86DISPATCHVPMVDMBP
 0010:0004CC80       EM86VDMBPDEFAULTDISPATCHER32
 0010:0004CC90       EM86VDMBPRECURSIVEDISPATCHER
 0010:0004CCD0       EM86VDMBPDEFAULTDISPATCHER
 0010:0004CD26       em86CheckVDMBP
 0010:0004CD78       em86CheckVPMBP
 0010:0004CDC8       em86opHLT
 0010:0004CDDE       em86misc$em86DispatchVPMBP
 0010:0004CE30       VDHWAITEVENTSEM
 0010:0004CE50       _ldr32UnpackPage
 0010:0004D178       em86int$em86opINT
 0010:0004D18C       em86opINTnn
 0010:0004D2AC       EM86INTHOOK
 0010:0004D344       EM86CHOOKSTUBINTH
 0010:0004D368       _PGAllocContext
 0010:0004D368       _EndSWAP32_12
 0010:0004D368       _StartSWAP32_13
 0010:0004D4A7       _pgwAllocPte
 0010:0004D518       _SELCopy
 0010:0004D62A       _selGetSeg
 0010:0004D70C       selwrk$g_selAllocSeg
 0010:0004D7CC       _VMMapAlias
 0010:0004DCCC       _VR32AllocSharedMem
 0010:0004DD9A       _VR32GetNamedSharedMem
 0010:0004DE2E       _VM32ApiAllocSharedMem
 0010:0004E030       _VM32ApiGetNamedSharedMem
 0010:0004E140       _VMInitTask
 0010:0004E1FF       _vmCreateArena
 0010:0004E444       _vmAllocNamedShrMem
 0010:0004E620       _vmGetNamedShrMem
 0010:0004E840       g_ValidateName
 0010:0004E845       ValidateName
 0010:0004E870       _vmFreeNamedSharedMem
 0010:0004E96C       _VMCreatePseudoHandle
 0010:0004EA04       _tkDupProcData
 0010:0004EA64       exec$tkInitSemPTDATbl
 0010:0004EA88       _tkAllocPTDA
 0010:0004EE0C       _tkExitList
 0010:0004EEA4       _tkAddExitListRoutine
 0010:0004EFFF       _VRExitList
 0010:0004F028       _tkLibiInitStatic
 0010:0004F07D       _TKLibiStartDispatch
 0010:0004F258       _ldrMatchStringsN
 0010:0004F274       _ldrIncDLDRecord
 0010:0004F33E       _ldrWasLoadModuled
 0010:0004F3A8       _LDRGetProcAddr
 0010:0004F5CC       _VR32QueryProcAddr
 0010:0004F5E8       _ldrCheckDLLTerm
 0010:0004F668       _ldrSetLoaded
 0010:0004F68A       _ldrGetModule
 0010:0004F7A7       _ldrGetMte
 0010:0004FEBF       _ldrFindModule
 0010:000500E8       _ldrIsAttached
 0010:000501F1       _ldrChkLoadType
 0010:00050244       g_w_loadmodule
 0010:00050738       _tkNewPid
 0010:000507D4       _tkStartProcess
 0010:000508C0       g_SELSegRealloc
 0010:000508C0       _StartSWAP32_14
 0010:000508C0       _EndSWAP32_13
 0010:000508C5       SELSegRealloc
 0010:000509E4       _VR32GiveSharedMem
 0010:00050B44       _TKLibiRecordMTE
 0010:00050CBB       _TKLibiInitNextDLL
 0010:000514D4       _LdrGetModIndx
 0010:00051504       _ldrGetFileName
 0010:00051554       _LDRCheckSig
 0010:00051586       _ldrAllocObjects
 0010:000517F2       _ldrProcessObjects
 0010:00051CF4       _ldrEachObjEntry
 0010:00051DFE       _LDRGetTKModuleInfo
 0010:000520F1       _LDRSetTKLibiFlags
 0010:00052150       _ldrLoadImports
 0010:0005229D       _ldrLinkMTE
 0010:00052352       _ldrCreateMte
 0010:00052DDC       _ldrMTEValidatePtrs
 0010:00052E20       _EndSWAP32_14
 0010:00052E20       _StartSWAP32_15
 0010:00052E20       _PGSetTypeLDT
 0010:00052E6E       _pgwSetTypeLDT
 0010:000530D0       _SELMemMapAlias
 0010:00053230       _SELMemUnmapAlias
 0010:00053318       _selInitLDTSub
 0010:0005344B       _selInitInfoSegLDT
 0010:00053499       _SELInitLDT
 0010:000534FC       selwrk$g_selCreateCSAlias
 0010:00053660       _VMSelAlias
 0010:0005371C       _calcTLMASize
 0010:00053782       _VR32IAllocThreadLocalMemory
 0010:00053954       _dhw_VMGlobalToProcess
 0010:00053ADC       demsvc$demSleep
 0010:00053B0C       _DbgRegisterSemList
 0010:00053D48       _DbgkDBRead
 0010:00053DDD       _DBG32ApiDebug
 0010:00054056       _VR32DEBUG
 0010:00054068       _DYNAttach
 0010:000540D0       g_tkExecPgm
 0010:00054514       exec$tkgetnewenviron
 0010:000546A0       _tkInheritLIBPATH
 0010:00054778       _tkSetPIB
 0010:00054821       _tkAllocPIB
 0010:0005489C       _VR32ExitList
 0010:000548B0       _tkSetPTDAVars
 0010:000549C5       _TKAllocR2Stacks
 0010:00054B48       _ldrTransPath
 0010:00054B98       _ldrASMpMTEFromHandle
 0010:00054BB3       _ldrGetCallGate
 0010:00054C1C       _ldrAllocCallGate
 0010:00054DE4       _LDRLoadExe
 0010:00054F69       _ldrCheckGlobal
 0010:00054FD6       _ldrGetModParams
 0010:000551B8       _StartSWAP32_16
 0010:000551B8       _EndSWAP32_15
 0010:000551B8       _SELAllocLDT
 0010:000551DC       _SELAddDiscRec
 0010:0005524C       selwrk$g_selAllocHuge
 0010:00055330       selwrk$g_selReallocHuge
 0010:00055560       _ldrStrCpyB
 0010:00055580       _VR32QueryProcType
 0010:000555A8       _ldrExpandRecord
 0010:0005566E       _ldrGet32TgtAddr
 0010:000558DD       _ldrApply32Fixups
 0010:00055ADD       _ldrGetTgtMte
 0010:00055B2B       _ldrGetOrdNum
 0010:00055CAD       _ldrGetOrdNumSub
 0010:00055D3D       _ldrGetImport
 0010:00055E74       _StartSWAP32_17
 0010:00055E74       selseg$g__SegAlloc
 0010:00055E74       _EndSWAP32_16
 0010:00055F84       VDHREQUESTMUTEXSEM
 0010:00055FA4       VDHRELEASEMUTEXSEM
 0010:00055FB0       _VR32RequestVDD
 0010:00055FE1       VDMMREQUESTVDD
 0010:000560B8       VDHLOCKMEM
 0010:000561A2       VDHUNLOCKMEM
 0010:00056204       VDHLOCKENTRY
 0010:0005636C       _VR32QuerySysInfo
 0010:0005647C       _tkLibiCleanup
 0010:0005653A       _tkLibiFreeHeap
 0010:000565C1       _tkLibiFreeModules
 0010:00056638       _ldrNextLibPath
 0010:00056704       _ldrSelFwdFlg
 0010:00056744       _ldrGetFwdEnt
 0010:00056900       _ldrCheckSpecific
 0010:0005697F       _ldrCheckInternalName
 0010:000569FC       _StartSWAP32_18
 0010:000569FC       VDHPUSHSTACK
 0010:000569FC       _EndSWAP32_17
 0010:00056A64       em86misc$em86PushStack
 0010:00056AE4       VDHPOPSTACK
 0010:00056B4C       em86misc$em86PopStack
 0010:00056BBC       EM86DispatchVDMBPHooks
 0010:00056C30       VDMMPROCFBGND
 0010:00056CA8       VDHQUERYSEL
 0010:00056D6C       QUERYDATATYPE
 0010:00056E68       VDMMSETSTATE
 0010:00056E98       VDHPUSHINT
 0010:00056EFC       VDHPOPINT
 0010:00056F58       em86ReflectInt
 0010:00056F65       EM86ReflectV86Exception
 0010:00056F65       em86ReflectV86Int
 0010:000570DC       em86int$em86CallPreIntHooks
 0010:00057148       VDHARMRETURNHOOK
 0010:000573FC       VDHPUSHREGS
 0010:000573FC       _StartSWAP32_19
 0010:000573FC       _EndSWAP32_18
 0010:00057464       VDHPOPREGS
 0010:00057500       VDMMMEMORYMAPPEDIN
 0010:00057517       VDMMMEMORYUNMAPPED
 0010:0005752E       VDMMPROCMEMMAPPED
 0010:00057568       VDHMAPPAGES
 0010:000575BC       EM86VPMREFLECTIONHOOK
 0010:00057630       VDHINSTALLIOHOOK
 0010:0005790E       EM86GROWIOPM
 0010:00057A87       VDHSETIOHOOKSTATE
 0010:00057B54       EM86SETIOHOOKSTATE
 0010:00057D2C       _StartSWAP32_20
 0010:00057D2C       _pgwQueryState
 0010:00057D2C       _EndSWAP32_19
 0010:00057DEC       demMapDSDX
 0010:00057DF0       demMapDS
 0010:00057E08       demMapESDI
 0010:00057E0B       demMapES
 0010:00057E24       demMapSegX
 0010:00057E44       demMapVirt
 0010:00057E74       demSetCurrentPDB
 0010:00057E8C       INT2FV86DISPATCHER
 0010:00057EF8       VDMMPDBCHANGE
 0010:00057F09       VDMMPROCPDB
 0010:00057F3C       VDHREQUESTVDD
 0010:00057F5F       REQUESTVDD
 0010:0005802C       VDHREALLOCPAGES
 0010:0005855C       EM86CHOOKSTUBPREINTH
 0010:00058580       VDHREMOVEIOHOOK
 0010:00058607       VDHALLOCHOOK
 0010:000586D9       VDHFREEHOOK
 0010:00058780       _EndSWAP32_20
 0010:00058780       _StartSWAP32_21
 0010:00058780       EM86LOADTR
 0010:0005879C       VDHINSTALLFAULTHANDLER
 0010:000587B0       LHFREEPAGES
 0010:0005887F       VDHFREEMEM
 0010:000588D5       VDHALLOCUSERMEM
 0010:0005890F       VDHFREEUSERMEM
 0010:00058927       VDHQUERYUSERMEM
 0010:00058943       VDHSETUSERMEM
 0010:00058961       VDHQUERYARENA
 0010:00058978       VDHSETMAXFILEHANDLES
 0010:00058990       CLOSEVDD
 0010:00058A40       VDHFREEPAGES
 0010:00058B34       _StartSWAP32_22
 0010:00058B34       DEMOPENFILE
 0010:00058B34       _EndSWAP32_21
 0010:00058BD4       DEMCLOSEFILE
 0010:00058C04       DEMREADFILE
 0010:00058C50       DEMSEEKFILE
 0010:00058C94       demGetBaseName
 0010:00058D0C       demOpen
 0010:00058DC9       demOpenAsciiz
 0010:00058DDF       demOpenLabel
 0010:00058E87       demParseLabel
 0010:00058F44       DemOpen_CDROM_hack
 0010:00058FE8       demSetDefaultDrive
 0010:00058FF0       demSetDTA
 0010:00059010       demWrite
 0010:00059014       demfile2$demDoIO
 0010:000590A0       demClose
 0010:00059104       dem_handle_Close
 0010:00059114       demMakeFcb
 0010:00059158       g_demMapSeg
 0010:0005915D       demMapSeg
 0010:0005916C       demSetEAField
 0010:000591D8       demIOCTL
 0010:00059210       VDHGETCODEPAGEFONT
 0010:0005941C       VDHRELEASECODEPAGEFONT
 0010:00059434       demnls$demSeekRead
 0010:00059480       demQueryCurrentDir
 0010:000594A0       demSetCurrentDir
 0010:000594B0       demGeneric
 0010:000597AC       _StartSWAP32_23
 0010:000597AC       _PGInitVDMContext
 0010:000597AC       _EndSWAP32_22
 0010:000598BD       _PGAllocSizeQuery
 0010:00059A1C       _PGQueryState
 0010:00059B04       _SELCheckAccess
 0010:00059BAE       _SELSuBuff
 0010:00059C10       _VMCopy
 0010:00059CC8       DEMTRANSPATH
 0010:00059D38       DEMNOINHERITFILE
 0010:00059D88       DEMSETPTDAFILESCOUNT
 0010:00059DBC       demDupJFT
 0010:00059E60       demRead
 0010:00059E6C       demChgFilePtr
 0010:00059EA0       demioc2$demiocGetDevData
 0010:00059EC8       demiocErrorExit
 0010:00059ECC       demExtHandle
 0010:00059EF0       demInitNLS
 0010:00059F1C       demSetCodePage
 0010:0005A010       demnls$demGetCodePageInfo
 0010:0005A10C       demnls$demReadCountryFile
 0010:0005A2D8       demnls$demGetCountryCDIB
 0010:0005A310       demnls$demSearchCDIB
 0010:0005A35C       demnls$demCopyCDIB2
 0010:0005A378       demnls$demCopyCDIB
 0010:0005A394       demGetVersion
 0010:0005A3B0       demSpecialEntries
 0010:0005A3F8       demsvc$demSetV86KernelAddr
 0010:0005A420       demsvc$demGetVisDrv
 0010:0005A44C       demsvc$demSetWriteVerify
 0010:0005A454       demsvc$demVplCallibrate
 0010:0005A480       demsvc$demGetLogicalDriveCnt
 0010:0005A48C       VDHSETDOSDEVICE
 0010:0005A4CC       em86opINB
 0010:0005A57C       em86opOUTB
 0010:0005A5BC       em86opOUTW
 0010:0005A630       EM86BYTEINPUT
 0010:0005A634       EM86BYTEOUTPUT
 0010:0005A638       VDHDETECTPROCESSOR
 0010:0005A6C4       VDHCREATESEM
 0010:0005A700       VDHSETTIMER0
 0010:0005A710       _VR32OpenVDD
 0010:0005A77E       VDMMOPENVDD
 0010:0005A7C4       VDMMPROCCREATEDONE
 0010:0005A7E4       _VDMMApiCreateVDM
 0010:0005A8F0       VDMMCREATEVDM
 0010:0005AB93       VDMMINITINSTANCE
 0010:0005AC12       VDMMCOPYPROPERTIES
 0010:0005AC5E       VDMMSTRDUP
 0010:0005AD36       VDMMFREETEMPBLOCKS
 0010:0005AD5D       VDMMINITDOSHEAP
 0010:0005AD78       VDMMFILLHOLES
 0010:0005AE02       VDMMINITUNDOLIST
 0010:0005AE28       VDMMADDUNDOITEM
 0010:0005AE80       LHCREATE
 0010:0005AEC0       LHCOPYLA
 0010:0005AF86       LHALLOCPAGE
 0010:0005B149       LHCREATERECORD
 0010:0005B1F7       LHCHECKFORINSTALLFAULT
 0010:0005B297       LHFINDFREEMEM
 0010:0005B38E       VDHALLOCMEM
 0010:0005B414       VDHALLOCDOSMEM
 0010:0005B4B4       VDHCOPYMEM
 0010:0005B658       VDMMCOPYMVDMINSTANCE
 0010:0005B72A       VDMMCOPYVDDINSTANCE
 0010:0005B7C3       VDMMACTUALCOPY
 0010:0005B94B       VDMMCREATESEL
 0010:0005BA00       VDHPUTSYSVALUE
 0010:0005BA9E       VDMMSTRCMPI
 0010:0005BB00       OPENVDD
 0010:0005BC07       VDMMGETVALUEFROMSTRING
 0010:0005BC89       VDMMVALIDATESTRING
 0010:0005BCF8       VDHALLOCPAGES
 0010:0005BF28       VDHFINDFREEPAGES
 0010:0005BFCC       VDHQUERYFREEPAGES
 0010:0005BFEC       VDHRESERVEPAGES
 0010:0005C09D       VDHINSTALLFAULTHOOK
 0010:0005C257       CREATEPFH
 0010:0005C2AC       _vdmCreatePropertyInstance
 0010:0005C50F       _vdmSetPropertyInstance
 0010:0005C51E       _vdmQueryProperty
 0010:0005C5FB       VDHQUERYPROPERTY
 0010:0005C6C1       _VR32QueryDOSProperty
 0010:0005C7AC       _queryPropertyDetail
 0010:0005C8FD       _PROPFindNameOrOrdinal
 0010:0005C961       _PROPFind
 0010:0005C9AB       _PROPFindOrdinal
 0010:0005C9D7       _PRINFind
 0010:0005C9F9       _clearScanBits
 0010:0005CA1C       _swpAlloc
 0010:0005CA4F       _swpStrDup
 0010:0005CA9C       _TKCreateVDMProcess
 0010:0005CBB8       _VRCreateThread
 0010:0005CC5C       g_ldrVersionLie
 0010:0005CC90       DEMCREATEVDM1
 0010:0005CD85       DEMCREATEVDM2
 0010:0005D252       DEMMAKEFAKELIST
 0010:0005D3CF       DEMGETAPPNAME
 0010:0005D475       DEMGETNUMBER
 0010:0005D563       DEMPROCESSENTRIES
 0010:0005D5C4       VDMMENTERCREATEVDM
 0010:0005D614       VDMMEXITCREATEVDM
 0010:0005D6A0       _vdmmStart
 0010:0005D711       VDMM_IRETD
 0010:0005D74C       EM86CREATEVDM
 0010:0005DAE2       VDHINSTALLINTHOOK
 0010:0005DC97       VDHARMBPHOOK
 0010:0005DD12       VDHREGISTERAPI
 0010:0005DE30       demOpenSem
 0010:0005DE3F       DEM32OPENEVENTSEM
 0010:0005DE54       _EndSWAP32_23
 0010:0005DE54       _SELFreeVdmSels
 0010:0005DE54       _StartSWAP32_24
 0010:0005DF78       demsvc$demGetVplAddr
 0010:0005DF9C       em86PopVPMIRET
 0010:0005E0E4       em86opCLI
 0010:0005E13C       em86opINBimm
 0010:0005E1A8       em86opOUTBimm
 0010:0005E1DC       em86io$em86CallPortHdlr
 0010:0005E1EF       em86io$em86CallIOH
 0010:0005E234       EM86SIMWORDOUTPUT
 0010:0005E254       EM86CHOOKSTUBBIH
 0010:0005E2AC       EM86CHOOKSTUBBOH
 0010:0005E308       VDHSWITCHTOVPM
 0010:0005E3B0       VDHSWITCHTOV86
 0010:0005E474       _em86LoadVPMIDT
 0010:0005E480       EM86MEMCPY
 0010:0005E4A4       VDHOPENVDD
 0010:0005E4BA       VDHCLOSEVDD
 0010:0005E4EC       VDHCREATESEL
 0010:0005E556       VDHDESTROYSEL
 0010:0005E58C       VDHGETSELBASE
 0010:0005E60D       VDHCHANGEVPMIF
 0010:0005E666       VDHREADUBUF
 0010:0005E778       VDHWRITEUBUF
 0010:0005E88B       VDHSTARTHWINT
 0010:0005E909       VDHCHECKVPMINTVECTOR
 0010:0005E958       VDHGETVPMINTVECTOR
 0010:0005E99F       VDHBEGINUSEVPMSTACK
 0010:0005E9F8       VDHENDUSEVPMSTACK
 0010:0005EA44       _ldrIsInternalFixup
 0010:0005EB48       EM86ReflectVPMInt
 0010:0005ECE0       EM86VPMINTBPHDLR
 0010:0005ECFC       EM86VPMINT2FHDLR
 0010:0005ED4C       EM86VPMINT31HDLR
 0010:0005ED54       EM86V86REFLECTIONHOOK
 0010:0005ED60       VDHPUSHFARCALL
 0010:0005EE18       _SELSwitchVdmLDT
 0010:0005EE18       _EndSWAP32_24
 0010:0005EE18       _StartSWAP32_25
 0010:0005EED3       _SELPrintVdmLdt
 0010:0005EF14       demFileTimes
 0010:0005EF56       DemTouchHack
 0010:0005F024       demFindFirst
 0010:0005F07C       demFindNext
 0010:0005F09C       dff_2ndpass
 0010:0005F134       demChMod
 0010:0005F164       demGetLin
 0010:0005F174       demioc2$demiocRemovableMedia
 0010:0005F200       demCDRom
 0010:0005F254       demioc2$demiocRedirBlock
 0010:0005F2A4       demioc2$demiocGetLogDrive
 0010:0005F2B2       demiocSetLogDrive
 0010:0005F2B4       demiocLogDrive
 0010:0005F330       demGetDriveInfo
 0010:0005F35C       em86inst$em86opMOVSeg
 0010:0005F3E0       _em86UpdateIDT
 0010:0005F4A0       VDHREAD
 0010:0005F564       VDHSEEK
 0010:0005F5CC       _VR32CloseVDD
 0010:0005F5E9       VDMMCLOSEVDD
 0010:0005F620       VDMMVPMBEGINEND
 0010:0005F650       _vdmmSetTitle
 0010:0005F6C4       VDHSETVPMEXCEPT
 0010:0005F718       VDHSETVPMINTVECTOR
 0010:0005F7B0       EM86REFLECTEXCEPTION
 0010:0005F7BD       EM86ReflectVPMException
 0010:0005F9E8       EM86VPMINT21HDLR
 0010:0005FA0C       EM86VPMEXCRETHOOK
 0010:0005FADC       _StartSWAP32_26
 0010:0005FADC       _SELCreateVdmLDT
 0010:0005FADC       _EndSWAP32_25
 0010:0005FB6D       _SELAllocVdmSels
 0010:0005FEF3       _SELGetVdmInfo
 0010:0005FF18       jft_dup_OS2_handle
 0010:0005FF74       em86inst$em86GetValidSel
 0010:0005FFB4       EM86DEFAULTOUTWORDHOOK
 0010:0005FFD0       EM86DEFAULTIOINHOOK
 0010:0005FFE4       EM86DEFAULTIOOUTHOOK
 0010:0005FFF4       em86DefaultIOHook
 0010:00060020       em86io$em86IsPortHooked
 0010:0006009C       _em86Is32Sel
 0010:000600B8       EM86STARTVPMEXECUTION
 0010:000601B2       _int2fGetVPMSwitchAddr
 0010:00060266       VPMINITDATA
 0010:0006036C       _em86AllocLDTIDT
 0010:000605C2       _em86AllocVPM
 0010:000607A6       _em86AllocSel
 0010:00060807       EM86GETPSP
 0010:00060868       _int2fChain
 0010:0006086D       _int2fGetVDDAPI
 0010:000609FC       VDMMALLOCTEMPBLOCK
 0010:00060A40       _vdmmGetTitle
 0010:00060A80       _getValue
 0010:00060BF2       _checkPSZ
 0010:00060C26       _findEnum
 0010:00060C72       _putBytes
 0010:00060CAF       _queryPropertyValue
 0010:00060D98       VDHGETVPMEXCEPT
 0010:00060DE8       VDHARMVPMBPHOOK
 0010:00060E9A       VDHPROBEUBUF
 0010:00060F95       VDHPOPVPMFARRET
 0010:00060FE8       demSetTitle
 0010:00060FF4       _EndSWAP32_26
 0010:00060FF4       _StartSWAP32_27
 0010:00060FF4       _PGFreeContext
 0010:00061181       _PGRemapUvirt
 0010:0006120C       _pgwRemapUvirt
 0010:00061280       _SELQueryFreeAlias
 0010:00061328       _SELRemDiscRec
 0010:000613C8       _vmFreeObjectAliases
 0010:000614BD       _vmHasDebugAlias
 0010:000615B4       _vmFreeArena
 0010:0006162B       _VMFreeTask
 0010:0006178A       _vmFreeAll
 0010:00061974       _VMFreePseudoHandle
 0010:000619D4       demTerminate
 0010:000619E8       demsvc$demDosAbort
 0010:00061A04       EM86VPMDESTROYVDM
 0010:00061A28       _em86FreeVPM
 0010:00061B14       VDHSETBOOST
 0010:00061B58       VDHDESTROYSEM
 0010:00061B64       PFNUNDOLA
 0010:00061B9D       PFNUNDOEM86
 0010:00061BA3       PFNUNDOVDD
 0010:00061BC7       PFNUNDOFAULTS
 0010:00061BEB       PFNUNDOFIXEDHEAP
 0010:00061C62       PFNUNDOSWAPHEAP
 0010:00061CD9       VDMMSWITCHBGND
 0010:00061CEC       VDMMSWITCHFGND
 0010:00061CFF       VDMMPDBDESTROY
 0010:00061D10       LHUNRESERVEPAGES
 0010:00061DAC       VDHUNRESERVEPAGES
 0010:00061E40       _vdmDestroyPropertyInstance
 0010:00061E50       _destroyPropInst
 0010:00061E9C       VDMMDISARMTIMERHOOKS
 0010:00061EDC       _tkInheritJIT
 0010:00061F92       _tkLaunchJITSession
 0010:00061FE0       _tkJITProcessLaunchRequest
 0010:00062364       _tkEvapPTDA
 0010:00062410       _tkNextExitListRoutine
 0010:0006293A       _tkCleanUpExitList
 0010:00062960       _VRExit
 0010:00062974       _tkFreeUserStacks
 0010:00062A26       _tkFreeTSD
 0010:00062A78       _LDRFreeTask
 0010:00062AF8       _ldrBlastDLDRecord
 0010:00062B33       _ldrDecDLDRecord
 0010:00062BB8       _VRFreeModule
 0010:00062BC9       _LDRFreeModule
 0010:00062E42       _LDRDLLExitList
 0010:00062F3C       DEMDESTROYVDM1
 0010:00062FC8       DEMDESTROYVDM2
 0010:00062FDD       DEMDESTROYFAKELIST
 0010:0006300C       VDMMENTERTERMINATEVDM
 0010:00063038       VDMMEXITTERMINATEVDM
 0010:00063070       EM86DESTROYVDM
 0010:0006326C       demCloseSem
 0010:00063289       DEM32CLOSEEVENTSEM
 0010:0006329C       _XCPTCheckExceptionHandler
 0010:00063364       _EndSWAP32_27
 0010:00063364       _selAllocPhys
 0010:00063364       _StartSWAP32_28
 0010:00063427       _SELDestroyVdmLDT
 0010:00063484       _dhw_VMAlloc
 0010:00063744       demExtInfo
 0010:00063764       demFindFirstFCB
 0010:000637B8       demGetDriveFreespace
 0010:00063818       demNameTrans
 0010:00063830       demsvc$demQueryDate
 0010:00063850       demsvc$demQueryTime
 0010:00063868       EM86ENDVPMEXECUTION
 0010:00063959       VPMFREETASKRESOURCES
 0010:00063A2A       _em86FreeLDTIDT
 0010:00063AC8       VDHWRITE
 0010:00063AD4       demDelete
 0010:00063B49       DemQuickenHack
 0010:00063BF0       demGSetMediaID
 0010:00063C08       _StartLOAD_TUNE1_SWP
 0010:00063C08       _w_SetExtLIBPATH
 0010:00063C08       _EndSWAP32_28
 0010:00063C08       _EndLOAD_TUNE1_SWP
 0010:00063C08       _StartLOAD_TUNE4_SWP
 0010:00063C97       _w_nt_SetExtLIBPATH
 0010:0006414E       _w_QueryExtLIBPATH
 0010:0006421E       _ldrFreeMTEFixups
 0010:00064324       _ldrBlastResource
 0010:000643D8       _EndLOAD_TUNE8_SWP
 0010:000643D8       _StartLOAD_TUNE9_SWP
 0010:000643D8       _StartLOAD_FTUNE2_SWP
 0010:000643D8       g_PrefLookupMFT
 0010:000643D8       _StartLOAD_FTUNE1_SWP
 0010:000643D8       _StartLOAD_TUNE8_SWP
 0010:000643D8       _EndLOAD_TUNE4_SWP
 0010:000643D8       _EndLOAD_FTUNE2_SWP
 0010:000643D8       _EndLOAD_TUNE9_SWP
 0010:000643DD       PrefLookupMFT
 0010:0006449C       _ldrAllocSegments
 0010:0006484C       _ldrAllocSegment
 0010:00064DD6       _ldrSegment
 0010:000656F0       _ldrGetHugeSel
 0010:0006586C       _ldrPreloadLDT
 0010:0006595A       _ldrExpandSegment
 0010:00065AE8       ldrrsrc$g_IsHugeRsrc
 0010:00065AED       ldrrsrc$IsHugeRsrc
 0010:00065B48       _ldrProcessRsrcSeg
 0010:00065BB8       _ldrGetRsrcSel
 0010:00065C00       _ldrFreeHuge
 0010:00065C78       _EndLOAD_FTUNE1_SWP
 0010:00065C78       _StartLOAD_TUNEDIT1_SWP
 0010:00065C78       _PGPreload
 0010:00065D55       _pgwPreload
 0010:00065EEC       SELLoadSegment
 0010:00065F20       _SELValidateLoaded
 0010:00065F50       selwrk$g_selUnlockSeg
 0010:00066000       selwrk$g_selLockSeg
 0010:000660A4       selwrk$selValidateLockSeg
 0010:00066128       _LDRGetSegment
 0010:00066230       _ldrLoadSegment
 0010:0006630C       ldrLoadSegment
 0010:00066698       load_iterated_data
 0010:0006684C       clear_segment
 0010:0006686C       dofixups
 0010:0006690C       fixup
 0010:000669E8       _ldrEditProLog
 0010:00066B0A       _ldrInitEntry
 0010:00066BAC       _ldrSegFixOpenRec
 0010:00066C09       _ldrSegFixAddRecord
 0010:00066DE4       _ldrSegFixStopChain
 0010:00066E12       _ldrSegFixCloseRec
 0010:0006704F       _segfix_ReallocBlock
 0010:000670DC       _load_error
 0010:00067109       _ldrWriteErrTxt
 0010:0006734C       _ldrCopyName
 0010:000673C0       PLDENTERCRITSEC
 0010:000673C0       _EndLOAD_TUNEDIT1_SWP
 0010:000673C0       _StartLOAD_TUNEDOS12_SWP
 0010:000673C0       _EndLOAD_TUNEDOS5_SWP
 0010:000673C0       _StartLOAD_TUNEDOS5_SWP
 0010:000673DC       PLDEXITCRITSEC
 0010:000673F8       _PLD_WaitDumpComplete
 0010:0006740C       _EndLOAD_TUNEDOS11_SWP
 0010:0006740C       _EndLOAD_TUNEDOS12_SWP
 0010:0006740C       VDHREGISTERVDD
 0010:0006740C       _StartLOAD_TUNEDOS11_SWP
 0010:0006740C       _StartLOAD_TUNEDOS4_SWP
 0010:00067570       VDHINSTALLUSERHOOK
 0010:00067668       VDMMFREEVDDEP
 0010:000676EC       PLDGETVERSTRING
 0010:0006770C       _EndLOAD_EXITDOS1_SWP
 0010:0006770C       _StartLOAD_BEEP_SWP
 0010:0006770C       _w_Beep
 0010:0006770C       _EndLOAD_TUNEDOS4_SWP
 0010:0006770C       _StartLOAD_EXITDOS1_SWP
 0010:000677E7       _BeepOpen
 0010:00067845       _BeepGetTaskID
 0010:00067860       _StartEXMGSWAP_TEXT
 0010:00067860       _EndLOAD_BEEP_SWP
 0010:00067860       _xcptFormatAndSendHardErr
 0010:00067864       _xcptStackOverRun
 0010:0006786B       _xcptFatalDispatchError
 0010:00067C58       xcptmisc$ClearRegDump
 0010:00067C6C       xcptmisc$ClearLimAccDump
 0010:00067C84       _xcptQueryFPState
 0010:00067CA4       _VR32IRaiseException
 0010:00067DFB       _xcptRestoreFPState
 0010:00067F6C       _VRQueryRASInfo
 0010:00067F6C       _EndEXMGSWAP_TEXT
 0010:00067F6C       _StartTKSWAP_TEXT
 0010:00068242       _PLD_QueryInfo
 0010:000684B3       _PLD_CollectOptions
 0010:00068577       _PLD_CollectPDProcess
 0010:00068750       _PLD_CollectPDIProcess
 0010:000688C0       _RAS_QueryTrace
 0010:00068B53       _RAS_CollectStatic
 0010:00068E7B       _RAS_StaticMajor
 0010:00068F2E       _RAS_StaticGetMinor
 0010:00069573       _RAS_StaticMinor
 0010:00069607       _RAS_CollectPIDs
 0010:00069710       _RAS_SavePtdaPids
 0010:00069738       _RAS_CollectPNames
 0010:0006986B       _RAS_CollectDynamic
 0010:00069931       _RAS_QuerySDump
 0010:000699CC       _TKCreateVDMThread
 0010:00069A6C       _tkDeleteExitListRoutine
 0010:00069AE2       _TKCheckExitListRef
 0010:00069BBC       _VRResumeThread
 0010:00069BCB       _VRSuspendThread
 0010:00069BDC       _TKLibiError
 0010:00069BED       _TKLibiCheckRef
 0010:00069C22       _tkLibiCheckReference
 0010:00069C98       _TKLibiSetupUnload
 0010:00069CF5       _TKLibiRecordUnload
 0010:00069D35       _TKLibiUnloadDone
 0010:00069D6C       _TKLibiDbgNextDLL
 0010:00069DFA       _TKLibiDbgDone
 0010:00069E68       _tkGetLibiDispatcherAddr
 0010:00069ED8       _tkIThrdRetError
 0010:00069EF1       _VR32KillThread
 0010:00069FA6       _VR32WaitThread
 0010:00069FF2       _TKUpdateLocalFPHandler
 0010:0006A05F       _VR32QueryThreadContext
 0010:0006A434       _VR32DumpProcess
 0010:0006A88C       _PLD_ValidateRequest
 0010:0006A95F       _PLD_ValidateRequestFlags
 0010:0006A9D9       _PLD_ValidatePathname
 0010:0006AA66       _PLD_ValidateOptions
 0010:0006AB96       _PLD_ValidateNewProcessList
 0010:0006AC94       _PLD_CheckDuplicatedProcess
 0010:0006AD0E       _PLD_CheckDuplicatedIProcess
 0010:0006AD7C       _PLD_ValidateNewIProcessList
 0010:0006AE35       _PLD_ValidateProcess
 0010:0006AF52       _PLD_ValidateProcessCount
 0010:0006AF7D       _PLD_ValidateProcCleanUp
 0010:0006AFA4       _PLD_ValidateIProcess
 0010:0006B07C       _PLD_CheckProcData
 0010:0006B110       _PLD_CheckIProcData
 0010:0006B1A6       _PLD_CleanUpAPIProc
 0010:0006B210       _PLD_CleanUpAPIIProc
 0010:0006B25F       _PLD_ValidatePacketInfo
 0010:0006B316       _PLD_SetProcesses
 0010:0006B642       _PLD_GetEndProcess
 0010:0006B65F       _PLD_CleanUpAPI
 0010:0006B703       _PLD_DDPGetStorage
 0010:0006B752       _PLD_SetDefaults
 0010:0006B849       _PLD_ResetDefaults
 0010:0006B899       _PLD_ResetProcesses
 0010:0006B9BD       _PLD_DeleteIProcess
 0010:0006BA12       _PLD_FindMatchProcess
 0010:0006BA65       _PLD_FindMatchIProcess
 0010:0006BAB8       _VR32SuppressPopUps
 0010:0006BB28       _PDLogPopUp
 0010:0006BD64       _PLD32ApiDump
 0010:0006C70E       _PLD_HotKey
 0010:0006C7A3       _PLD_Ring0Trap
 0010:0006C866       _PLD_Ring3Trap
 0010:0006C8F8       _PLD_DynTrace
 0010:0006C9A4       _PLD_DeterminePids
 0010:0006CADD       _PLD_CheckActiveProcesses
 0010:0006CD0F       _PLD_CheckDLL
 0010:0006CE27       _PLD_UpdateTable
 0010:0006CEC1       _PLD_FindMTEFromImports
 0010:0006CF1F       _PLD_GetShortMTEName
 0010:0006CF8F       _PLD_CompareNames
 0010:0006D199       _PLD_FindNameFromPath
 0010:0006D1F0       _PLD_Cleanup
 0010:0006D428       _PLD_AllocPidTable
 0010:0006D4A1       _PLD_AddPidToTable
 0010:0006D527       _PLD_GetPidRec
 0010:0006D571       _PLD_FindFirstPidRec
 0010:0006D5CE       _PLD_FindNextPidRec
 0010:0006D676       _PLD_FreeTables
 0010:0006D69C       _PLD_FindMTEFromName
 0010:0006D81D       _PLD_BlastCircRefBit
 0010:0006D833       _PLD_FindSecondary
 0010:0006D9AE       _PLD_GetParents
 0010:0006DA43       _PLD_GetChildren
 0010:0006DAF1       _PLD_FindOptions
 0010:0006E00C       _PLD_CopyOptions
 0010:0006E2EF       _PLD_FindPids
 0010:0006E45E       _PLD_AddDDRanges
 0010:0006E794       _PLD_WriteSMTEInfo
 0010:0006E813       _PLD_WriteSMTEInfoForImports
 0010:0006E861       _PLD_WriteMTEs
 0010:0006E914       _PLD_WriteLDR
 0010:0006E9A8       _PLD_WriteSYSLDR
 0010:0006E9E7       _PLD_WriteMem_IgnoreUncommitedPages
 0010:0006EA3F       _PLD_WriteArenaHeaders
 0010:0006EA58       _PLD_WriteSYSVM
 0010:0006EC13       _PLD_WriteSYSIO
 0010:0006ED82       _PLD_WritePgdataInfo
 0010:0006EF03       _PLD_WritePerProcessPgdataInfo
 0010:0006EF1A       _PLD_WriteSYSPG
 0010:0006F09F       _PLD_WritePMDFMem
 0010:0006F149       _PLD_WriteSYSMVDMWorker
 0010:0006F15D       _PLD_WriteSYSMVDM
 0010:0006F1B0       _PLD_WriteMVDMCommon
 0010:0006F2D4       _PLD_WriteMVDM
 0010:0006F3A6       _PLD_Quiesce
 0010:0006F468       _PLD_WriteTRACE
 0010:0006F4FA       _PLD_WriteSTRACE
 0010:0006F55F       _PLD_WriteSYSSUMMWorker
 0010:0006F570       _PLD_WriteSYSSUMM
 0010:0006F5A7       _PLD_WriteSYSTKWorker
 0010:0006F606       _PLD_WriteSYSTK
 0010:0006F63D       _PLD_Write3CodePages
 0010:0006F6F8       _PLD_Write3DataPages
 0010:0006F73D       _PLD_WriteRegContext
 0010:0006F8A2       _PLD_WriteReturnCode
 0010:0006FAA1       _PLD_WriteSUMM
 0010:0006FB69       _PLD_WriteSYSSEMWorker
 0010:0006FB7A       _PLD_WriteSYSSEM
 0010:0006FBB1       _PLD_WriteSEM
 0010:0006FCD0       _PLD_WriteTK
 0010:000700BF       _PLD_WriteSysRequired
 0010:00070217       _PLD_WriteRequired
 0010:0007025A       _PLD_WriteTSS
 0010:000702A0       _TKSuspendThread
 0010:000702F0       _TKResumeThread
 0010:00070388       tksubr$tkNewPidWorker
 0010:000703E4       _PLD_WriteMem
 0010:00070624       _PLD_MapPrivate
 0010:0007085E       _PLD_WritePhysMem
 0010:0007096F       _PLD_WriteDumpRec
 0010:000709C1       _PLD_CheckFreeSpace
 0010:00070A82       _PLD_WriteSYSFS
 0010:00070D47       _PLD_WriteMFT
 0010:00070D5C       _PLD_WriteKHEAPS
 0010:00070E3C       _PLD_WriteADDR
 0010:00070FC5       _PLD_WriteDefaults
 0010:00071127       _PLD_WritePathName
 0010:000711F3       _PLD_WriteProcReq
 0010:0007145F       _PLD_WriteProcColl
 0010:00071610       _PLD_CreateSystemDump
 0010:00071800       _PLD_CreateHeader
 0010:000718EE       _PLD_WriteHeader
 0010:00071965       _PLD_InitBM
 0010:00071A14       _PLD_ResetPrivateBM
 0010:00071A35       _PLD_WriteSAB
 0010:00071A71       _PLD_WriteGDT
 0010:00071A96       _PLD_WriteIDT
 0010:00071AB4       _PLD_WritePRIVATE
 0010:00071B88       _StartLDRSWAP_TEXT
 0010:00071B88       _EndTKSWAP_TEXT
 0010:00071B88       ldrinita$g_lfirest
 0010:00071B88       lfirest
 0010:00071BB4       _ldrIsPath
 0010:00071C24       _ldrStop
 0010:00071C68       _LDRIsMTEDetaching
 0010:00071C9B       _ldrGarbageCollect
 0010:00071D91       _ldrLibDetach
 0010:00071DB5       _ldrLibDetachSub
 0010:00071F78       _ldrFreeMTE
 0010:000723C8       _ldrFindDetach
 0010:000724B5       _ldrRecordDLLTerm
 0010:00072511       _ldrEnumDLLTerm
 0010:0007259B       _ldrRunGraph
 0010:000725DC       _ldrReloadSeg
 0010:00072691       _ldrGetPages
 0010:00072A62       _ldrUseDataCache
 0010:00072ACA       _ldrMakeDataCache
 0010:00072C4C       ldrGDTPreload
 0010:00072CB0       _LDRNumtoAddr
 0010:00072D52       _LDRTstnClrSem
 0010:00072D84       _LDRGetModuleType
 0010:00072E20       _VRDosQueryABIOSSupport
 0010:00072E28       _VRDosQueryModFromEIP
 0010:00073005       _VRDosQueryModFromCS
 0010:000731D8       _LDRGetDYNMteInfo
 0010:00073384       _ldrGetContextSub
 0010:000733A4       _LDRGetContext
 0010:0007343E       _VR32QueryResourceSize
 0010:00073593       _VR32QueryHeaderInfo
 0010:00073914       _VR32InitializePorthole
 0010:0007391F       _ldrAllocDD
 0010:00073A19       _LDRReallocDD
 0010:00073AA5       _LDRReallocDD2
 0010:00073B1F       _LDRCleanupDLLTerm
 0010:00073C23       _ldrDispatchDLLTerm
 0010:00073EC7       _ldrSetupDLLTerm
 0010:00073FA0       _VR32DLLTerm
 0010:00073FD8       _VR32ICacheModule
 0010:0007409C       _ldrForceResModule
 0010:000741CF       _ldrRegisterDLLTerm
 0010:00074200       _VRLdrDirtyWorker
 0010:00074212       _Ldr32DirtyWorker
 0010:00074274       _segfix_FreeTempFixups
 0010:000742E4       _ldrSegFixAddIterRec
 0010:000743F0       _ldrSegFixLoadIterated
 0010:00074634       _ReadIterations
 0010:000746E0       _ldrSegFixFixupPage
 0010:0007480C       _ldrNoMemGetOrdNum
 0010:00074932       _ldrGetGate
 0010:0007497F       _ldrMapOrdinal
 0010:000749AC       _ldrFreeCallGate
 0010:00074A39       _ldrFreeLDTGate
 0010:00074AE0       _ldrUnlinkMTE
 0010:00074BFA       _ldrPromoteMTE
 0010:00074C42       _ldrCheckForWLO
 0010:00074EDB       _LDRUpdateGlobalErrTxt
 0010:00074F00       _LDRGetLibNameToHeap
 0010:00074F70       g_DevhlpAllocGDTSel
 0010:00074F70       _EndLDRSWAP_TEXT
 0010:00074F70       _StartSELSWAP_TEXT
 0010:00075108       g_DevhlpFreeGDTSel
 0010:00075264       selmgra$selBaseAll
 0010:000752A0       selmgra$selBaseAllAlias
 0010:00075364       _SELReserveLDT
 0010:000754D8       _SELFreeLDT
 0010:0007561B       _SELFuBuff
 0010:0007567B       _SELFreeTaskLDT
 0010:0007579A       _selFreePhys
 0010:000757F6       _SELClearPreload
 0010:0007581E       _selGiveSeg
 0010:00075978       selCheckAllocParms
 0010:000759B4       _selIfsSegRealloc
 0010:000759DC       SegCheck
 0010:00075A4C       _SELIfsAlloc
 0010:00075B3B       _SELIfsFree
 0010:00075C6E       _SELIfsRealloc
 0010:00075D32       _SELIfsNoSwap
 0010:00075EC8       _EndSELSWAP_TEXT
 0010:00075EC8       _vmAliasToAlias
 0010:00075EC8       _StartVMSWAP_TEXT
 0010:00076001       _vmChangeAlias
 0010:0007615C       _vmHasDiscardablePages
 0010:000761BC       _VMMapDebugAlias
 0010:0007652C       _VMGetAliasOffset
 0010:000765AC       _VMReserveMem
 0010:000766C4       _VR32AliasMem
 0010:0007675C       _VR32AllocProtectedMem
 0010:0007681F       _VR32QueryMemState
 0010:000768E0       _VR32QueryPageUsage
 0010:00076DEA       _VM32ApiAliasMem
 0010:00076F16       _VM32ApiQueryMemState
 0010:00076F7F       _VR32IFreeThreadLocalMemory
 0010:00077074       _VR32ISysCtl
 0010:000773AC       _BMPInit
 0010:000774C4       _dhw_VMProcessToGlobal
 0010:00077560       _dhw_VMSetMem
 0010:000777D0       _VMFreeMemOb
 0010:00077824       _StartPGSWAP_TEXT
 0010:00077824       _PGMove
 0010:00077824       _EndVMSWAP_TEXT
 0010:00077BC0       _PGSetType
 0010:00077CC1       _PGDiscToSwap
 0010:00077D20       _pgwDiscToSwap
 0010:00077D68       _pgwDiscToZFill
 0010:00077DB1       _pgwSwapToRes
 0010:00077E95       _pgwResToSwap
 0010:00077F0E       _PGGetAccess
 0010:00077F6E       _pgwGetAccess
 0010:00077F8C       _StartMVDMSWAP_TEXT
 0010:00077F8C       DEMSETCDS
 0010:00077F8C       _EndPGSWAP_TEXT
 0010:00077FD8       demFCBOpen
 0010:000781D0       demFCBClose
 0010:00078300       demFCBLength
 0010:00078310       demFCBIO
 0010:00078320       demCopyEAs
 0010:000783C4       demCreateNew
 0010:000783D4       demCreateTemp
 0010:000783E4       demDiskReset
 0010:000783F0       demLockOper
 0010:00078410       demFindNextFCB
 0010:00078464       dem_FFHack
 0010:000784E4       demDup
 0010:000784FC       demCommit
 0010:00078508       demEnumAttrib
 0010:00078524       demQMaxEASize
 0010:000785CC       demMapSegFixup
 0010:000785E4       g_demMapSegLenCX
 0010:000785E9       demMapSegLenCX
 0010:000785FC       demiocQueryHandle
 0010:000785FC       demiocQueryBlock
 0010:000785FC       demioc2$demiocInvalidFunction
 0010:000785FC       demiocSetDevData
 0010:00078604       demioc2$demiocOutputStatus
 0010:00078604       demioc2$demiocInputStatus
 0010:00078688       demioc2$demiocReadHandle
 0010:0007868C       demioc2$demiocWriteHandle
 0010:0007868E       demioc2$demiocReadWriteHandle
 0010:000786BE       demioc2$demiocReadBlock
 0010:000786C7       demioc2$demiocWriteBlock
 0010:000786C9       demioc2$demiocReadWriteBlock
 0010:000786DB       demioc2$demiocReadWrite
 0010:0007875D       demioc2$demiocMapErr
 0010:00078770       demioc2$demiocRedirHandle
 0010:000787BC       demioc2$demiocSetRetries
 0010:000787E0       demioc2$demiocGenericHandle
 0010:00078850       demioc2$demiocGenericBlock
 0010:00078900       demGetDPB
 0010:00078910       demAbsDrd
 0010:00078918       demAbsDwrt
 0010:00078980       demGetCountryInfo
 0010:000789A4       demQNMPInfo
 0010:000789D4       demQNMPHandState
 0010:000789E0       demSetNMPHandState
 0010:000789F0       demPeekNMP
 0010:00078A5C       demTransactNMP
 0010:00078AB4       demCallNMP
 0010:00078B6C       demWaitNMP
 0010:00078B88       demRawReadNMP
 0010:00078BD0       demRawWriteNMP
 0010:00078C0C       demInternalError
 0010:00078C9C       demsvc$demSetDate
 0010:00078CDC       demsvc$demSetTime
 0010:00078D5C       demsvc$demGetCDS
 0010:00078DA0       demsvc$demGetSFT
 0010:00078E6C       demsvc$demBlockDD
 0010:00078E70       demsvc$demYield
 0010:00078E78       demsvc$demJSA
 0010:00078E94       demGetMessage
 0010:00078EC4       VDHGetFlags
 0010:00078F18       EM86GETFLAGS
 0010:00078F64       em86opPUSHF
 0010:00078FC0       EM86POPF16
 0010:00079004       em86opPOPF
 0010:00079011       em86if$em86POPF16Entry
 0010:00079078       em86opIRET
 0010:00079096       em86IRET16
 0010:00079120       EM86SETFLAGS
 0010:00079264       em86inst$em86opLOCKPrefix
 0010:00079264       em86inst$em86opGenericPrefix
 0010:00079278       em86inst$em86opREPPrefix
 0010:00079284       em86inst$em86opREPNEPrefix
 0010:00079290       em86inst$em86opCSPrefix
 0010:0007929C       em86inst$em86opDSPrefix
 0010:000792A8       em86inst$em86opESPrefix
 0010:000792B4       em86inst$em86opSSPrefix
 0010:000792C0       em86inst$em86opFSPrefix
 0010:000792CC       em86inst$em86opGSPrefix
 0010:000792D8       em86inst$em86opOPER32Prefix
 0010:000792E4       em86inst$em86opADDR32Prefix
 0010:0007930C       em86inst$em86op0F
 0010:0007935C       em86opGPFault
 0010:0007939E       em86opInvalid
 0010:000793E4       em86inst$em86opLMSW
 0010:00079408       em86inst$em86DecodeOperand
 0010:00079614       em86inst$em86opGetCRx
 0010:00079638       em86inst$em86opSetCRx
 0010:00079649       em86inst$em86opSetCR0
 0010:0007968C       em86inst$em86opGetDRx
 0010:00079694       em86inst$em86opSetDRx
 0010:0007969C       em86inst$em86opCLTS
 0010:000796A4       em86inst$em86opLxS
 0010:00079750       em86inst$adjustUserEIP
 0010:00079778       em86inst$em86opPOPSeg
 0010:00079818       em86inst$em86CreateWrtSel
 0010:00079878       em86opINW
 0010:000799A0       em86opINWimm
 0010:00079A7C       em86opOUTWimm
 0010:00079AE4       em86opINSB
 0010:00079AF0       em86opINSW
 0010:00079AFC       em86opOUTSB
 0010:00079B08       em86opOUTSW
 0010:00079B10       em86io$em86StringIO
 0010:00079B78       em86io$em86CallHashPortHdlr
 0010:00079BB8       EM86DEFAULTOTHERIOHOOK
 0010:00079C00       EM86DEFAULTINWORDHOOK
 0010:00079C1C       EM86DEFAULTIGNOREIOHOOK
 0010:00079C20       EM86SIMWORDINPUT
 0010:00079C44       EM86SIMOTHERIO
 0010:00079C5C       em86io$em86SimDwordInput
 0010:00079C80       em86io$em86SimDwordOutput
 0010:00079CA0       em86io$em86SimVPMByteStringInpu
 0010:00079D28       em86io$em86SimVPMByteStringOutp
 0010:00079DC4       em86io$em86SimVPMWordStringInpu
 0010:00079E4C       em86io$em86SimVPMWordStringOutp
 0010:00079EE8       em86io$em86SimVPMDwordStringInp
 0010:00079F70       em86io$em86SimVPMDwordStringOut
 0010:0007A00C       em86io$em86SimByteStringInput
 0010:0007A0BC       em86io$em86SimByteStringOutput
 0010:0007A180       em86io$em86SimWordStringInput
 0010:0007A230       em86io$em86SimWordStringOutput
 0010:0007A2F4       em86io$em86SimDwordStringInput
 0010:0007A3A4       em86io$em86SimDwordStringOutput
 0010:0007A468       em86io$em86SimInvalidType
 0010:0007A47C       EM86SIMDWORDIO
 0010:0007A48C       EM86CSIMDWORDIO
 0010:0007A4A0       EM86CHOOKSTUBWIH
 0010:0007A4F8       EM86CHOOKSTUBWOH
 0010:0007A554       EM86CHOOKSTUBOTH
 0010:0007A5C8       HANDLEEXC
 0010:0007A630       _em86VPMNpxSet
 0010:0007A674       _em86VPMNpxStatus
 0010:0007A6D4       EM86GETCR4
 0010:0007A6D8       EM86SETCR4
 0010:0007A6E8       VDHREGISTERDPMI
 0010:0007A7CF       _em86FreeSel
 0010:0007A7E4       _int2fGetMode
 0010:0007A7F8       VDHWAKERAMSEM
 0010:0007A828       VDHREQUESTRAMSEM
 0010:0007A864       VDHWAITRAMSEM
 0010:0007A89C       VDHOPEN
 0010:0007A9EC       VDHCLOSE
 0010:0007AA20       VDHDEVIOCTL
 0010:0007ABBC       VDHFSCTL
 0010:0007AD98       VDHPHYSICALDISK
 0010:0007AE84       VDHPOPUP
 0010:0007AF04       VDHKILLVDM
 0010:0007AF2C       VDHHALTSYSTEM
 0010:0007AF50       VDHYIELD
 0010:0007AF70       VDHASSERTINITONLY
 0010:0007AF98       VDHASSERTTASK
 0010:0007AFC9       VDHASSERTVDMTASK
 0010:0007B008       VDHASSERTTASKONLY
 0010:0007B030       VDHASSERTVDMTASKONLY
 0010:0007B066       VDHCHECKHVDM
 0010:0007B0C4       LHDESTROY
 0010:0007B0FA       LHUPDATERECORDSTATE
 0010:0007B13B       LHCHECKFORFAULT
 0010:0007B228       LHREALLOCPAGES
 0010:0007B271       LHQUERYRECORD
 0010:0007B2BA       VDHCREATEBLOCKPOOL
 0010:0007B319       CREATEBPH
 0010:0007B370       VDHALLOCBLOCK
 0010:0007B448       VDHFREEBLOCK
 0010:0007B4FF       VDHDESTROYBLOCKPOOL
 0010:0007B59E       FREEBLOCKS
 0010:0007B5D3       VDHEXCHANGEMEM
 0010:0007B6AB       VDHALLOCSHAREDMEM
 0010:0007B753       VDHFREESHAREDMEM
 0010:0007B780       VDMMCVICLEANUP
 0010:0007B7BD       VDMMZEROFILL
 0010:0007B813       PFNINFO
 0010:0007B884       VDHVALIDATEPID
 0010:0007B8AF       VDHVMGETHANDLE
 0010:0007B8F5       VDHVMATTACH
 0010:0007B913       VDHVMDETACH
 0010:0007B931       VDHHANDLEFROMPID
 0010:0007B968       VDMMUPPERCASE
 0010:0007B99C       VDMMTITLEEVENT
 0010:0007B9D6       VDHREGISTERPERFCTRS
 0010:0007B9FD       VDHDECODEPROPERTY
 0010:0007BAE2       VDMMDECODESTRING
 0010:0007BC12       VDHCREATETHREAD
 0010:0007BC3C       VDHEXITTHREAD
 0010:0007BC50       VDHRPUNDO
 0010:0007BCC2       VDHGETDIRTYPAGEINFO
 0010:0007BD59       VDHPROCESSTOGLOBAL
 0010:0007BDC3       VDHREMOVEFAULTHOOK
 0010:0007BF0E       FREEPFH
 0010:0007BF1F       VDHALLOCDMABUFFER
 0010:0007BFE9       VDHFREEDMABUFFER
 0010:0007C01A       VDHMAPMEMBLOCK
 0010:0007C148       _vdmPropertyInit
 0010:0007C166       _vdmSetPropertyDefaults
 0010:0007C3D8       _setPropertyDefault
 0010:0007C55A       FNVDHRPALWAYSGOOD
 0010:0007C55F       _skipValue
 0010:0007C5AF       VDHREGISTERPROPERTY
 0010:0007C87F       _VR32SetDOSProperty
 0010:0007CAC1       _queryPropertyNames
 0010:0007CB4E       _PROPCreate
 0010:0007CBB7       _PROPDestroy
 0010:0007CC16       _swpFreez
 0010:0007CC2D       _swpStrNDup
 0010:0007CC73       _myStrChr
 0010:0007CC94       _em86PGMoveStub
 0010:0007CCBA       _em86PGGetAccessStub
 0010:0007CCD8       VDHCHECKPAGEPERM
 0010:0007CCFD       VDHRAISEEXCEPTION
 0010:0007CD17       VDHCHECKVPMEXCEPT
 0010:0007CD7F       _em86DPMITaskSwitch
 0010:0007CE7A       VDHPREPVPMIRET
 0010:0007CF04       _VPMPgMapPhys
 0010:0007CFE4       DEMLOADV86KERNEL
 0010:0007D0D0       DEMGETV86KERNEL
 0010:0007D14C       DEMINITFCBSFT
 0010:0007D1F5       DEMALLOCFCBSFT
 0010:0007D273       DEMFREESELTEMP
 0010:0007D2BE       DEMINITV86AREA
 0010:0007D5E2       DEMSETFAKEVERSION
 0010:0007D628       VALIDATELASTDRIVE
 0010:0007D690       VALIDATEFILESCOUNT
 0010:0007D695       VALIDATEAUTOEXEC
 0010:0007D69A       _demParseLabel
 0010:0007D75C       VDMMGETFILEFROMPATH
 0010:0007D7B0       VDMMINITGDT_PTDA
 0010:0007D7BC       VDMMADJUSTERROR
 0010:0007D7D8       em86opINTO
 0010:0007D7F0       EM86VPMEXCBPTERMINATE
 0010:0007D800       EM86VPMEXCBPREFLECT
 0010:0007D810       VPMINTDISPATCHER
 0010:0007D8E8       EM86INT23HOOK
 0010:0007DE60       demDeleteDir
 0010:0007DE70       demCreateDir
 0010:0007DE9C       demDeleteFCB
 0010:0007DEBC       demRenameFCB
 0010:0007DECC       demRename
 0010:0007DEE0       demStartSession
 0010:0007E178       demMoveConvert
 0010:0007E194       demQFSAttach
 0010:0007E1D0       demEditName
 0010:0007E1F8       demCreateSem
 0010:0007E234       demCreateMuxWaitSem
 0010:0007E23C       demResetSem
 0010:0007E258       demWaitSem
 0010:0007E280       demWaitMuxWaitSem
 0010:0007E29C       demSubstPhys
 0010:0007E318       XCHGP32
 0010:0007E320       PDOPEN
 0010:0007E464       PLDCLOSE
 0010:0007E490       PDWRITE
 0010:0007E544       PDSEEK
 0010:0007E584       PDDEL
 0010:0007E600       PDPHYSTOVIRT
 0010:0007E644       PDCALLDD
 0010:0007E6C8       PDNEWSIZE
 0010:0007E6F8       PDDUMPINFO
 0010:0007E824       PDSHUTDOWN
 0010:0007E844       PDREBOOT
 0010:0007E84C       PDGETDISKSPACEINFO
 0010:0007E8B0       PDVPBSEM
 0010:0007E8DC       PDKILLPROC
 0010:0007E900       RASGETSTDA
 0010:0007E964       PDRASQUIESCE
 0010:0007E988       PLDGETDATETIME
 0010:0007E9B0       _qsSys16Sem
 0010:0007E9B0       _StartQUERYSWAP_TEXT
 0010:0007E9B0       _EndMVDMSWAP_TEXT
 0010:0007EAD0       _qs16ShrMem
 0010:0007EB98       _qsMemory
 0010:0007EC9C       _VR32QuerySysState
 0010:0007ECB8       _QSQuerySysState
 0010:0007EE28       _qsGlobal
 0010:0007EE79       _qsProcess
 0010:0007EED3       _qsReadPtda
 0010:0007F033       _qsProcSem
 0010:0007F0BD       _qsProcLib
 0010:0007F0DF       _qsProcShrMem
 0010:0007F11F       _qsProcFS
 0010:0007F1D8       _qsProcThrd
 0010:0007F26A       _qsSem
 0010:0007F2AB       _qsLib
 0010:0007F2CB       _qsMem
 0010:0007F2EE       _qsFile
 0010:0007F342       _qsReadMFT
 0010:0007F4C4       _qsDisk
 0010:0007F4CC       _qsHWConfig
 0010:0007F4D4       _qsNamedPipe
 0010:0007F4DC       _qsModVer
 0010:0007F552       _qsNotSupported
 0010:0007F55A       _qsInitCache
 0010:0007F5E5       _qsFreeCache
 0010:0007F623       _qsCheckCache
 0010:0007F677       _qsFlushCache
 0010:0007F6D1       _qsReserveCache
 0010:0007F707       _qsFlushResCache
 0010:0007F764       _qsUpdatePtrs
 0010:0007F784       _LDRSysMteInfo
 0010:0007FA4B       _LDRProcMteInfo
 0010:0007FAAB       _LDRExSysMteInfo
 0010:0007FC24       _EndQUERYSWAP_TEXT
 0010:0007FC24       _pvwWriteMsg
 0010:0007FC24       _StartPERFSWAP_TEXT
 0010:0007FD76       _pvwTestConfig
 0010:0007FDCA       _pvwRegKrnlInstance
 0010:0007FEDE       _PVWCreateInstance_Thd
 0010:0007FFAC       _pvwReadPtda
 0010:00080069       _PVWCreateInstance_preThd
 0010:00080084       _PVWKillInstance_Thd
 0010:00080124       _PVWDestroyLink
 0010:0008013A       _PVWCreateInstance_Fil
 0010:00080213       _PVWKillInstance_Fil
 0010:000802A9       _pvwCalCTimer
 0010:000802B6       _pvwGet032Addrs
 0010:000802F3       _pvwDupTextBlk
 0010:000805AA       _pvwFindRPDesc
 0010:00080650       _pvwDeconRPDesc
 0010:000807B4       _PVWRegisterPerfCtrs
 0010:00080D54       _pvwInitPersist
 0010:00080E3B       _pvwInitTransient
 0010:00080F45       _pvwAliasPerfBlk
 0010:00081000       _VR32ConfigurePerf
 0010:000815ED       _VR32DeconPerf
 0010:000815F3       _VR32AliasPerfCtrs
 0010:00081831       _VR32RegisterPerfCtrs
 0010:00081848       _PvwMtRouterTable
 0010:00081A28       _PvwMtStartLock
 0010:00081A28       pvwMt_Ct_cpu_Int_0
 0010:00081A38       pvwMt_ST_cpu_NotIdle_0
 0010:00081A54       pvwMt_Ct_mem_Discard_0
 0010:00081A60       pvwMt_Ct_mem_SwapIn_0
 0010:00081A6C       pvwMt_Ct_mem_Recovered_0
 0010:00081A78       pvwMt_Ct_mem_Idled_0
 0010:00081A84       pvwMt_Ct_mem_Reassigned_1
 0010:00081A94       pvwMt_EQ_mem_QFree_0
 0010:00081AB0       pvwMt_Init_LQ_mem_QUsed_0
 0010:00081AB0       pvwMt_Init_EQ_mem_QUsed_0
 0010:00081B04       pvwMt_EQ_mem_QUsed_0
 0010:00081B20       pvwMt_LQ_mem_QUsed_0
 0010:00081B3C       pvwMt_CtST_cal_Masm_0
 0010:00081B5C       pvwMt_ET_cal_Masm_0
 0010:00081B78       pvwMt_CtST_cal_C_0
 0010:00081B90       pvwMt_ET_cal_C_0
 0010:00081C1C       pvwMt_Init_Mt_mem_PageFault_0
 0010:00081C3C       pvwMt_Mt_mem_PageFault_0
 0010:00081C84       pvwMt_Init_Mt_mem_PageFault_1
 0010:00081CA4       pvwMt_Mt_mem_PageFault_1
 0010:00081CE8       pvwMt_Ct_mem_SwapOut_0
 0010:00081CFC       pvwMt_Init_EQ_mem_QFree_0
 0010:00081CFC       pvwMt_Init_LQ_mem_QFree_0
 0010:00081D40       pvwMt_LQ_mem_QFree_0
 0010:00081D74       pvwMt_Init_EQ_mem_QCTResident_0
 0010:00081D74       pvwMt_Init_LQ_mem_QCTResident_0
 0010:00081DBC       pvwMt_Ct_cpu_Sched_0
 0010:00081E68       pvwMt_ET_cpu_NotIdle_0
 0010:00081EDC       pvwMt_ET_spr_Spare1_0
 0010:00081EF8       pvwMt_ST_spr_Spare1_0
 0010:00081F14       pvwMt_CtST_spr_Spare1_0
 0010:00081F34       pvwMt_Ct_spr_Spare1_0
 0010:00081F44       pvwMt_ET_spr_Spare2_0
 0010:00081F60       pvwMt_ST_spr_Spare2_0
 0010:00081F7C       pvwMt_CtST_spr_Spare2_0
 0010:00081F9C       pvwMt_Ct_spr_Spare2_0
 0010:00081FAC       pvwMt_ET_spr_Spare3_0
 0010:00081FC8       pvwMt_ST_spr_Spare3_0
 0010:00081FE4       pvwMt_CtST_spr_Spare3_0
 0010:00082004       pvwMt_Ct_spr_Spare3_0
 0010:00082014       pvwMt_ET_spr_Spare4_0
 0010:00082030       pvwMt_ST_spr_Spare4_0
 0010:0008204C       pvwMt_CtST_spr_Spare4_0
 0010:0008206C       pvwMt_Ct_spr_Spare4_0
 0010:0008207C       pvwMt_ET_spr_Spare5_0
 0010:00082098       pvwMt_ST_spr_Spare5_0
 0010:000820B4       pvwMt_CtST_spr_Spare5_0
 0010:000820D4       pvwMt_Ct_spr_Spare5_0
 0010:000820E4       pvwMt_ET_spr_Spare6_0
 0010:00082100       pvwMt_ST_spr_Spare6_0
 0010:0008211C       pvwMt_CtST_spr_Spare6_0
 0010:0008213C       pvwMt_Ct_spr_Spare6_0
 0010:0008214C       pvwMt_ET_spr_Spare7_0
 0010:00082168       pvwMt_ST_spr_Spare7_0
 0010:00082184       pvwMt_CtST_spr_Spare7_0
 0010:000821A4       pvwMt_Ct_spr_Spare7_0
 0010:000821B4       pvwMt_ET_spr_Spare8_0
 0010:000821D0       pvwMt_ST_spr_Spare8_0
 0010:000821EC       pvwMt_CtST_spr_Spare8_0
 0010:0008220C       pvwMt_Ct_spr_Spare8_0
 0010:0008221C       pvwMt_ET_spr_Spare9_0
 0010:00082238       pvwMt_ST_spr_Spare9_0
 0010:00082254       pvwMt_CtST_spr_Spare9_0
 0010:00082274       pvwMt_Ct_spr_Spare9_0
 0010:00082284       pvwMt_ET_spr_Spare10_0
 0010:000822A4       pvwMt_ST_spr_Spare10_0
 0010:000822C4       pvwMt_CtST_spr_Spare10_0
 0010:000822EC       pvwMt_Ct_spr_Spare10_0
 0010:00082300       _pvwStopTimers
 0010:00082334       _pvwCalibrateTimers
 0010:00082388       _VR32DYNAMICTRACE
 0010:00082388       _PvwMtEndLock
 0010:00082388       _EndPERFSWAP_TEXT
 0010:00082388       _StartDYNSWAP_TEXT
 0010:000823B3       _DYNDynamicTrace
 0010:00082474       _dynAPIInsert
 0010:000825AA       _dynAPIRemove
 0010:0008263A       _dynAPIClearAll
 0010:00082699       _dynAPIGetVar
 0010:00082862       _dynAPIQuery
 0010:00082962       _RAS_dynAPIQuery
 0010:00082A29       _dynAPIGetDTO
 0010:00082B29       _DYNDetach
 0010:00082B7A       _DYNAttachCheck
 0010:00082BF7       _DYNAttachError
 0010:00082C42       _DYNPurgeRange
 0010:00082CBA       _dynAPIVerify
 0010:00082D9A       _dynInitialize
 0010:00082F55       _dynShutdown
 0010:00083088       _dynDTOLink
 0010:000830CB       _dynDTOUnLink
 0010:000831F0       _dynDTORead11
 0010:0008342A       _dynDTORead20
 0010:00083539       _dynDTOVerify
 0010:000835E7       _dynDTOFixup
 0010:00083662       _dynDTOSet
 0010:000836DA       _dynDTOUnSet
 0010:0008372E       _dynDTODetach
 0010:000837F4       _dynDTOAttachCheck
 0010:0008387C       _dynDTOAttach
 0010:00083A36       _dynDTOAttachError
 0010:00083A81       _dynDTOPurgeRange
 0010:00083ABD       _dynDTOMakeSwappable
 0010:00083B1E       _dynDTOMakeResident
 0010:00083B8D       _dynDTODestroy
 0010:00083BD2       _dynDTOFree
 0010:00083C25       _dynDTOGetVar
 0010:00083DB5       _dynDTOQuery
 0010:00083E63       _RAS_dynDTOCount
 0010:00083EFB       _RAS_dynDTOInfo
 0010:00084067       _dynDTOGetDTO
 0010:0008416E       _dynDTONullProc
 0010:0008418F       _dynDTOScan
 0010:000842E8       _dynGetObjNum
 0010:00084347       _dynDTRFixup
 0010:00084403       _dynDTRSet
 0010:000844CC       _dynDTRUnSet
 0010:00084570       _dynDTRDetach
 0010:000845D7       _dynDTRMove
 0010:00084661       _dynDTRPurge
 0010:000846A3       _dynDTRMapAlias
 0010:00084810       _dynDTRUnMapAlias
 0010:00084868       _dynDTRSkipScan
 0010:000848C1       _dynDTRScan
 0010:00084AAD       _RAS_dynDTRInfo
 0010:00084DD0       _dynDTRCompile
 0010:00084EAC       dyndtra$dynAddTarget
 0010:00084F10       _dynDTRValidate
 0010:00084FD8       _StartDYNLOCK_TEXT
 0010:00084FD8       _EndDYNSWAP_TEXT
 0010:00084FD8       _dynInterpreter
 0010:00085344       tci_PushEAX
 0010:00085354       tci_PushECX
 0010:00085364       tci_PushEDX
 0010:00085374       tci_PushEBX
 0010:00085384       tci_PushESP
 0010:000853A0       tci_PushEBP
 0010:000853B0       tci_PushESI
 0010:000853C0       tci_PushEDI
 0010:000853D0       tci_PushCS
 0010:000853E4       tci_PushSS
 0010:00085404       tci_PushEFlags
 0010:00085414       tci_PushEIP
 0010:00085428       tci_PushDS
 0010:0008543C       tci_PushES
 0010:00085450       tci_PushFS
 0010:00085464       tci_PushGS
 0010:00085478       tci_PushW
 0010:0008548C       tci_PushOXS
 0010:000854B4       tci_PushWIS
 0010:000854E4       tci_PushSIS
 0010:00085528       tci_LogWN
 0010:00085548       tci_LogMRS
 0010:000855A4       tci_Add
 0010:000855BC       tci_POP1W
 0010:000855C4       tci_LogARS
 0010:00085624       tci_PushD
 0010:00085634       tci_PushOXF
 0010:00085658       tci_PushFIF
 0010:00085674       tci_CnvrtFXS
 0010:000856C8       tci_CnvrtSXF
 0010:00085708       tci_CnvrtDXS
 0010:00085730       tci_CnvrtSXD
 0010:00085754       tci_LogDN
 0010:00085774       tci_LogMRF
 0010:000857B8       tci_LogARF
 0010:00085800       tci_Sub
 0010:00085818       tci_Mul
 0010:00085838       tci_PopN
 0010:00085840       tci_MoveV
 0010:00085858       tci_PushV
 0010:00085874       tci_IncV
 0010:00085884       tci_MoveVIi
 0010:000858B4       tci_PushVIi
 0010:000858E0       tci_IncVIi
 0010:00085900       tci_JmpN
 0010:00085908       tci_JmpZN
 0010:0008591C       tci_JmpNN
 0010:00085930       tci_JmpPN
 0010:00085944       tci_Remove
 0010:0008594C       tci_Abort
 0010:0008595C       tci_OrV
 0010:00085974       tci_And
 0010:0008598C       tci_Or
 0010:000859A4       tci_Xor
 0010:000859BC       tci_Not
 0010:000859C8       tci_ProcDump
 0010:000859D8       tci_ExitOk
 0010:000859DC       tci_SetMinW
 0010:000859E8       tci_SetMajW
 0010:000859F4       tci_SetMin
 0010:00085A08       tci_SetMaj
 0010:00085A1C       tci_Xchg
 0010:00085A48       tci_CallKDB
 0010:00085A5C       tci_CallDD
 0010:00085BDC       tci_CallDBG
 0010:00085BE8       tci_DupN
 0010:00085C0C       tci_Dup
 0010:00085C40       tci_EnterBIF
 0010:00085C64       tci_EnterWIF
 0010:00085C88       tci_EnterDIF
 0010:00085CAC       tci_EnterBIS
 0010:00085CE0       tci_EnterWIS
 0010:00085D14       tci_EnterDIS
 0010:00085D48       tci_PushBIF
 0010:00085D64       tci_PushBIS
 0010:00085D94       tci_PushDIS
 0010:00085DC4       tci_PushWIF
 0010:00085DE0       tci_PushTSC
 0010:00085E1C       tci_PushTID
 0010:00085E34       tci_PushPID
 0010:00085E50       tci_PushProcID
 0010:00085E60       tci_PushSlot
 0010:00085E78       tci_PushpTCB
 0010:00085E8C       tci_PushpPTDA
 0010:00085EA0       tci_PushpPCB
 0010:00085EB0       tci_Suspend
 0010:00085EC0       tci_Resume
 0010:00085ED0       tci_RolN
 0010:00085EEC       tci_RorN
 0010:00085F08       tci_ShlN
 0010:00085F24       tci_ShrN
 0010:00085F40       tci_Rol
 0010:00085F64       tci_Ror
 0010:00085F88       tci_Shl
 0010:00085FAC       tci_Shr
 0010:00085FD0       tci_VFA
 0010:00086000       tci_VSA
 0010:00086040       tci_PushKEAX
 0010:00086058       tci_PushKEBX
 0010:00086070       tci_PushKECX
 0010:00086088       tci_PushKEDX
 0010:000860A0       tci_PushKESP
 0010:000860B8       tci_PushKEBP
 0010:000860D0       tci_PushKESI
 0010:000860E8       tci_PushKEDI
 0010:00086100       tci_PushKES
 0010:00086118       tci_PushKCS
 0010:00086130       tci_PushKSS
 0010:00086148       tci_PushKDS
 0010:00086160       tci_PushKEFlags
 0010:00086178       tci_PushKEIP
 0010:00086190       tci_PushKFS
 0010:000861A8       tci_PushKGS
 0010:000861C0       tci_PushKReg
 0010:000861F8       tci_EnterEAX
 0010:00086208       tci_EnterEBX
 0010:00086218       tci_EnterECX
 0010:00086228       tci_EnterEDX
 0010:00086238       tci_EnterESI
 0010:00086248       tci_EnterEDI
 0010:00086258       tci_EnterEBP
 0010:00086268       tci_EnterDS
 0010:0008627C       tci_EnterES
 0010:00086290       tci_EnterFS
 0010:000862A4       tci_EnterGS
 0010:000862B8       tci_PushCR0
 0010:000862C8       tci_PushCR2
 0010:000862D8       tci_PushCR3
 0010:000862E8       tci_PushCR4
 0010:00086304       tci_PushDR0
 0010:00086314       tci_PushDR1
 0010:00086324       tci_PushDR2
 0010:00086334       tci_PushDR3
 0010:00086344       tci_PushDR6
 0010:00086354       tci_PushDR7
 0010:00086364       tci_PushTR
 0010:00086378       tci_PushLDTR
 0010:0008638C       tci_PushGDTR
 0010:000863B8       tci_PushIDTR
 0010:000863E4       tci_PushMSR
 0010:00086430       tci_PushPMC
 0010:00086470       tci_PushCPUID
 0010:000864E8       tci_LogFault
 0010:000865EC       tci_GPFault
 0010:00086688       tci_PageFault
 0010:000866D8       tci_FixFault
 0010:000866E4       tci_SysDump
 0010:00086804       _DYNTrap3
 0010:000868A3       DRAS3
 0010:00086900       _dynSStep
 0010:00086A60       _dynEmulateCLD
 0010:00086A69       _dynEmulateSTC
 0010:00086A6F       _dynEmulateCMC
 0010:00086A76       _dynEmulateCLC
 0010:00086A7A       _dynEmulateNOP
 0010:00086A80       _DYNRecordPoint
 0010:00086ABC       _StartDEBUGLOCK_TEXT
 0010:00086ABC       _EndDYNLOCK_TEXT
 0010:00086ABC       _DbgAliasFree
 0010:00086B56       _DbgProcTerm
 0010:00086C6E       _DbgEvent
 0010:00086D4C       _DbgWatchpoint
 0010:00086EB6       _DbgHandler
 0010:000870DE       _DbgNotify
 0010:00087266       _DbgBlock
 0010:000872AD       _DbgEnterCrit
 0010:0008737B       _DbgExitCrit
 0010:00087418       _DbgProcessSemList
 0010:00087BF5       _DbgSeverConnection
 0010:00087DAE       _DbgDetachConnection
 0010:00087EB8       _DbgReadReg
 0010:00088171       _dbgVerifySel
 0010:000881C2       _DbgWriteReg
 0010:00088413       _DbgSStep
 0010:0008859C       _DbgStop
 0010:0008860D       _DbgFreezeThaw
 0010:00088781       _DbgCoRegs
 0010:0008890F       _DbgThrdStat
 0010:00088A56       _DbgContinue
 0010:00088B3E       _dbgXchgOpcode
 0010:00088CDB       _DbgCall
 0010:00088DD7       _DbgKillDebuggees
 0010:00088EBD       _DbgKillJITDebuggee
 0010:00088F45       _DbgGetDCB
 0010:00089010       _DbgReleaseDCB
 0010:000890A0       _DbgValidateDR7
 0010:000890C4       _DbgDR7LeGe
 0010:000890E8       _DbgWPAlloc
 0010:000892B2       _dbgGlobalWPFree
 0010:0008947C       _dbgLocalWPFree
 0010:00089646       _DbgWPFree
 0010:000896AC       _DbgWPSet
 0010:00089863       _DbgWPHit
 0010:000899C4       g__DbgProcTerm
 0010:000899CF       g__DbgKillDebuggees
 0010:000899DC       _StartDEBUGSWAP_TEXT
 0010:000899DC       _EndDEBUGLOCK_TEXT
 0010:000899DC       _dbgUserCSEIP
 0010:00089A95       _dbgFinishXchgOp
 0010:00089B6C       _DbgTrap
 0010:00089E25       _DbgException
 0010:00089F95       _DbgNewProc
 0010:00089FC1       _DbgThreadCreate
 0010:00089FF3       _DbgThreadNotify
 0010:0008A04D       _DbgModuleNotify
 0010:0008A08D       _DbgModuleEvent
 0010:0008A0A2       _DBGEntryEvent
 0010:0008A0ED       _DbgLibLoad
 0010:0008A14A       _DbgLibFree
 0010:0008A1A7       _DbgDLLEvent
 0010:0008A1F4       _DbgValidateTF
 0010:0008A330       _DbgNull
 0010:0008A367       _dbgReadWrite
 0010:0008A48C       _DbgRWMem
 0010:0008A4EF       _DbgReadWord
 0010:0008A53A       _DbgWriteWord
 0010:0008A57E       _DbgReadBuf
 0010:0008A5C2       _DbgWriteBuf
 0010:0008A606       _DbgGo
 0010:0008A6A8       _DbgTerm
 0010:0008A714       _DbgNumToAddr
 0010:0008A765       _DbgAlias
 0010:0008A890       _DbgConnect
 0010:0008A94B       _DbgCreateAttachEntry
 0010:0008AA1E       _DbgAttach
 0010:0008AAE7       _DbgDetach
 0010:0008AB9C       _DbgRegisterPerProcessJITDebugger
 0010:0008AE85       _DbgRegisterGlobalJITDebugger
 0010:0008B109       _DbgQueryJITDebugger
 0010:0008B304       _DbgSetWatch
 0010:0008B3E8       _DbgClearWatch
 0010:0008B42D       _DbgAddrToObject
 0010:0008B4EF       _DbgLinearToSel
 0010:0008B591       _DbgSelToLinear
 0010:0008B648       _DbgkDBWrite
 0010:0008B693       _DbgEnable
 0010:0008B77C       _DbgDisable
 0010:0008B7E8       _DBGWPAllocVDM
 0010:0008BA0F       _DBGWPFreeVDM
 0010:0008BBF2       _DBGDR6QueryVDM
 0010:0008BCF8       _PTraceCmd
 0010:0008BECB       _PTPidToPTDA
 0010:0008BF18       _PT_CvtOUTBuff
 0010:0008C6CC       _PT_CvtINBuff
 0010:0008CDAE       _PTSelToLin
 0010:0008CE75       _PTLinToSel
 0010:0008CEFD       _PTAlias
 0010:0008D144       _PT_FPRegs
 0010:0008D294       _PTCheck
 0010:0008D9B4       _EndDEBUGSWAP_TEXT
 0010:0008D9B4       g_dh32_MonFlush
 0010:0008D9B4       _StartMON32SWAP_TEXT
 0010:0008DA1C       g_dh32_MonitorCreate
 0010:0008DA9C       g_dh32_Register
 0010:0008DB08       g_dh32_DeRegister
 0010:0008DB64       _ArrayToFlat
 0010:0008DC88       _MonitorFromBufferI
 0010:0008DCEA       _MonitorFromBufferO
 0010:0008DD4D       _MD32IMONREAD
 0010:0008DE8F       _MD32IMONWRITE
 0010:0008DFE8       _access_ubuffers
 0010:0008E080       _dhw_MonitorCreate
 0010:0008E5C2       _dhw_Register
 0010:0008EA85       _dhw_Deregister
 0010:0008ECDC       _FindMonFromPid
 0010:0008ED05       _UseChain
 0010:0008ED65       _UnUseChain
 0010:0008ED80       _StartMON32LOCK_TEXT
 0010:0008ED80       _dhw_MonWrite
 0010:0008ED80       _EndMON32SWAP_TEXT
 0010:0008EEB3       _FlatToArray
 0010:0008F004       _FindChain
 0010:0008F034       _Notify32MonNotify
 0010:0008F068       _StartPROFLOCK_TEXT
 0010:0008F068       _PROSysArena
 0010:0008F068       _EndMON32LOCK_TEXT
 0010:0008F08D       _PROShrArena
 0010:0008F0B4       proLogProfileData
 0010:0008F198       _proError
 0010:0008F1A8       _StartPROFSWAP_TEXT
 0010:0008F1A8       _EndPROFLOCK_TEXT
 0010:0008F1A8       _VR32Profile
 0010:0008F237       _proCreate
 0010:0008F86E       _proStart
 0010:0008F8A7       _proStop
 0010:0008F8D8       _proClear
 0010:0008F9D8       _proDump
 0010:0008FE2B       _PRODestroyPCB
 0010:0008FFB8       _proGetPPCB
 0010:0009002A       _proDestroyDeadThrdPCBs
 0010:00090086       _PROAllocThrdPCB
 0010:000902CF       _PROSaveThrdPCB
 0010:00090394       _proSetTimer
 0010:000903C0       _proCollectOn
 0010:000903E4       _proCollectOff
 0010:00090408       _hyberYankIdlePF
 0010:0009054D       _hyberPageOut
 0010:00090668       _hyberGetOldrPage
 0010:00090747       _hyberGiveUp
 0010:00090788       _hybernate
 0010:000910C5       _hyberInitInfo
 0010:0009115B       _hyberMapPhysMem
 0010:0009124D       _hyberRestart
 0010:00091293       _hyberOK
 0010:00091402       _hyberFileCheck
 0010:00091501       _hyberFreeSwapper
 0010:0009153C       _hyberFreezeSys
 0010:0009155B       _hyberIOinit
 0010:000915EA       _hyberDumpTheSystem
 0010:000917AF       _hyberSetMultiple
 0010:000917EC       _hyberStartio
 0010:000918DC       _hyberDummy
 0010:000918E0       _hyberGrabState
 0010:00091A60       hyberCommState
 0010:00091A9C       _hyberChksumPage
 0010:00091AC0       _hyberPgCopy
 0010:00091AF0       _hyberDone
 0010:00091AF8       _hyberSpcl
 0010:00091B04       _getSwapperPath
 0010:00091B28       _getSFTExtent
 0010:00091B60       _BootDos32
 0010:00091B80       _hyberReboot
 0010:00091B88       _inb
 0010:00091B90       _outb
 0010:00091BA4       _hyberDelay
 0010:00091BB0       _hdWaitReady
 0010:00091BD0       _hdWaitNotBusy
 0010:00091BE0       _hdWaitForIRQ14
 0010:00091BEC       _hdReadBlock
 0010:00091C38       _hdWriteBlock
 0010:00091CD0       _hdEnd
 0010:00091CD4       g_InitCodeLocks
 0010:00091CD4       _StartCINIT_TEXT
 0010:00091CD4       _EndPROFSWAP_TEXT
 0010:00091D78       _FSD_SetSwap
 0010:00091D98       _FSD_OpenPageFile
 0010:00091E88       _FSD_GetPageMediaInfo
 0010:00091EB0       _BufInit
 0010:00092079       _FinishBufInit
 0010:000921D8       _Sec1
 0010:000921FC       _Sec2
 0010:000922AC       _SYISaveMessage
 0010:00092404       _SYISaveMessageSub
 0010:00092420       _SYISaveMessageID
 0010:00092438       _SYIIniPLD
 0010:000925C0       _PGAllocHighMem
 0010:00092815       _pgAllocPFHighMem
 0010:000929BC       _selFixCallGates
 0010:00092A0C       _selLockHandleInit
 0010:00092A68       _SELDiscSegInit
 0010:00092AC0       _SMReinit
 0010:00092D80       _smIncreaseBitmapForInmemFile
 0010:00092DD4       _smSIOInit
 0010:000932AC       _vmInitAliasRec
 0010:00093318       _dhw_VMInitAlloc
 0010:0009339A       _vmdh_AllocAddList
 0010:000933EE       _vmdh_AllocRemoveList
 0010:00093445       _VMDH_AllocRemoveAccess
 0010:00093478       _VMInit
 0010:000940FC       _vmInitAlloc
 0010:000941B6       _vmInitBMPInit
 0010:0009424F       _VMExchangeSel
 0010:00094360       _VMInitProtect
 0010:000944FC       g__LDRDisableDirtyHooks
 0010:00094507       g__PGInitBuf
 0010:00094512       g__PGInitInfoSegs
 0010:0009451D       g__VMInitProtect
 0010:00094528       _vmNameShareInit
 0010:00094580       _vmDonateHighCode
 0010:0009460C       _vmInitPublicHeaps
 0010:000947C7       _VMRemoveUserAccessKHB
 0010:00094A7B       _VMDonateKHB
 0010:00094BB3       _vmDonateFragKH
 0010:00094EC0       _VMCreateKH
 0010:000951F4       _vmCreateKSH
 0010:00095464       _selLockDD
 0010:000954CF       _SELRemoveAccess
 0010:00095698       VDMMINIT
 0010:000957C6       INITTIME
 0010:000957F2       INITALLOCSEM
 0010:00095858       INITGLOBALMAP
 0010:000958D1       INITMAPID
 0010:000958DE       INITINSTANCE
 0010:00095923       INITCHECKVDDLOADING
 0010:00095961       LOADVDDS
 0010:00095B3E       VDMMFAILMESSAGE
 0010:00095B72       UNLOADVDDS
 0010:00095C06       VDMMLOADINGVDD
 0010:00095C56       VDMMUNLOADINGVDD
 0010:00095D67       INITGETVDMINTERRUPTHANDLER
 0010:00095DA3       _VDMMDHRegisterPDD
 0010:00095F85       VDMMGETPOSREGS
 0010:00095FEE       VDMMFREEREGISTERPDDBLOCKS
 0010:0009601D       INITSYSCONFIGTABLE
 0010:00096054       LHSETUPINST
 0010:00096114       INITASSIGNADDRESS
 0010:00096233       FIXASSIGNADDRESS
 0010:00096304       FREEINITHEAP
 0010:00096334       HEAPFREEHEAP
 0010:0009635B       QUERYOBJTYPE
 0010:00096398       VDMMASSIGNADDRESS
 0010:000963E3       VDMMGETFIXUP
 0010:00096433       HEAPALLOC
 0010:000966E4       VDMMDEASSIGNADDRESS
 0010:00096831       HEAPFREEHB
 0010:00096847       HEAPCOALESCEHB
 0010:00096894       HEAPALLOCHB
 0010:000968EC       VDHOPENPDD
 0010:00096970       VDMMINITTIMER
 0010:000969BC       _VDMInt13CreateMiniVDM
 0010:00096A05       _VDMInt13CreateMiniVDMSub
 0010:00097033       _VDMInt13DestroyMiniVDM
 0010:00097154       g_InitNPXEM
 0010:000972C4       npx$NPXPtdaFixup
 0010:000972EC       g_InitNPX
 0010:000973B0       _SEMInitShrTbl
 0010:000974C4       _TIMInit
 0010:0009756C       _TKPreInit
 0010:000975F4       _TKSchedInit
 0010:00097658       _TKInit
 0010:00097985       _tkInitSysInfo
 0010:00097A74       g_INTInit
 0010:00097AB4       g_INTInit2
 0010:00097AF4       int$intAllocStack
 0010:00097B80       g__DevhlpDisableAccess
 0010:00097BE4       inidin2$SysInitThread3Thunk
 0010:00097BF0       SIReadAt
 0010:00097C44       SIOpen
 0010:00097CA8       SIClose
 0010:00097CC0       SIIOSftTransPath
 0010:00097D14       SIldrGetMedia
 0010:00097D1C       _LDRInit
 0010:00097E43       _LDRDisableDirtyHooks
 0010:00097E7E       _LDRFreeVDDMTEs
 0010:00097EBC       g_PreLoadInit
 0010:00097EC8       g_LDRLibPathAlloc
 0010:00097F24       g_ldrLieListAlloc
 0010:00097FE0       _LDRInitOTE
 0010:0009813C       ldrinita$InitMTEs
 0010:00098180       g_FreeDynLink
 0010:000981B8       EditDynLink
 0010:00098244       g__LDRFreeInit
 0010:000984B8       ldrinita$_ldrFreeSegInit
 0010:00098510       _CheckABIOS
 0010:00098518       LDRSetMiniFileIO
 0010:0009856C       g_LDRUnSetMiniFileIO
 0010:000985C4       _LDREnableCVK
 0010:000985CC       _ldrCopyVDD
 0010:00098641       _ldrResetDD
 0010:000986B0       _PGSwitchContextInit
 0010:00098858       _PGSwitchInit
 0010:00098944       _pgInitDosTable
 0010:00098964       _PGInit
 0010:00099B5E       _PGAllocCRPTE
 0010:00099BFB       _PGInitBuf
 0010:00099E3F       _PGInitSwap
 0010:00099E85       _pgAllocArena
 0010:0009A04A       _pgFreeArena
 0010:0009A071       _pgDecommitArena
 0010:0009A10E       _PGInitHob
 0010:0009A277       _pgInitPrt
 0010:0009A37A       _pgSetBoundary
 0010:0009A3F3       _PGInitInfoSegs
 0010:0009A6BB       _PGInitHighMem
 0010:0009A89F       _PGAgerInit
 0010:0009A9C6       _pgTrap2BootFix
 0010:0009AB0C       _SELInit
 0010:0009AD48       g__SELReinit
 0010:0009AF18       g__SELEndInit
 0010:0009AFCC       selinit$selMapHigh
 0010:0009B080       _LDRINITInfo
 0010:0009B0FC       _LDRINITSetGDT_DPL0
 0010:0009B1C8       _LDRLoadVDD
 0010:0009B2E0       _LDRUnloadVDD
 0010:0009B338       DEMINIT
 0010:0009B3FC       g_VDMMINITTIMER
 0010:0009B407       g_VDMMGETPOSREGS
 0010:0009B414       g_MVDMINIT
 0010:0009B59C       vdmma$vdmmBuildPSZZ
 0010:0009B640       vdmma$vdmmStrCpy
 0010:0009B654       vdmma$vdmmStrLen
 0010:0009B67C       vdmma$vdmmGetMachineInfo
 0010:0009B67C       VDMMGETMACHINEINFO
 0010:0009B6A4       VDMMSEM
 0010:0009B6E4       VDMMREMOVESYMMTE
 0010:0009B704       vdmma$Clear96
 0010:0009B70C       vdmma$POSRead
 0010:0009B71C       VDMMGETSLOTPOS
 0010:0009B758       VDMMGETPLANARPOS
 0010:0009B79C       VDMMGETVIDEOPOS
 0010:0009B7D8       VDMMGETPORT90
 0010:0009B7DC       VDMMGETPORT92
 0010:0009B7E0       EM86INIT
 0010:0009B7F4       g__TKPreInit
 0010:0009B7FF       g__TKSchedInit
 0010:0009B80A       g__TKInit
 0010:0009B818       _DebugPagingEnabled
 0010:0009B844       SIDebugLoadSymDosFS
 0010:0009B89C       SIDebugLoadSymModule
 0010:0009B8DC       _EndCINIT_TEXT
 0010:0009B8DC       _StartTHUNKINIT_TEXT
 0010:0009BA24       _StartENDHIGH32CODE
 0010:0009BA24       _EndTHUNKINIT_TEXT

Program entry point at 0002:00006118
